Component: ARM Compiler 5.06 update 1 (build 61) Tool: armlink [4d35a8]

==============================================================================

Section Cross References

    system_stm32f7xx.o(i.SystemCoreClockUpdate) refers to system_stm32f7xx.o(.data) for .data
    stm32f7xx_hal.o(i.HAL_DeInit) refers to stm32f7xx_hal.o(i.HAL_MspDeInit) for HAL_MspDeInit
    stm32f7xx_hal.o(i.HAL_Delay) refers to stm32f7xx_hal.o(i.HAL_GetTick) for HAL_GetTick
    stm32f7xx_hal.o(i.HAL_GetTick) refers to stm32f7xx_hal.o(.data) for .data
    stm32f7xx_hal.o(i.HAL_IncTick) refers to stm32f7xx_hal.o(.data) for .data
    stm32f7xx_hal.o(i.HAL_Init) refers to stm32f7xx_hal_cortex.o(i.HAL_NVIC_SetPriorityGrouping) for HAL_NVIC_SetPriorityGrouping
    stm32f7xx_hal.o(i.HAL_Init) refers to stm32f7xx_hal.o(i.HAL_InitTick) for HAL_InitTick
    stm32f7xx_hal.o(i.HAL_Init) refers to stm32f7xx_hal.o(i.HAL_MspInit) for HAL_MspInit
    stm32f7xx_hal.o(i.HAL_InitTick) refers to stm32f7xx_hal_rcc.o(i.HAL_RCC_GetHCLKFreq) for HAL_RCC_GetHCLKFreq
    stm32f7xx_hal.o(i.HAL_InitTick) refers to stm32f7xx_hal_cortex.o(i.HAL_SYSTICK_Config) for HAL_SYSTICK_Config
    stm32f7xx_hal.o(i.HAL_InitTick) refers to stm32f7xx_hal_cortex.o(i.HAL_NVIC_SetPriority) for HAL_NVIC_SetPriority
    stm32f7xx_hal_cortex.o(i.HAL_NVIC_SetPriority) refers to stm32f7xx_hal_cortex.o(i.NVIC_SetPriority) for NVIC_SetPriority
    stm32f7xx_hal_cortex.o(i.HAL_SYSTICK_Config) refers to stm32f7xx_hal_cortex.o(i.NVIC_SetPriority) for NVIC_SetPriority
    stm32f7xx_hal_cortex.o(i.HAL_SYSTICK_IRQHandler) refers to stm32f7xx_hal_cortex.o(i.HAL_SYSTICK_Callback) for HAL_SYSTICK_Callback
    stm32f7xx_ll_usb.o(i.USB_ActivateDedicatedEndpoint) refers to stm32f7xx_ll_usb.o(.data) for .data
    stm32f7xx_ll_usb.o(i.USB_CoreInit) refers to stm32f7xx_ll_usb.o(i.USB_CoreReset) for USB_CoreReset
    stm32f7xx_ll_usb.o(i.USB_DevConnect) refers to stm32f7xx_hal.o(i.HAL_Delay) for HAL_Delay
    stm32f7xx_ll_usb.o(i.USB_DevDisconnect) refers to stm32f7xx_hal.o(i.HAL_Delay) for HAL_Delay
    stm32f7xx_ll_usb.o(i.USB_DevInit) refers to stm32f7xx_ll_usb.o(i.USB_FlushTxFifo) for USB_FlushTxFifo
    stm32f7xx_ll_usb.o(i.USB_DevInit) refers to stm32f7xx_ll_usb.o(i.USB_FlushRxFifo) for USB_FlushRxFifo
    stm32f7xx_ll_usb.o(i.USB_EPStartXfer) refers to stm32f7xx_ll_usb.o(i.USB_WritePacket) for USB_WritePacket
    stm32f7xx_ll_usb.o(i.USB_HC_StartXfer) refers to stm32f7xx_ll_usb.o(i.USB_DoPing) for USB_DoPing
    stm32f7xx_ll_usb.o(i.USB_HC_StartXfer) refers to stm32f7xx_ll_usb.o(i.USB_WritePacket) for USB_WritePacket
    stm32f7xx_ll_usb.o(i.USB_HostInit) refers to stm32f7xx_ll_usb.o(i.USB_FlushTxFifo) for USB_FlushTxFifo
    stm32f7xx_ll_usb.o(i.USB_HostInit) refers to stm32f7xx_ll_usb.o(i.USB_FlushRxFifo) for USB_FlushRxFifo
    stm32f7xx_ll_usb.o(i.USB_HostInit) refers to stm32f7xx_ll_usb.o(i.USB_DriveVbus) for USB_DriveVbus
    stm32f7xx_ll_usb.o(i.USB_HostInit) refers to stm32f7xx_hal.o(i.HAL_Delay) for HAL_Delay
    stm32f7xx_ll_usb.o(i.USB_ResetPort) refers to stm32f7xx_hal.o(i.HAL_Delay) for HAL_Delay
    stm32f7xx_ll_usb.o(i.USB_SetCurrentMode) refers to stm32f7xx_hal.o(i.HAL_Delay) for HAL_Delay
    stm32f7xx_ll_usb.o(i.USB_StopDevice) refers to stm32f7xx_ll_usb.o(i.USB_FlushRxFifo) for USB_FlushRxFifo
    stm32f7xx_ll_usb.o(i.USB_StopDevice) refers to stm32f7xx_ll_usb.o(i.USB_FlushTxFifo) for USB_FlushTxFifo
    stm32f7xx_ll_usb.o(i.USB_StopHost) refers to stm32f7xx_ll_usb.o(i.USB_FlushTxFifo) for USB_FlushTxFifo
    stm32f7xx_ll_usb.o(i.USB_StopHost) refers to stm32f7xx_ll_usb.o(i.USB_FlushRxFifo) for USB_FlushRxFifo
    stm32f7xx_hal_flash.o(i.FLASH_SetErrorCode) refers to stm32f7xx_hal_flash.o(.bss) for .bss
    stm32f7xx_hal_flash.o(i.FLASH_WaitForLastOperation) refers to stm32f7xx_hal.o(i.HAL_GetTick) for HAL_GetTick
    stm32f7xx_hal_flash.o(i.FLASH_WaitForLastOperation) refers to stm32f7xx_hal_flash.o(i.FLASH_SetErrorCode) for FLASH_SetErrorCode
    stm32f7xx_hal_flash.o(i.FLASH_WaitForLastOperation) refers to stm32f7xx_hal_flash.o(.bss) for .bss
    stm32f7xx_hal_flash.o(i.HAL_FLASH_GetError) refers to stm32f7xx_hal_flash.o(.bss) for .bss
    stm32f7xx_hal_flash.o(i.HAL_FLASH_IRQHandler) refers to stm32f7xx_hal_flash.o(i.HAL_FLASH_EndOfOperationCallback) for HAL_FLASH_EndOfOperationCallback
    stm32f7xx_hal_flash.o(i.HAL_FLASH_IRQHandler) refers to stm32f7xx_hal_flash_ex.o(i.FLASH_Erase_Sector) for FLASH_Erase_Sector
    stm32f7xx_hal_flash.o(i.HAL_FLASH_IRQHandler) refers to stm32f7xx_hal_flash.o(i.FLASH_SetErrorCode) for FLASH_SetErrorCode
    stm32f7xx_hal_flash.o(i.HAL_FLASH_IRQHandler) refers to stm32f7xx_hal_flash.o(i.HAL_FLASH_OperationErrorCallback) for HAL_FLASH_OperationErrorCallback
    stm32f7xx_hal_flash.o(i.HAL_FLASH_IRQHandler) refers to stm32f7xx_hal_flash.o(.bss) for .bss
    stm32f7xx_hal_flash.o(i.HAL_FLASH_OB_Launch) refers to stm32f7xx_hal_flash.o(i.FLASH_WaitForLastOperation) for FLASH_WaitForLastOperation
    stm32f7xx_hal_flash.o(i.HAL_FLASH_Program) refers to stm32f7xx_hal_flash.o(i.FLASH_WaitForLastOperation) for FLASH_WaitForLastOperation
    stm32f7xx_hal_flash.o(i.HAL_FLASH_Program) refers to stm32f7xx_hal_flash.o(i.FLASH_Program_Byte) for FLASH_Program_Byte
    stm32f7xx_hal_flash.o(i.HAL_FLASH_Program) refers to stm32f7xx_hal_flash.o(i.FLASH_Program_HalfWord) for FLASH_Program_HalfWord
    stm32f7xx_hal_flash.o(i.HAL_FLASH_Program) refers to stm32f7xx_hal_flash.o(i.FLASH_Program_Word) for FLASH_Program_Word
    stm32f7xx_hal_flash.o(i.HAL_FLASH_Program) refers to stm32f7xx_hal_flash.o(i.FLASH_Program_DoubleWord) for FLASH_Program_DoubleWord
    stm32f7xx_hal_flash.o(i.HAL_FLASH_Program) refers to stm32f7xx_hal_flash.o(.bss) for .bss
    stm32f7xx_hal_flash.o(i.HAL_FLASH_Program_IT) refers to stm32f7xx_hal_flash.o(i.FLASH_Program_Byte) for FLASH_Program_Byte
    stm32f7xx_hal_flash.o(i.HAL_FLASH_Program_IT) refers to stm32f7xx_hal_flash.o(i.FLASH_Program_HalfWord) for FLASH_Program_HalfWord
    stm32f7xx_hal_flash.o(i.HAL_FLASH_Program_IT) refers to stm32f7xx_hal_flash.o(i.FLASH_Program_Word) for FLASH_Program_Word
    stm32f7xx_hal_flash.o(i.HAL_FLASH_Program_IT) refers to stm32f7xx_hal_flash.o(i.FLASH_Program_DoubleWord) for FLASH_Program_DoubleWord
    stm32f7xx_hal_flash.o(i.HAL_FLASH_Program_IT) refers to stm32f7xx_hal_flash.o(.bss) for .bss
    stm32f7xx_hal_pwr_ex.o(i.HAL_PWREx_ControlVoltageScaling) refers to stm32f7xx_hal.o(i.HAL_GetTick) for HAL_GetTick
    stm32f7xx_hal_pwr_ex.o(i.HAL_PWREx_DisableBkUpReg) refers to stm32f7xx_hal.o(i.HAL_GetTick) for HAL_GetTick
    stm32f7xx_hal_pwr_ex.o(i.HAL_PWREx_DisableOverDrive) refers to stm32f7xx_hal.o(i.HAL_GetTick) for HAL_GetTick
    stm32f7xx_hal_pwr_ex.o(i.HAL_PWREx_EnableBkUpReg) refers to stm32f7xx_hal.o(i.HAL_GetTick) for HAL_GetTick
    stm32f7xx_hal_pwr_ex.o(i.HAL_PWREx_EnableOverDrive) refers to stm32f7xx_hal.o(i.HAL_GetTick) for HAL_GetTick
    stm32f7xx_hal_pwr_ex.o(i.HAL_PWREx_EnterUnderDriveSTOPMode) refers to stm32f7xx_hal.o(i.HAL_GetTick) for HAL_GetTick
    stm32f7xx_hal_rcc.o(i.HAL_RCC_ClockConfig) refers to stm32f7xx_hal.o(i.HAL_GetTick) for HAL_GetTick
    stm32f7xx_hal_rcc.o(i.HAL_RCC_ClockConfig) refers to stm32f7xx_hal.o(i.HAL_InitTick) for HAL_InitTick
    stm32f7xx_hal_rcc.o(i.HAL_RCC_GetHCLKFreq) refers to stm32f7xx_hal_rcc.o(i.HAL_RCC_GetSysClockFreq) for HAL_RCC_GetSysClockFreq
    stm32f7xx_hal_rcc.o(i.HAL_RCC_GetHCLKFreq) refers to system_stm32f7xx.o(.data) for SystemCoreClock
    stm32f7xx_hal_rcc.o(i.HAL_RCC_GetHCLKFreq) refers to stm32f7xx_hal_rcc.o(.constdata) for .constdata
    stm32f7xx_hal_rcc.o(i.HAL_RCC_GetPCLK1Freq) refers to stm32f7xx_hal_rcc.o(i.HAL_RCC_GetHCLKFreq) for HAL_RCC_GetHCLKFreq
    stm32f7xx_hal_rcc.o(i.HAL_RCC_GetPCLK1Freq) refers to stm32f7xx_hal_rcc.o(.constdata) for .constdata
    stm32f7xx_hal_rcc.o(i.HAL_RCC_GetPCLK2Freq) refers to stm32f7xx_hal_rcc.o(i.HAL_RCC_GetHCLKFreq) for HAL_RCC_GetHCLKFreq
    stm32f7xx_hal_rcc.o(i.HAL_RCC_GetPCLK2Freq) refers to stm32f7xx_hal_rcc.o(.constdata) for .constdata
    stm32f7xx_hal_rcc.o(i.HAL_RCC_MCOConfig) refers to stm32f7xx_hal_gpio.o(i.HAL_GPIO_Init) for HAL_GPIO_Init
    stm32f7xx_hal_rcc.o(i.HAL_RCC_NMI_IRQHandler) refers to stm32f7xx_hal_rcc.o(i.HAL_RCC_CSSCallback) for HAL_RCC_CSSCallback
    stm32f7xx_hal_rcc.o(i.HAL_RCC_OscConfig) refers to stm32f7xx_hal.o(i.HAL_GetTick) for HAL_GetTick
    stm32f7xx_hal_tim_ex.o(i.HAL_TIMEx_ConfigCommutationEvent_DMA) refers to stm32f7xx_hal_tim_ex.o(i.TIMEx_DMACommutationCplt) for TIMEx_DMACommutationCplt
    stm32f7xx_hal_tim_ex.o(i.HAL_TIMEx_ConfigCommutationEvent_DMA) refers to stm32f7xx_hal_tim.o(i.TIM_DMAError) for TIM_DMAError
    stm32f7xx_hal_tim_ex.o(i.HAL_TIMEx_HallSensor_DeInit) refers to stm32f7xx_hal_tim_ex.o(i.HAL_TIMEx_HallSensor_MspDeInit) for HAL_TIMEx_HallSensor_MspDeInit
    stm32f7xx_hal_tim_ex.o(i.HAL_TIMEx_HallSensor_Init) refers to stm32f7xx_hal_tim_ex.o(i.HAL_TIMEx_HallSensor_MspInit) for HAL_TIMEx_HallSensor_MspInit
    stm32f7xx_hal_tim_ex.o(i.HAL_TIMEx_HallSensor_Init) refers to stm32f7xx_hal_tim.o(i.TIM_Base_SetConfig) for TIM_Base_SetConfig
    stm32f7xx_hal_tim_ex.o(i.HAL_TIMEx_HallSensor_Init) refers to stm32f7xx_hal_tim.o(i.TIM_TI1_SetConfig) for TIM_TI1_SetConfig
    stm32f7xx_hal_tim_ex.o(i.HAL_TIMEx_HallSensor_Init) refers to stm32f7xx_hal_tim.o(i.TIM_OC2_SetConfig) for TIM_OC2_SetConfig
    stm32f7xx_hal_tim_ex.o(i.HAL_TIMEx_HallSensor_Start) refers to stm32f7xx_hal_tim.o(i.TIM_CCxChannelCmd) for TIM_CCxChannelCmd
    stm32f7xx_hal_tim_ex.o(i.HAL_TIMEx_HallSensor_Start_DMA) refers to stm32f7xx_hal_tim.o(i.TIM_CCxChannelCmd) for TIM_CCxChannelCmd
    stm32f7xx_hal_tim_ex.o(i.HAL_TIMEx_HallSensor_Start_DMA) refers to stm32f7xx_hal_dma.o(i.HAL_DMA_Start_IT) for HAL_DMA_Start_IT
    stm32f7xx_hal_tim_ex.o(i.HAL_TIMEx_HallSensor_Start_DMA) refers to stm32f7xx_hal_tim.o(i.TIM_DMACaptureCplt) for TIM_DMACaptureCplt
    stm32f7xx_hal_tim_ex.o(i.HAL_TIMEx_HallSensor_Start_DMA) refers to stm32f7xx_hal_tim.o(i.TIM_DMAError) for TIM_DMAError
    stm32f7xx_hal_tim_ex.o(i.HAL_TIMEx_HallSensor_Start_IT) refers to stm32f7xx_hal_tim.o(i.TIM_CCxChannelCmd) for TIM_CCxChannelCmd
    stm32f7xx_hal_tim_ex.o(i.HAL_TIMEx_HallSensor_Stop) refers to stm32f7xx_hal_tim.o(i.TIM_CCxChannelCmd) for TIM_CCxChannelCmd
    stm32f7xx_hal_tim_ex.o(i.HAL_TIMEx_HallSensor_Stop_DMA) refers to stm32f7xx_hal_tim.o(i.TIM_CCxChannelCmd) for TIM_CCxChannelCmd
    stm32f7xx_hal_tim_ex.o(i.HAL_TIMEx_HallSensor_Stop_IT) refers to stm32f7xx_hal_tim.o(i.TIM_CCxChannelCmd) for TIM_CCxChannelCmd
    stm32f7xx_hal_tim_ex.o(i.HAL_TIMEx_OCN_Start) refers to stm32f7xx_hal_tim_ex.o(i.TIM_CCxNChannelCmd) for TIM_CCxNChannelCmd
    stm32f7xx_hal_tim_ex.o(i.HAL_TIMEx_OCN_Start_DMA) refers to stm32f7xx_hal_dma.o(i.HAL_DMA_Start_IT) for HAL_DMA_Start_IT
    stm32f7xx_hal_tim_ex.o(i.HAL_TIMEx_OCN_Start_DMA) refers to stm32f7xx_hal_tim_ex.o(i.TIM_CCxNChannelCmd) for TIM_CCxNChannelCmd
    stm32f7xx_hal_tim_ex.o(i.HAL_TIMEx_OCN_Start_DMA) refers to stm32f7xx_hal_tim.o(i.TIM_DMADelayPulseCplt) for TIM_DMADelayPulseCplt
    stm32f7xx_hal_tim_ex.o(i.HAL_TIMEx_OCN_Start_DMA) refers to stm32f7xx_hal_tim.o(i.TIM_DMAError) for TIM_DMAError
    stm32f7xx_hal_tim_ex.o(i.HAL_TIMEx_OCN_Start_IT) refers to stm32f7xx_hal_tim_ex.o(i.TIM_CCxNChannelCmd) for TIM_CCxNChannelCmd
    stm32f7xx_hal_tim_ex.o(i.HAL_TIMEx_OCN_Stop) refers to stm32f7xx_hal_tim_ex.o(i.TIM_CCxNChannelCmd) for TIM_CCxNChannelCmd
    stm32f7xx_hal_tim_ex.o(i.HAL_TIMEx_OCN_Stop_DMA) refers to stm32f7xx_hal_tim_ex.o(i.TIM_CCxNChannelCmd) for TIM_CCxNChannelCmd
    stm32f7xx_hal_tim_ex.o(i.HAL_TIMEx_OCN_Stop_IT) refers to stm32f7xx_hal_tim_ex.o(i.TIM_CCxNChannelCmd) for TIM_CCxNChannelCmd
    stm32f7xx_hal_tim_ex.o(i.HAL_TIMEx_OnePulseN_Start) refers to stm32f7xx_hal_tim_ex.o(i.TIM_CCxNChannelCmd) for TIM_CCxNChannelCmd
    stm32f7xx_hal_tim_ex.o(i.HAL_TIMEx_OnePulseN_Start_IT) refers to stm32f7xx_hal_tim_ex.o(i.TIM_CCxNChannelCmd) for TIM_CCxNChannelCmd
    stm32f7xx_hal_tim_ex.o(i.HAL_TIMEx_OnePulseN_Stop) refers to stm32f7xx_hal_tim_ex.o(i.TIM_CCxNChannelCmd) for TIM_CCxNChannelCmd
    stm32f7xx_hal_tim_ex.o(i.HAL_TIMEx_OnePulseN_Stop_IT) refers to stm32f7xx_hal_tim_ex.o(i.TIM_CCxNChannelCmd) for TIM_CCxNChannelCmd
    stm32f7xx_hal_tim_ex.o(i.HAL_TIMEx_PWMN_Start) refers to stm32f7xx_hal_tim_ex.o(i.TIM_CCxNChannelCmd) for TIM_CCxNChannelCmd
    stm32f7xx_hal_tim_ex.o(i.HAL_TIMEx_PWMN_Start_DMA) refers to stm32f7xx_hal_dma.o(i.HAL_DMA_Start_IT) for HAL_DMA_Start_IT
    stm32f7xx_hal_tim_ex.o(i.HAL_TIMEx_PWMN_Start_DMA) refers to stm32f7xx_hal_tim_ex.o(i.TIM_CCxNChannelCmd) for TIM_CCxNChannelCmd
    stm32f7xx_hal_tim_ex.o(i.HAL_TIMEx_PWMN_Start_DMA) refers to stm32f7xx_hal_tim.o(i.TIM_DMADelayPulseCplt) for TIM_DMADelayPulseCplt
    stm32f7xx_hal_tim_ex.o(i.HAL_TIMEx_PWMN_Start_DMA) refers to stm32f7xx_hal_tim.o(i.TIM_DMAError) for TIM_DMAError
    stm32f7xx_hal_tim_ex.o(i.HAL_TIMEx_PWMN_Start_IT) refers to stm32f7xx_hal_tim_ex.o(i.TIM_CCxNChannelCmd) for TIM_CCxNChannelCmd
    stm32f7xx_hal_tim_ex.o(i.HAL_TIMEx_PWMN_Stop) refers to stm32f7xx_hal_tim_ex.o(i.TIM_CCxNChannelCmd) for TIM_CCxNChannelCmd
    stm32f7xx_hal_tim_ex.o(i.HAL_TIMEx_PWMN_Stop_DMA) refers to stm32f7xx_hal_tim_ex.o(i.TIM_CCxNChannelCmd) for TIM_CCxNChannelCmd
    stm32f7xx_hal_tim_ex.o(i.HAL_TIMEx_PWMN_Stop_IT) refers to stm32f7xx_hal_tim_ex.o(i.TIM_CCxNChannelCmd) for TIM_CCxNChannelCmd
    stm32f7xx_hal_tim_ex.o(i.HAL_TIM_ConfigOCrefClear) refers to stm32f7xx_hal_tim.o(i.TIM_ETR_SetConfig) for TIM_ETR_SetConfig
    stm32f7xx_hal_tim_ex.o(i.HAL_TIM_OC_ConfigChannel) refers to stm32f7xx_hal_tim.o(i.TIM_OC1_SetConfig) for TIM_OC1_SetConfig
    stm32f7xx_hal_tim_ex.o(i.HAL_TIM_OC_ConfigChannel) refers to stm32f7xx_hal_tim.o(i.TIM_OC2_SetConfig) for TIM_OC2_SetConfig
    stm32f7xx_hal_tim_ex.o(i.HAL_TIM_OC_ConfigChannel) refers to stm32f7xx_hal_tim.o(i.TIM_OC3_SetConfig) for TIM_OC3_SetConfig
    stm32f7xx_hal_tim_ex.o(i.HAL_TIM_OC_ConfigChannel) refers to stm32f7xx_hal_tim.o(i.TIM_OC4_SetConfig) for TIM_OC4_SetConfig
    stm32f7xx_hal_tim_ex.o(i.HAL_TIM_OC_ConfigChannel) refers to stm32f7xx_hal_tim_ex.o(i.TIM_OC5_SetConfig) for TIM_OC5_SetConfig
    stm32f7xx_hal_tim_ex.o(i.HAL_TIM_OC_ConfigChannel) refers to stm32f7xx_hal_tim_ex.o(i.TIM_OC6_SetConfig) for TIM_OC6_SetConfig
    stm32f7xx_hal_tim_ex.o(i.HAL_TIM_PWM_ConfigChannel) refers to stm32f7xx_hal_tim.o(i.TIM_OC1_SetConfig) for TIM_OC1_SetConfig
    stm32f7xx_hal_tim_ex.o(i.HAL_TIM_PWM_ConfigChannel) refers to stm32f7xx_hal_tim.o(i.TIM_OC2_SetConfig) for TIM_OC2_SetConfig
    stm32f7xx_hal_tim_ex.o(i.HAL_TIM_PWM_ConfigChannel) refers to stm32f7xx_hal_tim.o(i.TIM_OC3_SetConfig) for TIM_OC3_SetConfig
    stm32f7xx_hal_tim_ex.o(i.HAL_TIM_PWM_ConfigChannel) refers to stm32f7xx_hal_tim.o(i.TIM_OC4_SetConfig) for TIM_OC4_SetConfig
    stm32f7xx_hal_tim_ex.o(i.HAL_TIM_PWM_ConfigChannel) refers to stm32f7xx_hal_tim_ex.o(i.TIM_OC5_SetConfig) for TIM_OC5_SetConfig
    stm32f7xx_hal_tim_ex.o(i.HAL_TIM_PWM_ConfigChannel) refers to stm32f7xx_hal_tim_ex.o(i.TIM_OC6_SetConfig) for TIM_OC6_SetConfig
    stm32f7xx_hal_tim_ex.o(i.TIMEx_DMACommutationCplt) refers to stm32f7xx_hal_tim_ex.o(i.HAL_TIMEx_CommutationCallback) for HAL_TIMEx_CommutationCallback
    stm32f7xx_hal_sai_ex.o(i.SAI_GetInputClock) refers to stm32f7xx_hal_rcc_ex.o(i.HAL_RCCEx_GetPeriphCLKFreq) for HAL_RCCEx_GetPeriphCLKFreq
    stm32f7xx_hal_pcd.o(i.HAL_PCD_DeInit) refers to stm32f7xx_hal_pcd.o(i.HAL_PCD_Stop) for HAL_PCD_Stop
    stm32f7xx_hal_pcd.o(i.HAL_PCD_DeInit) refers to usbd_conf.o(i.HAL_PCD_MspDeInit) for HAL_PCD_MspDeInit
    stm32f7xx_hal_pcd.o(i.HAL_PCD_DevConnect) refers to stm32f7xx_ll_usb.o(i.USB_DevConnect) for USB_DevConnect
    stm32f7xx_hal_pcd.o(i.HAL_PCD_DevDisconnect) refers to stm32f7xx_ll_usb.o(i.USB_DevDisconnect) for USB_DevDisconnect
    stm32f7xx_hal_pcd.o(i.HAL_PCD_EP_Close) refers to stm32f7xx_ll_usb.o(i.USB_DeactivateEndpoint) for USB_DeactivateEndpoint
    stm32f7xx_hal_pcd.o(i.HAL_PCD_EP_ClrStall) refers to stm32f7xx_ll_usb.o(i.USB_EPClearStall) for USB_EPClearStall
    stm32f7xx_hal_pcd.o(i.HAL_PCD_EP_Flush) refers to stm32f7xx_ll_usb.o(i.USB_FlushTxFifo) for USB_FlushTxFifo
    stm32f7xx_hal_pcd.o(i.HAL_PCD_EP_Flush) refers to stm32f7xx_ll_usb.o(i.USB_FlushRxFifo) for USB_FlushRxFifo
    stm32f7xx_hal_pcd.o(i.HAL_PCD_EP_Open) refers to stm32f7xx_ll_usb.o(i.USB_ActivateEndpoint) for USB_ActivateEndpoint
    stm32f7xx_hal_pcd.o(i.HAL_PCD_EP_Receive) refers to stm32f7xx_ll_usb.o(i.USB_EPStartXfer) for USB_EPStartXfer
    stm32f7xx_hal_pcd.o(i.HAL_PCD_EP_Receive) refers to stm32f7xx_ll_usb.o(i.USB_EP0StartXfer) for USB_EP0StartXfer
    stm32f7xx_hal_pcd.o(i.HAL_PCD_EP_SetStall) refers to stm32f7xx_ll_usb.o(i.USB_EPSetStall) for USB_EPSetStall
    stm32f7xx_hal_pcd.o(i.HAL_PCD_EP_SetStall) refers to stm32f7xx_ll_usb.o(i.USB_EP0_OutStart) for USB_EP0_OutStart
    stm32f7xx_hal_pcd.o(i.HAL_PCD_EP_Transmit) refers to stm32f7xx_ll_usb.o(i.USB_EPStartXfer) for USB_EPStartXfer
    stm32f7xx_hal_pcd.o(i.HAL_PCD_EP_Transmit) refers to stm32f7xx_ll_usb.o(i.USB_EP0StartXfer) for USB_EP0StartXfer
    stm32f7xx_hal_pcd.o(i.HAL_PCD_IRQHandler) refers to stm32f7xx_ll_usb.o(i.USB_GetMode) for USB_GetMode
    stm32f7xx_hal_pcd.o(i.HAL_PCD_IRQHandler) refers to stm32f7xx_ll_usb.o(i.USB_ReadInterrupts) for USB_ReadInterrupts
    stm32f7xx_hal_pcd.o(i.HAL_PCD_IRQHandler) refers to stm32f7xx_ll_usb.o(i.USB_ReadDevAllOutEpInterrupt) for USB_ReadDevAllOutEpInterrupt
    stm32f7xx_hal_pcd.o(i.HAL_PCD_IRQHandler) refers to stm32f7xx_ll_usb.o(i.USB_ReadDevOutEPInterrupt) for USB_ReadDevOutEPInterrupt
    stm32f7xx_hal_pcd.o(i.HAL_PCD_IRQHandler) refers to usbd_conf.o(i.HAL_PCD_DataOutStageCallback) for HAL_PCD_DataOutStageCallback
    stm32f7xx_hal_pcd.o(i.HAL_PCD_IRQHandler) refers to stm32f7xx_ll_usb.o(i.USB_EP0_OutStart) for USB_EP0_OutStart
    stm32f7xx_hal_pcd.o(i.HAL_PCD_IRQHandler) refers to usbd_conf.o(i.HAL_PCD_SetupStageCallback) for HAL_PCD_SetupStageCallback
    stm32f7xx_hal_pcd.o(i.HAL_PCD_IRQHandler) refers to stm32f7xx_ll_usb.o(i.USB_ReadDevAllInEpInterrupt) for USB_ReadDevAllInEpInterrupt
    stm32f7xx_hal_pcd.o(i.HAL_PCD_IRQHandler) refers to stm32f7xx_ll_usb.o(i.USB_ReadDevInEPInterrupt) for USB_ReadDevInEPInterrupt
    stm32f7xx_hal_pcd.o(i.HAL_PCD_IRQHandler) refers to usbd_conf.o(i.HAL_PCD_DataInStageCallback) for HAL_PCD_DataInStageCallback
    stm32f7xx_hal_pcd.o(i.HAL_PCD_IRQHandler) refers to stm32f7xx_hal_pcd.o(i.PCD_WriteEmptyTxFifo) for PCD_WriteEmptyTxFifo
    stm32f7xx_hal_pcd.o(i.HAL_PCD_IRQHandler) refers to usbd_conf.o(i.HAL_PCD_ResumeCallback) for HAL_PCD_ResumeCallback
    stm32f7xx_hal_pcd.o(i.HAL_PCD_IRQHandler) refers to usbd_conf.o(i.HAL_PCD_SuspendCallback) for HAL_PCD_SuspendCallback
    stm32f7xx_hal_pcd.o(i.HAL_PCD_IRQHandler) refers to stm32f7xx_ll_usb.o(i.USB_FlushTxFifo) for USB_FlushTxFifo
    stm32f7xx_hal_pcd.o(i.HAL_PCD_IRQHandler) refers to stm32f7xx_hal_pcd_ex.o(i.HAL_PCDEx_LPM_Callback) for HAL_PCDEx_LPM_Callback
    stm32f7xx_hal_pcd.o(i.HAL_PCD_IRQHandler) refers to stm32f7xx_ll_usb.o(i.USB_ActivateSetup) for USB_ActivateSetup
    stm32f7xx_hal_pcd.o(i.HAL_PCD_IRQHandler) refers to stm32f7xx_ll_usb.o(i.USB_GetDevSpeed) for USB_GetDevSpeed
    stm32f7xx_hal_pcd.o(i.HAL_PCD_IRQHandler) refers to usbd_conf.o(i.HAL_PCD_ResetCallback) for HAL_PCD_ResetCallback
    stm32f7xx_hal_pcd.o(i.HAL_PCD_IRQHandler) refers to stm32f7xx_ll_usb.o(i.USB_ReadPacket) for USB_ReadPacket
    stm32f7xx_hal_pcd.o(i.HAL_PCD_IRQHandler) refers to usbd_conf.o(i.HAL_PCD_SOFCallback) for HAL_PCD_SOFCallback
    stm32f7xx_hal_pcd.o(i.HAL_PCD_IRQHandler) refers to usbd_conf.o(i.HAL_PCD_ISOINIncompleteCallback) for HAL_PCD_ISOINIncompleteCallback
    stm32f7xx_hal_pcd.o(i.HAL_PCD_IRQHandler) refers to usbd_conf.o(i.HAL_PCD_ISOOUTIncompleteCallback) for HAL_PCD_ISOOUTIncompleteCallback
    stm32f7xx_hal_pcd.o(i.HAL_PCD_IRQHandler) refers to usbd_conf.o(i.HAL_PCD_ConnectCallback) for HAL_PCD_ConnectCallback
    stm32f7xx_hal_pcd.o(i.HAL_PCD_IRQHandler) refers to usbd_conf.o(i.HAL_PCD_DisconnectCallback) for HAL_PCD_DisconnectCallback
    stm32f7xx_hal_pcd.o(i.HAL_PCD_Init) refers to usbd_conf.o(i.HAL_PCD_MspInit) for HAL_PCD_MspInit
    stm32f7xx_hal_pcd.o(i.HAL_PCD_Init) refers to stm32f7xx_ll_usb.o(i.USB_DisableGlobalInt) for USB_DisableGlobalInt
    stm32f7xx_hal_pcd.o(i.HAL_PCD_Init) refers to memcpya.o(.text) for __aeabi_memcpy4
    stm32f7xx_hal_pcd.o(i.HAL_PCD_Init) refers to stm32f7xx_ll_usb.o(i.USB_CoreInit) for USB_CoreInit
    stm32f7xx_hal_pcd.o(i.HAL_PCD_Init) refers to stm32f7xx_ll_usb.o(i.USB_SetCurrentMode) for USB_SetCurrentMode
    stm32f7xx_hal_pcd.o(i.HAL_PCD_Init) refers to stm32f7xx_ll_usb.o(i.USB_DevInit) for USB_DevInit
    stm32f7xx_hal_pcd.o(i.HAL_PCD_Init) refers to stm32f7xx_hal_pcd_ex.o(i.HAL_PCDEx_ActivateLPM) for HAL_PCDEx_ActivateLPM
    stm32f7xx_hal_pcd.o(i.HAL_PCD_Init) refers to stm32f7xx_ll_usb.o(i.USB_DevDisconnect) for USB_DevDisconnect
    stm32f7xx_hal_pcd.o(i.HAL_PCD_SetAddress) refers to stm32f7xx_ll_usb.o(i.USB_SetDevAddress) for USB_SetDevAddress
    stm32f7xx_hal_pcd.o(i.HAL_PCD_Start) refers to stm32f7xx_ll_usb.o(i.USB_DevConnect) for USB_DevConnect
    stm32f7xx_hal_pcd.o(i.HAL_PCD_Start) refers to stm32f7xx_ll_usb.o(i.USB_EnableGlobalInt) for USB_EnableGlobalInt
    stm32f7xx_hal_pcd.o(i.HAL_PCD_Stop) refers to stm32f7xx_ll_usb.o(i.USB_DisableGlobalInt) for USB_DisableGlobalInt
    stm32f7xx_hal_pcd.o(i.HAL_PCD_Stop) refers to stm32f7xx_ll_usb.o(i.USB_StopDevice) for USB_StopDevice
    stm32f7xx_hal_pcd.o(i.HAL_PCD_Stop) refers to stm32f7xx_ll_usb.o(i.USB_DevDisconnect) for USB_DevDisconnect
    stm32f7xx_hal_pcd.o(i.PCD_WriteEmptyTxFifo) refers to stm32f7xx_ll_usb.o(i.USB_WritePacket) for USB_WritePacket
    stm32f7xx_hal_pwr.o(i.HAL_PWR_PVD_IRQHandler) refers to stm32f7xx_hal_pwr.o(i.HAL_PWR_PVDCallback) for HAL_PWR_PVDCallback
    stm32f7xx_hal_sai.o(i.HAL_SAI_Abort) refers to stm32f7xx_hal_dma.o(i.HAL_DMA_Abort) for HAL_DMA_Abort
    stm32f7xx_hal_sai.o(i.HAL_SAI_Abort) refers to stm32f7xx_hal_sai.o(i.SAI_Disable) for SAI_Disable
    stm32f7xx_hal_sai.o(i.HAL_SAI_DMAStop) refers to stm32f7xx_hal_dma.o(i.HAL_DMA_Abort) for HAL_DMA_Abort
    stm32f7xx_hal_sai.o(i.HAL_SAI_DMAStop) refers to stm32f7xx_hal_sai.o(i.SAI_Disable) for SAI_Disable
    stm32f7xx_hal_sai.o(i.HAL_SAI_DeInit) refers to stm32f7xx_hal_sai.o(i.SAI_Disable) for SAI_Disable
    stm32f7xx_hal_sai.o(i.HAL_SAI_DeInit) refers to stm32f7xx_hal_sai.o(i.HAL_SAI_MspDeInit) for HAL_SAI_MspDeInit
    stm32f7xx_hal_sai.o(i.HAL_SAI_IRQHandler) refers to stm32746g_discovery_audio.o(i.HAL_SAI_ErrorCallback) for HAL_SAI_ErrorCallback
    stm32f7xx_hal_sai.o(i.HAL_SAI_IRQHandler) refers to stm32f7xx_hal_sai.o(i.HAL_SAI_Abort) for HAL_SAI_Abort
    stm32f7xx_hal_sai.o(i.HAL_SAI_Init) refers to stm32f7xx_hal_sai.o(i.HAL_SAI_MspInit) for HAL_SAI_MspInit
    stm32f7xx_hal_sai.o(i.HAL_SAI_Init) refers to stm32f7xx_hal_sai.o(i.SAI_Disable) for SAI_Disable
    stm32f7xx_hal_sai.o(i.HAL_SAI_Init) refers to stm32f7xx_hal_sai_ex.o(i.SAI_BlockSynchroConfig) for SAI_BlockSynchroConfig
    stm32f7xx_hal_sai.o(i.HAL_SAI_Init) refers to stm32f7xx_hal_sai_ex.o(i.SAI_GetInputClock) for SAI_GetInputClock
    stm32f7xx_hal_sai.o(i.HAL_SAI_InitProtocol) refers to stm32f7xx_hal_sai.o(i.SAI_InitI2S) for SAI_InitI2S
    stm32f7xx_hal_sai.o(i.HAL_SAI_InitProtocol) refers to stm32f7xx_hal_sai.o(i.SAI_InitPCM) for SAI_InitPCM
    stm32f7xx_hal_sai.o(i.HAL_SAI_InitProtocol) refers to stm32f7xx_hal_sai.o(i.HAL_SAI_Init) for HAL_SAI_Init
    stm32f7xx_hal_sai.o(i.HAL_SAI_Receive) refers to stm32f7xx_hal.o(i.HAL_GetTick) for HAL_GetTick
    stm32f7xx_hal_sai.o(i.HAL_SAI_Receive_DMA) refers to stm32f7xx_hal_dma.o(i.HAL_DMA_Start_IT) for HAL_DMA_Start_IT
    stm32f7xx_hal_sai.o(i.HAL_SAI_Receive_DMA) refers to stm32f7xx_hal_sai.o(i.SAI_InterruptFlag) for SAI_InterruptFlag
    stm32f7xx_hal_sai.o(i.HAL_SAI_Receive_DMA) refers to stm32f7xx_hal_sai.o(i.SAI_DMARxHalfCplt) for SAI_DMARxHalfCplt
    stm32f7xx_hal_sai.o(i.HAL_SAI_Receive_DMA) refers to stm32f7xx_hal_sai.o(i.SAI_DMARxCplt) for SAI_DMARxCplt
    stm32f7xx_hal_sai.o(i.HAL_SAI_Receive_DMA) refers to stm32f7xx_hal_sai.o(i.SAI_DMAError) for SAI_DMAError
    stm32f7xx_hal_sai.o(i.HAL_SAI_Receive_IT) refers to stm32f7xx_hal_sai.o(i.SAI_InterruptFlag) for SAI_InterruptFlag
    stm32f7xx_hal_sai.o(i.HAL_SAI_Receive_IT) refers to stm32f7xx_hal_sai.o(i.SAI_Receive_IT16Bit) for SAI_Receive_IT16Bit
    stm32f7xx_hal_sai.o(i.HAL_SAI_Receive_IT) refers to stm32f7xx_hal_sai.o(i.SAI_Receive_IT8Bit) for SAI_Receive_IT8Bit
    stm32f7xx_hal_sai.o(i.HAL_SAI_Receive_IT) refers to stm32f7xx_hal_sai.o(i.SAI_Receive_IT32Bit) for SAI_Receive_IT32Bit
    stm32f7xx_hal_sai.o(i.HAL_SAI_Transmit) refers to stm32f7xx_hal.o(i.HAL_GetTick) for HAL_GetTick
    stm32f7xx_hal_sai.o(i.HAL_SAI_Transmit) refers to stm32f7xx_hal_sai.o(i.SAI_FillFifo) for SAI_FillFifo
    stm32f7xx_hal_sai.o(i.HAL_SAI_Transmit_DMA) refers to stm32f7xx_hal_dma.o(i.HAL_DMA_Start_IT) for HAL_DMA_Start_IT
    stm32f7xx_hal_sai.o(i.HAL_SAI_Transmit_DMA) refers to stm32f7xx_hal_sai.o(i.SAI_InterruptFlag) for SAI_InterruptFlag
    stm32f7xx_hal_sai.o(i.HAL_SAI_Transmit_DMA) refers to stm32f7xx_hal_sai.o(i.SAI_DMATxHalfCplt) for SAI_DMATxHalfCplt
    stm32f7xx_hal_sai.o(i.HAL_SAI_Transmit_DMA) refers to stm32f7xx_hal_sai.o(i.SAI_DMATxCplt) for SAI_DMATxCplt
    stm32f7xx_hal_sai.o(i.HAL_SAI_Transmit_DMA) refers to stm32f7xx_hal_sai.o(i.SAI_DMAError) for SAI_DMAError
    stm32f7xx_hal_sai.o(i.HAL_SAI_Transmit_IT) refers to stm32f7xx_hal_sai.o(i.SAI_FillFifo) for SAI_FillFifo
    stm32f7xx_hal_sai.o(i.HAL_SAI_Transmit_IT) refers to stm32f7xx_hal_sai.o(i.SAI_InterruptFlag) for SAI_InterruptFlag
    stm32f7xx_hal_sai.o(i.HAL_SAI_Transmit_IT) refers to stm32f7xx_hal_sai.o(i.SAI_Transmit_IT16Bit) for SAI_Transmit_IT16Bit
    stm32f7xx_hal_sai.o(i.HAL_SAI_Transmit_IT) refers to stm32f7xx_hal_sai.o(i.SAI_Transmit_IT8Bit) for SAI_Transmit_IT8Bit
    stm32f7xx_hal_sai.o(i.HAL_SAI_Transmit_IT) refers to stm32f7xx_hal_sai.o(i.SAI_Transmit_IT32Bit) for SAI_Transmit_IT32Bit
    stm32f7xx_hal_sai.o(i.SAI_DMAError) refers to stm32f7xx_hal_sai.o(i.HAL_SAI_DMAStop) for HAL_SAI_DMAStop
    stm32f7xx_hal_sai.o(i.SAI_DMAError) refers to stm32746g_discovery_audio.o(i.HAL_SAI_ErrorCallback) for HAL_SAI_ErrorCallback
    stm32f7xx_hal_sai.o(i.SAI_DMARxCplt) refers to stm32f7xx_hal_sai.o(i.SAI_InterruptFlag) for SAI_InterruptFlag
    stm32f7xx_hal_sai.o(i.SAI_DMARxCplt) refers to stm32746g_discovery_audio.o(i.HAL_SAI_RxCpltCallback) for HAL_SAI_RxCpltCallback
    stm32f7xx_hal_sai.o(i.SAI_DMARxHalfCplt) refers to stm32746g_discovery_audio.o(i.HAL_SAI_RxHalfCpltCallback) for HAL_SAI_RxHalfCpltCallback
    stm32f7xx_hal_sai.o(i.SAI_DMATxCplt) refers to stm32f7xx_hal_sai.o(i.SAI_InterruptFlag) for SAI_InterruptFlag
    stm32f7xx_hal_sai.o(i.SAI_DMATxCplt) refers to stm32746g_discovery_audio.o(i.HAL_SAI_TxCpltCallback) for HAL_SAI_TxCpltCallback
    stm32f7xx_hal_sai.o(i.SAI_DMATxHalfCplt) refers to stm32746g_discovery_audio.o(i.HAL_SAI_TxHalfCpltCallback) for HAL_SAI_TxHalfCpltCallback
    stm32f7xx_hal_sai.o(i.SAI_Disable) refers to stm32f7xx_hal.o(i.HAL_GetTick) for HAL_GetTick
    stm32f7xx_hal_sai.o(i.SAI_Receive_IT16Bit) refers to stm32f7xx_hal_sai.o(i.SAI_InterruptFlag) for SAI_InterruptFlag
    stm32f7xx_hal_sai.o(i.SAI_Receive_IT16Bit) refers to stm32746g_discovery_audio.o(i.HAL_SAI_RxCpltCallback) for HAL_SAI_RxCpltCallback
    stm32f7xx_hal_sai.o(i.SAI_Receive_IT32Bit) refers to stm32f7xx_hal_sai.o(i.SAI_InterruptFlag) for SAI_InterruptFlag
    stm32f7xx_hal_sai.o(i.SAI_Receive_IT32Bit) refers to stm32746g_discovery_audio.o(i.HAL_SAI_RxCpltCallback) for HAL_SAI_RxCpltCallback
    stm32f7xx_hal_sai.o(i.SAI_Receive_IT8Bit) refers to stm32f7xx_hal_sai.o(i.SAI_InterruptFlag) for SAI_InterruptFlag
    stm32f7xx_hal_sai.o(i.SAI_Receive_IT8Bit) refers to stm32746g_discovery_audio.o(i.HAL_SAI_RxCpltCallback) for HAL_SAI_RxCpltCallback
    stm32f7xx_hal_sai.o(i.SAI_Transmit_IT16Bit) refers to stm32f7xx_hal_sai.o(i.SAI_InterruptFlag) for SAI_InterruptFlag
    stm32f7xx_hal_sai.o(i.SAI_Transmit_IT16Bit) refers to stm32746g_discovery_audio.o(i.HAL_SAI_TxCpltCallback) for HAL_SAI_TxCpltCallback
    stm32f7xx_hal_sai.o(i.SAI_Transmit_IT32Bit) refers to stm32f7xx_hal_sai.o(i.SAI_InterruptFlag) for SAI_InterruptFlag
    stm32f7xx_hal_sai.o(i.SAI_Transmit_IT32Bit) refers to stm32746g_discovery_audio.o(i.HAL_SAI_TxCpltCallback) for HAL_SAI_TxCpltCallback
    stm32f7xx_hal_sai.o(i.SAI_Transmit_IT8Bit) refers to stm32f7xx_hal_sai.o(i.SAI_InterruptFlag) for SAI_InterruptFlag
    stm32f7xx_hal_sai.o(i.SAI_Transmit_IT8Bit) refers to stm32746g_discovery_audio.o(i.HAL_SAI_TxCpltCallback) for HAL_SAI_TxCpltCallback
    stm32f7xx_hal_i2c.o(i.HAL_I2C_DeInit) refers to stm32f7xx_hal_i2c.o(i.HAL_I2C_MspDeInit) for HAL_I2C_MspDeInit
    stm32f7xx_hal_i2c.o(i.HAL_I2C_ER_IRQHandler) refers to stm32f7xx_hal_i2c.o(i.HAL_I2C_ErrorCallback) for HAL_I2C_ErrorCallback
    stm32f7xx_hal_i2c.o(i.HAL_I2C_EV_IRQHandler) refers to stm32f7xx_hal_i2c.o(i.I2C_SlaveTransmit_ISR) for I2C_SlaveTransmit_ISR
    stm32f7xx_hal_i2c.o(i.HAL_I2C_EV_IRQHandler) refers to stm32f7xx_hal_i2c.o(i.I2C_MasterTransmit_ISR) for I2C_MasterTransmit_ISR
    stm32f7xx_hal_i2c.o(i.HAL_I2C_EV_IRQHandler) refers to stm32f7xx_hal_i2c.o(i.I2C_SlaveReceive_ISR) for I2C_SlaveReceive_ISR
    stm32f7xx_hal_i2c.o(i.HAL_I2C_EV_IRQHandler) refers to stm32f7xx_hal_i2c.o(i.I2C_MasterReceive_ISR) for I2C_MasterReceive_ISR
    stm32f7xx_hal_i2c.o(i.HAL_I2C_Init) refers to stm32f7xx_hal_i2c.o(i.HAL_I2C_MspInit) for HAL_I2C_MspInit
    stm32f7xx_hal_i2c.o(i.HAL_I2C_IsDeviceReady) refers to stm32f7xx_hal.o(i.HAL_GetTick) for HAL_GetTick
    stm32f7xx_hal_i2c.o(i.HAL_I2C_IsDeviceReady) refers to stm32f7xx_hal_i2c.o(i.I2C_WaitOnFlagUntilTimeout) for I2C_WaitOnFlagUntilTimeout
    stm32f7xx_hal_i2c.o(i.HAL_I2C_Master_Receive) refers to stm32f7xx_hal_i2c.o(i.I2C_TransferConfig) for I2C_TransferConfig
    stm32f7xx_hal_i2c.o(i.HAL_I2C_Master_Receive) refers to stm32f7xx_hal_i2c.o(i.I2C_WaitOnRXNEFlagUntilTimeout) for I2C_WaitOnRXNEFlagUntilTimeout
    stm32f7xx_hal_i2c.o(i.HAL_I2C_Master_Receive) refers to stm32f7xx_hal_i2c.o(i.I2C_WaitOnSTOPFlagUntilTimeout) for I2C_WaitOnSTOPFlagUntilTimeout
    stm32f7xx_hal_i2c.o(i.HAL_I2C_Master_Receive) refers to stm32f7xx_hal_i2c.o(i.I2C_WaitOnFlagUntilTimeout) for I2C_WaitOnFlagUntilTimeout
    stm32f7xx_hal_i2c.o(i.HAL_I2C_Master_Receive_DMA) refers to stm32f7xx_hal_dma.o(i.HAL_DMA_Start_IT) for HAL_DMA_Start_IT
    stm32f7xx_hal_i2c.o(i.HAL_I2C_Master_Receive_DMA) refers to stm32f7xx_hal_i2c.o(i.I2C_TransferConfig) for I2C_TransferConfig
    stm32f7xx_hal_i2c.o(i.HAL_I2C_Master_Receive_DMA) refers to stm32f7xx_hal_i2c.o(i.I2C_WaitOnRXNEFlagUntilTimeout) for I2C_WaitOnRXNEFlagUntilTimeout
    stm32f7xx_hal_i2c.o(i.HAL_I2C_Master_Receive_DMA) refers to stm32f7xx_hal_dma.o(i.HAL_DMA_Abort) for HAL_DMA_Abort
    stm32f7xx_hal_i2c.o(i.HAL_I2C_Master_Receive_DMA) refers to stm32f7xx_hal_i2c.o(i.I2C_DMAMasterReceiveCplt) for I2C_DMAMasterReceiveCplt
    stm32f7xx_hal_i2c.o(i.HAL_I2C_Master_Receive_DMA) refers to stm32f7xx_hal_i2c.o(i.I2C_DMAError) for I2C_DMAError
    stm32f7xx_hal_i2c.o(i.HAL_I2C_Master_Receive_IT) refers to stm32f7xx_hal_i2c.o(i.I2C_TransferConfig) for I2C_TransferConfig
    stm32f7xx_hal_i2c.o(i.HAL_I2C_Master_Transmit) refers to stm32f7xx_hal_i2c.o(i.I2C_TransferConfig) for I2C_TransferConfig
    stm32f7xx_hal_i2c.o(i.HAL_I2C_Master_Transmit) refers to stm32f7xx_hal_i2c.o(i.I2C_WaitOnTXISFlagUntilTimeout) for I2C_WaitOnTXISFlagUntilTimeout
    stm32f7xx_hal_i2c.o(i.HAL_I2C_Master_Transmit) refers to stm32f7xx_hal_i2c.o(i.I2C_WaitOnSTOPFlagUntilTimeout) for I2C_WaitOnSTOPFlagUntilTimeout
    stm32f7xx_hal_i2c.o(i.HAL_I2C_Master_Transmit) refers to stm32f7xx_hal_i2c.o(i.I2C_WaitOnFlagUntilTimeout) for I2C_WaitOnFlagUntilTimeout
    stm32f7xx_hal_i2c.o(i.HAL_I2C_Master_Transmit_DMA) refers to stm32f7xx_hal_dma.o(i.HAL_DMA_Start_IT) for HAL_DMA_Start_IT
    stm32f7xx_hal_i2c.o(i.HAL_I2C_Master_Transmit_DMA) refers to stm32f7xx_hal_i2c.o(i.I2C_TransferConfig) for I2C_TransferConfig
    stm32f7xx_hal_i2c.o(i.HAL_I2C_Master_Transmit_DMA) refers to stm32f7xx_hal_i2c.o(i.I2C_WaitOnTXISFlagUntilTimeout) for I2C_WaitOnTXISFlagUntilTimeout
    stm32f7xx_hal_i2c.o(i.HAL_I2C_Master_Transmit_DMA) refers to stm32f7xx_hal_dma.o(i.HAL_DMA_Abort) for HAL_DMA_Abort
    stm32f7xx_hal_i2c.o(i.HAL_I2C_Master_Transmit_DMA) refers to stm32f7xx_hal_i2c.o(i.I2C_DMAMasterTransmitCplt) for I2C_DMAMasterTransmitCplt
    stm32f7xx_hal_i2c.o(i.HAL_I2C_Master_Transmit_DMA) refers to stm32f7xx_hal_i2c.o(i.I2C_DMAError) for I2C_DMAError
    stm32f7xx_hal_i2c.o(i.HAL_I2C_Master_Transmit_IT) refers to stm32f7xx_hal_i2c.o(i.I2C_TransferConfig) for I2C_TransferConfig
    stm32f7xx_hal_i2c.o(i.HAL_I2C_Mem_Read) refers to stm32f7xx_hal_i2c.o(i.I2C_RequestMemoryRead) for I2C_RequestMemoryRead
    stm32f7xx_hal_i2c.o(i.HAL_I2C_Mem_Read) refers to stm32f7xx_hal_i2c.o(i.I2C_TransferConfig) for I2C_TransferConfig
    stm32f7xx_hal_i2c.o(i.HAL_I2C_Mem_Read) refers to stm32f7xx_hal_i2c.o(i.I2C_WaitOnFlagUntilTimeout) for I2C_WaitOnFlagUntilTimeout
    stm32f7xx_hal_i2c.o(i.HAL_I2C_Mem_Read) refers to stm32f7xx_hal_i2c.o(i.I2C_WaitOnSTOPFlagUntilTimeout) for I2C_WaitOnSTOPFlagUntilTimeout
    stm32f7xx_hal_i2c.o(i.HAL_I2C_Mem_Read_DMA) refers to stm32f7xx_hal_dma.o(i.HAL_DMA_Start_IT) for HAL_DMA_Start_IT
    stm32f7xx_hal_i2c.o(i.HAL_I2C_Mem_Read_DMA) refers to stm32f7xx_hal_i2c.o(i.I2C_RequestMemoryRead) for I2C_RequestMemoryRead
    stm32f7xx_hal_i2c.o(i.HAL_I2C_Mem_Read_DMA) refers to stm32f7xx_hal_i2c.o(i.I2C_TransferConfig) for I2C_TransferConfig
    stm32f7xx_hal_i2c.o(i.HAL_I2C_Mem_Read_DMA) refers to stm32f7xx_hal_i2c.o(i.I2C_WaitOnFlagUntilTimeout) for I2C_WaitOnFlagUntilTimeout
    stm32f7xx_hal_i2c.o(i.HAL_I2C_Mem_Read_DMA) refers to stm32f7xx_hal_i2c.o(i.I2C_DMAMemReceiveCplt) for I2C_DMAMemReceiveCplt
    stm32f7xx_hal_i2c.o(i.HAL_I2C_Mem_Read_DMA) refers to stm32f7xx_hal_i2c.o(i.I2C_DMAError) for I2C_DMAError
    stm32f7xx_hal_i2c.o(i.HAL_I2C_Mem_Read_IT) refers to stm32f7xx_hal_i2c.o(i.I2C_RequestMemoryRead) for I2C_RequestMemoryRead
    stm32f7xx_hal_i2c.o(i.HAL_I2C_Mem_Read_IT) refers to stm32f7xx_hal_i2c.o(i.I2C_TransferConfig) for I2C_TransferConfig
    stm32f7xx_hal_i2c.o(i.HAL_I2C_Mem_Write) refers to stm32f7xx_hal_i2c.o(i.I2C_RequestMemoryWrite) for I2C_RequestMemoryWrite
    stm32f7xx_hal_i2c.o(i.HAL_I2C_Mem_Write) refers to stm32f7xx_hal_i2c.o(i.I2C_TransferConfig) for I2C_TransferConfig
    stm32f7xx_hal_i2c.o(i.HAL_I2C_Mem_Write) refers to stm32f7xx_hal_i2c.o(i.I2C_WaitOnTXISFlagUntilTimeout) for I2C_WaitOnTXISFlagUntilTimeout
    stm32f7xx_hal_i2c.o(i.HAL_I2C_Mem_Write) refers to stm32f7xx_hal_i2c.o(i.I2C_WaitOnSTOPFlagUntilTimeout) for I2C_WaitOnSTOPFlagUntilTimeout
    stm32f7xx_hal_i2c.o(i.HAL_I2C_Mem_Write) refers to stm32f7xx_hal_i2c.o(i.I2C_WaitOnFlagUntilTimeout) for I2C_WaitOnFlagUntilTimeout
    stm32f7xx_hal_i2c.o(i.HAL_I2C_Mem_Write_DMA) refers to stm32f7xx_hal_dma.o(i.HAL_DMA_Start_IT) for HAL_DMA_Start_IT
    stm32f7xx_hal_i2c.o(i.HAL_I2C_Mem_Write_DMA) refers to stm32f7xx_hal_i2c.o(i.I2C_RequestMemoryWrite) for I2C_RequestMemoryWrite
    stm32f7xx_hal_i2c.o(i.HAL_I2C_Mem_Write_DMA) refers to stm32f7xx_hal_i2c.o(i.I2C_TransferConfig) for I2C_TransferConfig
    stm32f7xx_hal_i2c.o(i.HAL_I2C_Mem_Write_DMA) refers to stm32f7xx_hal_i2c.o(i.I2C_WaitOnTXISFlagUntilTimeout) for I2C_WaitOnTXISFlagUntilTimeout
    stm32f7xx_hal_i2c.o(i.HAL_I2C_Mem_Write_DMA) refers to stm32f7xx_hal_i2c.o(i.I2C_DMAMemTransmitCplt) for I2C_DMAMemTransmitCplt
    stm32f7xx_hal_i2c.o(i.HAL_I2C_Mem_Write_DMA) refers to stm32f7xx_hal_i2c.o(i.I2C_DMAError) for I2C_DMAError
    stm32f7xx_hal_i2c.o(i.HAL_I2C_Mem_Write_IT) refers to stm32f7xx_hal_i2c.o(i.I2C_RequestMemoryWrite) for I2C_RequestMemoryWrite
    stm32f7xx_hal_i2c.o(i.HAL_I2C_Mem_Write_IT) refers to stm32f7xx_hal_i2c.o(i.I2C_TransferConfig) for I2C_TransferConfig
    stm32f7xx_hal_i2c.o(i.HAL_I2C_Slave_Receive) refers to stm32f7xx_hal_i2c.o(i.I2C_WaitOnFlagUntilTimeout) for I2C_WaitOnFlagUntilTimeout
    stm32f7xx_hal_i2c.o(i.HAL_I2C_Slave_Receive) refers to stm32f7xx_hal_i2c.o(i.I2C_WaitOnRXNEFlagUntilTimeout) for I2C_WaitOnRXNEFlagUntilTimeout
    stm32f7xx_hal_i2c.o(i.HAL_I2C_Slave_Receive) refers to stm32f7xx_hal_i2c.o(i.I2C_WaitOnSTOPFlagUntilTimeout) for I2C_WaitOnSTOPFlagUntilTimeout
    stm32f7xx_hal_i2c.o(i.HAL_I2C_Slave_Receive_DMA) refers to stm32f7xx_hal_dma.o(i.HAL_DMA_Start_IT) for HAL_DMA_Start_IT
    stm32f7xx_hal_i2c.o(i.HAL_I2C_Slave_Receive_DMA) refers to stm32f7xx_hal_i2c.o(i.I2C_WaitOnFlagUntilTimeout) for I2C_WaitOnFlagUntilTimeout
    stm32f7xx_hal_i2c.o(i.HAL_I2C_Slave_Receive_DMA) refers to stm32f7xx_hal_i2c.o(i.I2C_DMASlaveReceiveCplt) for I2C_DMASlaveReceiveCplt
    stm32f7xx_hal_i2c.o(i.HAL_I2C_Slave_Receive_DMA) refers to stm32f7xx_hal_i2c.o(i.I2C_DMAError) for I2C_DMAError
    stm32f7xx_hal_i2c.o(i.HAL_I2C_Slave_Transmit) refers to stm32f7xx_hal_i2c.o(i.I2C_WaitOnFlagUntilTimeout) for I2C_WaitOnFlagUntilTimeout
    stm32f7xx_hal_i2c.o(i.HAL_I2C_Slave_Transmit) refers to stm32f7xx_hal_i2c.o(i.I2C_WaitOnTXISFlagUntilTimeout) for I2C_WaitOnTXISFlagUntilTimeout
    stm32f7xx_hal_i2c.o(i.HAL_I2C_Slave_Transmit) refers to stm32f7xx_hal_i2c.o(i.I2C_WaitOnSTOPFlagUntilTimeout) for I2C_WaitOnSTOPFlagUntilTimeout
    stm32f7xx_hal_i2c.o(i.HAL_I2C_Slave_Transmit_DMA) refers to stm32f7xx_hal_dma.o(i.HAL_DMA_Start_IT) for HAL_DMA_Start_IT
    stm32f7xx_hal_i2c.o(i.HAL_I2C_Slave_Transmit_DMA) refers to stm32f7xx_hal_i2c.o(i.I2C_WaitOnFlagUntilTimeout) for I2C_WaitOnFlagUntilTimeout
    stm32f7xx_hal_i2c.o(i.HAL_I2C_Slave_Transmit_DMA) refers to stm32f7xx_hal_i2c.o(i.I2C_DMASlaveTransmitCplt) for I2C_DMASlaveTransmitCplt
    stm32f7xx_hal_i2c.o(i.HAL_I2C_Slave_Transmit_DMA) refers to stm32f7xx_hal_i2c.o(i.I2C_DMAError) for I2C_DMAError
    stm32f7xx_hal_i2c.o(i.I2C_DMAError) refers to stm32f7xx_hal_i2c.o(i.HAL_I2C_ErrorCallback) for HAL_I2C_ErrorCallback
    stm32f7xx_hal_i2c.o(i.I2C_DMAMasterReceiveCplt) refers to stm32f7xx_hal_i2c.o(i.I2C_WaitOnFlagUntilTimeout) for I2C_WaitOnFlagUntilTimeout
    stm32f7xx_hal_i2c.o(i.I2C_DMAMasterReceiveCplt) refers to stm32f7xx_hal_dma.o(i.HAL_DMA_Start_IT) for HAL_DMA_Start_IT
    stm32f7xx_hal_i2c.o(i.I2C_DMAMasterReceiveCplt) refers to stm32f7xx_hal_i2c.o(i.I2C_TransferConfig) for I2C_TransferConfig
    stm32f7xx_hal_i2c.o(i.I2C_DMAMasterReceiveCplt) refers to stm32f7xx_hal_i2c.o(i.I2C_WaitOnSTOPFlagUntilTimeout) for I2C_WaitOnSTOPFlagUntilTimeout
    stm32f7xx_hal_i2c.o(i.I2C_DMAMasterReceiveCplt) refers to stm32f7xx_hal_i2c.o(i.HAL_I2C_ErrorCallback) for HAL_I2C_ErrorCallback
    stm32f7xx_hal_i2c.o(i.I2C_DMAMasterReceiveCplt) refers to stm32f7xx_hal_i2c.o(i.HAL_I2C_MasterRxCpltCallback) for HAL_I2C_MasterRxCpltCallback
    stm32f7xx_hal_i2c.o(i.I2C_DMAMasterTransmitCplt) refers to stm32f7xx_hal_i2c.o(i.I2C_WaitOnFlagUntilTimeout) for I2C_WaitOnFlagUntilTimeout
    stm32f7xx_hal_i2c.o(i.I2C_DMAMasterTransmitCplt) refers to stm32f7xx_hal_dma.o(i.HAL_DMA_Start_IT) for HAL_DMA_Start_IT
    stm32f7xx_hal_i2c.o(i.I2C_DMAMasterTransmitCplt) refers to stm32f7xx_hal_i2c.o(i.I2C_TransferConfig) for I2C_TransferConfig
    stm32f7xx_hal_i2c.o(i.I2C_DMAMasterTransmitCplt) refers to stm32f7xx_hal_i2c.o(i.I2C_WaitOnTXISFlagUntilTimeout) for I2C_WaitOnTXISFlagUntilTimeout
    stm32f7xx_hal_i2c.o(i.I2C_DMAMasterTransmitCplt) refers to stm32f7xx_hal_i2c.o(i.I2C_WaitOnSTOPFlagUntilTimeout) for I2C_WaitOnSTOPFlagUntilTimeout
    stm32f7xx_hal_i2c.o(i.I2C_DMAMasterTransmitCplt) refers to stm32f7xx_hal_i2c.o(i.HAL_I2C_ErrorCallback) for HAL_I2C_ErrorCallback
    stm32f7xx_hal_i2c.o(i.I2C_DMAMasterTransmitCplt) refers to stm32f7xx_hal_i2c.o(i.HAL_I2C_MasterTxCpltCallback) for HAL_I2C_MasterTxCpltCallback
    stm32f7xx_hal_i2c.o(i.I2C_DMAMemReceiveCplt) refers to stm32f7xx_hal_i2c.o(i.I2C_WaitOnFlagUntilTimeout) for I2C_WaitOnFlagUntilTimeout
    stm32f7xx_hal_i2c.o(i.I2C_DMAMemReceiveCplt) refers to stm32f7xx_hal_dma.o(i.HAL_DMA_Start_IT) for HAL_DMA_Start_IT
    stm32f7xx_hal_i2c.o(i.I2C_DMAMemReceiveCplt) refers to stm32f7xx_hal_i2c.o(i.I2C_TransferConfig) for I2C_TransferConfig
    stm32f7xx_hal_i2c.o(i.I2C_DMAMemReceiveCplt) refers to stm32f7xx_hal_i2c.o(i.I2C_WaitOnSTOPFlagUntilTimeout) for I2C_WaitOnSTOPFlagUntilTimeout
    stm32f7xx_hal_i2c.o(i.I2C_DMAMemReceiveCplt) refers to stm32f7xx_hal_i2c.o(i.HAL_I2C_ErrorCallback) for HAL_I2C_ErrorCallback
    stm32f7xx_hal_i2c.o(i.I2C_DMAMemReceiveCplt) refers to stm32f7xx_hal_i2c.o(i.HAL_I2C_MemRxCpltCallback) for HAL_I2C_MemRxCpltCallback
    stm32f7xx_hal_i2c.o(i.I2C_DMAMemTransmitCplt) refers to stm32f7xx_hal_i2c.o(i.I2C_WaitOnFlagUntilTimeout) for I2C_WaitOnFlagUntilTimeout
    stm32f7xx_hal_i2c.o(i.I2C_DMAMemTransmitCplt) refers to stm32f7xx_hal_dma.o(i.HAL_DMA_Start_IT) for HAL_DMA_Start_IT
    stm32f7xx_hal_i2c.o(i.I2C_DMAMemTransmitCplt) refers to stm32f7xx_hal_i2c.o(i.I2C_TransferConfig) for I2C_TransferConfig
    stm32f7xx_hal_i2c.o(i.I2C_DMAMemTransmitCplt) refers to stm32f7xx_hal_i2c.o(i.I2C_WaitOnTXISFlagUntilTimeout) for I2C_WaitOnTXISFlagUntilTimeout
    stm32f7xx_hal_i2c.o(i.I2C_DMAMemTransmitCplt) refers to stm32f7xx_hal_i2c.o(i.I2C_WaitOnSTOPFlagUntilTimeout) for I2C_WaitOnSTOPFlagUntilTimeout
    stm32f7xx_hal_i2c.o(i.I2C_DMAMemTransmitCplt) refers to stm32f7xx_hal_i2c.o(i.HAL_I2C_ErrorCallback) for HAL_I2C_ErrorCallback
    stm32f7xx_hal_i2c.o(i.I2C_DMAMemTransmitCplt) refers to stm32f7xx_hal_i2c.o(i.HAL_I2C_MemTxCpltCallback) for HAL_I2C_MemTxCpltCallback
    stm32f7xx_hal_i2c.o(i.I2C_DMASlaveReceiveCplt) refers to stm32f7xx_hal_i2c.o(i.I2C_WaitOnSTOPFlagUntilTimeout) for I2C_WaitOnSTOPFlagUntilTimeout
    stm32f7xx_hal_i2c.o(i.I2C_DMASlaveReceiveCplt) refers to stm32f7xx_hal_i2c.o(i.I2C_WaitOnFlagUntilTimeout) for I2C_WaitOnFlagUntilTimeout
    stm32f7xx_hal_i2c.o(i.I2C_DMASlaveReceiveCplt) refers to stm32f7xx_hal_i2c.o(i.HAL_I2C_ErrorCallback) for HAL_I2C_ErrorCallback
    stm32f7xx_hal_i2c.o(i.I2C_DMASlaveReceiveCplt) refers to stm32f7xx_hal_i2c.o(i.HAL_I2C_SlaveRxCpltCallback) for HAL_I2C_SlaveRxCpltCallback
    stm32f7xx_hal_i2c.o(i.I2C_DMASlaveTransmitCplt) refers to stm32f7xx_hal_i2c.o(i.I2C_WaitOnSTOPFlagUntilTimeout) for I2C_WaitOnSTOPFlagUntilTimeout
    stm32f7xx_hal_i2c.o(i.I2C_DMASlaveTransmitCplt) refers to stm32f7xx_hal_i2c.o(i.I2C_WaitOnFlagUntilTimeout) for I2C_WaitOnFlagUntilTimeout
    stm32f7xx_hal_i2c.o(i.I2C_DMASlaveTransmitCplt) refers to stm32f7xx_hal_i2c.o(i.HAL_I2C_ErrorCallback) for HAL_I2C_ErrorCallback
    stm32f7xx_hal_i2c.o(i.I2C_DMASlaveTransmitCplt) refers to stm32f7xx_hal_i2c.o(i.HAL_I2C_SlaveTxCpltCallback) for HAL_I2C_SlaveTxCpltCallback
    stm32f7xx_hal_i2c.o(i.I2C_IsAcknowledgeFailed) refers to stm32f7xx_hal.o(i.HAL_GetTick) for HAL_GetTick
    stm32f7xx_hal_i2c.o(i.I2C_MasterReceive_ISR) refers to stm32f7xx_hal_i2c.o(i.I2C_TransferConfig) for I2C_TransferConfig
    stm32f7xx_hal_i2c.o(i.I2C_MasterReceive_ISR) refers to stm32f7xx_hal_i2c.o(i.HAL_I2C_MasterRxCpltCallback) for HAL_I2C_MasterRxCpltCallback
    stm32f7xx_hal_i2c.o(i.I2C_MasterReceive_ISR) refers to stm32f7xx_hal_i2c.o(i.HAL_I2C_MemRxCpltCallback) for HAL_I2C_MemRxCpltCallback
    stm32f7xx_hal_i2c.o(i.I2C_MasterReceive_ISR) refers to stm32f7xx_hal_i2c.o(i.HAL_I2C_ErrorCallback) for HAL_I2C_ErrorCallback
    stm32f7xx_hal_i2c.o(i.I2C_MasterTransmit_ISR) refers to stm32f7xx_hal_i2c.o(i.I2C_TransferConfig) for I2C_TransferConfig
    stm32f7xx_hal_i2c.o(i.I2C_MasterTransmit_ISR) refers to stm32f7xx_hal_i2c.o(i.HAL_I2C_MasterTxCpltCallback) for HAL_I2C_MasterTxCpltCallback
    stm32f7xx_hal_i2c.o(i.I2C_MasterTransmit_ISR) refers to stm32f7xx_hal_i2c.o(i.HAL_I2C_MemTxCpltCallback) for HAL_I2C_MemTxCpltCallback
    stm32f7xx_hal_i2c.o(i.I2C_MasterTransmit_ISR) refers to stm32f7xx_hal_i2c.o(i.HAL_I2C_ErrorCallback) for HAL_I2C_ErrorCallback
    stm32f7xx_hal_i2c.o(i.I2C_RequestMemoryRead) refers to stm32f7xx_hal_i2c.o(i.I2C_TransferConfig) for I2C_TransferConfig
    stm32f7xx_hal_i2c.o(i.I2C_RequestMemoryRead) refers to stm32f7xx_hal_i2c.o(i.I2C_WaitOnTXISFlagUntilTimeout) for I2C_WaitOnTXISFlagUntilTimeout
    stm32f7xx_hal_i2c.o(i.I2C_RequestMemoryRead) refers to stm32f7xx_hal_i2c.o(i.I2C_WaitOnFlagUntilTimeout) for I2C_WaitOnFlagUntilTimeout
    stm32f7xx_hal_i2c.o(i.I2C_RequestMemoryWrite) refers to stm32f7xx_hal_i2c.o(i.I2C_TransferConfig) for I2C_TransferConfig
    stm32f7xx_hal_i2c.o(i.I2C_RequestMemoryWrite) refers to stm32f7xx_hal_i2c.o(i.I2C_WaitOnTXISFlagUntilTimeout) for I2C_WaitOnTXISFlagUntilTimeout
    stm32f7xx_hal_i2c.o(i.I2C_RequestMemoryWrite) refers to stm32f7xx_hal_i2c.o(i.I2C_WaitOnFlagUntilTimeout) for I2C_WaitOnFlagUntilTimeout
    stm32f7xx_hal_i2c.o(i.I2C_SlaveReceive_ISR) refers to stm32f7xx_hal_i2c.o(i.HAL_I2C_ErrorCallback) for HAL_I2C_ErrorCallback
    stm32f7xx_hal_i2c.o(i.I2C_SlaveReceive_ISR) refers to stm32f7xx_hal_i2c.o(i.HAL_I2C_SlaveRxCpltCallback) for HAL_I2C_SlaveRxCpltCallback
    stm32f7xx_hal_i2c.o(i.I2C_SlaveTransmit_ISR) refers to stm32f7xx_hal_i2c.o(i.HAL_I2C_ErrorCallback) for HAL_I2C_ErrorCallback
    stm32f7xx_hal_i2c.o(i.I2C_SlaveTransmit_ISR) refers to stm32f7xx_hal_i2c.o(i.HAL_I2C_SlaveTxCpltCallback) for HAL_I2C_SlaveTxCpltCallback
    stm32f7xx_hal_i2c.o(i.I2C_WaitOnFlagUntilTimeout) refers to stm32f7xx_hal.o(i.HAL_GetTick) for HAL_GetTick
    stm32f7xx_hal_i2c.o(i.I2C_WaitOnRXNEFlagUntilTimeout) refers to stm32f7xx_hal.o(i.HAL_GetTick) for HAL_GetTick
    stm32f7xx_hal_i2c.o(i.I2C_WaitOnRXNEFlagUntilTimeout) refers to stm32f7xx_hal_i2c.o(i.I2C_IsAcknowledgeFailed) for I2C_IsAcknowledgeFailed
    stm32f7xx_hal_i2c.o(i.I2C_WaitOnSTOPFlagUntilTimeout) refers to stm32f7xx_hal.o(i.HAL_GetTick) for HAL_GetTick
    stm32f7xx_hal_i2c.o(i.I2C_WaitOnSTOPFlagUntilTimeout) refers to stm32f7xx_hal_i2c.o(i.I2C_IsAcknowledgeFailed) for I2C_IsAcknowledgeFailed
    stm32f7xx_hal_i2c.o(i.I2C_WaitOnTXISFlagUntilTimeout) refers to stm32f7xx_hal.o(i.HAL_GetTick) for HAL_GetTick
    stm32f7xx_hal_i2c.o(i.I2C_WaitOnTXISFlagUntilTimeout) refers to stm32f7xx_hal_i2c.o(i.I2C_IsAcknowledgeFailed) for I2C_IsAcknowledgeFailed
    stm32f7xx_hal_gpio.o(i.HAL_GPIO_EXTI_IRQHandler) refers to stm32f7xx_hal_gpio.o(i.HAL_GPIO_EXTI_Callback) for HAL_GPIO_EXTI_Callback
    stm32f7xx_hal_rcc_ex.o(i.HAL_RCCEx_PeriphCLKConfig) refers to stm32f7xx_hal.o(i.HAL_GetTick) for HAL_GetTick
    stm32f7xx_hal_tim.o(i.HAL_TIM_Base_DeInit) refers to stm32f7xx_hal_tim.o(i.HAL_TIM_Base_MspDeInit) for HAL_TIM_Base_MspDeInit
    stm32f7xx_hal_tim.o(i.HAL_TIM_Base_Init) refers to stm32f7xx_hal_tim.o(i.HAL_TIM_Base_MspInit) for HAL_TIM_Base_MspInit
    stm32f7xx_hal_tim.o(i.HAL_TIM_Base_Init) refers to stm32f7xx_hal_tim.o(i.TIM_Base_SetConfig) for TIM_Base_SetConfig
    stm32f7xx_hal_tim.o(i.HAL_TIM_Base_Start_DMA) refers to stm32f7xx_hal_dma.o(i.HAL_DMA_Start_IT) for HAL_DMA_Start_IT
    stm32f7xx_hal_tim.o(i.HAL_TIM_Base_Start_DMA) refers to stm32f7xx_hal_tim.o(i.TIM_DMAPeriodElapsedCplt) for TIM_DMAPeriodElapsedCplt
    stm32f7xx_hal_tim.o(i.HAL_TIM_Base_Start_DMA) refers to stm32f7xx_hal_tim.o(i.TIM_DMAError) for TIM_DMAError
    stm32f7xx_hal_tim.o(i.HAL_TIM_ConfigClockSource) refers to stm32f7xx_hal_tim.o(i.TIM_ETR_SetConfig) for TIM_ETR_SetConfig
    stm32f7xx_hal_tim.o(i.HAL_TIM_ConfigClockSource) refers to stm32f7xx_hal_tim.o(i.TIM_TI1_ConfigInputStage) for TIM_TI1_ConfigInputStage
    stm32f7xx_hal_tim.o(i.HAL_TIM_ConfigClockSource) refers to stm32f7xx_hal_tim.o(i.TIM_TI2_ConfigInputStage) for TIM_TI2_ConfigInputStage
    stm32f7xx_hal_tim.o(i.HAL_TIM_ConfigClockSource) refers to stm32f7xx_hal_tim.o(i.TIM_ITRx_SetConfig) for TIM_ITRx_SetConfig
    stm32f7xx_hal_tim.o(i.HAL_TIM_ConfigOCrefClear) refers to stm32f7xx_hal_tim.o(i.TIM_ETR_SetConfig) for TIM_ETR_SetConfig
    stm32f7xx_hal_tim.o(i.HAL_TIM_DMABurst_ReadStart) refers to stm32f7xx_hal_dma.o(i.HAL_DMA_Start_IT) for HAL_DMA_Start_IT
    stm32f7xx_hal_tim.o(i.HAL_TIM_DMABurst_ReadStart) refers to stm32f7xx_hal_tim.o(i.TIM_DMAError) for TIM_DMAError
    stm32f7xx_hal_tim.o(i.HAL_TIM_DMABurst_ReadStart) refers to stm32f7xx_hal_tim.o(i.TIM_DMACaptureCplt) for TIM_DMACaptureCplt
    stm32f7xx_hal_tim.o(i.HAL_TIM_DMABurst_ReadStart) refers to stm32f7xx_hal_tim.o(i.TIM_DMAPeriodElapsedCplt) for TIM_DMAPeriodElapsedCplt
    stm32f7xx_hal_tim.o(i.HAL_TIM_DMABurst_ReadStart) refers to stm32f7xx_hal_tim_ex.o(i.TIMEx_DMACommutationCplt) for TIMEx_DMACommutationCplt
    stm32f7xx_hal_tim.o(i.HAL_TIM_DMABurst_ReadStart) refers to stm32f7xx_hal_tim.o(i.TIM_DMATriggerCplt) for TIM_DMATriggerCplt
    stm32f7xx_hal_tim.o(i.HAL_TIM_DMABurst_ReadStop) refers to stm32f7xx_hal_dma.o(i.HAL_DMA_Abort) for HAL_DMA_Abort
    stm32f7xx_hal_tim.o(i.HAL_TIM_DMABurst_WriteStart) refers to stm32f7xx_hal_dma.o(i.HAL_DMA_Start_IT) for HAL_DMA_Start_IT
    stm32f7xx_hal_tim.o(i.HAL_TIM_DMABurst_WriteStart) refers to stm32f7xx_hal_tim.o(i.TIM_DMAError) for TIM_DMAError
    stm32f7xx_hal_tim.o(i.HAL_TIM_DMABurst_WriteStart) refers to stm32f7xx_hal_tim.o(i.TIM_DMADelayPulseCplt) for TIM_DMADelayPulseCplt
    stm32f7xx_hal_tim.o(i.HAL_TIM_DMABurst_WriteStart) refers to stm32f7xx_hal_tim.o(i.TIM_DMAPeriodElapsedCplt) for TIM_DMAPeriodElapsedCplt
    stm32f7xx_hal_tim.o(i.HAL_TIM_DMABurst_WriteStart) refers to stm32f7xx_hal_tim_ex.o(i.TIMEx_DMACommutationCplt) for TIMEx_DMACommutationCplt
    stm32f7xx_hal_tim.o(i.HAL_TIM_DMABurst_WriteStart) refers to stm32f7xx_hal_tim.o(i.TIM_DMATriggerCplt) for TIM_DMATriggerCplt
    stm32f7xx_hal_tim.o(i.HAL_TIM_DMABurst_WriteStop) refers to stm32f7xx_hal_dma.o(i.HAL_DMA_Abort) for HAL_DMA_Abort
    stm32f7xx_hal_tim.o(i.HAL_TIM_Encoder_DeInit) refers to stm32f7xx_hal_tim.o(i.HAL_TIM_Encoder_MspDeInit) for HAL_TIM_Encoder_MspDeInit
    stm32f7xx_hal_tim.o(i.HAL_TIM_Encoder_Init) refers to stm32f7xx_hal_tim.o(i.HAL_TIM_Encoder_MspInit) for HAL_TIM_Encoder_MspInit
    stm32f7xx_hal_tim.o(i.HAL_TIM_Encoder_Init) refers to stm32f7xx_hal_tim.o(i.TIM_Base_SetConfig) for TIM_Base_SetConfig
    stm32f7xx_hal_tim.o(i.HAL_TIM_Encoder_Start) refers to stm32f7xx_hal_tim.o(i.TIM_CCxChannelCmd) for TIM_CCxChannelCmd
    stm32f7xx_hal_tim.o(i.HAL_TIM_Encoder_Start_DMA) refers to stm32f7xx_hal_dma.o(i.HAL_DMA_Start_IT) for HAL_DMA_Start_IT
    stm32f7xx_hal_tim.o(i.HAL_TIM_Encoder_Start_DMA) refers to stm32f7xx_hal_tim.o(i.TIM_CCxChannelCmd) for TIM_CCxChannelCmd
    stm32f7xx_hal_tim.o(i.HAL_TIM_Encoder_Start_DMA) refers to stm32f7xx_hal_tim.o(i.TIM_DMACaptureCplt) for TIM_DMACaptureCplt
    stm32f7xx_hal_tim.o(i.HAL_TIM_Encoder_Start_DMA) refers to stm32f7xx_hal_tim.o(i.TIM_DMAError) for TIM_DMAError
    stm32f7xx_hal_tim.o(i.HAL_TIM_Encoder_Start_IT) refers to stm32f7xx_hal_tim.o(i.TIM_CCxChannelCmd) for TIM_CCxChannelCmd
    stm32f7xx_hal_tim.o(i.HAL_TIM_Encoder_Stop) refers to stm32f7xx_hal_tim.o(i.TIM_CCxChannelCmd) for TIM_CCxChannelCmd
    stm32f7xx_hal_tim.o(i.HAL_TIM_Encoder_Stop_DMA) refers to stm32f7xx_hal_tim.o(i.TIM_CCxChannelCmd) for TIM_CCxChannelCmd
    stm32f7xx_hal_tim.o(i.HAL_TIM_Encoder_Stop_IT) refers to stm32f7xx_hal_tim.o(i.TIM_CCxChannelCmd) for TIM_CCxChannelCmd
    stm32f7xx_hal_tim.o(i.HAL_TIM_IC_ConfigChannel) refers to stm32f7xx_hal_tim.o(i.TIM_TI1_SetConfig) for TIM_TI1_SetConfig
    stm32f7xx_hal_tim.o(i.HAL_TIM_IC_ConfigChannel) refers to stm32f7xx_hal_tim.o(i.TIM_TI2_SetConfig) for TIM_TI2_SetConfig
    stm32f7xx_hal_tim.o(i.HAL_TIM_IC_DeInit) refers to stm32f7xx_hal_tim.o(i.HAL_TIM_IC_MspDeInit) for HAL_TIM_IC_MspDeInit
    stm32f7xx_hal_tim.o(i.HAL_TIM_IC_Init) refers to stm32f7xx_hal_tim.o(i.HAL_TIM_IC_MspInit) for HAL_TIM_IC_MspInit
    stm32f7xx_hal_tim.o(i.HAL_TIM_IC_Init) refers to stm32f7xx_hal_tim.o(i.TIM_Base_SetConfig) for TIM_Base_SetConfig
    stm32f7xx_hal_tim.o(i.HAL_TIM_IC_Start) refers to stm32f7xx_hal_tim.o(i.TIM_CCxChannelCmd) for TIM_CCxChannelCmd
    stm32f7xx_hal_tim.o(i.HAL_TIM_IC_Start_DMA) refers to stm32f7xx_hal_dma.o(i.HAL_DMA_Start_IT) for HAL_DMA_Start_IT
    stm32f7xx_hal_tim.o(i.HAL_TIM_IC_Start_DMA) refers to stm32f7xx_hal_tim.o(i.TIM_CCxChannelCmd) for TIM_CCxChannelCmd
    stm32f7xx_hal_tim.o(i.HAL_TIM_IC_Start_DMA) refers to stm32f7xx_hal_tim.o(i.TIM_DMACaptureCplt) for TIM_DMACaptureCplt
    stm32f7xx_hal_tim.o(i.HAL_TIM_IC_Start_DMA) refers to stm32f7xx_hal_tim.o(i.TIM_DMAError) for TIM_DMAError
    stm32f7xx_hal_tim.o(i.HAL_TIM_IC_Start_IT) refers to stm32f7xx_hal_tim.o(i.TIM_CCxChannelCmd) for TIM_CCxChannelCmd
    stm32f7xx_hal_tim.o(i.HAL_TIM_IC_Stop) refers to stm32f7xx_hal_tim.o(i.TIM_CCxChannelCmd) for TIM_CCxChannelCmd
    stm32f7xx_hal_tim.o(i.HAL_TIM_IC_Stop_DMA) refers to stm32f7xx_hal_tim.o(i.TIM_CCxChannelCmd) for TIM_CCxChannelCmd
    stm32f7xx_hal_tim.o(i.HAL_TIM_IC_Stop_IT) refers to stm32f7xx_hal_tim.o(i.TIM_CCxChannelCmd) for TIM_CCxChannelCmd
    stm32f7xx_hal_tim.o(i.HAL_TIM_IRQHandler) refers to stm32f7xx_hal_tim.o(i.HAL_TIM_IC_CaptureCallback) for HAL_TIM_IC_CaptureCallback
    stm32f7xx_hal_tim.o(i.HAL_TIM_IRQHandler) refers to stm32f7xx_hal_tim.o(i.HAL_TIM_OC_DelayElapsedCallback) for HAL_TIM_OC_DelayElapsedCallback
    stm32f7xx_hal_tim.o(i.HAL_TIM_IRQHandler) refers to stm32f7xx_hal_tim.o(i.HAL_TIM_PWM_PulseFinishedCallback) for HAL_TIM_PWM_PulseFinishedCallback
    stm32f7xx_hal_tim.o(i.HAL_TIM_IRQHandler) refers to stm32f7xx_hal_tim.o(i.HAL_TIM_PeriodElapsedCallback) for HAL_TIM_PeriodElapsedCallback
    stm32f7xx_hal_tim.o(i.HAL_TIM_IRQHandler) refers to stm32f7xx_hal_tim_ex.o(i.HAL_TIMEx_BreakCallback) for HAL_TIMEx_BreakCallback
    stm32f7xx_hal_tim.o(i.HAL_TIM_IRQHandler) refers to stm32f7xx_hal_tim.o(i.HAL_TIM_TriggerCallback) for HAL_TIM_TriggerCallback
    stm32f7xx_hal_tim.o(i.HAL_TIM_IRQHandler) refers to stm32f7xx_hal_tim_ex.o(i.HAL_TIMEx_CommutationCallback) for HAL_TIMEx_CommutationCallback
    stm32f7xx_hal_tim.o(i.HAL_TIM_OC_ConfigChannel) refers to stm32f7xx_hal_tim.o(i.TIM_OC1_SetConfig) for TIM_OC1_SetConfig
    stm32f7xx_hal_tim.o(i.HAL_TIM_OC_ConfigChannel) refers to stm32f7xx_hal_tim.o(i.TIM_OC2_SetConfig) for TIM_OC2_SetConfig
    stm32f7xx_hal_tim.o(i.HAL_TIM_OC_ConfigChannel) refers to stm32f7xx_hal_tim.o(i.TIM_OC3_SetConfig) for TIM_OC3_SetConfig
    stm32f7xx_hal_tim.o(i.HAL_TIM_OC_ConfigChannel) refers to stm32f7xx_hal_tim.o(i.TIM_OC4_SetConfig) for TIM_OC4_SetConfig
    stm32f7xx_hal_tim.o(i.HAL_TIM_OC_DeInit) refers to stm32f7xx_hal_tim.o(i.HAL_TIM_OC_MspDeInit) for HAL_TIM_OC_MspDeInit
    stm32f7xx_hal_tim.o(i.HAL_TIM_OC_Init) refers to stm32f7xx_hal_tim.o(i.HAL_TIM_OC_MspInit) for HAL_TIM_OC_MspInit
    stm32f7xx_hal_tim.o(i.HAL_TIM_OC_Init) refers to stm32f7xx_hal_tim.o(i.TIM_Base_SetConfig) for TIM_Base_SetConfig
    stm32f7xx_hal_tim.o(i.HAL_TIM_OC_Start) refers to stm32f7xx_hal_tim.o(i.TIM_CCxChannelCmd) for TIM_CCxChannelCmd
    stm32f7xx_hal_tim.o(i.HAL_TIM_OC_Start_DMA) refers to stm32f7xx_hal_dma.o(i.HAL_DMA_Start_IT) for HAL_DMA_Start_IT
    stm32f7xx_hal_tim.o(i.HAL_TIM_OC_Start_DMA) refers to stm32f7xx_hal_tim.o(i.TIM_CCxChannelCmd) for TIM_CCxChannelCmd
    stm32f7xx_hal_tim.o(i.HAL_TIM_OC_Start_DMA) refers to stm32f7xx_hal_tim.o(i.TIM_DMADelayPulseCplt) for TIM_DMADelayPulseCplt
    stm32f7xx_hal_tim.o(i.HAL_TIM_OC_Start_DMA) refers to stm32f7xx_hal_tim.o(i.TIM_DMAError) for TIM_DMAError
    stm32f7xx_hal_tim.o(i.HAL_TIM_OC_Start_IT) refers to stm32f7xx_hal_tim.o(i.TIM_CCxChannelCmd) for TIM_CCxChannelCmd
    stm32f7xx_hal_tim.o(i.HAL_TIM_OC_Stop) refers to stm32f7xx_hal_tim.o(i.TIM_CCxChannelCmd) for TIM_CCxChannelCmd
    stm32f7xx_hal_tim.o(i.HAL_TIM_OC_Stop_DMA) refers to stm32f7xx_hal_tim.o(i.TIM_CCxChannelCmd) for TIM_CCxChannelCmd
    stm32f7xx_hal_tim.o(i.HAL_TIM_OC_Stop_IT) refers to stm32f7xx_hal_tim.o(i.TIM_CCxChannelCmd) for TIM_CCxChannelCmd
    stm32f7xx_hal_tim.o(i.HAL_TIM_OnePulse_ConfigChannel) refers to stm32f7xx_hal_tim.o(i.TIM_OC1_SetConfig) for TIM_OC1_SetConfig
    stm32f7xx_hal_tim.o(i.HAL_TIM_OnePulse_ConfigChannel) refers to stm32f7xx_hal_tim.o(i.TIM_OC2_SetConfig) for TIM_OC2_SetConfig
    stm32f7xx_hal_tim.o(i.HAL_TIM_OnePulse_ConfigChannel) refers to stm32f7xx_hal_tim.o(i.TIM_TI1_SetConfig) for TIM_TI1_SetConfig
    stm32f7xx_hal_tim.o(i.HAL_TIM_OnePulse_ConfigChannel) refers to stm32f7xx_hal_tim.o(i.TIM_TI2_SetConfig) for TIM_TI2_SetConfig
    stm32f7xx_hal_tim.o(i.HAL_TIM_OnePulse_DeInit) refers to stm32f7xx_hal_tim.o(i.HAL_TIM_OnePulse_MspDeInit) for HAL_TIM_OnePulse_MspDeInit
    stm32f7xx_hal_tim.o(i.HAL_TIM_OnePulse_Init) refers to stm32f7xx_hal_tim.o(i.HAL_TIM_OnePulse_MspInit) for HAL_TIM_OnePulse_MspInit
    stm32f7xx_hal_tim.o(i.HAL_TIM_OnePulse_Init) refers to stm32f7xx_hal_tim.o(i.TIM_Base_SetConfig) for TIM_Base_SetConfig
    stm32f7xx_hal_tim.o(i.HAL_TIM_OnePulse_Start) refers to stm32f7xx_hal_tim.o(i.TIM_CCxChannelCmd) for TIM_CCxChannelCmd
    stm32f7xx_hal_tim.o(i.HAL_TIM_OnePulse_Start_IT) refers to stm32f7xx_hal_tim.o(i.TIM_CCxChannelCmd) for TIM_CCxChannelCmd
    stm32f7xx_hal_tim.o(i.HAL_TIM_OnePulse_Stop) refers to stm32f7xx_hal_tim.o(i.TIM_CCxChannelCmd) for TIM_CCxChannelCmd
    stm32f7xx_hal_tim.o(i.HAL_TIM_OnePulse_Stop_IT) refers to stm32f7xx_hal_tim.o(i.TIM_CCxChannelCmd) for TIM_CCxChannelCmd
    stm32f7xx_hal_tim.o(i.HAL_TIM_PWM_ConfigChannel) refers to stm32f7xx_hal_tim.o(i.TIM_OC1_SetConfig) for TIM_OC1_SetConfig
    stm32f7xx_hal_tim.o(i.HAL_TIM_PWM_ConfigChannel) refers to stm32f7xx_hal_tim.o(i.TIM_OC2_SetConfig) for TIM_OC2_SetConfig
    stm32f7xx_hal_tim.o(i.HAL_TIM_PWM_ConfigChannel) refers to stm32f7xx_hal_tim.o(i.TIM_OC3_SetConfig) for TIM_OC3_SetConfig
    stm32f7xx_hal_tim.o(i.HAL_TIM_PWM_ConfigChannel) refers to stm32f7xx_hal_tim.o(i.TIM_OC4_SetConfig) for TIM_OC4_SetConfig
    stm32f7xx_hal_tim.o(i.HAL_TIM_PWM_DeInit) refers to stm32f7xx_hal_tim.o(i.HAL_TIM_PWM_MspDeInit) for HAL_TIM_PWM_MspDeInit
    stm32f7xx_hal_tim.o(i.HAL_TIM_PWM_Init) refers to stm32f7xx_hal_tim.o(i.HAL_TIM_PWM_MspInit) for HAL_TIM_PWM_MspInit
    stm32f7xx_hal_tim.o(i.HAL_TIM_PWM_Init) refers to stm32f7xx_hal_tim.o(i.TIM_Base_SetConfig) for TIM_Base_SetConfig
    stm32f7xx_hal_tim.o(i.HAL_TIM_PWM_Start) refers to stm32f7xx_hal_tim.o(i.TIM_CCxChannelCmd) for TIM_CCxChannelCmd
    stm32f7xx_hal_tim.o(i.HAL_TIM_PWM_Start_DMA) refers to stm32f7xx_hal_dma.o(i.HAL_DMA_Start_IT) for HAL_DMA_Start_IT
    stm32f7xx_hal_tim.o(i.HAL_TIM_PWM_Start_DMA) refers to stm32f7xx_hal_tim.o(i.TIM_CCxChannelCmd) for TIM_CCxChannelCmd
    stm32f7xx_hal_tim.o(i.HAL_TIM_PWM_Start_DMA) refers to stm32f7xx_hal_tim.o(i.TIM_DMADelayPulseCplt) for TIM_DMADelayPulseCplt
    stm32f7xx_hal_tim.o(i.HAL_TIM_PWM_Start_DMA) refers to stm32f7xx_hal_tim.o(i.TIM_DMAError) for TIM_DMAError
    stm32f7xx_hal_tim.o(i.HAL_TIM_PWM_Start_IT) refers to stm32f7xx_hal_tim.o(i.TIM_CCxChannelCmd) for TIM_CCxChannelCmd
    stm32f7xx_hal_tim.o(i.HAL_TIM_PWM_Stop) refers to stm32f7xx_hal_tim.o(i.TIM_CCxChannelCmd) for TIM_CCxChannelCmd
    stm32f7xx_hal_tim.o(i.HAL_TIM_PWM_Stop_DMA) refers to stm32f7xx_hal_tim.o(i.TIM_CCxChannelCmd) for TIM_CCxChannelCmd
    stm32f7xx_hal_tim.o(i.HAL_TIM_PWM_Stop_IT) refers to stm32f7xx_hal_tim.o(i.TIM_CCxChannelCmd) for TIM_CCxChannelCmd
    stm32f7xx_hal_tim.o(i.HAL_TIM_SlaveConfigSynchronization) refers to stm32f7xx_hal_tim.o(i.TIM_ETR_SetConfig) for TIM_ETR_SetConfig
    stm32f7xx_hal_tim.o(i.HAL_TIM_SlaveConfigSynchronization) refers to stm32f7xx_hal_tim.o(i.TIM_TI1_ConfigInputStage) for TIM_TI1_ConfigInputStage
    stm32f7xx_hal_tim.o(i.HAL_TIM_SlaveConfigSynchronization) refers to stm32f7xx_hal_tim.o(i.TIM_TI2_ConfigInputStage) for TIM_TI2_ConfigInputStage
    stm32f7xx_hal_tim.o(i.HAL_TIM_SlaveConfigSynchronization_IT) refers to stm32f7xx_hal_tim.o(i.TIM_SlaveTimer_SetConfig) for TIM_SlaveTimer_SetConfig
    stm32f7xx_hal_tim.o(i.TIM_DMACaptureCplt) refers to stm32f7xx_hal_tim.o(i.HAL_TIM_IC_CaptureCallback) for HAL_TIM_IC_CaptureCallback
    stm32f7xx_hal_tim.o(i.TIM_DMADelayPulseCplt) refers to stm32f7xx_hal_tim.o(i.HAL_TIM_PWM_PulseFinishedCallback) for HAL_TIM_PWM_PulseFinishedCallback
    stm32f7xx_hal_tim.o(i.TIM_DMAError) refers to stm32f7xx_hal_tim.o(i.HAL_TIM_ErrorCallback) for HAL_TIM_ErrorCallback
    stm32f7xx_hal_tim.o(i.TIM_DMAPeriodElapsedCplt) refers to stm32f7xx_hal_tim.o(i.HAL_TIM_PeriodElapsedCallback) for HAL_TIM_PeriodElapsedCallback
    stm32f7xx_hal_tim.o(i.TIM_DMATriggerCplt) refers to stm32f7xx_hal_tim.o(i.HAL_TIM_TriggerCallback) for HAL_TIM_TriggerCallback
    stm32f7xx_hal_tim.o(i.TIM_SlaveTimer_SetConfig) refers to stm32f7xx_hal_tim.o(i.TIM_ETR_SetConfig) for TIM_ETR_SetConfig
    stm32f7xx_hal_tim.o(i.TIM_SlaveTimer_SetConfig) refers to stm32f7xx_hal_tim.o(i.TIM_TI1_ConfigInputStage) for TIM_TI1_ConfigInputStage
    stm32f7xx_hal_tim.o(i.TIM_SlaveTimer_SetConfig) refers to stm32f7xx_hal_tim.o(i.TIM_TI2_ConfigInputStage) for TIM_TI2_ConfigInputStage
    stm32f7xx_hal_dma.o(i.DMA_CalcBaseAndBitshift) refers to stm32f7xx_hal_dma.o(.constdata) for .constdata
    stm32f7xx_hal_dma.o(i.HAL_DMA_Abort) refers to stm32f7xx_hal.o(i.HAL_GetTick) for HAL_GetTick
    stm32f7xx_hal_dma.o(i.HAL_DMA_DeInit) refers to stm32f7xx_hal_dma.o(i.DMA_CalcBaseAndBitshift) for DMA_CalcBaseAndBitshift
    stm32f7xx_hal_dma.o(i.HAL_DMA_Init) refers to stm32f7xx_hal_dma.o(i.DMA_CalcBaseAndBitshift) for DMA_CalcBaseAndBitshift
    stm32f7xx_hal_dma.o(i.HAL_DMA_PollForTransfer) refers to stm32f7xx_hal.o(i.HAL_GetTick) for HAL_GetTick
    stm32f7xx_hal_dma.o(i.HAL_DMA_Start) refers to stm32f7xx_hal_dma.o(i.DMA_SetConfig) for DMA_SetConfig
    stm32f7xx_hal_dma.o(i.HAL_DMA_Start_IT) refers to stm32f7xx_hal_dma.o(i.DMA_SetConfig) for DMA_SetConfig
    stm32f7xx_hal_flash_ex.o(i.FLASH_OB_BootAddressConfig) refers to stm32f7xx_hal_flash.o(i.FLASH_WaitForLastOperation) for FLASH_WaitForLastOperation
    stm32f7xx_hal_flash_ex.o(i.HAL_FLASHEx_Erase) refers to stm32f7xx_hal_flash.o(i.FLASH_WaitForLastOperation) for FLASH_WaitForLastOperation
    stm32f7xx_hal_flash_ex.o(i.HAL_FLASHEx_Erase) refers to stm32f7xx_hal_flash_ex.o(i.FLASH_MassErase) for FLASH_MassErase
    stm32f7xx_hal_flash_ex.o(i.HAL_FLASHEx_Erase) refers to stm32f7xx_hal_flash_ex.o(i.FLASH_Erase_Sector) for FLASH_Erase_Sector
    stm32f7xx_hal_flash_ex.o(i.HAL_FLASHEx_Erase) refers to stm32f7xx_hal_flash.o(.bss) for pFlash
    stm32f7xx_hal_flash_ex.o(i.HAL_FLASHEx_Erase_IT) refers to stm32f7xx_hal_flash_ex.o(i.FLASH_Erase_Sector) for FLASH_Erase_Sector
    stm32f7xx_hal_flash_ex.o(i.HAL_FLASHEx_Erase_IT) refers to stm32f7xx_hal_flash_ex.o(i.FLASH_MassErase) for FLASH_MassErase
    stm32f7xx_hal_flash_ex.o(i.HAL_FLASHEx_Erase_IT) refers to stm32f7xx_hal_flash.o(.bss) for pFlash
    stm32f7xx_hal_flash_ex.o(i.HAL_FLASHEx_OBGetConfig) refers to stm32f7xx_hal_flash_ex.o(i.FLASH_OB_GetBootAddress) for FLASH_OB_GetBootAddress
    stm32f7xx_hal_flash_ex.o(i.HAL_FLASHEx_OBProgram) refers to stm32f7xx_hal_flash.o(i.FLASH_WaitForLastOperation) for FLASH_WaitForLastOperation
    stm32f7xx_hal_flash_ex.o(i.HAL_FLASHEx_OBProgram) refers to stm32f7xx_hal_flash_ex.o(i.FLASH_OB_BootAddressConfig) for FLASH_OB_BootAddressConfig
    stm32f7xx_hal_flash_ex.o(i.HAL_FLASHEx_OBProgram) refers to stm32f7xx_hal_flash.o(.bss) for pFlash
    stm32f7xx_hal_usart.o(i.HAL_USART_DMAStop) refers to stm32f7xx_hal_dma.o(i.HAL_DMA_Abort) for HAL_DMA_Abort
    stm32f7xx_hal_usart.o(i.HAL_USART_DeInit) refers to stm32f7xx_hal_usart.o(i.HAL_USART_MspDeInit) for HAL_USART_MspDeInit
    stm32f7xx_hal_usart.o(i.HAL_USART_IRQHandler) refers to stm32f7xx_hal_usart.o(i.HAL_USART_ErrorCallback) for HAL_USART_ErrorCallback
    stm32f7xx_hal_usart.o(i.HAL_USART_IRQHandler) refers to stm32f7xx_hal_usart.o(i.USART_TransmitReceive_IT) for USART_TransmitReceive_IT
    stm32f7xx_hal_usart.o(i.HAL_USART_IRQHandler) refers to stm32f7xx_hal_usart.o(i.HAL_USART_TxCpltCallback) for HAL_USART_TxCpltCallback
    stm32f7xx_hal_usart.o(i.HAL_USART_IRQHandler) refers to stm32f7xx_hal_usart.o(i.USART_Receive_IT) for USART_Receive_IT
    stm32f7xx_hal_usart.o(i.HAL_USART_Init) refers to stm32f7xx_hal_usart.o(i.HAL_USART_MspInit) for HAL_USART_MspInit
    stm32f7xx_hal_usart.o(i.HAL_USART_Init) refers to stm32f7xx_hal_usart.o(i.USART_SetConfig) for USART_SetConfig
    stm32f7xx_hal_usart.o(i.HAL_USART_Init) refers to stm32f7xx_hal_usart.o(i.USART_WaitOnFlagUntilTimeout) for USART_WaitOnFlagUntilTimeout
    stm32f7xx_hal_usart.o(i.HAL_USART_Receive) refers to stm32f7xx_hal_usart.o(i.USART_WaitOnFlagUntilTimeout) for USART_WaitOnFlagUntilTimeout
    stm32f7xx_hal_usart.o(i.HAL_USART_Receive_DMA) refers to stm32f7xx_hal_dma.o(i.HAL_DMA_Start_IT) for HAL_DMA_Start_IT
    stm32f7xx_hal_usart.o(i.HAL_USART_Receive_DMA) refers to stm32f7xx_hal_usart.o(i.USART_DMAReceiveCplt) for USART_DMAReceiveCplt
    stm32f7xx_hal_usart.o(i.HAL_USART_Receive_DMA) refers to stm32f7xx_hal_usart.o(i.USART_DMARxHalfCplt) for USART_DMARxHalfCplt
    stm32f7xx_hal_usart.o(i.HAL_USART_Receive_DMA) refers to stm32f7xx_hal_usart.o(i.USART_DMAError) for USART_DMAError
    stm32f7xx_hal_usart.o(i.HAL_USART_Transmit) refers to stm32f7xx_hal_usart.o(i.USART_WaitOnFlagUntilTimeout) for USART_WaitOnFlagUntilTimeout
    stm32f7xx_hal_usart.o(i.HAL_USART_TransmitReceive) refers to stm32f7xx_hal_usart.o(i.USART_WaitOnFlagUntilTimeout) for USART_WaitOnFlagUntilTimeout
    stm32f7xx_hal_usart.o(i.HAL_USART_TransmitReceive_DMA) refers to stm32f7xx_hal_dma.o(i.HAL_DMA_Start_IT) for HAL_DMA_Start_IT
    stm32f7xx_hal_usart.o(i.HAL_USART_TransmitReceive_DMA) refers to stm32f7xx_hal_usart.o(i.USART_DMAError) for USART_DMAError
    stm32f7xx_hal_usart.o(i.HAL_USART_TransmitReceive_DMA) refers to stm32f7xx_hal_usart.o(i.USART_DMAReceiveCplt) for USART_DMAReceiveCplt
    stm32f7xx_hal_usart.o(i.HAL_USART_TransmitReceive_DMA) refers to stm32f7xx_hal_usart.o(i.USART_DMARxHalfCplt) for USART_DMARxHalfCplt
    stm32f7xx_hal_usart.o(i.HAL_USART_TransmitReceive_DMA) refers to stm32f7xx_hal_usart.o(i.USART_DMATransmitCplt) for USART_DMATransmitCplt
    stm32f7xx_hal_usart.o(i.HAL_USART_TransmitReceive_DMA) refers to stm32f7xx_hal_usart.o(i.USART_DMATxHalfCplt) for USART_DMATxHalfCplt
    stm32f7xx_hal_usart.o(i.HAL_USART_Transmit_DMA) refers to stm32f7xx_hal_dma.o(i.HAL_DMA_Start_IT) for HAL_DMA_Start_IT
    stm32f7xx_hal_usart.o(i.HAL_USART_Transmit_DMA) refers to stm32f7xx_hal_usart.o(i.USART_DMATransmitCplt) for USART_DMATransmitCplt
    stm32f7xx_hal_usart.o(i.HAL_USART_Transmit_DMA) refers to stm32f7xx_hal_usart.o(i.USART_DMATxHalfCplt) for USART_DMATxHalfCplt
    stm32f7xx_hal_usart.o(i.HAL_USART_Transmit_DMA) refers to stm32f7xx_hal_usart.o(i.USART_DMAError) for USART_DMAError
    stm32f7xx_hal_usart.o(i.USART_DMAError) refers to stm32f7xx_hal_usart.o(i.HAL_USART_ErrorCallback) for HAL_USART_ErrorCallback
    stm32f7xx_hal_usart.o(i.USART_DMAReceiveCplt) refers to stm32f7xx_hal_usart.o(i.HAL_USART_TxRxCpltCallback) for HAL_USART_TxRxCpltCallback
    stm32f7xx_hal_usart.o(i.USART_DMAReceiveCplt) refers to stm32f7xx_hal_usart.o(i.HAL_USART_RxCpltCallback) for HAL_USART_RxCpltCallback
    stm32f7xx_hal_usart.o(i.USART_DMARxHalfCplt) refers to stm32f7xx_hal_usart.o(i.HAL_USART_RxHalfCpltCallback) for HAL_USART_RxHalfCpltCallback
    stm32f7xx_hal_usart.o(i.USART_DMATransmitCplt) refers to stm32f7xx_hal_usart.o(i.HAL_USART_TxCpltCallback) for HAL_USART_TxCpltCallback
    stm32f7xx_hal_usart.o(i.USART_DMATxHalfCplt) refers to stm32f7xx_hal_usart.o(i.HAL_USART_TxHalfCpltCallback) for HAL_USART_TxHalfCpltCallback
    stm32f7xx_hal_usart.o(i.USART_Receive_IT) refers to stm32f7xx_hal_usart.o(i.HAL_USART_RxCpltCallback) for HAL_USART_RxCpltCallback
    stm32f7xx_hal_usart.o(i.USART_SetConfig) refers to stm32f7xx_hal_rcc.o(i.HAL_RCC_GetPCLK1Freq) for HAL_RCC_GetPCLK1Freq
    stm32f7xx_hal_usart.o(i.USART_SetConfig) refers to stm32f7xx_hal_rcc.o(i.HAL_RCC_GetPCLK2Freq) for HAL_RCC_GetPCLK2Freq
    stm32f7xx_hal_usart.o(i.USART_SetConfig) refers to stm32f7xx_hal_rcc.o(i.HAL_RCC_GetSysClockFreq) for HAL_RCC_GetSysClockFreq
    stm32f7xx_hal_usart.o(i.USART_TransmitReceive_IT) refers to stm32f7xx_hal_usart.o(i.HAL_USART_TxRxCpltCallback) for HAL_USART_TxRxCpltCallback
    stm32f7xx_hal_usart.o(i.USART_WaitOnFlagUntilTimeout) refers to stm32f7xx_hal.o(i.HAL_GetTick) for HAL_GetTick
    stm32f7xx_hal_uart.o(i.HAL_HalfDuplex_Init) refers to main.o(i.HAL_UART_MspInit) for HAL_UART_MspInit
    stm32f7xx_hal_uart.o(i.HAL_HalfDuplex_Init) refers to stm32f7xx_hal_uart.o(i.UART_SetConfig) for UART_SetConfig
    stm32f7xx_hal_uart.o(i.HAL_HalfDuplex_Init) refers to stm32f7xx_hal_uart.o(i.UART_AdvFeatureConfig) for UART_AdvFeatureConfig
    stm32f7xx_hal_uart.o(i.HAL_HalfDuplex_Init) refers to stm32f7xx_hal_uart.o(i.UART_CheckIdleState) for UART_CheckIdleState
    stm32f7xx_hal_uart.o(i.HAL_LIN_Init) refers to main.o(i.HAL_UART_MspInit) for HAL_UART_MspInit
    stm32f7xx_hal_uart.o(i.HAL_LIN_Init) refers to stm32f7xx_hal_uart.o(i.UART_SetConfig) for UART_SetConfig
    stm32f7xx_hal_uart.o(i.HAL_LIN_Init) refers to stm32f7xx_hal_uart.o(i.UART_AdvFeatureConfig) for UART_AdvFeatureConfig
    stm32f7xx_hal_uart.o(i.HAL_LIN_Init) refers to stm32f7xx_hal_uart.o(i.UART_CheckIdleState) for UART_CheckIdleState
    stm32f7xx_hal_uart.o(i.HAL_MultiProcessor_DisableMuteMode) refers to stm32f7xx_hal_uart.o(i.UART_CheckIdleState) for UART_CheckIdleState
    stm32f7xx_hal_uart.o(i.HAL_MultiProcessor_EnableMuteMode) refers to stm32f7xx_hal_uart.o(i.UART_CheckIdleState) for UART_CheckIdleState
    stm32f7xx_hal_uart.o(i.HAL_MultiProcessor_Init) refers to main.o(i.HAL_UART_MspInit) for HAL_UART_MspInit
    stm32f7xx_hal_uart.o(i.HAL_MultiProcessor_Init) refers to stm32f7xx_hal_uart.o(i.UART_SetConfig) for UART_SetConfig
    stm32f7xx_hal_uart.o(i.HAL_MultiProcessor_Init) refers to stm32f7xx_hal_uart.o(i.UART_AdvFeatureConfig) for UART_AdvFeatureConfig
    stm32f7xx_hal_uart.o(i.HAL_MultiProcessor_Init) refers to stm32f7xx_hal_uart.o(i.UART_CheckIdleState) for UART_CheckIdleState
    stm32f7xx_hal_uart.o(i.HAL_UART_DMAStop) refers to stm32f7xx_hal_dma.o(i.HAL_DMA_Abort) for HAL_DMA_Abort
    stm32f7xx_hal_uart.o(i.HAL_UART_DeInit) refers to main.o(i.HAL_UART_MspDeInit) for HAL_UART_MspDeInit
    stm32f7xx_hal_uart.o(i.HAL_UART_IRQHandler) refers to stm32f7xx_hal_uart.o(i.HAL_UART_ErrorCallback) for HAL_UART_ErrorCallback
    stm32f7xx_hal_uart.o(i.HAL_UART_IRQHandler) refers to stm32f7xx_hal_uart.o(i.UART_Receive_IT) for UART_Receive_IT
    stm32f7xx_hal_uart.o(i.HAL_UART_IRQHandler) refers to stm32f7xx_hal_uart.o(i.UART_Transmit_IT) for UART_Transmit_IT
    stm32f7xx_hal_uart.o(i.HAL_UART_IRQHandler) refers to stm32f7xx_hal_uart.o(i.HAL_UART_TxCpltCallback) for HAL_UART_TxCpltCallback
    stm32f7xx_hal_uart.o(i.HAL_UART_Init) refers to main.o(i.HAL_UART_MspInit) for HAL_UART_MspInit
    stm32f7xx_hal_uart.o(i.HAL_UART_Init) refers to stm32f7xx_hal_uart.o(i.UART_SetConfig) for UART_SetConfig
    stm32f7xx_hal_uart.o(i.HAL_UART_Init) refers to stm32f7xx_hal_uart.o(i.UART_AdvFeatureConfig) for UART_AdvFeatureConfig
    stm32f7xx_hal_uart.o(i.HAL_UART_Init) refers to stm32f7xx_hal_uart.o(i.UART_CheckIdleState) for UART_CheckIdleState
    stm32f7xx_hal_uart.o(i.HAL_UART_Receive) refers to stm32f7xx_hal_uart.o(i.UART_WaitOnFlagUntilTimeout) for UART_WaitOnFlagUntilTimeout
    stm32f7xx_hal_uart.o(i.HAL_UART_Receive_DMA) refers to stm32f7xx_hal_dma.o(i.HAL_DMA_Start_IT) for HAL_DMA_Start_IT
    stm32f7xx_hal_uart.o(i.HAL_UART_Receive_DMA) refers to stm32f7xx_hal_uart.o(i.UART_DMAReceiveCplt) for UART_DMAReceiveCplt
    stm32f7xx_hal_uart.o(i.HAL_UART_Receive_DMA) refers to stm32f7xx_hal_uart.o(i.UART_DMARxHalfCplt) for UART_DMARxHalfCplt
    stm32f7xx_hal_uart.o(i.HAL_UART_Receive_DMA) refers to stm32f7xx_hal_uart.o(i.UART_DMAError) for UART_DMAError
    stm32f7xx_hal_uart.o(i.HAL_UART_Transmit) refers to stm32f7xx_hal_uart.o(i.UART_WaitOnFlagUntilTimeout) for UART_WaitOnFlagUntilTimeout
    stm32f7xx_hal_uart.o(i.HAL_UART_Transmit_DMA) refers to stm32f7xx_hal_dma.o(i.HAL_DMA_Start_IT) for HAL_DMA_Start_IT
    stm32f7xx_hal_uart.o(i.HAL_UART_Transmit_DMA) refers to stm32f7xx_hal_uart.o(i.UART_DMATransmitCplt) for UART_DMATransmitCplt
    stm32f7xx_hal_uart.o(i.HAL_UART_Transmit_DMA) refers to stm32f7xx_hal_uart.o(i.UART_DMATxHalfCplt) for UART_DMATxHalfCplt
    stm32f7xx_hal_uart.o(i.HAL_UART_Transmit_DMA) refers to stm32f7xx_hal_uart.o(i.UART_DMAError) for UART_DMAError
    stm32f7xx_hal_uart.o(i.UART_CheckIdleState) refers to stm32f7xx_hal_uart.o(i.UART_WaitOnFlagUntilTimeout) for UART_WaitOnFlagUntilTimeout
    stm32f7xx_hal_uart.o(i.UART_DMAError) refers to stm32f7xx_hal_uart.o(i.HAL_UART_ErrorCallback) for HAL_UART_ErrorCallback
    stm32f7xx_hal_uart.o(i.UART_DMAReceiveCplt) refers to stm32f7xx_hal_uart.o(i.HAL_UART_RxCpltCallback) for HAL_UART_RxCpltCallback
    stm32f7xx_hal_uart.o(i.UART_DMARxHalfCplt) refers to stm32f7xx_hal_uart.o(i.HAL_UART_RxHalfCpltCallback) for HAL_UART_RxHalfCpltCallback
    stm32f7xx_hal_uart.o(i.UART_DMATransmitCplt) refers to stm32f7xx_hal_uart.o(i.HAL_UART_TxCpltCallback) for HAL_UART_TxCpltCallback
    stm32f7xx_hal_uart.o(i.UART_DMATxHalfCplt) refers to stm32f7xx_hal_uart.o(i.HAL_UART_TxHalfCpltCallback) for HAL_UART_TxHalfCpltCallback
    stm32f7xx_hal_uart.o(i.UART_Receive_IT) refers to stm32f7xx_hal_uart.o(i.HAL_UART_RxCpltCallback) for HAL_UART_RxCpltCallback
    stm32f7xx_hal_uart.o(i.UART_SetConfig) refers to stm32f7xx_hal_rcc.o(i.HAL_RCC_GetPCLK1Freq) for HAL_RCC_GetPCLK1Freq
    stm32f7xx_hal_uart.o(i.UART_SetConfig) refers to stm32f7xx_hal_rcc.o(i.HAL_RCC_GetPCLK2Freq) for HAL_RCC_GetPCLK2Freq
    stm32f7xx_hal_uart.o(i.UART_SetConfig) refers to stm32f7xx_hal_rcc.o(i.HAL_RCC_GetSysClockFreq) for HAL_RCC_GetSysClockFreq
    stm32f7xx_hal_uart.o(i.UART_Transmit_IT) refers to stm32f7xx_hal_uart.o(i.UART_WaitOnFlagUntilTimeout) for UART_WaitOnFlagUntilTimeout
    stm32f7xx_hal_uart.o(i.UART_Transmit_IT) refers to stm32f7xx_hal_uart.o(i.HAL_UART_TxCpltCallback) for HAL_UART_TxCpltCallback
    stm32f7xx_hal_uart.o(i.UART_WaitOnFlagUntilTimeout) refers to stm32f7xx_hal.o(i.HAL_GetTick) for HAL_GetTick
    stm32f7xx_hal_i2s.o(i.HAL_I2S_DMAStop) refers to stm32f7xx_hal_dma.o(i.HAL_DMA_Abort) for HAL_DMA_Abort
    stm32f7xx_hal_i2s.o(i.HAL_I2S_DeInit) refers to stm32f7xx_hal_i2s.o(i.HAL_I2S_MspDeInit) for HAL_I2S_MspDeInit
    stm32f7xx_hal_i2s.o(i.HAL_I2S_IRQHandler) refers to stm32f7xx_hal_i2s.o(i.HAL_I2S_RxCpltCallback) for HAL_I2S_RxCpltCallback
    stm32f7xx_hal_i2s.o(i.HAL_I2S_IRQHandler) refers to stm32f7xx_hal_i2s.o(i.HAL_I2S_TxCpltCallback) for HAL_I2S_TxCpltCallback
    stm32f7xx_hal_i2s.o(i.HAL_I2S_IRQHandler) refers to stm32f7xx_hal_i2s.o(i.HAL_I2S_ErrorCallback) for HAL_I2S_ErrorCallback
    stm32f7xx_hal_i2s.o(i.HAL_I2S_Init) refers to stm32f7xx_hal_i2s.o(i.HAL_I2S_MspInit) for HAL_I2S_MspInit
    stm32f7xx_hal_i2s.o(i.HAL_I2S_Receive) refers to stm32f7xx_hal_i2s.o(i.I2S_WaitFlagStateUntilTimeout) for I2S_WaitFlagStateUntilTimeout
    stm32f7xx_hal_i2s.o(i.HAL_I2S_Receive) refers to stm32f7xx_hal_i2s.o(i.HAL_I2S_ErrorCallback) for HAL_I2S_ErrorCallback
    stm32f7xx_hal_i2s.o(i.HAL_I2S_Receive_DMA) refers to stm32f7xx_hal_dma.o(i.HAL_DMA_Start_IT) for HAL_DMA_Start_IT
    stm32f7xx_hal_i2s.o(i.HAL_I2S_Receive_DMA) refers to stm32f7xx_hal_i2s.o(i.I2S_DMARxHalfCplt) for I2S_DMARxHalfCplt
    stm32f7xx_hal_i2s.o(i.HAL_I2S_Receive_DMA) refers to stm32f7xx_hal_i2s.o(i.I2S_DMARxCplt) for I2S_DMARxCplt
    stm32f7xx_hal_i2s.o(i.HAL_I2S_Receive_DMA) refers to stm32f7xx_hal_i2s.o(i.I2S_DMAError) for I2S_DMAError
    stm32f7xx_hal_i2s.o(i.HAL_I2S_Transmit) refers to stm32f7xx_hal_i2s.o(i.I2S_WaitFlagStateUntilTimeout) for I2S_WaitFlagStateUntilTimeout
    stm32f7xx_hal_i2s.o(i.HAL_I2S_Transmit) refers to stm32f7xx_hal_i2s.o(i.HAL_I2S_ErrorCallback) for HAL_I2S_ErrorCallback
    stm32f7xx_hal_i2s.o(i.HAL_I2S_Transmit_DMA) refers to stm32f7xx_hal_dma.o(i.HAL_DMA_Start_IT) for HAL_DMA_Start_IT
    stm32f7xx_hal_i2s.o(i.HAL_I2S_Transmit_DMA) refers to stm32f7xx_hal_i2s.o(i.I2S_DMATxHalfCplt) for I2S_DMATxHalfCplt
    stm32f7xx_hal_i2s.o(i.HAL_I2S_Transmit_DMA) refers to stm32f7xx_hal_i2s.o(i.I2S_DMATxCplt) for I2S_DMATxCplt
    stm32f7xx_hal_i2s.o(i.HAL_I2S_Transmit_DMA) refers to stm32f7xx_hal_i2s.o(i.I2S_DMAError) for I2S_DMAError
    stm32f7xx_hal_i2s.o(i.I2S_DMAError) refers to stm32f7xx_hal_i2s.o(i.HAL_I2S_ErrorCallback) for HAL_I2S_ErrorCallback
    stm32f7xx_hal_i2s.o(i.I2S_DMARxCplt) refers to stm32f7xx_hal_i2s.o(i.HAL_I2S_RxCpltCallback) for HAL_I2S_RxCpltCallback
    stm32f7xx_hal_i2s.o(i.I2S_DMARxHalfCplt) refers to stm32f7xx_hal_i2s.o(i.HAL_I2S_RxHalfCpltCallback) for HAL_I2S_RxHalfCpltCallback
    stm32f7xx_hal_i2s.o(i.I2S_DMATxCplt) refers to stm32f7xx_hal_i2s.o(i.HAL_I2S_TxCpltCallback) for HAL_I2S_TxCpltCallback
    stm32f7xx_hal_i2s.o(i.I2S_DMATxHalfCplt) refers to stm32f7xx_hal_i2s.o(i.HAL_I2S_TxHalfCpltCallback) for HAL_I2S_TxHalfCpltCallback
    stm32f7xx_hal_i2s.o(i.I2S_WaitFlagStateUntilTimeout) refers to stm32f7xx_hal.o(i.HAL_GetTick) for HAL_GetTick
    wm8994.o(i.CODEC_IO_Write) refers to stm32746g_discovery.o(i.AUDIO_IO_Write) for AUDIO_IO_Write
    wm8994.o(i.wm8994_DeInit) refers to stm32746g_discovery.o(i.AUDIO_IO_DeInit) for AUDIO_IO_DeInit
    wm8994.o(i.wm8994_Init) refers to stm32746g_discovery.o(i.AUDIO_IO_Init) for AUDIO_IO_Init
    wm8994.o(i.wm8994_Init) refers to wm8994.o(i.CODEC_IO_Write) for CODEC_IO_Write
    wm8994.o(i.wm8994_Init) refers to stm32746g_discovery.o(i.AUDIO_IO_Delay) for AUDIO_IO_Delay
    wm8994.o(i.wm8994_Init) refers to wm8994.o(i.wm8994_SetVolume) for wm8994_SetVolume
    wm8994.o(i.wm8994_Init) refers to wm8994.o(.data) for .data
    wm8994.o(i.wm8994_Pause) refers to wm8994.o(i.wm8994_SetMute) for wm8994_SetMute
    wm8994.o(i.wm8994_Pause) refers to wm8994.o(i.CODEC_IO_Write) for CODEC_IO_Write
    wm8994.o(i.wm8994_Play) refers to wm8994.o(i.wm8994_SetMute) for wm8994_SetMute
    wm8994.o(i.wm8994_ReadID) refers to stm32746g_discovery.o(i.AUDIO_IO_Init) for AUDIO_IO_Init
    wm8994.o(i.wm8994_ReadID) refers to stm32746g_discovery.o(i.AUDIO_IO_Read) for AUDIO_IO_Read
    wm8994.o(i.wm8994_Reset) refers to wm8994.o(i.CODEC_IO_Write) for CODEC_IO_Write
    wm8994.o(i.wm8994_Reset) refers to wm8994.o(.data) for .data
    wm8994.o(i.wm8994_Resume) refers to wm8994.o(i.wm8994_SetMute) for wm8994_SetMute
    wm8994.o(i.wm8994_SetFrequency) refers to wm8994.o(i.CODEC_IO_Write) for CODEC_IO_Write
    wm8994.o(i.wm8994_SetMute) refers to wm8994.o(i.CODEC_IO_Write) for CODEC_IO_Write
    wm8994.o(i.wm8994_SetMute) refers to wm8994.o(.data) for .data
    wm8994.o(i.wm8994_SetOutputMode) refers to wm8994.o(i.CODEC_IO_Write) for CODEC_IO_Write
    wm8994.o(i.wm8994_SetVolume) refers to wm8994.o(i.wm8994_SetMute) for wm8994_SetMute
    wm8994.o(i.wm8994_SetVolume) refers to wm8994.o(i.CODEC_IO_Write) for CODEC_IO_Write
    wm8994.o(i.wm8994_SetVolume) refers to wm8994.o(.data) for .data
    wm8994.o(i.wm8994_Stop) refers to wm8994.o(i.wm8994_SetMute) for wm8994_SetMute
    wm8994.o(i.wm8994_Stop) refers to wm8994.o(i.CODEC_IO_Write) for CODEC_IO_Write
    wm8994.o(i.wm8994_Stop) refers to wm8994.o(.data) for .data
    wm8994.o(.data) refers to wm8994.o(i.wm8994_Init) for wm8994_Init
    wm8994.o(.data) refers to wm8994.o(i.wm8994_DeInit) for wm8994_DeInit
    wm8994.o(.data) refers to wm8994.o(i.wm8994_ReadID) for wm8994_ReadID
    wm8994.o(.data) refers to wm8994.o(i.wm8994_Play) for wm8994_Play
    wm8994.o(.data) refers to wm8994.o(i.wm8994_Pause) for wm8994_Pause
    wm8994.o(.data) refers to wm8994.o(i.wm8994_Resume) for wm8994_Resume
    wm8994.o(.data) refers to wm8994.o(i.wm8994_Stop) for wm8994_Stop
    wm8994.o(.data) refers to wm8994.o(i.wm8994_SetFrequency) for wm8994_SetFrequency
    wm8994.o(.data) refers to wm8994.o(i.wm8994_SetVolume) for wm8994_SetVolume
    wm8994.o(.data) refers to wm8994.o(i.wm8994_SetMute) for wm8994_SetMute
    wm8994.o(.data) refers to wm8994.o(i.wm8994_SetOutputMode) for wm8994_SetOutputMode
    wm8994.o(.data) refers to wm8994.o(i.wm8994_Reset) for wm8994_Reset
    startup_stm32f746xx.o(RESET) refers to startup_stm32f746xx.o(STACK) for __initial_sp
    startup_stm32f746xx.o(RESET) refers to startup_stm32f746xx.o(.text) for Reset_Handler
    startup_stm32f746xx.o(RESET) refers to stm32f7xx_it.o(i.NMI_Handler) for NMI_Handler
    startup_stm32f746xx.o(RESET) refers to stm32f7xx_it.o(i.HardFault_Handler) for HardFault_Handler
    startup_stm32f746xx.o(RESET) refers to stm32f7xx_it.o(i.MemManage_Handler) for MemManage_Handler
    startup_stm32f746xx.o(RESET) refers to stm32f7xx_it.o(i.BusFault_Handler) for BusFault_Handler
    startup_stm32f746xx.o(RESET) refers to stm32f7xx_it.o(i.UsageFault_Handler) for UsageFault_Handler
    startup_stm32f746xx.o(RESET) refers to stm32f7xx_it.o(i.SVC_Handler) for SVC_Handler
    startup_stm32f746xx.o(RESET) refers to stm32f7xx_it.o(i.DebugMon_Handler) for DebugMon_Handler
    startup_stm32f746xx.o(RESET) refers to stm32f7xx_it.o(i.PendSV_Handler) for PendSV_Handler
    startup_stm32f746xx.o(RESET) refers to stm32f7xx_it.o(i.SysTick_Handler) for SysTick_Handler
    startup_stm32f746xx.o(RESET) refers to stm32f7xx_it.o(i.DMA2_Stream4_IRQHandler) for DMA2_Stream4_IRQHandler
    startup_stm32f746xx.o(RESET) refers to stm32f7xx_it.o(i.OTG_FS_IRQHandler) for OTG_FS_IRQHandler
    startup_stm32f746xx.o(.text) refers to system_stm32f7xx.o(i.SystemInit) for SystemInit
    startup_stm32f746xx.o(.text) refers to entry.o(.ARM.Collect$$$$00000000) for __main
    usbd_audio_if.o(i.Audio_DeInit) refers to stm32746g_discovery_audio.o(i.BSP_AUDIO_OUT_Stop) for BSP_AUDIO_OUT_Stop
    usbd_audio_if.o(i.Audio_Init) refers to stm32746g_discovery_audio.o(i.BSP_AUDIO_OUT_Init) for BSP_AUDIO_OUT_Init
    usbd_audio_if.o(i.Audio_Init) refers to stm32746g_discovery_audio.o(i.BSP_AUDIO_OUT_SetAudioFrameSlot) for BSP_AUDIO_OUT_SetAudioFrameSlot
    usbd_audio_if.o(i.Audio_MuteCtl) refers to stm32746g_discovery_audio.o(i.BSP_AUDIO_OUT_SetMute) for BSP_AUDIO_OUT_SetMute
    usbd_audio_if.o(i.Audio_PlaybackCmd) refers to stm32746g_discovery_audio.o(i.BSP_AUDIO_OUT_Play) for BSP_AUDIO_OUT_Play
    usbd_audio_if.o(i.Audio_PlaybackCmd) refers to stm32746g_discovery_audio.o(i.BSP_AUDIO_OUT_ChangeBuffer) for BSP_AUDIO_OUT_ChangeBuffer
    usbd_audio_if.o(i.Audio_PlaybackCmd) refers to usbd_audio_if.o(.data) for .data
    usbd_audio_if.o(i.Audio_VolumeCtl) refers to stm32746g_discovery_audio.o(i.BSP_AUDIO_OUT_SetVolume) for BSP_AUDIO_OUT_SetVolume
    usbd_audio_if.o(i.BSP_AUDIO_OUT_HalfTransfer_CallBack) refers to usbd_audio.o(i.USBD_AUDIO_Sync) for USBD_AUDIO_Sync
    usbd_audio_if.o(i.BSP_AUDIO_OUT_HalfTransfer_CallBack) refers to main.o(.bss) for USBD_Device
    usbd_audio_if.o(i.BSP_AUDIO_OUT_TransferComplete_CallBack) refers to usbd_audio.o(i.USBD_AUDIO_Sync) for USBD_AUDIO_Sync
    usbd_audio_if.o(i.BSP_AUDIO_OUT_TransferComplete_CallBack) refers to main.o(.bss) for USBD_Device
    usbd_audio_if.o(.data) refers to usbd_audio_if.o(i.Audio_Init) for Audio_Init
    usbd_audio_if.o(.data) refers to usbd_audio_if.o(i.Audio_DeInit) for Audio_DeInit
    usbd_audio_if.o(.data) refers to usbd_audio_if.o(i.Audio_PlaybackCmd) for Audio_PlaybackCmd
    usbd_audio_if.o(.data) refers to usbd_audio_if.o(i.Audio_VolumeCtl) for Audio_VolumeCtl
    usbd_audio_if.o(.data) refers to usbd_audio_if.o(i.Audio_MuteCtl) for Audio_MuteCtl
    usbd_audio_if.o(.data) refers to usbd_audio_if.o(i.Audio_PeriodicTC) for Audio_PeriodicTC
    usbd_audio_if.o(.data) refers to usbd_audio_if.o(i.Audio_GetState) for Audio_GetState
    usbd_conf.o(i.HAL_PCD_ConnectCallback) refers to usbd_core.o(i.USBD_LL_DevConnected) for USBD_LL_DevConnected
    usbd_conf.o(i.HAL_PCD_DataInStageCallback) refers to usbd_core.o(i.USBD_LL_DataInStage) for USBD_LL_DataInStage
    usbd_conf.o(i.HAL_PCD_DataOutStageCallback) refers to usbd_core.o(i.USBD_LL_DataOutStage) for USBD_LL_DataOutStage
    usbd_conf.o(i.HAL_PCD_DisconnectCallback) refers to usbd_core.o(i.USBD_LL_DevDisconnected) for USBD_LL_DevDisconnected
    usbd_conf.o(i.HAL_PCD_ISOINIncompleteCallback) refers to usbd_core.o(i.USBD_LL_IsoINIncomplete) for USBD_LL_IsoINIncomplete
    usbd_conf.o(i.HAL_PCD_ISOOUTIncompleteCallback) refers to usbd_core.o(i.USBD_LL_IsoOUTIncomplete) for USBD_LL_IsoOUTIncomplete
    usbd_conf.o(i.HAL_PCD_MspInit) refers to stm32f7xx_hal_gpio.o(i.HAL_GPIO_Init) for HAL_GPIO_Init
    usbd_conf.o(i.HAL_PCD_MspInit) refers to stm32f7xx_hal_cortex.o(i.HAL_NVIC_SetPriority) for HAL_NVIC_SetPriority
    usbd_conf.o(i.HAL_PCD_MspInit) refers to stm32f7xx_hal_cortex.o(i.HAL_NVIC_EnableIRQ) for HAL_NVIC_EnableIRQ
    usbd_conf.o(i.HAL_PCD_ResetCallback) refers to usbd_core.o(i.USBD_LL_Reset) for USBD_LL_Reset
    usbd_conf.o(i.HAL_PCD_ResetCallback) refers to usbd_core.o(i.USBD_LL_SetSpeed) for USBD_LL_SetSpeed
    usbd_conf.o(i.HAL_PCD_ResumeCallback) refers to usbd_core.o(i.USBD_LL_Resume) for USBD_LL_Resume
    usbd_conf.o(i.HAL_PCD_SOFCallback) refers to usbd_core.o(i.USBD_LL_SOF) for USBD_LL_SOF
    usbd_conf.o(i.HAL_PCD_SetupStageCallback) refers to usbd_core.o(i.USBD_LL_SetupStage) for USBD_LL_SetupStage
    usbd_conf.o(i.HAL_PCD_SuspendCallback) refers to usbd_core.o(i.USBD_LL_Suspend) for USBD_LL_Suspend
    usbd_conf.o(i.USBD_LL_ClearStallEP) refers to stm32f7xx_hal_pcd.o(i.HAL_PCD_EP_ClrStall) for HAL_PCD_EP_ClrStall
    usbd_conf.o(i.USBD_LL_CloseEP) refers to stm32f7xx_hal_pcd.o(i.HAL_PCD_EP_Close) for HAL_PCD_EP_Close
    usbd_conf.o(i.USBD_LL_DeInit) refers to stm32f7xx_hal_pcd.o(i.HAL_PCD_DeInit) for HAL_PCD_DeInit
    usbd_conf.o(i.USBD_LL_Delay) refers to stm32f7xx_hal.o(i.HAL_Delay) for HAL_Delay
    usbd_conf.o(i.USBD_LL_FlushEP) refers to stm32f7xx_hal_pcd.o(i.HAL_PCD_EP_Flush) for HAL_PCD_EP_Flush
    usbd_conf.o(i.USBD_LL_GetRxDataSize) refers to stm32f7xx_hal_pcd.o(i.HAL_PCD_EP_GetRxCount) for HAL_PCD_EP_GetRxCount
    usbd_conf.o(i.USBD_LL_Init) refers to stm32f7xx_hal_pcd.o(i.HAL_PCD_Init) for HAL_PCD_Init
    usbd_conf.o(i.USBD_LL_Init) refers to stm32f7xx_hal_pcd_ex.o(i.HAL_PCDEx_SetRxFiFo) for HAL_PCDEx_SetRxFiFo
    usbd_conf.o(i.USBD_LL_Init) refers to stm32f7xx_hal_pcd_ex.o(i.HAL_PCDEx_SetTxFiFo) for HAL_PCDEx_SetTxFiFo
    usbd_conf.o(i.USBD_LL_Init) refers to usbd_conf.o(.bss) for .bss
    usbd_conf.o(i.USBD_LL_OpenEP) refers to stm32f7xx_hal_pcd.o(i.HAL_PCD_EP_Open) for HAL_PCD_EP_Open
    usbd_conf.o(i.USBD_LL_PrepareReceive) refers to stm32f7xx_hal_pcd.o(i.HAL_PCD_EP_Receive) for HAL_PCD_EP_Receive
    usbd_conf.o(i.USBD_LL_SetUSBAddress) refers to stm32f7xx_hal_pcd.o(i.HAL_PCD_SetAddress) for HAL_PCD_SetAddress
    usbd_conf.o(i.USBD_LL_StallEP) refers to stm32f7xx_hal_pcd.o(i.HAL_PCD_EP_SetStall) for HAL_PCD_EP_SetStall
    usbd_conf.o(i.USBD_LL_Start) refers to stm32f7xx_hal_pcd.o(i.HAL_PCD_Start) for HAL_PCD_Start
    usbd_conf.o(i.USBD_LL_Stop) refers to stm32f7xx_hal_pcd.o(i.HAL_PCD_Stop) for HAL_PCD_Stop
    usbd_conf.o(i.USBD_LL_Transmit) refers to stm32f7xx_hal_pcd.o(i.HAL_PCD_EP_Transmit) for HAL_PCD_EP_Transmit
    usbd_desc.o(i.USBD_AUDIO_ConfigStrDescriptor) refers to usbd_ctlreq.o(i.USBD_GetString) for USBD_GetString
    usbd_desc.o(i.USBD_AUDIO_ConfigStrDescriptor) refers to usbd_desc.o(.bss) for .bss
    usbd_desc.o(i.USBD_AUDIO_DeviceDescriptor) refers to usbd_desc.o(.data) for .data
    usbd_desc.o(i.USBD_AUDIO_InterfaceStrDescriptor) refers to usbd_ctlreq.o(i.USBD_GetString) for USBD_GetString
    usbd_desc.o(i.USBD_AUDIO_InterfaceStrDescriptor) refers to usbd_desc.o(.bss) for .bss
    usbd_desc.o(i.USBD_AUDIO_LangIDStrDescriptor) refers to usbd_desc.o(.data) for .data
    usbd_desc.o(i.USBD_AUDIO_ManufacturerStrDescriptor) refers to usbd_ctlreq.o(i.USBD_GetString) for USBD_GetString
    usbd_desc.o(i.USBD_AUDIO_ManufacturerStrDescriptor) refers to usbd_desc.o(.bss) for .bss
    usbd_desc.o(i.USBD_AUDIO_ProductStrDescriptor) refers to usbd_ctlreq.o(i.USBD_GetString) for USBD_GetString
    usbd_desc.o(i.USBD_AUDIO_ProductStrDescriptor) refers to usbd_desc.o(.bss) for .bss
    usbd_desc.o(i.USBD_AUDIO_SerialStrDescriptor) refers to usbd_desc.o(i.IntToUnicode) for IntToUnicode
    usbd_desc.o(i.USBD_AUDIO_SerialStrDescriptor) refers to usbd_desc.o(.data) for .data
    usbd_desc.o(.data) refers to usbd_desc.o(i.USBD_AUDIO_DeviceDescriptor) for USBD_AUDIO_DeviceDescriptor
    usbd_desc.o(.data) refers to usbd_desc.o(i.USBD_AUDIO_LangIDStrDescriptor) for USBD_AUDIO_LangIDStrDescriptor
    usbd_desc.o(.data) refers to usbd_desc.o(i.USBD_AUDIO_ManufacturerStrDescriptor) for USBD_AUDIO_ManufacturerStrDescriptor
    usbd_desc.o(.data) refers to usbd_desc.o(i.USBD_AUDIO_ProductStrDescriptor) for USBD_AUDIO_ProductStrDescriptor
    usbd_desc.o(.data) refers to usbd_desc.o(i.USBD_AUDIO_SerialStrDescriptor) for USBD_AUDIO_SerialStrDescriptor
    usbd_desc.o(.data) refers to usbd_desc.o(i.USBD_AUDIO_ConfigStrDescriptor) for USBD_AUDIO_ConfigStrDescriptor
    usbd_desc.o(.data) refers to usbd_desc.o(i.USBD_AUDIO_InterfaceStrDescriptor) for USBD_AUDIO_InterfaceStrDescriptor
    main.o(i.BSP_AUDIO_OUT_ClockConfig) refers to stm32f7xx_hal_rcc_ex.o(i.HAL_RCCEx_GetPeriphCLKConfig) for HAL_RCCEx_GetPeriphCLKConfig
    main.o(i.BSP_AUDIO_OUT_ClockConfig) refers to stm32f7xx_hal_rcc_ex.o(i.HAL_RCCEx_PeriphCLKConfig) for HAL_RCCEx_PeriphCLKConfig
    main.o(i.HAL_UART_MspDeInit) refers to stm32f7xx_hal_gpio.o(i.HAL_GPIO_DeInit) for HAL_GPIO_DeInit
    main.o(i.HAL_UART_MspInit) refers to stm32f7xx_hal_gpio.o(i.HAL_GPIO_Init) for HAL_GPIO_Init
    main.o(i.main) refers to main.o(i.CPU_CACHE_Enable) for CPU_CACHE_Enable
    main.o(i.main) refers to stm32f7xx_hal.o(i.HAL_Init) for HAL_Init
    main.o(i.main) refers to stm32f7xx_hal_rcc.o(i.HAL_RCC_OscConfig) for HAL_RCC_OscConfig
    main.o(i.main) refers to stm32f7xx_hal_pwr_ex.o(i.HAL_PWREx_EnableOverDrive) for HAL_PWREx_EnableOverDrive
    main.o(i.main) refers to stm32f7xx_hal_rcc.o(i.HAL_RCC_ClockConfig) for HAL_RCC_ClockConfig
    main.o(i.main) refers to stm32746g_discovery.o(i.BSP_LED_Init) for BSP_LED_Init
    main.o(i.main) refers to stm32f7xx_hal_uart.o(i.HAL_UART_DeInit) for HAL_UART_DeInit
    main.o(i.main) refers to stm32f7xx_hal_uart.o(i.HAL_UART_Init) for HAL_UART_Init
    main.o(i.main) refers to usbd_core.o(i.USBD_Init) for USBD_Init
    main.o(i.main) refers to usbd_core.o(i.USBD_RegisterClass) for USBD_RegisterClass
    main.o(i.main) refers to usbd_audio.o(i.USBD_AUDIO_RegisterInterface) for USBD_AUDIO_RegisterInterface
    main.o(i.main) refers to usbd_core.o(i.USBD_Start) for USBD_Start
    main.o(i.main) refers to stm32f7xx_hal_uart.o(i.HAL_UART_Transmit) for HAL_UART_Transmit
    main.o(i.main) refers to stm32746g_discovery.o(i.BSP_LED_Toggle) for BSP_LED_Toggle
    main.o(i.main) refers to main.o(.bss) for .bss
    main.o(i.main) refers to usbd_desc.o(.data) for AUDIO_Desc
    main.o(i.main) refers to usbd_audio.o(.data) for USBD_AUDIO
    main.o(i.main) refers to usbd_audio_if.o(.data) for USBD_AUDIO_fops
    main.o(i.main) refers to main.o(.data) for .data
    main.o(i.main) refers to usbd_audio_if.o(.data) for Buffer_USART_Senden
    stm32f7xx_it.o(i.DMA2_Stream4_IRQHandler) refers to stm32f7xx_hal_dma.o(i.HAL_DMA_IRQHandler) for HAL_DMA_IRQHandler
    stm32f7xx_it.o(i.DMA2_Stream4_IRQHandler) refers to stm32746g_discovery_audio.o(.bss) for haudio_out_sai
    stm32f7xx_it.o(i.OTG_FS_IRQHandler) refers to stm32f7xx_hal_pcd.o(i.HAL_PCD_IRQHandler) for HAL_PCD_IRQHandler
    stm32f7xx_it.o(i.OTG_FS_IRQHandler) refers to usbd_conf.o(.bss) for hpcd
    stm32f7xx_it.o(i.SysTick_Handler) refers to stm32f7xx_hal.o(i.HAL_IncTick) for HAL_IncTick
    usbd_ctlreq.o(i.USBD_CtlError) refers to usbd_conf.o(i.USBD_LL_StallEP) for USBD_LL_StallEP
    usbd_ctlreq.o(i.USBD_GetDescriptor) refers to usbd_ctlreq.o(i.USBD_CtlError) for USBD_CtlError
    usbd_ctlreq.o(i.USBD_GetDescriptor) refers to usbd_ioreq.o(i.USBD_CtlSendData) for USBD_CtlSendData
    usbd_ctlreq.o(i.USBD_SetConfig) refers to usbd_core.o(i.USBD_ClrClassConfig) for USBD_ClrClassConfig
    usbd_ctlreq.o(i.USBD_SetConfig) refers to usbd_core.o(i.USBD_SetClassConfig) for USBD_SetClassConfig
    usbd_ctlreq.o(i.USBD_SetConfig) refers to usbd_ioreq.o(i.USBD_CtlSendStatus) for USBD_CtlSendStatus
    usbd_ctlreq.o(i.USBD_SetConfig) refers to usbd_ctlreq.o(i.USBD_CtlError) for USBD_CtlError
    usbd_ctlreq.o(i.USBD_SetConfig) refers to usbd_ctlreq.o(.data) for .data
    usbd_ctlreq.o(i.USBD_StdDevReq) refers to usbd_ctlreq.o(i.USBD_GetDescriptor) for USBD_GetDescriptor
    usbd_ctlreq.o(i.USBD_StdDevReq) refers to usbd_conf.o(i.USBD_LL_SetUSBAddress) for USBD_LL_SetUSBAddress
    usbd_ctlreq.o(i.USBD_StdDevReq) refers to usbd_ioreq.o(i.USBD_CtlSendStatus) for USBD_CtlSendStatus
    usbd_ctlreq.o(i.USBD_StdDevReq) refers to usbd_ctlreq.o(i.USBD_SetConfig) for USBD_SetConfig
    usbd_ctlreq.o(i.USBD_StdDevReq) refers to usbd_ctlreq.o(i.USBD_CtlError) for USBD_CtlError
    usbd_ctlreq.o(i.USBD_StdDevReq) refers to usbd_ioreq.o(i.USBD_CtlSendData) for USBD_CtlSendData
    usbd_ctlreq.o(i.USBD_StdEPReq) refers to usbd_conf.o(i.USBD_LL_StallEP) for USBD_LL_StallEP
    usbd_ctlreq.o(i.USBD_StdEPReq) refers to usbd_conf.o(i.USBD_LL_ClearStallEP) for USBD_LL_ClearStallEP
    usbd_ctlreq.o(i.USBD_StdEPReq) refers to usbd_ioreq.o(i.USBD_CtlSendStatus) for USBD_CtlSendStatus
    usbd_ctlreq.o(i.USBD_StdEPReq) refers to usbd_ctlreq.o(i.USBD_CtlError) for USBD_CtlError
    usbd_ctlreq.o(i.USBD_StdEPReq) refers to usbd_conf.o(i.USBD_LL_IsStallEP) for USBD_LL_IsStallEP
    usbd_ctlreq.o(i.USBD_StdEPReq) refers to usbd_ioreq.o(i.USBD_CtlSendData) for USBD_CtlSendData
    usbd_ctlreq.o(i.USBD_StdItfReq) refers to usbd_ioreq.o(i.USBD_CtlSendStatus) for USBD_CtlSendStatus
    usbd_ctlreq.o(i.USBD_StdItfReq) refers to usbd_ctlreq.o(i.USBD_CtlError) for USBD_CtlError
    usbd_ioreq.o(i.USBD_CtlContinueRx) refers to usbd_conf.o(i.USBD_LL_PrepareReceive) for USBD_LL_PrepareReceive
    usbd_ioreq.o(i.USBD_CtlContinueSendData) refers to usbd_conf.o(i.USBD_LL_Transmit) for USBD_LL_Transmit
    usbd_ioreq.o(i.USBD_CtlPrepareRx) refers to usbd_conf.o(i.USBD_LL_PrepareReceive) for USBD_LL_PrepareReceive
    usbd_ioreq.o(i.USBD_CtlReceiveStatus) refers to usbd_conf.o(i.USBD_LL_PrepareReceive) for USBD_LL_PrepareReceive
    usbd_ioreq.o(i.USBD_CtlSendData) refers to usbd_conf.o(i.USBD_LL_Transmit) for USBD_LL_Transmit
    usbd_ioreq.o(i.USBD_CtlSendStatus) refers to usbd_conf.o(i.USBD_LL_Transmit) for USBD_LL_Transmit
    usbd_ioreq.o(i.USBD_GetRxCount) refers to usbd_conf.o(i.USBD_LL_GetRxDataSize) for USBD_LL_GetRxDataSize
    usbd_core.o(i.USBD_DeInit) refers to usbd_conf.o(i.USBD_LL_Stop) for USBD_LL_Stop
    usbd_core.o(i.USBD_DeInit) refers to usbd_conf.o(i.USBD_LL_DeInit) for USBD_LL_DeInit
    usbd_core.o(i.USBD_Init) refers to usbd_conf.o(i.USBD_LL_Init) for USBD_LL_Init
    usbd_core.o(i.USBD_LL_DataInStage) refers to usbd_ioreq.o(i.USBD_CtlContinueSendData) for USBD_CtlContinueSendData
    usbd_core.o(i.USBD_LL_DataInStage) refers to usbd_conf.o(i.USBD_LL_PrepareReceive) for USBD_LL_PrepareReceive
    usbd_core.o(i.USBD_LL_DataInStage) refers to usbd_ioreq.o(i.USBD_CtlReceiveStatus) for USBD_CtlReceiveStatus
    usbd_core.o(i.USBD_LL_DataOutStage) refers to usbd_ioreq.o(i.USBD_CtlContinueRx) for USBD_CtlContinueRx
    usbd_core.o(i.USBD_LL_DataOutStage) refers to usbd_ioreq.o(i.USBD_CtlSendStatus) for USBD_CtlSendStatus
    usbd_core.o(i.USBD_LL_Reset) refers to usbd_conf.o(i.USBD_LL_OpenEP) for USBD_LL_OpenEP
    usbd_core.o(i.USBD_LL_SetupStage) refers to usbd_ctlreq.o(i.USBD_ParseSetupRequest) for USBD_ParseSetupRequest
    usbd_core.o(i.USBD_LL_SetupStage) refers to usbd_conf.o(i.USBD_LL_StallEP) for USBD_LL_StallEP
    usbd_core.o(i.USBD_LL_SetupStage) refers to usbd_ctlreq.o(i.USBD_StdDevReq) for USBD_StdDevReq
    usbd_core.o(i.USBD_LL_SetupStage) refers to usbd_ctlreq.o(i.USBD_StdItfReq) for USBD_StdItfReq
    usbd_core.o(i.USBD_LL_SetupStage) refers to usbd_ctlreq.o(i.USBD_StdEPReq) for USBD_StdEPReq
    usbd_core.o(i.USBD_Start) refers to usbd_conf.o(i.USBD_LL_Start) for USBD_LL_Start
    usbd_core.o(i.USBD_Stop) refers to usbd_conf.o(i.USBD_LL_Stop) for USBD_LL_Stop
    stm32746g_discovery_audio.o(i.BSP_AUDIO_IN_DeInit) refers to stm32746g_discovery_audio.o(i.SAIx_In_DeInit) for SAIx_In_DeInit
    stm32746g_discovery_audio.o(i.BSP_AUDIO_IN_DeInit) refers to stm32746g_discovery_audio.o(i.BSP_AUDIO_IN_MspDeInit) for BSP_AUDIO_IN_MspDeInit
    stm32746g_discovery_audio.o(i.BSP_AUDIO_IN_DeInit) refers to stm32746g_discovery_audio.o(.bss) for .bss
    stm32746g_discovery_audio.o(i.BSP_AUDIO_IN_Init) refers to stm32746g_discovery_audio.o(i.SAIx_In_DeInit) for SAIx_In_DeInit
    stm32746g_discovery_audio.o(i.BSP_AUDIO_IN_Init) refers to main.o(i.BSP_AUDIO_OUT_ClockConfig) for BSP_AUDIO_OUT_ClockConfig
    stm32746g_discovery_audio.o(i.BSP_AUDIO_IN_Init) refers to stm32f7xx_hal_sai.o(i.HAL_SAI_GetState) for HAL_SAI_GetState
    stm32746g_discovery_audio.o(i.BSP_AUDIO_IN_Init) refers to stm32746g_discovery_audio.o(i.BSP_AUDIO_OUT_MspInit) for BSP_AUDIO_OUT_MspInit
    stm32746g_discovery_audio.o(i.BSP_AUDIO_IN_Init) refers to stm32746g_discovery_audio.o(i.BSP_AUDIO_IN_MspInit) for BSP_AUDIO_IN_MspInit
    stm32746g_discovery_audio.o(i.BSP_AUDIO_IN_Init) refers to stm32746g_discovery_audio.o(i.SAIx_In_Init) for SAIx_In_Init
    stm32746g_discovery_audio.o(i.BSP_AUDIO_IN_Init) refers to stm32746g_discovery_audio.o(.bss) for .bss
    stm32746g_discovery_audio.o(i.BSP_AUDIO_IN_Init) refers to wm8994.o(.data) for wm8994_drv
    stm32746g_discovery_audio.o(i.BSP_AUDIO_IN_Init) refers to stm32746g_discovery_audio.o(.data) for .data
    stm32746g_discovery_audio.o(i.BSP_AUDIO_IN_MspDeInit) refers to stm32f7xx_hal_cortex.o(i.HAL_NVIC_DisableIRQ) for HAL_NVIC_DisableIRQ
    stm32746g_discovery_audio.o(i.BSP_AUDIO_IN_MspDeInit) refers to stm32f7xx_hal_dma.o(i.HAL_DMA_DeInit) for HAL_DMA_DeInit
    stm32746g_discovery_audio.o(i.BSP_AUDIO_IN_MspDeInit) refers to stm32f7xx_hal_gpio.o(i.HAL_GPIO_DeInit) for HAL_GPIO_DeInit
    stm32746g_discovery_audio.o(i.BSP_AUDIO_IN_MspDeInit) refers to stm32746g_discovery_audio.o(.bss) for .bss
    stm32746g_discovery_audio.o(i.BSP_AUDIO_IN_MspInit) refers to stm32f7xx_hal_gpio.o(i.HAL_GPIO_Init) for HAL_GPIO_Init
    stm32746g_discovery_audio.o(i.BSP_AUDIO_IN_MspInit) refers to stm32f7xx_hal_dma.o(i.HAL_DMA_DeInit) for HAL_DMA_DeInit
    stm32746g_discovery_audio.o(i.BSP_AUDIO_IN_MspInit) refers to stm32f7xx_hal_dma.o(i.HAL_DMA_Init) for HAL_DMA_Init
    stm32746g_discovery_audio.o(i.BSP_AUDIO_IN_MspInit) refers to stm32f7xx_hal_cortex.o(i.HAL_NVIC_SetPriority) for HAL_NVIC_SetPriority
    stm32746g_discovery_audio.o(i.BSP_AUDIO_IN_MspInit) refers to stm32f7xx_hal_cortex.o(i.HAL_NVIC_EnableIRQ) for HAL_NVIC_EnableIRQ
    stm32746g_discovery_audio.o(i.BSP_AUDIO_IN_MspInit) refers to stm32746g_discovery_audio.o(.bss) for .bss
    stm32746g_discovery_audio.o(i.BSP_AUDIO_IN_OUT_Init) refers to stm32746g_discovery_audio.o(i.SAIx_In_DeInit) for SAIx_In_DeInit
    stm32746g_discovery_audio.o(i.BSP_AUDIO_IN_OUT_Init) refers to stm32746g_discovery_audio.o(i.SAIx_Out_DeInit) for SAIx_Out_DeInit
    stm32746g_discovery_audio.o(i.BSP_AUDIO_IN_OUT_Init) refers to main.o(i.BSP_AUDIO_OUT_ClockConfig) for BSP_AUDIO_OUT_ClockConfig
    stm32746g_discovery_audio.o(i.BSP_AUDIO_IN_OUT_Init) refers to stm32f7xx_hal_sai.o(i.HAL_SAI_GetState) for HAL_SAI_GetState
    stm32746g_discovery_audio.o(i.BSP_AUDIO_IN_OUT_Init) refers to stm32746g_discovery_audio.o(i.BSP_AUDIO_IN_MspInit) for BSP_AUDIO_IN_MspInit
    stm32746g_discovery_audio.o(i.BSP_AUDIO_IN_OUT_Init) refers to stm32746g_discovery_audio.o(i.BSP_AUDIO_OUT_MspInit) for BSP_AUDIO_OUT_MspInit
    stm32746g_discovery_audio.o(i.BSP_AUDIO_IN_OUT_Init) refers to stm32746g_discovery_audio.o(i.SAIx_In_Init) for SAIx_In_Init
    stm32746g_discovery_audio.o(i.BSP_AUDIO_IN_OUT_Init) refers to stm32746g_discovery_audio.o(.bss) for .bss
    stm32746g_discovery_audio.o(i.BSP_AUDIO_IN_OUT_Init) refers to wm8994.o(.data) for wm8994_drv
    stm32746g_discovery_audio.o(i.BSP_AUDIO_IN_OUT_Init) refers to stm32746g_discovery_audio.o(.data) for .data
    stm32746g_discovery_audio.o(i.BSP_AUDIO_IN_Pause) refers to stm32f7xx_hal_sai.o(i.HAL_SAI_DMAPause) for HAL_SAI_DMAPause
    stm32746g_discovery_audio.o(i.BSP_AUDIO_IN_Pause) refers to stm32746g_discovery_audio.o(.bss) for .bss
    stm32746g_discovery_audio.o(i.BSP_AUDIO_IN_Record) refers to stm32f7xx_hal_sai.o(i.HAL_SAI_Receive_DMA) for HAL_SAI_Receive_DMA
    stm32746g_discovery_audio.o(i.BSP_AUDIO_IN_Record) refers to stm32746g_discovery_audio.o(.bss) for .bss
    stm32746g_discovery_audio.o(i.BSP_AUDIO_IN_Resume) refers to stm32f7xx_hal_sai.o(i.HAL_SAI_DMAResume) for HAL_SAI_DMAResume
    stm32746g_discovery_audio.o(i.BSP_AUDIO_IN_Resume) refers to stm32746g_discovery_audio.o(.bss) for .bss
    stm32746g_discovery_audio.o(i.BSP_AUDIO_IN_SetVolume) refers to stm32746g_discovery_audio.o(.data) for .data
    stm32746g_discovery_audio.o(i.BSP_AUDIO_IN_Stop) refers to stm32f7xx_hal_sai.o(i.HAL_SAI_DMAStop) for HAL_SAI_DMAStop
    stm32746g_discovery_audio.o(i.BSP_AUDIO_IN_Stop) refers to stm32f7xx_hal.o(i.HAL_Delay) for HAL_Delay
    stm32746g_discovery_audio.o(i.BSP_AUDIO_IN_Stop) refers to stm32746g_discovery_audio.o(.bss) for .bss
    stm32746g_discovery_audio.o(i.BSP_AUDIO_IN_Stop) refers to stm32746g_discovery_audio.o(.data) for .data
    stm32746g_discovery_audio.o(i.BSP_AUDIO_OUT_ChangeBuffer) refers to stm32f7xx_hal_sai.o(i.HAL_SAI_Transmit_DMA) for HAL_SAI_Transmit_DMA
    stm32746g_discovery_audio.o(i.BSP_AUDIO_OUT_ChangeBuffer) refers to stm32746g_discovery_audio.o(.bss) for .bss
    stm32746g_discovery_audio.o(i.BSP_AUDIO_OUT_ClockConfig) refers to stm32f7xx_hal_rcc_ex.o(i.HAL_RCCEx_GetPeriphCLKConfig) for HAL_RCCEx_GetPeriphCLKConfig
    stm32746g_discovery_audio.o(i.BSP_AUDIO_OUT_ClockConfig) refers to stm32f7xx_hal_rcc_ex.o(i.HAL_RCCEx_PeriphCLKConfig) for HAL_RCCEx_PeriphCLKConfig
    stm32746g_discovery_audio.o(i.BSP_AUDIO_OUT_DeInit) refers to stm32746g_discovery_audio.o(i.SAIx_Out_DeInit) for SAIx_Out_DeInit
    stm32746g_discovery_audio.o(i.BSP_AUDIO_OUT_DeInit) refers to stm32746g_discovery_audio.o(i.BSP_AUDIO_OUT_MspDeInit) for BSP_AUDIO_OUT_MspDeInit
    stm32746g_discovery_audio.o(i.BSP_AUDIO_OUT_DeInit) refers to stm32746g_discovery_audio.o(.bss) for .bss
    stm32746g_discovery_audio.o(i.BSP_AUDIO_OUT_Init) refers to stm32746g_discovery_audio.o(i.SAIx_Out_DeInit) for SAIx_Out_DeInit
    stm32746g_discovery_audio.o(i.BSP_AUDIO_OUT_Init) refers to main.o(i.BSP_AUDIO_OUT_ClockConfig) for BSP_AUDIO_OUT_ClockConfig
    stm32746g_discovery_audio.o(i.BSP_AUDIO_OUT_Init) refers to stm32f7xx_hal_sai.o(i.HAL_SAI_GetState) for HAL_SAI_GetState
    stm32746g_discovery_audio.o(i.BSP_AUDIO_OUT_Init) refers to stm32746g_discovery_audio.o(i.BSP_AUDIO_OUT_MspInit) for BSP_AUDIO_OUT_MspInit
    stm32746g_discovery_audio.o(i.BSP_AUDIO_OUT_Init) refers to stm32746g_discovery_audio.o(i.SAIx_Out_Init) for SAIx_Out_Init
    stm32746g_discovery_audio.o(i.BSP_AUDIO_OUT_Init) refers to stm32746g_discovery_audio.o(.bss) for .bss
    stm32746g_discovery_audio.o(i.BSP_AUDIO_OUT_Init) refers to wm8994.o(.data) for wm8994_drv
    stm32746g_discovery_audio.o(i.BSP_AUDIO_OUT_Init) refers to stm32746g_discovery_audio.o(.data) for .data
    stm32746g_discovery_audio.o(i.BSP_AUDIO_OUT_MspDeInit) refers to stm32f7xx_hal_cortex.o(i.HAL_NVIC_DisableIRQ) for HAL_NVIC_DisableIRQ
    stm32746g_discovery_audio.o(i.BSP_AUDIO_OUT_MspDeInit) refers to stm32f7xx_hal_dma.o(i.HAL_DMA_DeInit) for HAL_DMA_DeInit
    stm32746g_discovery_audio.o(i.BSP_AUDIO_OUT_MspDeInit) refers to stm32f7xx_hal_gpio.o(i.HAL_GPIO_DeInit) for HAL_GPIO_DeInit
    stm32746g_discovery_audio.o(i.BSP_AUDIO_OUT_MspInit) refers to stm32f7xx_hal_gpio.o(i.HAL_GPIO_Init) for HAL_GPIO_Init
    stm32746g_discovery_audio.o(i.BSP_AUDIO_OUT_MspInit) refers to stm32f7xx_hal_dma.o(i.HAL_DMA_DeInit) for HAL_DMA_DeInit
    stm32746g_discovery_audio.o(i.BSP_AUDIO_OUT_MspInit) refers to stm32f7xx_hal_dma.o(i.HAL_DMA_Init) for HAL_DMA_Init
    stm32746g_discovery_audio.o(i.BSP_AUDIO_OUT_MspInit) refers to stm32f7xx_hal_cortex.o(i.HAL_NVIC_SetPriority) for HAL_NVIC_SetPriority
    stm32746g_discovery_audio.o(i.BSP_AUDIO_OUT_MspInit) refers to stm32f7xx_hal_cortex.o(i.HAL_NVIC_EnableIRQ) for HAL_NVIC_EnableIRQ
    stm32746g_discovery_audio.o(i.BSP_AUDIO_OUT_MspInit) refers to stm32746g_discovery_audio.o(.bss) for .bss
    stm32746g_discovery_audio.o(i.BSP_AUDIO_OUT_Pause) refers to stm32f7xx_hal_sai.o(i.HAL_SAI_DMAPause) for HAL_SAI_DMAPause
    stm32746g_discovery_audio.o(i.BSP_AUDIO_OUT_Pause) refers to stm32746g_discovery_audio.o(.data) for .data
    stm32746g_discovery_audio.o(i.BSP_AUDIO_OUT_Pause) refers to stm32746g_discovery_audio.o(.bss) for .bss
    stm32746g_discovery_audio.o(i.BSP_AUDIO_OUT_Play) refers to stm32f7xx_hal_sai.o(i.HAL_SAI_Transmit_DMA) for HAL_SAI_Transmit_DMA
    stm32746g_discovery_audio.o(i.BSP_AUDIO_OUT_Play) refers to stm32746g_discovery_audio.o(.data) for .data
    stm32746g_discovery_audio.o(i.BSP_AUDIO_OUT_Play) refers to stm32746g_discovery_audio.o(.bss) for .bss
    stm32746g_discovery_audio.o(i.BSP_AUDIO_OUT_Resume) refers to stm32f7xx_hal_sai.o(i.HAL_SAI_DMAResume) for HAL_SAI_DMAResume
    stm32746g_discovery_audio.o(i.BSP_AUDIO_OUT_Resume) refers to stm32746g_discovery_audio.o(.data) for .data
    stm32746g_discovery_audio.o(i.BSP_AUDIO_OUT_Resume) refers to stm32746g_discovery_audio.o(.bss) for .bss
    stm32746g_discovery_audio.o(i.BSP_AUDIO_OUT_SetAudioFrameSlot) refers to stm32f7xx_hal_sai.o(i.HAL_SAI_Init) for HAL_SAI_Init
    stm32746g_discovery_audio.o(i.BSP_AUDIO_OUT_SetAudioFrameSlot) refers to stm32746g_discovery_audio.o(.bss) for .bss
    stm32746g_discovery_audio.o(i.BSP_AUDIO_OUT_SetFrequency) refers to main.o(i.BSP_AUDIO_OUT_ClockConfig) for BSP_AUDIO_OUT_ClockConfig
    stm32746g_discovery_audio.o(i.BSP_AUDIO_OUT_SetFrequency) refers to stm32f7xx_hal_sai.o(i.HAL_SAI_Init) for HAL_SAI_Init
    stm32746g_discovery_audio.o(i.BSP_AUDIO_OUT_SetFrequency) refers to stm32746g_discovery_audio.o(.bss) for .bss
    stm32746g_discovery_audio.o(i.BSP_AUDIO_OUT_SetMute) refers to stm32746g_discovery_audio.o(.data) for .data
    stm32746g_discovery_audio.o(i.BSP_AUDIO_OUT_SetOutputMode) refers to stm32746g_discovery_audio.o(.data) for .data
    stm32746g_discovery_audio.o(i.BSP_AUDIO_OUT_SetVolume) refers to stm32746g_discovery_audio.o(.data) for .data
    stm32746g_discovery_audio.o(i.BSP_AUDIO_OUT_Stop) refers to stm32f7xx_hal_sai.o(i.HAL_SAI_DMAStop) for HAL_SAI_DMAStop
    stm32746g_discovery_audio.o(i.BSP_AUDIO_OUT_Stop) refers to stm32f7xx_hal.o(i.HAL_Delay) for HAL_Delay
    stm32746g_discovery_audio.o(i.BSP_AUDIO_OUT_Stop) refers to stm32746g_discovery_audio.o(.bss) for .bss
    stm32746g_discovery_audio.o(i.BSP_AUDIO_OUT_Stop) refers to stm32746g_discovery_audio.o(.data) for .data
    stm32746g_discovery_audio.o(i.HAL_SAI_ErrorCallback) refers to stm32f7xx_hal_sai.o(i.HAL_SAI_GetState) for HAL_SAI_GetState
    stm32746g_discovery_audio.o(i.HAL_SAI_ErrorCallback) refers to stm32746g_discovery_audio.o(i.BSP_AUDIO_OUT_Error_CallBack) for BSP_AUDIO_OUT_Error_CallBack
    stm32746g_discovery_audio.o(i.HAL_SAI_ErrorCallback) refers to stm32746g_discovery_audio.o(i.BSP_AUDIO_IN_Error_CallBack) for BSP_AUDIO_IN_Error_CallBack
    stm32746g_discovery_audio.o(i.HAL_SAI_ErrorCallback) refers to stm32746g_discovery_audio.o(.bss) for .bss
    stm32746g_discovery_audio.o(i.HAL_SAI_RxCpltCallback) refers to stm32746g_discovery_audio.o(i.BSP_AUDIO_IN_TransferComplete_CallBack) for BSP_AUDIO_IN_TransferComplete_CallBack
    stm32746g_discovery_audio.o(i.HAL_SAI_RxHalfCpltCallback) refers to stm32746g_discovery_audio.o(i.BSP_AUDIO_IN_HalfTransfer_CallBack) for BSP_AUDIO_IN_HalfTransfer_CallBack
    stm32746g_discovery_audio.o(i.HAL_SAI_TxCpltCallback) refers to usbd_audio_if.o(i.BSP_AUDIO_OUT_TransferComplete_CallBack) for BSP_AUDIO_OUT_TransferComplete_CallBack
    stm32746g_discovery_audio.o(i.HAL_SAI_TxHalfCpltCallback) refers to usbd_audio_if.o(i.BSP_AUDIO_OUT_HalfTransfer_CallBack) for BSP_AUDIO_OUT_HalfTransfer_CallBack
    stm32746g_discovery_audio.o(i.SAIx_In_DeInit) refers to stm32f7xx_hal_sai.o(i.HAL_SAI_DeInit) for HAL_SAI_DeInit
    stm32746g_discovery_audio.o(i.SAIx_In_DeInit) refers to stm32746g_discovery_audio.o(.bss) for .bss
    stm32746g_discovery_audio.o(i.SAIx_In_Init) refers to stm32f7xx_hal_sai.o(i.HAL_SAI_Init) for HAL_SAI_Init
    stm32746g_discovery_audio.o(i.SAIx_In_Init) refers to stm32746g_discovery_audio.o(.bss) for .bss
    stm32746g_discovery_audio.o(i.SAIx_Out_DeInit) refers to stm32f7xx_hal_sai.o(i.HAL_SAI_DeInit) for HAL_SAI_DeInit
    stm32746g_discovery_audio.o(i.SAIx_Out_DeInit) refers to stm32746g_discovery_audio.o(.bss) for .bss
    stm32746g_discovery_audio.o(i.SAIx_Out_Init) refers to stm32f7xx_hal_sai.o(i.HAL_SAI_Init) for HAL_SAI_Init
    stm32746g_discovery_audio.o(i.SAIx_Out_Init) refers to stm32746g_discovery_audio.o(.bss) for .bss
    stm32746g_discovery.o(i.AUDIO_IO_Delay) refers to stm32f7xx_hal.o(i.HAL_Delay) for HAL_Delay
    stm32746g_discovery.o(i.AUDIO_IO_Init) refers to stm32746g_discovery.o(i.I2Cx_Init) for I2Cx_Init
    stm32746g_discovery.o(i.AUDIO_IO_Init) refers to stm32746g_discovery.o(.bss) for .bss
    stm32746g_discovery.o(i.AUDIO_IO_Read) refers to stm32746g_discovery.o(i.I2Cx_ReadMultiple) for I2Cx_ReadMultiple
    stm32746g_discovery.o(i.AUDIO_IO_Read) refers to stm32746g_discovery.o(.bss) for .bss
    stm32746g_discovery.o(i.AUDIO_IO_Write) refers to stm32746g_discovery.o(i.I2Cx_WriteMultiple) for I2Cx_WriteMultiple
    stm32746g_discovery.o(i.AUDIO_IO_Write) refers to stm32746g_discovery.o(.bss) for .bss
    stm32746g_discovery.o(i.BSP_COM_DeInit) refers to stm32f7xx_hal_uart.o(i.HAL_UART_DeInit) for HAL_UART_DeInit
    stm32746g_discovery.o(i.BSP_COM_DeInit) refers to stm32746g_discovery.o(.data) for .data
    stm32746g_discovery.o(i.BSP_COM_Init) refers to stm32f7xx_hal_gpio.o(i.HAL_GPIO_Init) for HAL_GPIO_Init
    stm32746g_discovery.o(i.BSP_COM_Init) refers to stm32f7xx_hal_uart.o(i.HAL_UART_Init) for HAL_UART_Init
    stm32746g_discovery.o(i.BSP_COM_Init) refers to stm32746g_discovery.o(.constdata) for .constdata
    stm32746g_discovery.o(i.BSP_COM_Init) refers to stm32746g_discovery.o(.data) for .data
    stm32746g_discovery.o(i.BSP_LED_DeInit) refers to stm32f7xx_hal_gpio.o(i.HAL_GPIO_WritePin) for HAL_GPIO_WritePin
    stm32746g_discovery.o(i.BSP_LED_DeInit) refers to stm32f7xx_hal_gpio.o(i.HAL_GPIO_DeInit) for HAL_GPIO_DeInit
    stm32746g_discovery.o(i.BSP_LED_DeInit) refers to stm32746g_discovery.o(.constdata) for .constdata
    stm32746g_discovery.o(i.BSP_LED_Init) refers to stm32f7xx_hal_gpio.o(i.HAL_GPIO_Init) for HAL_GPIO_Init
    stm32746g_discovery.o(i.BSP_LED_Init) refers to stm32f7xx_hal_gpio.o(i.HAL_GPIO_WritePin) for HAL_GPIO_WritePin
    stm32746g_discovery.o(i.BSP_LED_Init) refers to stm32746g_discovery.o(.constdata) for .constdata
    stm32746g_discovery.o(i.BSP_LED_Off) refers to stm32f7xx_hal_gpio.o(i.HAL_GPIO_WritePin) for HAL_GPIO_WritePin
    stm32746g_discovery.o(i.BSP_LED_Off) refers to stm32746g_discovery.o(.constdata) for .constdata
    stm32746g_discovery.o(i.BSP_LED_On) refers to stm32f7xx_hal_gpio.o(i.HAL_GPIO_WritePin) for HAL_GPIO_WritePin
    stm32746g_discovery.o(i.BSP_LED_On) refers to stm32746g_discovery.o(.constdata) for .constdata
    stm32746g_discovery.o(i.BSP_LED_Toggle) refers to stm32f7xx_hal_gpio.o(i.HAL_GPIO_TogglePin) for HAL_GPIO_TogglePin
    stm32746g_discovery.o(i.BSP_LED_Toggle) refers to stm32746g_discovery.o(.constdata) for .constdata
    stm32746g_discovery.o(i.BSP_PB_DeInit) refers to stm32f7xx_hal_cortex.o(i.HAL_NVIC_DisableIRQ) for HAL_NVIC_DisableIRQ
    stm32746g_discovery.o(i.BSP_PB_DeInit) refers to stm32f7xx_hal_gpio.o(i.HAL_GPIO_DeInit) for HAL_GPIO_DeInit
    stm32746g_discovery.o(i.BSP_PB_DeInit) refers to stm32746g_discovery.o(.constdata) for .constdata
    stm32746g_discovery.o(i.BSP_PB_DeInit) refers to stm32746g_discovery.o(.data) for .data
    stm32746g_discovery.o(i.BSP_PB_GetState) refers to stm32f7xx_hal_gpio.o(i.HAL_GPIO_ReadPin) for HAL_GPIO_ReadPin
    stm32746g_discovery.o(i.BSP_PB_GetState) refers to stm32746g_discovery.o(.constdata) for .constdata
    stm32746g_discovery.o(i.BSP_PB_GetState) refers to stm32746g_discovery.o(.data) for .data
    stm32746g_discovery.o(i.BSP_PB_Init) refers to stm32f7xx_hal_gpio.o(i.HAL_GPIO_Init) for HAL_GPIO_Init
    stm32746g_discovery.o(i.BSP_PB_Init) refers to stm32f7xx_hal_cortex.o(i.HAL_NVIC_SetPriority) for HAL_NVIC_SetPriority
    stm32746g_discovery.o(i.BSP_PB_Init) refers to stm32f7xx_hal_cortex.o(i.HAL_NVIC_EnableIRQ) for HAL_NVIC_EnableIRQ
    stm32746g_discovery.o(i.BSP_PB_Init) refers to stm32746g_discovery.o(.constdata) for .constdata
    stm32746g_discovery.o(i.BSP_PB_Init) refers to stm32746g_discovery.o(.data) for .data
    stm32746g_discovery.o(i.CAMERA_Delay) refers to stm32f7xx_hal.o(i.HAL_Delay) for HAL_Delay
    stm32746g_discovery.o(i.CAMERA_IO_Init) refers to stm32746g_discovery.o(i.I2Cx_Init) for I2Cx_Init
    stm32746g_discovery.o(i.CAMERA_IO_Init) refers to stm32746g_discovery.o(.bss) for .bss
    stm32746g_discovery.o(i.CAMERA_IO_Read) refers to stm32746g_discovery.o(i.I2Cx_ReadMultiple) for I2Cx_ReadMultiple
    stm32746g_discovery.o(i.CAMERA_IO_Read) refers to stm32746g_discovery.o(.bss) for .bss
    stm32746g_discovery.o(i.CAMERA_IO_Write) refers to stm32746g_discovery.o(i.I2Cx_WriteMultiple) for I2Cx_WriteMultiple
    stm32746g_discovery.o(i.CAMERA_IO_Write) refers to stm32746g_discovery.o(.bss) for .bss
    stm32746g_discovery.o(i.EEPROM_IO_Init) refers to stm32746g_discovery.o(i.I2Cx_Init) for I2Cx_Init
    stm32746g_discovery.o(i.EEPROM_IO_Init) refers to stm32746g_discovery.o(.bss) for .bss
    stm32746g_discovery.o(i.EEPROM_IO_IsDeviceReady) refers to stm32f7xx_hal_i2c.o(i.HAL_I2C_IsDeviceReady) for HAL_I2C_IsDeviceReady
    stm32746g_discovery.o(i.EEPROM_IO_IsDeviceReady) refers to stm32746g_discovery.o(.bss) for .bss
    stm32746g_discovery.o(i.EEPROM_IO_ReadData) refers to stm32746g_discovery.o(i.I2Cx_ReadMultiple) for I2Cx_ReadMultiple
    stm32746g_discovery.o(i.EEPROM_IO_ReadData) refers to stm32746g_discovery.o(.bss) for .bss
    stm32746g_discovery.o(i.EEPROM_IO_WriteData) refers to stm32746g_discovery.o(i.I2Cx_WriteMultiple) for I2Cx_WriteMultiple
    stm32746g_discovery.o(i.EEPROM_IO_WriteData) refers to stm32746g_discovery.o(.bss) for .bss
    stm32746g_discovery.o(i.I2Cx_Error) refers to stm32f7xx_hal_i2c.o(i.HAL_I2C_DeInit) for HAL_I2C_DeInit
    stm32746g_discovery.o(i.I2Cx_Error) refers to stm32746g_discovery.o(i.I2Cx_Init) for I2Cx_Init
    stm32746g_discovery.o(i.I2Cx_Init) refers to stm32f7xx_hal_i2c.o(i.HAL_I2C_GetState) for HAL_I2C_GetState
    stm32746g_discovery.o(i.I2Cx_Init) refers to stm32746g_discovery.o(i.I2Cx_MspInit) for I2Cx_MspInit
    stm32746g_discovery.o(i.I2Cx_Init) refers to stm32f7xx_hal_i2c.o(i.HAL_I2C_Init) for HAL_I2C_Init
    stm32746g_discovery.o(i.I2Cx_Init) refers to stm32746g_discovery.o(.bss) for .bss
    stm32746g_discovery.o(i.I2Cx_MspInit) refers to stm32f7xx_hal_gpio.o(i.HAL_GPIO_Init) for HAL_GPIO_Init
    stm32746g_discovery.o(i.I2Cx_MspInit) refers to stm32f7xx_hal_cortex.o(i.HAL_NVIC_SetPriority) for HAL_NVIC_SetPriority
    stm32746g_discovery.o(i.I2Cx_MspInit) refers to stm32f7xx_hal_cortex.o(i.HAL_NVIC_EnableIRQ) for HAL_NVIC_EnableIRQ
    stm32746g_discovery.o(i.I2Cx_MspInit) refers to stm32746g_discovery.o(.bss) for .bss
    stm32746g_discovery.o(i.I2Cx_ReadMultiple) refers to stm32f7xx_hal_i2c.o(i.HAL_I2C_Mem_Read) for HAL_I2C_Mem_Read
    stm32746g_discovery.o(i.I2Cx_ReadMultiple) refers to stm32746g_discovery.o(i.I2Cx_Error) for I2Cx_Error
    stm32746g_discovery.o(i.I2Cx_WriteMultiple) refers to stm32f7xx_hal_i2c.o(i.HAL_I2C_Mem_Write) for HAL_I2C_Mem_Write
    stm32746g_discovery.o(i.I2Cx_WriteMultiple) refers to stm32746g_discovery.o(i.I2Cx_Error) for I2Cx_Error
    stm32746g_discovery.o(i.TS_IO_Delay) refers to stm32f7xx_hal.o(i.HAL_Delay) for HAL_Delay
    stm32746g_discovery.o(i.TS_IO_Init) refers to stm32746g_discovery.o(i.I2Cx_Init) for I2Cx_Init
    stm32746g_discovery.o(i.TS_IO_Init) refers to stm32746g_discovery.o(.bss) for .bss
    stm32746g_discovery.o(i.TS_IO_Read) refers to stm32746g_discovery.o(i.I2Cx_ReadMultiple) for I2Cx_ReadMultiple
    stm32746g_discovery.o(i.TS_IO_Read) refers to stm32746g_discovery.o(.bss) for .bss
    stm32746g_discovery.o(i.TS_IO_Write) refers to stm32746g_discovery.o(i.I2Cx_WriteMultiple) for I2Cx_WriteMultiple
    stm32746g_discovery.o(i.TS_IO_Write) refers to stm32746g_discovery.o(.bss) for .bss
    usbd_audio.o(i.USBD_AUDIO_DataOut) refers to usbd_conf.o(i.USBD_LL_PrepareReceive) for USBD_LL_PrepareReceive
    usbd_audio.o(i.USBD_AUDIO_DeInit) refers to usbd_conf.o(i.USBD_LL_CloseEP) for USBD_LL_CloseEP
    usbd_audio.o(i.USBD_AUDIO_DeInit) refers to malloc.o(i.free) for free
    usbd_audio.o(i.USBD_AUDIO_GetCfgDesc) refers to usbd_audio.o(.data) for .data
    usbd_audio.o(i.USBD_AUDIO_GetDeviceQualifierDesc) refers to usbd_audio.o(.data) for .data
    usbd_audio.o(i.USBD_AUDIO_Init) refers to usbd_conf.o(i.USBD_LL_OpenEP) for USBD_LL_OpenEP
    usbd_audio.o(i.USBD_AUDIO_Init) refers to malloc.o(i.malloc) for malloc
    usbd_audio.o(i.USBD_AUDIO_Init) refers to usbd_conf.o(i.USBD_LL_PrepareReceive) for USBD_LL_PrepareReceive
    usbd_audio.o(i.USBD_AUDIO_Setup) refers to memseta.o(.text) for __aeabi_memclr
    usbd_audio.o(i.USBD_AUDIO_Setup) refers to usbd_ioreq.o(i.USBD_CtlPrepareRx) for USBD_CtlPrepareRx
    usbd_audio.o(i.USBD_AUDIO_Setup) refers to usbd_ctlreq.o(i.USBD_CtlError) for USBD_CtlError
    usbd_audio.o(i.USBD_AUDIO_Setup) refers to usbd_ioreq.o(i.USBD_CtlSendData) for USBD_CtlSendData
    usbd_audio.o(i.USBD_AUDIO_Setup) refers to usbd_audio.o(.data) for .data
    usbd_audio.o(.data) refers to usbd_audio.o(i.USBD_AUDIO_Init) for USBD_AUDIO_Init
    usbd_audio.o(.data) refers to usbd_audio.o(i.USBD_AUDIO_DeInit) for USBD_AUDIO_DeInit
    usbd_audio.o(.data) refers to usbd_audio.o(i.USBD_AUDIO_Setup) for USBD_AUDIO_Setup
    usbd_audio.o(.data) refers to usbd_audio.o(i.USBD_AUDIO_EP0_TxReady) for USBD_AUDIO_EP0_TxReady
    usbd_audio.o(.data) refers to usbd_audio.o(i.USBD_AUDIO_EP0_RxReady) for USBD_AUDIO_EP0_RxReady
    usbd_audio.o(.data) refers to usbd_audio.o(i.USBD_AUDIO_DataIn) for USBD_AUDIO_DataIn
    usbd_audio.o(.data) refers to usbd_audio.o(i.USBD_AUDIO_DataOut) for USBD_AUDIO_DataOut
    usbd_audio.o(.data) refers to usbd_audio.o(i.USBD_AUDIO_SOF) for USBD_AUDIO_SOF
    usbd_audio.o(.data) refers to usbd_audio.o(i.USBD_AUDIO_IsoINIncomplete) for USBD_AUDIO_IsoINIncomplete
    usbd_audio.o(.data) refers to usbd_audio.o(i.USBD_AUDIO_IsoOutIncomplete) for USBD_AUDIO_IsoOutIncomplete
    usbd_audio.o(.data) refers to usbd_audio.o(i.USBD_AUDIO_GetCfgDesc) for USBD_AUDIO_GetCfgDesc
    usbd_audio.o(.data) refers to usbd_audio.o(i.USBD_AUDIO_GetDeviceQualifierDesc) for USBD_AUDIO_GetDeviceQualifierDesc
    entry.o(.ARM.Collect$$$$00000000) refers (Special) to entry10a.o(.ARM.Collect$$$$0000000D) for __rt_final_cpp
    entry.o(.ARM.Collect$$$$00000000) refers (Special) to entry11a.o(.ARM.Collect$$$$0000000F) for __rt_final_exit
    entry.o(.ARM.Collect$$$$00000000) refers (Special) to entry7b.o(.ARM.Collect$$$$00000008) for _main_clock
    entry.o(.ARM.Collect$$$$00000000) refers (Special) to entry8b.o(.ARM.Collect$$$$0000000A) for _main_cpp_init
    entry.o(.ARM.Collect$$$$00000000) refers (Special) to entry9a.o(.ARM.Collect$$$$0000000B) for _main_init
    entry.o(.ARM.Collect$$$$00000000) refers (Special) to entry5.o(.ARM.Collect$$$$00000004) for _main_scatterload
    entry.o(.ARM.Collect$$$$00000000) refers (Special) to entry2.o(.ARM.Collect$$$$00000001) for _main_stk
    malloc.o(i.free) refers to mvars.o(.data) for __microlib_freelist
    malloc.o(i.malloc) refers to mvars.o(.data) for __microlib_freelist_initialised
    malloc.o(i.malloc) refers to mvars.o(.data) for __microlib_freelist
    malloc.o(i.malloc) refers to startup_stm32f746xx.o(HEAP) for __heap_base
    mallocr.o(i.__free$realloc) refers to mvars.o(.data) for __microlib_freelist
    mallocr.o(i.__malloc$realloc) refers to mallocr.o(i.internal_alloc) for internal_alloc
    mallocr.o(i.__malloc$realloc) refers to mvars.o(.data) for __microlib_freelist_initialised
    mallocr.o(i.__malloc$realloc) refers to startup_stm32f746xx.o(HEAP) for __heap_base
    mallocr.o(i.__malloc$realloc) refers to mvars.o(.data) for __microlib_freelist
    mallocr.o(i.internal_alloc) refers to memcpya.o(.text) for __aeabi_memcpy
    mallocr.o(i.internal_alloc) refers to mvars.o(.data) for __microlib_freelist
    mallocr.o(i.realloc) refers to mallocr.o(i.__free$realloc) for __free$realloc
    mallocr.o(i.realloc) refers to mallocr.o(i.internal_alloc) for internal_alloc
    mallocr.o(i.realloc) refers to mallocr.o(i.__malloc$realloc) for __malloc$realloc
    mallocr.o(i.realloc) refers to mvars.o(.data) for __microlib_freelist
    malloca.o(i.__aligned_malloc) refers to mvars.o(.data) for __microlib_freelist_initialised
    malloca.o(i.__aligned_malloc) refers to mvars.o(.data) for __microlib_freelist
    malloca.o(i.__aligned_malloc) refers to startup_stm32f746xx.o(HEAP) for __heap_base
    malloca.o(i.__free$memalign) refers to mvars.o(.data) for __microlib_freelist
    malloca.o(i.__malloc$memalign) refers to malloca.o(i.__aligned_malloc) for __aligned_malloc
    mallocra.o(i.__aligned_malloc$realloc) refers to mallocra.o(i.internal_alloc) for internal_alloc
    mallocra.o(i.__aligned_malloc$realloc) refers to mvars.o(.data) for __microlib_freelist_initialised
    mallocra.o(i.__aligned_malloc$realloc) refers to startup_stm32f746xx.o(HEAP) for __heap_base
    mallocra.o(i.__aligned_malloc$realloc) refers to mvars.o(.data) for __microlib_freelist
    mallocra.o(i.__free$realloc$memalign) refers to mvars.o(.data) for __microlib_freelist
    mallocra.o(i.__malloc$realloc$memalign) refers to mallocra.o(i.__aligned_malloc$realloc) for __aligned_malloc$realloc
    mallocra.o(i.__realloc$memalign) refers to mallocra.o(i.__free$realloc$memalign) for __free$realloc$memalign
    mallocra.o(i.__realloc$memalign) refers to mallocra.o(i.internal_alloc) for internal_alloc
    mallocra.o(i.__realloc$memalign) refers to mallocra.o(i.__malloc$realloc$memalign) for __malloc$realloc$memalign
    mallocra.o(i.__realloc$memalign) refers to mvars.o(.data) for __microlib_freelist
    mallocra.o(i.internal_alloc) refers to memcpya.o(.text) for __aeabi_memcpy
    mallocra.o(i.internal_alloc) refers to mvars.o(.data) for __microlib_freelist
    entry2.o(.ARM.Collect$$$$00000001) refers to entry2.o(.ARM.Collect$$$$00002712) for __lit__00000000
    entry2.o(.ARM.Collect$$$$00002712) refers to startup_stm32f746xx.o(STACK) for __initial_sp
    entry2.o(__vectab_stack_and_reset_area) refers to startup_stm32f746xx.o(STACK) for __initial_sp
    entry2.o(__vectab_stack_and_reset_area) refers to entry.o(.ARM.Collect$$$$00000000) for __main
    entry5.o(.ARM.Collect$$$$00000004) refers to init.o(.text) for __scatterload
    entry9a.o(.ARM.Collect$$$$0000000B) refers to main.o(i.main) for main
    entry9b.o(.ARM.Collect$$$$0000000C) refers to main.o(i.main) for main
    init.o(.text) refers to entry5.o(.ARM.Collect$$$$00000004) for __main_after_scatterload


==============================================================================

Removing Unused input sections from the image.

    Removing system_stm32f7xx.o(.rev16_text), (4 bytes).
    Removing system_stm32f7xx.o(.revsh_text), (4 bytes).
    Removing system_stm32f7xx.o(.rrx_text), (6 bytes).
    Removing system_stm32f7xx.o(i.SystemCoreClockUpdate), (128 bytes).
    Removing stm32f7xx_hal.o(.rev16_text), (4 bytes).
    Removing stm32f7xx_hal.o(.revsh_text), (4 bytes).
    Removing stm32f7xx_hal.o(.rrx_text), (6 bytes).
    Removing stm32f7xx_hal.o(i.HAL_DBGMCU_DisableDBGSleepMode), (16 bytes).
    Removing stm32f7xx_hal.o(i.HAL_DBGMCU_DisableDBGStandbyMode), (16 bytes).
    Removing stm32f7xx_hal.o(i.HAL_DBGMCU_DisableDBGStopMode), (16 bytes).
    Removing stm32f7xx_hal.o(i.HAL_DBGMCU_EnableDBGSleepMode), (16 bytes).
    Removing stm32f7xx_hal.o(i.HAL_DBGMCU_EnableDBGStandbyMode), (16 bytes).
    Removing stm32f7xx_hal.o(i.HAL_DBGMCU_EnableDBGStopMode), (16 bytes).
    Removing stm32f7xx_hal.o(i.HAL_DeInit), (52 bytes).
    Removing stm32f7xx_hal.o(i.HAL_DisableCompensationCell), (16 bytes).
    Removing stm32f7xx_hal.o(i.HAL_DisableFMCMemorySwapping), (16 bytes).
    Removing stm32f7xx_hal.o(i.HAL_EnableCompensationCell), (16 bytes).
    Removing stm32f7xx_hal.o(i.HAL_EnableFMCMemorySwapping), (16 bytes).
    Removing stm32f7xx_hal.o(i.HAL_GetDEVID), (16 bytes).
    Removing stm32f7xx_hal.o(i.HAL_GetHalVersion), (8 bytes).
    Removing stm32f7xx_hal.o(i.HAL_GetREVID), (12 bytes).
    Removing stm32f7xx_hal.o(i.HAL_MspDeInit), (8 bytes).
    Removing stm32f7xx_hal.o(i.HAL_ResumeTick), (14 bytes).
    Removing stm32f7xx_hal.o(i.HAL_SuspendTick), (14 bytes).
    Removing stm32f7xx_hal_cortex.o(.rev16_text), (4 bytes).
    Removing stm32f7xx_hal_cortex.o(.revsh_text), (4 bytes).
    Removing stm32f7xx_hal_cortex.o(.rrx_text), (6 bytes).
    Removing stm32f7xx_hal_cortex.o(i.HAL_MPU_ConfigRegion), (92 bytes).
    Removing stm32f7xx_hal_cortex.o(i.HAL_NVIC_ClearPendingIRQ), (22 bytes).
    Removing stm32f7xx_hal_cortex.o(i.HAL_NVIC_DisableIRQ), (22 bytes).
    Removing stm32f7xx_hal_cortex.o(i.HAL_NVIC_GetActive), (32 bytes).
    Removing stm32f7xx_hal_cortex.o(i.HAL_NVIC_GetPendingIRQ), (32 bytes).
    Removing stm32f7xx_hal_cortex.o(i.HAL_NVIC_GetPriority), (82 bytes).
    Removing stm32f7xx_hal_cortex.o(i.HAL_NVIC_GetPriorityGrouping), (16 bytes).
    Removing stm32f7xx_hal_cortex.o(i.HAL_NVIC_SetPendingIRQ), (22 bytes).
    Removing stm32f7xx_hal_cortex.o(i.HAL_NVIC_SystemReset), (36 bytes).
    Removing stm32f7xx_hal_cortex.o(i.HAL_SYSTICK_CLKSourceConfig), (24 bytes).
    Removing stm32f7xx_hal_cortex.o(i.HAL_SYSTICK_Callback), (8 bytes).
    Removing stm32f7xx_hal_cortex.o(i.HAL_SYSTICK_IRQHandler), (8 bytes).
    Removing stm32f7xx_ll_usb.o(.rev16_text), (4 bytes).
    Removing stm32f7xx_ll_usb.o(.revsh_text), (4 bytes).
    Removing stm32f7xx_ll_usb.o(.rrx_text), (6 bytes).
    Removing stm32f7xx_ll_usb.o(i.USB_ActivateDedicatedEndpoint), (220 bytes).
    Removing stm32f7xx_ll_usb.o(i.USB_ClearInterrupts), (8 bytes).
    Removing stm32f7xx_ll_usb.o(i.USB_DeactivateDedicatedEndpoint), (78 bytes).
    Removing stm32f7xx_ll_usb.o(i.USB_DoPing), (64 bytes).
    Removing stm32f7xx_ll_usb.o(i.USB_DriveVbus), (44 bytes).
    Removing stm32f7xx_ll_usb.o(i.USB_GetCurrentFrame), (8 bytes).
    Removing stm32f7xx_ll_usb.o(i.USB_GetHostSpeed), (14 bytes).
    Removing stm32f7xx_ll_usb.o(i.USB_HC_Halt), (376 bytes).
    Removing stm32f7xx_ll_usb.o(i.USB_HC_Init), (230 bytes).
    Removing stm32f7xx_ll_usb.o(i.USB_HC_ReadInterrupt), (12 bytes).
    Removing stm32f7xx_ll_usb.o(i.USB_HC_StartXfer), (392 bytes).
    Removing stm32f7xx_ll_usb.o(i.USB_HostInit), (196 bytes).
    Removing stm32f7xx_ll_usb.o(i.USB_InitFSLSPClkSel), (56 bytes).
    Removing stm32f7xx_ll_usb.o(i.USB_ResetPort), (44 bytes).
    Removing stm32f7xx_ll_usb.o(i.USB_SetDevSpeed), (14 bytes).
    Removing stm32f7xx_ll_usb.o(i.USB_StopDevice), (64 bytes).
    Removing stm32f7xx_ll_usb.o(i.USB_StopHost), (178 bytes).
    Removing stm32f7xx_ll_usb.o(.data), (4 bytes).
    Removing stm32f7xx_hal_flash.o(.rev16_text), (4 bytes).
    Removing stm32f7xx_hal_flash.o(.revsh_text), (4 bytes).
    Removing stm32f7xx_hal_flash.o(.rrx_text), (6 bytes).
    Removing stm32f7xx_hal_flash.o(i.FLASH_Program_Byte), (36 bytes).
    Removing stm32f7xx_hal_flash.o(i.FLASH_Program_DoubleWord), (44 bytes).
    Removing stm32f7xx_hal_flash.o(i.FLASH_Program_HalfWord), (40 bytes).
    Removing stm32f7xx_hal_flash.o(i.FLASH_Program_Word), (40 bytes).
    Removing stm32f7xx_hal_flash.o(i.FLASH_SetErrorCode), (84 bytes).
    Removing stm32f7xx_hal_flash.o(i.FLASH_WaitForLastOperation), (72 bytes).
    Removing stm32f7xx_hal_flash.o(i.HAL_FLASH_EndOfOperationCallback), (8 bytes).
    Removing stm32f7xx_hal_flash.o(i.HAL_FLASH_GetError), (12 bytes).
    Removing stm32f7xx_hal_flash.o(i.HAL_FLASH_IRQHandler), (256 bytes).
    Removing stm32f7xx_hal_flash.o(i.HAL_FLASH_Lock), (20 bytes).
    Removing stm32f7xx_hal_flash.o(i.HAL_FLASH_OB_Launch), (24 bytes).
    Removing stm32f7xx_hal_flash.o(i.HAL_FLASH_OB_Lock), (20 bytes).
    Removing stm32f7xx_hal_flash.o(i.HAL_FLASH_OB_Unlock), (40 bytes).
    Removing stm32f7xx_hal_flash.o(i.HAL_FLASH_OperationErrorCallback), (8 bytes).
    Removing stm32f7xx_hal_flash.o(i.HAL_FLASH_Program), (132 bytes).
    Removing stm32f7xx_hal_flash.o(i.HAL_FLASH_Program_IT), (132 bytes).
    Removing stm32f7xx_hal_flash.o(i.HAL_FLASH_Unlock), (40 bytes).
    Removing stm32f7xx_hal_flash.o(.bss), (28 bytes).
    Removing stm32f7xx_hal_pwr_ex.o(.rev16_text), (4 bytes).
    Removing stm32f7xx_hal_pwr_ex.o(.revsh_text), (4 bytes).
    Removing stm32f7xx_hal_pwr_ex.o(.rrx_text), (6 bytes).
    Removing stm32f7xx_hal_pwr_ex.o(i.HAL_PWREx_ControlVoltageScaling), (176 bytes).
    Removing stm32f7xx_hal_pwr_ex.o(i.HAL_PWREx_DisableBkUpReg), (56 bytes).
    Removing stm32f7xx_hal_pwr_ex.o(i.HAL_PWREx_DisableFlashPowerDown), (16 bytes).
    Removing stm32f7xx_hal_pwr_ex.o(i.HAL_PWREx_DisableLowRegulatorLowVoltage), (16 bytes).
    Removing stm32f7xx_hal_pwr_ex.o(i.HAL_PWREx_DisableMainRegulatorLowVoltage), (16 bytes).
    Removing stm32f7xx_hal_pwr_ex.o(i.HAL_PWREx_DisableOverDrive), (108 bytes).
    Removing stm32f7xx_hal_pwr_ex.o(i.HAL_PWREx_EnableBkUpReg), (56 bytes).
    Removing stm32f7xx_hal_pwr_ex.o(i.HAL_PWREx_EnableFlashPowerDown), (16 bytes).
    Removing stm32f7xx_hal_pwr_ex.o(i.HAL_PWREx_EnableLowRegulatorLowVoltage), (16 bytes).
    Removing stm32f7xx_hal_pwr_ex.o(i.HAL_PWREx_EnableMainRegulatorLowVoltage), (16 bytes).
    Removing stm32f7xx_hal_pwr_ex.o(i.HAL_PWREx_EnterUnderDriveSTOPMode), (144 bytes).
    Removing stm32f7xx_hal_pwr_ex.o(i.HAL_PWREx_GetVoltageRange), (16 bytes).
    Removing stm32f7xx_hal_rcc.o(.rev16_text), (4 bytes).
    Removing stm32f7xx_hal_rcc.o(.revsh_text), (4 bytes).
    Removing stm32f7xx_hal_rcc.o(.rrx_text), (6 bytes).
    Removing stm32f7xx_hal_rcc.o(i.HAL_RCC_CSSCallback), (8 bytes).
    Removing stm32f7xx_hal_rcc.o(i.HAL_RCC_DeInit), (88 bytes).
    Removing stm32f7xx_hal_rcc.o(i.HAL_RCC_DisableCSS), (16 bytes).
    Removing stm32f7xx_hal_rcc.o(i.HAL_RCC_EnableCSS), (16 bytes).
    Removing stm32f7xx_hal_rcc.o(i.HAL_RCC_GetClockConfig), (64 bytes).
    Removing stm32f7xx_hal_rcc.o(i.HAL_RCC_GetOscConfig), (228 bytes).
    Removing stm32f7xx_hal_rcc.o(i.HAL_RCC_MCOConfig), (148 bytes).
    Removing stm32f7xx_hal_rcc.o(i.HAL_RCC_NMI_IRQHandler), (28 bytes).
    Removing stm32f7xx_hal_tim_ex.o(.rev16_text), (4 bytes).
    Removing stm32f7xx_hal_tim_ex.o(.revsh_text), (4 bytes).
    Removing stm32f7xx_hal_tim_ex.o(.rrx_text), (6 bytes).
    Removing stm32f7xx_hal_tim_ex.o(i.HAL_TIMEx_BreakCallback), (2 bytes).
    Removing stm32f7xx_hal_tim_ex.o(i.HAL_TIMEx_CommutationCallback), (2 bytes).
    Removing stm32f7xx_hal_tim_ex.o(i.HAL_TIMEx_ConfigBreakDeadTime), (98 bytes).
    Removing stm32f7xx_hal_tim_ex.o(i.HAL_TIMEx_ConfigCommutationEvent), (92 bytes).
    Removing stm32f7xx_hal_tim_ex.o(i.HAL_TIMEx_ConfigCommutationEvent_DMA), (124 bytes).
    Removing stm32f7xx_hal_tim_ex.o(i.HAL_TIMEx_ConfigCommutationEvent_IT), (102 bytes).
    Removing stm32f7xx_hal_tim_ex.o(i.HAL_TIMEx_GroupChannel5), (58 bytes).
    Removing stm32f7xx_hal_tim_ex.o(i.HAL_TIMEx_HallSensor_DeInit), (56 bytes).
    Removing stm32f7xx_hal_tim_ex.o(i.HAL_TIMEx_HallSensor_GetState), (6 bytes).
    Removing stm32f7xx_hal_tim_ex.o(i.HAL_TIMEx_HallSensor_Init), (180 bytes).
    Removing stm32f7xx_hal_tim_ex.o(i.HAL_TIMEx_HallSensor_MspDeInit), (2 bytes).
    Removing stm32f7xx_hal_tim_ex.o(i.HAL_TIMEx_HallSensor_MspInit), (2 bytes).
    Removing stm32f7xx_hal_tim_ex.o(i.HAL_TIMEx_HallSensor_Start), (28 bytes).
    Removing stm32f7xx_hal_tim_ex.o(i.HAL_TIMEx_HallSensor_Start_DMA), (104 bytes).
    Removing stm32f7xx_hal_tim_ex.o(i.HAL_TIMEx_HallSensor_Start_IT), (38 bytes).
    Removing stm32f7xx_hal_tim_ex.o(i.HAL_TIMEx_HallSensor_Stop), (46 bytes).
    Removing stm32f7xx_hal_tim_ex.o(i.HAL_TIMEx_HallSensor_Stop_DMA), (56 bytes).
    Removing stm32f7xx_hal_tim_ex.o(i.HAL_TIMEx_HallSensor_Stop_IT), (56 bytes).
    Removing stm32f7xx_hal_tim_ex.o(i.HAL_TIMEx_MasterConfigSynchronization), (88 bytes).
    Removing stm32f7xx_hal_tim_ex.o(i.HAL_TIMEx_OCN_Start), (36 bytes).
    Removing stm32f7xx_hal_tim_ex.o(i.HAL_TIMEx_OCN_Start_DMA), (220 bytes).
    Removing stm32f7xx_hal_tim_ex.o(i.HAL_TIMEx_OCN_Start_IT), (96 bytes).
    Removing stm32f7xx_hal_tim_ex.o(i.HAL_TIMEx_OCN_Stop), (66 bytes).
    Removing stm32f7xx_hal_tim_ex.o(i.HAL_TIMEx_OCN_Stop_DMA), (122 bytes).
    Removing stm32f7xx_hal_tim_ex.o(i.HAL_TIMEx_OCN_Stop_IT), (134 bytes).
    Removing stm32f7xx_hal_tim_ex.o(i.HAL_TIMEx_OnePulseN_Start), (26 bytes).
    Removing stm32f7xx_hal_tim_ex.o(i.HAL_TIMEx_OnePulseN_Start_IT), (46 bytes).
    Removing stm32f7xx_hal_tim_ex.o(i.HAL_TIMEx_OnePulseN_Stop), (66 bytes).
    Removing stm32f7xx_hal_tim_ex.o(i.HAL_TIMEx_OnePulseN_Stop_IT), (86 bytes).
    Removing stm32f7xx_hal_tim_ex.o(i.HAL_TIMEx_PWMN_Start), (36 bytes).
    Removing stm32f7xx_hal_tim_ex.o(i.HAL_TIMEx_PWMN_Start_DMA), (220 bytes).
    Removing stm32f7xx_hal_tim_ex.o(i.HAL_TIMEx_PWMN_Start_IT), (96 bytes).
    Removing stm32f7xx_hal_tim_ex.o(i.HAL_TIMEx_PWMN_Stop), (66 bytes).
    Removing stm32f7xx_hal_tim_ex.o(i.HAL_TIMEx_PWMN_Stop_DMA), (122 bytes).
    Removing stm32f7xx_hal_tim_ex.o(i.HAL_TIMEx_PWMN_Stop_IT), (134 bytes).
    Removing stm32f7xx_hal_tim_ex.o(i.HAL_TIMEx_RemapConfig), (34 bytes).
    Removing stm32f7xx_hal_tim_ex.o(i.HAL_TIM_ConfigOCrefClear), (252 bytes).
    Removing stm32f7xx_hal_tim_ex.o(i.HAL_TIM_OC_ConfigChannel), (114 bytes).
    Removing stm32f7xx_hal_tim_ex.o(i.HAL_TIM_PWM_ConfigChannel), (296 bytes).
    Removing stm32f7xx_hal_tim_ex.o(i.TIMEx_DMACommutationCplt), (16 bytes).
    Removing stm32f7xx_hal_tim_ex.o(i.TIM_CCxNChannelCmd), (22 bytes).
    Removing stm32f7xx_hal_tim_ex.o(i.TIM_OC5_SetConfig), (88 bytes).
    Removing stm32f7xx_hal_tim_ex.o(i.TIM_OC6_SetConfig), (88 bytes).
    Removing stm32f7xx_hal_sai_ex.o(.rev16_text), (4 bytes).
    Removing stm32f7xx_hal_sai_ex.o(.revsh_text), (4 bytes).
    Removing stm32f7xx_hal_sai_ex.o(.rrx_text), (6 bytes).
    Removing stm32f7xx_hal_pcd.o(.rev16_text), (4 bytes).
    Removing stm32f7xx_hal_pcd.o(.revsh_text), (4 bytes).
    Removing stm32f7xx_hal_pcd.o(.rrx_text), (6 bytes).
    Removing stm32f7xx_hal_pcd.o(i.HAL_PCD_ActivateRemoteWakeup), (26 bytes).
    Removing stm32f7xx_hal_pcd.o(i.HAL_PCD_ConnectCallback), (2 bytes).
    Removing stm32f7xx_hal_pcd.o(i.HAL_PCD_DataInStageCallback), (2 bytes).
    Removing stm32f7xx_hal_pcd.o(i.HAL_PCD_DataOutStageCallback), (2 bytes).
    Removing stm32f7xx_hal_pcd.o(i.HAL_PCD_DeActivateRemoteWakeup), (18 bytes).
    Removing stm32f7xx_hal_pcd.o(i.HAL_PCD_DeInit), (36 bytes).
    Removing stm32f7xx_hal_pcd.o(i.HAL_PCD_DevConnect), (36 bytes).
    Removing stm32f7xx_hal_pcd.o(i.HAL_PCD_DevDisconnect), (36 bytes).
    Removing stm32f7xx_hal_pcd.o(i.HAL_PCD_DisconnectCallback), (2 bytes).
    Removing stm32f7xx_hal_pcd.o(i.HAL_PCD_EP_Flush), (50 bytes).
    Removing stm32f7xx_hal_pcd.o(i.HAL_PCD_EP_GetRxCount), (20 bytes).
    Removing stm32f7xx_hal_pcd.o(i.HAL_PCD_GetState), (6 bytes).
    Removing stm32f7xx_hal_pcd.o(i.HAL_PCD_ISOINIncompleteCallback), (2 bytes).
    Removing stm32f7xx_hal_pcd.o(i.HAL_PCD_ISOOUTIncompleteCallback), (2 bytes).
    Removing stm32f7xx_hal_pcd.o(i.HAL_PCD_MspDeInit), (2 bytes).
    Removing stm32f7xx_hal_pcd.o(i.HAL_PCD_MspInit), (2 bytes).
    Removing stm32f7xx_hal_pcd.o(i.HAL_PCD_ResetCallback), (2 bytes).
    Removing stm32f7xx_hal_pcd.o(i.HAL_PCD_ResumeCallback), (2 bytes).
    Removing stm32f7xx_hal_pcd.o(i.HAL_PCD_SOFCallback), (2 bytes).
    Removing stm32f7xx_hal_pcd.o(i.HAL_PCD_SetupStageCallback), (2 bytes).
    Removing stm32f7xx_hal_pcd.o(i.HAL_PCD_Stop), (48 bytes).
    Removing stm32f7xx_hal_pcd.o(i.HAL_PCD_SuspendCallback), (2 bytes).
    Removing stm32f7xx_hal_pwr.o(.rev16_text), (4 bytes).
    Removing stm32f7xx_hal_pwr.o(.revsh_text), (4 bytes).
    Removing stm32f7xx_hal_pwr.o(.rrx_text), (6 bytes).
    Removing stm32f7xx_hal_pwr.o(i.HAL_PWR_ConfigPVD), (124 bytes).
    Removing stm32f7xx_hal_pwr.o(i.HAL_PWR_DeInit), (24 bytes).
    Removing stm32f7xx_hal_pwr.o(i.HAL_PWR_DisableBkUpAccess), (16 bytes).
    Removing stm32f7xx_hal_pwr.o(i.HAL_PWR_DisablePVD), (16 bytes).
    Removing stm32f7xx_hal_pwr.o(i.HAL_PWR_DisableSEVOnPend), (16 bytes).
    Removing stm32f7xx_hal_pwr.o(i.HAL_PWR_DisableSleepOnExit), (16 bytes).
    Removing stm32f7xx_hal_pwr.o(i.HAL_PWR_DisableWakeUpPin), (16 bytes).
    Removing stm32f7xx_hal_pwr.o(i.HAL_PWR_EnableBkUpAccess), (16 bytes).
    Removing stm32f7xx_hal_pwr.o(i.HAL_PWR_EnablePVD), (16 bytes).
    Removing stm32f7xx_hal_pwr.o(i.HAL_PWR_EnableSEVOnPend), (16 bytes).
    Removing stm32f7xx_hal_pwr.o(i.HAL_PWR_EnableSleepOnExit), (16 bytes).
    Removing stm32f7xx_hal_pwr.o(i.HAL_PWR_EnableWakeUpPin), (28 bytes).
    Removing stm32f7xx_hal_pwr.o(i.HAL_PWR_EnterSLEEPMode), (32 bytes).
    Removing stm32f7xx_hal_pwr.o(i.HAL_PWR_EnterSTANDBYMode), (32 bytes).
    Removing stm32f7xx_hal_pwr.o(i.HAL_PWR_EnterSTOPMode), (60 bytes).
    Removing stm32f7xx_hal_pwr.o(i.HAL_PWR_PVDCallback), (8 bytes).
    Removing stm32f7xx_hal_pwr.o(i.HAL_PWR_PVD_IRQHandler), (28 bytes).
    Removing stm32f7xx_hal_sai.o(.rev16_text), (4 bytes).
    Removing stm32f7xx_hal_sai.o(.revsh_text), (4 bytes).
    Removing stm32f7xx_hal_sai.o(.rrx_text), (6 bytes).
    Removing stm32f7xx_hal_sai.o(i.HAL_SAI_Abort), (80 bytes).
    Removing stm32f7xx_hal_sai.o(i.HAL_SAI_DMAPause), (38 bytes).
    Removing stm32f7xx_hal_sai.o(i.HAL_SAI_DMAResume), (54 bytes).
    Removing stm32f7xx_hal_sai.o(i.HAL_SAI_DisableRxMuteMode), (28 bytes).
    Removing stm32f7xx_hal_sai.o(i.HAL_SAI_DisableTxMuteMode), (24 bytes).
    Removing stm32f7xx_hal_sai.o(i.HAL_SAI_EnableRxMuteMode), (60 bytes).
    Removing stm32f7xx_hal_sai.o(i.HAL_SAI_EnableTxMuteMode), (36 bytes).
    Removing stm32f7xx_hal_sai.o(i.HAL_SAI_ErrorCallback), (2 bytes).
    Removing stm32f7xx_hal_sai.o(i.HAL_SAI_GetError), (6 bytes).
    Removing stm32f7xx_hal_sai.o(i.HAL_SAI_IRQHandler), (198 bytes).
    Removing stm32f7xx_hal_sai.o(i.HAL_SAI_InitProtocol), (54 bytes).
    Removing stm32f7xx_hal_sai.o(i.HAL_SAI_Receive), (234 bytes).
    Removing stm32f7xx_hal_sai.o(i.HAL_SAI_Receive_DMA), (164 bytes).
    Removing stm32f7xx_hal_sai.o(i.HAL_SAI_Receive_IT), (144 bytes).
    Removing stm32f7xx_hal_sai.o(i.HAL_SAI_RxCpltCallback), (2 bytes).
    Removing stm32f7xx_hal_sai.o(i.HAL_SAI_RxHalfCpltCallback), (2 bytes).
    Removing stm32f7xx_hal_sai.o(i.HAL_SAI_Transmit), (244 bytes).
    Removing stm32f7xx_hal_sai.o(i.HAL_SAI_Transmit_IT), (148 bytes).
    Removing stm32f7xx_hal_sai.o(i.HAL_SAI_TxCpltCallback), (2 bytes).
    Removing stm32f7xx_hal_sai.o(i.HAL_SAI_TxHalfCpltCallback), (2 bytes).
    Removing stm32f7xx_hal_sai.o(i.SAI_DMARxCplt), (58 bytes).
    Removing stm32f7xx_hal_sai.o(i.SAI_DMARxHalfCplt), (10 bytes).
    Removing stm32f7xx_hal_sai.o(i.SAI_FillFifo), (86 bytes).
    Removing stm32f7xx_hal_sai.o(i.SAI_InitI2S), (154 bytes).
    Removing stm32f7xx_hal_sai.o(i.SAI_InitPCM), (108 bytes).
    Removing stm32f7xx_hal_sai.o(i.SAI_Receive_IT16Bit), (70 bytes).
    Removing stm32f7xx_hal_sai.o(i.SAI_Receive_IT32Bit), (70 bytes).
    Removing stm32f7xx_hal_sai.o(i.SAI_Receive_IT8Bit), (68 bytes).
    Removing stm32f7xx_hal_sai.o(i.SAI_Transmit_IT16Bit), (68 bytes).
    Removing stm32f7xx_hal_sai.o(i.SAI_Transmit_IT32Bit), (68 bytes).
    Removing stm32f7xx_hal_sai.o(i.SAI_Transmit_IT8Bit), (66 bytes).
    Removing stm32f7xx_hal_i2c.o(.rev16_text), (4 bytes).
    Removing stm32f7xx_hal_i2c.o(.revsh_text), (4 bytes).
    Removing stm32f7xx_hal_i2c.o(.rrx_text), (6 bytes).
    Removing stm32f7xx_hal_i2c.o(i.HAL_I2C_ER_IRQHandler), (116 bytes).
    Removing stm32f7xx_hal_i2c.o(i.HAL_I2C_EV_IRQHandler), (298 bytes).
    Removing stm32f7xx_hal_i2c.o(i.HAL_I2C_ErrorCallback), (2 bytes).
    Removing stm32f7xx_hal_i2c.o(i.HAL_I2C_GetError), (4 bytes).
    Removing stm32f7xx_hal_i2c.o(i.HAL_I2C_IsDeviceReady), (292 bytes).
    Removing stm32f7xx_hal_i2c.o(i.HAL_I2C_MasterRxCpltCallback), (2 bytes).
    Removing stm32f7xx_hal_i2c.o(i.HAL_I2C_MasterTxCpltCallback), (2 bytes).
    Removing stm32f7xx_hal_i2c.o(i.HAL_I2C_Master_Receive), (240 bytes).
    Removing stm32f7xx_hal_i2c.o(i.HAL_I2C_Master_Receive_DMA), (196 bytes).
    Removing stm32f7xx_hal_i2c.o(i.HAL_I2C_Master_Receive_IT), (134 bytes).
    Removing stm32f7xx_hal_i2c.o(i.HAL_I2C_Master_Transmit), (240 bytes).
    Removing stm32f7xx_hal_i2c.o(i.HAL_I2C_Master_Transmit_DMA), (212 bytes).
    Removing stm32f7xx_hal_i2c.o(i.HAL_I2C_Master_Transmit_IT), (134 bytes).
    Removing stm32f7xx_hal_i2c.o(i.HAL_I2C_MemRxCpltCallback), (2 bytes).
    Removing stm32f7xx_hal_i2c.o(i.HAL_I2C_MemTxCpltCallback), (2 bytes).
    Removing stm32f7xx_hal_i2c.o(i.HAL_I2C_Mem_Read_DMA), (216 bytes).
    Removing stm32f7xx_hal_i2c.o(i.HAL_I2C_Mem_Read_IT), (162 bytes).
    Removing stm32f7xx_hal_i2c.o(i.HAL_I2C_Mem_Write_DMA), (228 bytes).
    Removing stm32f7xx_hal_i2c.o(i.HAL_I2C_Mem_Write_IT), (162 bytes).
    Removing stm32f7xx_hal_i2c.o(i.HAL_I2C_SlaveRxCpltCallback), (2 bytes).
    Removing stm32f7xx_hal_i2c.o(i.HAL_I2C_SlaveTxCpltCallback), (2 bytes).
    Removing stm32f7xx_hal_i2c.o(i.HAL_I2C_Slave_Receive), (258 bytes).
    Removing stm32f7xx_hal_i2c.o(i.HAL_I2C_Slave_Receive_DMA), (172 bytes).
    Removing stm32f7xx_hal_i2c.o(i.HAL_I2C_Slave_Receive_IT), (80 bytes).
    Removing stm32f7xx_hal_i2c.o(i.HAL_I2C_Slave_Transmit), (274 bytes).
    Removing stm32f7xx_hal_i2c.o(i.HAL_I2C_Slave_Transmit_DMA), (200 bytes).
    Removing stm32f7xx_hal_i2c.o(i.HAL_I2C_Slave_Transmit_IT), (80 bytes).
    Removing stm32f7xx_hal_i2c.o(i.I2C_DMAError), (38 bytes).
    Removing stm32f7xx_hal_i2c.o(i.I2C_DMAMasterReceiveCplt), (336 bytes).
    Removing stm32f7xx_hal_i2c.o(i.I2C_DMAMasterTransmitCplt), (316 bytes).
    Removing stm32f7xx_hal_i2c.o(i.I2C_DMAMemReceiveCplt), (336 bytes).
    Removing stm32f7xx_hal_i2c.o(i.I2C_DMAMemTransmitCplt), (316 bytes).
    Removing stm32f7xx_hal_i2c.o(i.I2C_DMASlaveReceiveCplt), (112 bytes).
    Removing stm32f7xx_hal_i2c.o(i.I2C_DMASlaveTransmitCplt), (102 bytes).
    Removing stm32f7xx_hal_i2c.o(i.I2C_MasterReceive_ISR), (300 bytes).
    Removing stm32f7xx_hal_i2c.o(i.I2C_MasterTransmit_ISR), (312 bytes).
    Removing stm32f7xx_hal_i2c.o(i.I2C_SlaveReceive_ISR), (158 bytes).
    Removing stm32f7xx_hal_i2c.o(i.I2C_SlaveTransmit_ISR), (166 bytes).
    Removing stm32f7xx_hal_i2c.o(i.I2C_WaitOnRXNEFlagUntilTimeout), (128 bytes).
    Removing stm32f7xx_hal_gpio.o(.rev16_text), (4 bytes).
    Removing stm32f7xx_hal_gpio.o(.revsh_text), (4 bytes).
    Removing stm32f7xx_hal_gpio.o(.rrx_text), (6 bytes).
    Removing stm32f7xx_hal_gpio.o(i.HAL_GPIO_EXTI_Callback), (8 bytes).
    Removing stm32f7xx_hal_gpio.o(i.HAL_GPIO_EXTI_IRQHandler), (24 bytes).
    Removing stm32f7xx_hal_gpio.o(i.HAL_GPIO_LockPin), (34 bytes).
    Removing stm32f7xx_hal_gpio.o(i.HAL_GPIO_ReadPin), (10 bytes).
    Removing stm32f7xx_hal_rcc_ex.o(.rev16_text), (4 bytes).
    Removing stm32f7xx_hal_rcc_ex.o(.revsh_text), (4 bytes).
    Removing stm32f7xx_hal_rcc_ex.o(.rrx_text), (6 bytes).
    Removing stm32f7xx_hal_tim.o(.rev16_text), (4 bytes).
    Removing stm32f7xx_hal_tim.o(.revsh_text), (4 bytes).
    Removing stm32f7xx_hal_tim.o(.rrx_text), (6 bytes).
    Removing stm32f7xx_hal_tim.o(i.HAL_TIM_Base_DeInit), (56 bytes).
    Removing stm32f7xx_hal_tim.o(i.HAL_TIM_Base_GetState), (6 bytes).
    Removing stm32f7xx_hal_tim.o(i.HAL_TIM_Base_Init), (48 bytes).
    Removing stm32f7xx_hal_tim.o(i.HAL_TIM_Base_MspDeInit), (2 bytes).
    Removing stm32f7xx_hal_tim.o(i.HAL_TIM_Base_MspInit), (2 bytes).
    Removing stm32f7xx_hal_tim.o(i.HAL_TIM_Base_Start), (26 bytes).
    Removing stm32f7xx_hal_tim.o(i.HAL_TIM_Base_Start_DMA), (92 bytes).
    Removing stm32f7xx_hal_tim.o(i.HAL_TIM_Base_Start_IT), (24 bytes).
    Removing stm32f7xx_hal_tim.o(i.HAL_TIM_Base_Stop), (44 bytes).
    Removing stm32f7xx_hal_tim.o(i.HAL_TIM_Base_Stop_DMA), (48 bytes).
    Removing stm32f7xx_hal_tim.o(i.HAL_TIM_Base_Stop_IT), (42 bytes).
    Removing stm32f7xx_hal_tim.o(i.HAL_TIM_ConfigClockSource), (252 bytes).
    Removing stm32f7xx_hal_tim.o(i.HAL_TIM_ConfigOCrefClear), (170 bytes).
    Removing stm32f7xx_hal_tim.o(i.HAL_TIM_ConfigTI1Input), (16 bytes).
    Removing stm32f7xx_hal_tim.o(i.HAL_TIM_DMABurst_ReadStart), (260 bytes).
    Removing stm32f7xx_hal_tim.o(i.HAL_TIM_DMABurst_ReadStop), (96 bytes).
    Removing stm32f7xx_hal_tim.o(i.HAL_TIM_DMABurst_WriteStart), (260 bytes).
    Removing stm32f7xx_hal_tim.o(i.HAL_TIM_DMABurst_WriteStop), (96 bytes).
    Removing stm32f7xx_hal_tim.o(i.HAL_TIM_Encoder_DeInit), (56 bytes).
    Removing stm32f7xx_hal_tim.o(i.HAL_TIM_Encoder_GetState), (6 bytes).
    Removing stm32f7xx_hal_tim.o(i.HAL_TIM_Encoder_Init), (168 bytes).
    Removing stm32f7xx_hal_tim.o(i.HAL_TIM_Encoder_MspDeInit), (2 bytes).
    Removing stm32f7xx_hal_tim.o(i.HAL_TIM_Encoder_MspInit), (2 bytes).
    Removing stm32f7xx_hal_tim.o(i.HAL_TIM_Encoder_Start), (52 bytes).
    Removing stm32f7xx_hal_tim.o(i.HAL_TIM_Encoder_Start_DMA), (272 bytes).
    Removing stm32f7xx_hal_tim.o(i.HAL_TIM_Encoder_Start_IT), (92 bytes).
    Removing stm32f7xx_hal_tim.o(i.HAL_TIM_Encoder_Stop), (70 bytes).
    Removing stm32f7xx_hal_tim.o(i.HAL_TIM_Encoder_Stop_DMA), (116 bytes).
    Removing stm32f7xx_hal_tim.o(i.HAL_TIM_Encoder_Stop_IT), (116 bytes).
    Removing stm32f7xx_hal_tim.o(i.HAL_TIM_ErrorCallback), (2 bytes).
    Removing stm32f7xx_hal_tim.o(i.HAL_TIM_GenerateEvent), (40 bytes).
    Removing stm32f7xx_hal_tim.o(i.HAL_TIM_IC_CaptureCallback), (2 bytes).
    Removing stm32f7xx_hal_tim.o(i.HAL_TIM_IC_ConfigChannel), (288 bytes).
    Removing stm32f7xx_hal_tim.o(i.HAL_TIM_IC_DeInit), (56 bytes).
    Removing stm32f7xx_hal_tim.o(i.HAL_TIM_IC_GetState), (6 bytes).
    Removing stm32f7xx_hal_tim.o(i.HAL_TIM_IC_Init), (54 bytes).
    Removing stm32f7xx_hal_tim.o(i.HAL_TIM_IC_MspDeInit), (2 bytes).
    Removing stm32f7xx_hal_tim.o(i.HAL_TIM_IC_MspInit), (2 bytes).
    Removing stm32f7xx_hal_tim.o(i.HAL_TIM_IC_Start), (26 bytes).
    Removing stm32f7xx_hal_tim.o(i.HAL_TIM_IC_Start_DMA), (200 bytes).
    Removing stm32f7xx_hal_tim.o(i.HAL_TIM_IC_Start_IT), (76 bytes).
    Removing stm32f7xx_hal_tim.o(i.HAL_TIM_IC_Stop), (44 bytes).
    Removing stm32f7xx_hal_tim.o(i.HAL_TIM_IC_Stop_DMA), (100 bytes).
    Removing stm32f7xx_hal_tim.o(i.HAL_TIM_IC_Stop_IT), (94 bytes).
    Removing stm32f7xx_hal_tim.o(i.HAL_TIM_IRQHandler), (382 bytes).
    Removing stm32f7xx_hal_tim.o(i.HAL_TIM_OC_ConfigChannel), (86 bytes).
    Removing stm32f7xx_hal_tim.o(i.HAL_TIM_OC_DeInit), (56 bytes).
    Removing stm32f7xx_hal_tim.o(i.HAL_TIM_OC_DelayElapsedCallback), (2 bytes).
    Removing stm32f7xx_hal_tim.o(i.HAL_TIM_OC_GetState), (6 bytes).
    Removing stm32f7xx_hal_tim.o(i.HAL_TIM_OC_Init), (54 bytes).
    Removing stm32f7xx_hal_tim.o(i.HAL_TIM_OC_MspDeInit), (2 bytes).
    Removing stm32f7xx_hal_tim.o(i.HAL_TIM_OC_MspInit), (2 bytes).
    Removing stm32f7xx_hal_tim.o(i.HAL_TIM_OC_Start), (56 bytes).
    Removing stm32f7xx_hal_tim.o(i.HAL_TIM_OC_Start_DMA), (240 bytes).
    Removing stm32f7xx_hal_tim.o(i.HAL_TIM_OC_Start_IT), (108 bytes).
    Removing stm32f7xx_hal_tim.o(i.HAL_TIM_OC_Stop), (88 bytes).
    Removing stm32f7xx_hal_tim.o(i.HAL_TIM_OC_Stop_DMA), (144 bytes).
    Removing stm32f7xx_hal_tim.o(i.HAL_TIM_OC_Stop_IT), (136 bytes).
    Removing stm32f7xx_hal_tim.o(i.HAL_TIM_OnePulse_ConfigChannel), (224 bytes).
    Removing stm32f7xx_hal_tim.o(i.HAL_TIM_OnePulse_DeInit), (56 bytes).
    Removing stm32f7xx_hal_tim.o(i.HAL_TIM_OnePulse_GetState), (6 bytes).
    Removing stm32f7xx_hal_tim.o(i.HAL_TIM_OnePulse_Init), (74 bytes).
    Removing stm32f7xx_hal_tim.o(i.HAL_TIM_OnePulse_MspDeInit), (2 bytes).
    Removing stm32f7xx_hal_tim.o(i.HAL_TIM_OnePulse_MspInit), (2 bytes).
    Removing stm32f7xx_hal_tim.o(i.HAL_TIM_OnePulse_Start), (60 bytes).
    Removing stm32f7xx_hal_tim.o(i.HAL_TIM_OnePulse_Start_IT), (80 bytes).
    Removing stm32f7xx_hal_tim.o(i.HAL_TIM_OnePulse_Stop), (100 bytes).
    Removing stm32f7xx_hal_tim.o(i.HAL_TIM_OnePulse_Stop_IT), (120 bytes).
    Removing stm32f7xx_hal_tim.o(i.HAL_TIM_PWM_ConfigChannel), (208 bytes).
    Removing stm32f7xx_hal_tim.o(i.HAL_TIM_PWM_DeInit), (56 bytes).
    Removing stm32f7xx_hal_tim.o(i.HAL_TIM_PWM_GetState), (6 bytes).
    Removing stm32f7xx_hal_tim.o(i.HAL_TIM_PWM_Init), (54 bytes).
    Removing stm32f7xx_hal_tim.o(i.HAL_TIM_PWM_MspDeInit), (2 bytes).
    Removing stm32f7xx_hal_tim.o(i.HAL_TIM_PWM_MspInit), (2 bytes).
    Removing stm32f7xx_hal_tim.o(i.HAL_TIM_PWM_PulseFinishedCallback), (2 bytes).
    Removing stm32f7xx_hal_tim.o(i.HAL_TIM_PWM_Start), (56 bytes).
    Removing stm32f7xx_hal_tim.o(i.HAL_TIM_PWM_Start_DMA), (240 bytes).
    Removing stm32f7xx_hal_tim.o(i.HAL_TIM_PWM_Start_IT), (108 bytes).
    Removing stm32f7xx_hal_tim.o(i.HAL_TIM_PWM_Stop), (92 bytes).
    Removing stm32f7xx_hal_tim.o(i.HAL_TIM_PWM_Stop_DMA), (144 bytes).
    Removing stm32f7xx_hal_tim.o(i.HAL_TIM_PWM_Stop_IT), (136 bytes).
    Removing stm32f7xx_hal_tim.o(i.HAL_TIM_PeriodElapsedCallback), (2 bytes).
    Removing stm32f7xx_hal_tim.o(i.HAL_TIM_ReadCapturedValue), (68 bytes).
    Removing stm32f7xx_hal_tim.o(i.HAL_TIM_SlaveConfigSynchronization), (168 bytes).
    Removing stm32f7xx_hal_tim.o(i.HAL_TIM_SlaveConfigSynchronization_IT), (68 bytes).
    Removing stm32f7xx_hal_tim.o(i.HAL_TIM_TriggerCallback), (2 bytes).
    Removing stm32f7xx_hal_tim.o(i.TIM_Base_SetConfig), (196 bytes).
    Removing stm32f7xx_hal_tim.o(i.TIM_CCxChannelCmd), (22 bytes).
    Removing stm32f7xx_hal_tim.o(i.TIM_DMACaptureCplt), (62 bytes).
    Removing stm32f7xx_hal_tim.o(i.TIM_DMADelayPulseCplt), (62 bytes).
    Removing stm32f7xx_hal_tim.o(i.TIM_DMAError), (16 bytes).
    Removing stm32f7xx_hal_tim.o(i.TIM_DMAPeriodElapsedCplt), (16 bytes).
    Removing stm32f7xx_hal_tim.o(i.TIM_DMATriggerCplt), (16 bytes).
    Removing stm32f7xx_hal_tim.o(i.TIM_ETR_SetConfig), (18 bytes).
    Removing stm32f7xx_hal_tim.o(i.TIM_ITRx_SetConfig), (16 bytes).
    Removing stm32f7xx_hal_tim.o(i.TIM_OC1_SetConfig), (104 bytes).
    Removing stm32f7xx_hal_tim.o(i.TIM_OC2_SetConfig), (108 bytes).
    Removing stm32f7xx_hal_tim.o(i.TIM_OC3_SetConfig), (108 bytes).
    Removing stm32f7xx_hal_tim.o(i.TIM_OC4_SetConfig), (88 bytes).
    Removing stm32f7xx_hal_tim.o(i.TIM_SlaveTimer_SetConfig), (128 bytes).
    Removing stm32f7xx_hal_tim.o(i.TIM_TI1_ConfigInputStage), (34 bytes).
    Removing stm32f7xx_hal_tim.o(i.TIM_TI1_SetConfig), (128 bytes).
    Removing stm32f7xx_hal_tim.o(i.TIM_TI2_ConfigInputStage), (36 bytes).
    Removing stm32f7xx_hal_tim.o(i.TIM_TI2_SetConfig), (54 bytes).
    Removing stm32f7xx_hal_pcd_ex.o(.rev16_text), (4 bytes).
    Removing stm32f7xx_hal_pcd_ex.o(.revsh_text), (4 bytes).
    Removing stm32f7xx_hal_pcd_ex.o(.rrx_text), (6 bytes).
    Removing stm32f7xx_hal_pcd_ex.o(i.HAL_PCDEx_DeActivateLPM), (32 bytes).
    Removing stm32f7xx_hal_dma.o(.rev16_text), (4 bytes).
    Removing stm32f7xx_hal_dma.o(.revsh_text), (4 bytes).
    Removing stm32f7xx_hal_dma.o(.rrx_text), (6 bytes).
    Removing stm32f7xx_hal_dma.o(i.HAL_DMA_GetError), (4 bytes).
    Removing stm32f7xx_hal_dma.o(i.HAL_DMA_GetState), (6 bytes).
    Removing stm32f7xx_hal_dma.o(i.HAL_DMA_PollForTransfer), (328 bytes).
    Removing stm32f7xx_hal_dma.o(i.HAL_DMA_Start), (58 bytes).
    Removing stm32f7xx_hal_flash_ex.o(.rev16_text), (4 bytes).
    Removing stm32f7xx_hal_flash_ex.o(.revsh_text), (4 bytes).
    Removing stm32f7xx_hal_flash_ex.o(.rrx_text), (6 bytes).
    Removing stm32f7xx_hal_flash_ex.o(i.FLASH_Erase_Sector), (96 bytes).
    Removing stm32f7xx_hal_flash_ex.o(i.FLASH_MassErase), (44 bytes).
    Removing stm32f7xx_hal_flash_ex.o(i.FLASH_OB_BootAddressConfig), (48 bytes).
    Removing stm32f7xx_hal_flash_ex.o(i.FLASH_OB_GetBootAddress), (20 bytes).
    Removing stm32f7xx_hal_flash_ex.o(i.HAL_FLASHEx_Erase), (148 bytes).
    Removing stm32f7xx_hal_flash_ex.o(i.HAL_FLASHEx_Erase_IT), (100 bytes).
    Removing stm32f7xx_hal_flash_ex.o(i.HAL_FLASHEx_OBGetConfig), (80 bytes).
    Removing stm32f7xx_hal_flash_ex.o(i.HAL_FLASHEx_OBProgram), (236 bytes).
    Removing stm32f7xx_hal_usart.o(.rev16_text), (4 bytes).
    Removing stm32f7xx_hal_usart.o(.revsh_text), (4 bytes).
    Removing stm32f7xx_hal_usart.o(.rrx_text), (6 bytes).
    Removing stm32f7xx_hal_usart.o(i.HAL_USART_DMAPause), (78 bytes).
    Removing stm32f7xx_hal_usart.o(i.HAL_USART_DMAResume), (90 bytes).
    Removing stm32f7xx_hal_usart.o(i.HAL_USART_DMAStop), (50 bytes).
    Removing stm32f7xx_hal_usart.o(i.HAL_USART_DeInit), (50 bytes).
    Removing stm32f7xx_hal_usart.o(i.HAL_USART_ErrorCallback), (2 bytes).
    Removing stm32f7xx_hal_usart.o(i.HAL_USART_GetError), (4 bytes).
    Removing stm32f7xx_hal_usart.o(i.HAL_USART_GetState), (6 bytes).
    Removing stm32f7xx_hal_usart.o(i.HAL_USART_IRQHandler), (316 bytes).
    Removing stm32f7xx_hal_usart.o(i.HAL_USART_Init), (170 bytes).
    Removing stm32f7xx_hal_usart.o(i.HAL_USART_MspDeInit), (2 bytes).
    Removing stm32f7xx_hal_usart.o(i.HAL_USART_MspInit), (2 bytes).
    Removing stm32f7xx_hal_usart.o(i.HAL_USART_Receive), (226 bytes).
    Removing stm32f7xx_hal_usart.o(i.HAL_USART_Receive_DMA), (152 bytes).
    Removing stm32f7xx_hal_usart.o(i.HAL_USART_Receive_IT), (164 bytes).
    Removing stm32f7xx_hal_usart.o(i.HAL_USART_RxCpltCallback), (2 bytes).
    Removing stm32f7xx_hal_usart.o(i.HAL_USART_RxHalfCpltCallback), (2 bytes).
    Removing stm32f7xx_hal_usart.o(i.HAL_USART_Transmit), (152 bytes).
    Removing stm32f7xx_hal_usart.o(i.HAL_USART_TransmitReceive), (262 bytes).
    Removing stm32f7xx_hal_usart.o(i.HAL_USART_TransmitReceive_DMA), (188 bytes).
    Removing stm32f7xx_hal_usart.o(i.HAL_USART_TransmitReceive_IT), (162 bytes).
    Removing stm32f7xx_hal_usart.o(i.HAL_USART_Transmit_DMA), (124 bytes).
    Removing stm32f7xx_hal_usart.o(i.HAL_USART_Transmit_IT), (62 bytes).
    Removing stm32f7xx_hal_usart.o(i.HAL_USART_TxCpltCallback), (2 bytes).
    Removing stm32f7xx_hal_usart.o(i.HAL_USART_TxHalfCpltCallback), (2 bytes).
    Removing stm32f7xx_hal_usart.o(i.HAL_USART_TxRxCpltCallback), (2 bytes).
    Removing stm32f7xx_hal_usart.o(i.USART_DMAError), (30 bytes).
    Removing stm32f7xx_hal_usart.o(i.USART_DMAReceiveCplt), (86 bytes).
    Removing stm32f7xx_hal_usart.o(i.USART_DMARxHalfCplt), (10 bytes).
    Removing stm32f7xx_hal_usart.o(i.USART_DMATransmitCplt), (60 bytes).
    Removing stm32f7xx_hal_usart.o(i.USART_DMATxHalfCplt), (10 bytes).
    Removing stm32f7xx_hal_usart.o(i.USART_Receive_IT), (124 bytes).
    Removing stm32f7xx_hal_usart.o(i.USART_SetConfig), (296 bytes).
    Removing stm32f7xx_hal_usart.o(i.USART_TransmitReceive_IT), (206 bytes).
    Removing stm32f7xx_hal_usart.o(i.USART_WaitOnFlagUntilTimeout), (146 bytes).
    Removing stm32f7xx_hal_uart.o(.rev16_text), (4 bytes).
    Removing stm32f7xx_hal_uart.o(.revsh_text), (4 bytes).
    Removing stm32f7xx_hal_uart.o(.rrx_text), (6 bytes).
    Removing stm32f7xx_hal_uart.o(i.HAL_HalfDuplex_EnableReceiver), (60 bytes).
    Removing stm32f7xx_hal_uart.o(i.HAL_HalfDuplex_EnableTransmitter), (60 bytes).
    Removing stm32f7xx_hal_uart.o(i.HAL_HalfDuplex_Init), (116 bytes).
    Removing stm32f7xx_hal_uart.o(i.HAL_LIN_Init), (130 bytes).
    Removing stm32f7xx_hal_uart.o(i.HAL_LIN_SendBreak), (48 bytes).
    Removing stm32f7xx_hal_uart.o(i.HAL_MultiProcessor_DisableMuteMode), (42 bytes).
    Removing stm32f7xx_hal_uart.o(i.HAL_MultiProcessor_EnableMuteMode), (42 bytes).
    Removing stm32f7xx_hal_uart.o(i.HAL_MultiProcessor_EnterMuteMode), (12 bytes).
    Removing stm32f7xx_hal_uart.o(i.HAL_MultiProcessor_Init), (138 bytes).
    Removing stm32f7xx_hal_uart.o(i.HAL_UART_DMAPause), (86 bytes).
    Removing stm32f7xx_hal_uart.o(i.HAL_UART_DMAResume), (108 bytes).
    Removing stm32f7xx_hal_uart.o(i.HAL_UART_DMAStop), (50 bytes).
    Removing stm32f7xx_hal_uart.o(i.HAL_UART_ErrorCallback), (2 bytes).
    Removing stm32f7xx_hal_uart.o(i.HAL_UART_GetError), (4 bytes).
    Removing stm32f7xx_hal_uart.o(i.HAL_UART_GetState), (6 bytes).
    Removing stm32f7xx_hal_uart.o(i.HAL_UART_IRQHandler), (234 bytes).
    Removing stm32f7xx_hal_uart.o(i.HAL_UART_MspDeInit), (2 bytes).
    Removing stm32f7xx_hal_uart.o(i.HAL_UART_MspInit), (2 bytes).
    Removing stm32f7xx_hal_uart.o(i.HAL_UART_Receive), (268 bytes).
    Removing stm32f7xx_hal_uart.o(i.HAL_UART_Receive_DMA), (144 bytes).
    Removing stm32f7xx_hal_uart.o(i.HAL_UART_Receive_IT), (174 bytes).
    Removing stm32f7xx_hal_uart.o(i.HAL_UART_RxCpltCallback), (2 bytes).
    Removing stm32f7xx_hal_uart.o(i.HAL_UART_RxHalfCpltCallback), (2 bytes).
    Removing stm32f7xx_hal_uart.o(i.HAL_UART_Transmit_DMA), (152 bytes).
    Removing stm32f7xx_hal_uart.o(i.HAL_UART_Transmit_IT), (104 bytes).
    Removing stm32f7xx_hal_uart.o(i.HAL_UART_TxCpltCallback), (2 bytes).
    Removing stm32f7xx_hal_uart.o(i.HAL_UART_TxHalfCpltCallback), (2 bytes).
    Removing stm32f7xx_hal_uart.o(i.UART_DMAError), (34 bytes).
    Removing stm32f7xx_hal_uart.o(i.UART_DMAReceiveCplt), (54 bytes).
    Removing stm32f7xx_hal_uart.o(i.UART_DMARxHalfCplt), (10 bytes).
    Removing stm32f7xx_hal_uart.o(i.UART_DMATransmitCplt), (46 bytes).
    Removing stm32f7xx_hal_uart.o(i.UART_DMATxHalfCplt), (10 bytes).
    Removing stm32f7xx_hal_uart.o(i.UART_Receive_IT), (148 bytes).
    Removing stm32f7xx_hal_uart.o(i.UART_Transmit_IT), (146 bytes).
    Removing stm32f7xx_hal_i2s.o(.rev16_text), (4 bytes).
    Removing stm32f7xx_hal_i2s.o(.revsh_text), (4 bytes).
    Removing stm32f7xx_hal_i2s.o(.rrx_text), (6 bytes).
    Removing stm32f7xx_hal_i2s.o(i.HAL_I2S_DMAPause), (88 bytes).
    Removing stm32f7xx_hal_i2s.o(i.HAL_I2S_DMAResume), (82 bytes).
    Removing stm32f7xx_hal_i2s.o(i.HAL_I2S_DMAStop), (106 bytes).
    Removing stm32f7xx_hal_i2s.o(i.HAL_I2S_DeInit), (36 bytes).
    Removing stm32f7xx_hal_i2s.o(i.HAL_I2S_ErrorCallback), (2 bytes).
    Removing stm32f7xx_hal_i2s.o(i.HAL_I2S_GetError), (4 bytes).
    Removing stm32f7xx_hal_i2s.o(i.HAL_I2S_GetState), (6 bytes).
    Removing stm32f7xx_hal_i2s.o(i.HAL_I2S_IRQHandler), (220 bytes).
    Removing stm32f7xx_hal_i2s.o(i.HAL_I2S_Init), (296 bytes).
    Removing stm32f7xx_hal_i2s.o(i.HAL_I2S_MspDeInit), (2 bytes).
    Removing stm32f7xx_hal_i2s.o(i.HAL_I2S_MspInit), (2 bytes).
    Removing stm32f7xx_hal_i2s.o(i.HAL_I2S_Receive), (228 bytes).
    Removing stm32f7xx_hal_i2s.o(i.HAL_I2S_Receive_DMA), (192 bytes).
    Removing stm32f7xx_hal_i2s.o(i.HAL_I2S_Receive_IT), (116 bytes).
    Removing stm32f7xx_hal_i2s.o(i.HAL_I2S_RxCpltCallback), (2 bytes).
    Removing stm32f7xx_hal_i2s.o(i.HAL_I2S_RxHalfCpltCallback), (2 bytes).
    Removing stm32f7xx_hal_i2s.o(i.HAL_I2S_Transmit), (248 bytes).
    Removing stm32f7xx_hal_i2s.o(i.HAL_I2S_Transmit_DMA), (172 bytes).
    Removing stm32f7xx_hal_i2s.o(i.HAL_I2S_Transmit_IT), (116 bytes).
    Removing stm32f7xx_hal_i2s.o(i.HAL_I2S_TxCpltCallback), (2 bytes).
    Removing stm32f7xx_hal_i2s.o(i.HAL_I2S_TxHalfCpltCallback), (2 bytes).
    Removing stm32f7xx_hal_i2s.o(i.I2S_DMAError), (40 bytes).
    Removing stm32f7xx_hal_i2s.o(i.I2S_DMARxCplt), (50 bytes).
    Removing stm32f7xx_hal_i2s.o(i.I2S_DMARxHalfCplt), (10 bytes).
    Removing stm32f7xx_hal_i2s.o(i.I2S_DMATxCplt), (50 bytes).
    Removing stm32f7xx_hal_i2s.o(i.I2S_DMATxHalfCplt), (10 bytes).
    Removing stm32f7xx_hal_i2s.o(i.I2S_WaitFlagStateUntilTimeout), (106 bytes).
    Removing usbd_audio_if.o(.rev16_text), (4 bytes).
    Removing usbd_audio_if.o(.revsh_text), (4 bytes).
    Removing usbd_audio_if.o(.rrx_text), (6 bytes).
    Removing usbd_conf.o(.rev16_text), (4 bytes).
    Removing usbd_conf.o(.revsh_text), (4 bytes).
    Removing usbd_conf.o(.rrx_text), (6 bytes).
    Removing usbd_conf.o(i.HAL_PCD_MspDeInit), (60 bytes).
    Removing usbd_conf.o(i.USBD_LL_DeInit), (14 bytes).
    Removing usbd_conf.o(i.USBD_LL_Delay), (4 bytes).
    Removing usbd_conf.o(i.USBD_LL_FlushEP), (14 bytes).
    Removing usbd_conf.o(i.USBD_LL_GetRxDataSize), (8 bytes).
    Removing usbd_conf.o(i.USBD_LL_Stop), (14 bytes).
    Removing usbd_desc.o(.rev16_text), (4 bytes).
    Removing usbd_desc.o(.revsh_text), (4 bytes).
    Removing usbd_desc.o(.rrx_text), (6 bytes).
    Removing main.o(.rev16_text), (4 bytes).
    Removing main.o(.revsh_text), (4 bytes).
    Removing main.o(.rrx_text), (6 bytes).
    Removing main.o(.data), (10 bytes).
    Removing stm32f7xx_it.o(.rev16_text), (4 bytes).
    Removing stm32f7xx_it.o(.revsh_text), (4 bytes).
    Removing stm32f7xx_it.o(.rrx_text), (6 bytes).
    Removing usbd_ctlreq.o(.rev16_text), (4 bytes).
    Removing usbd_ctlreq.o(.revsh_text), (4 bytes).
    Removing usbd_ctlreq.o(.rrx_text), (6 bytes).
    Removing usbd_ioreq.o(.rev16_text), (4 bytes).
    Removing usbd_ioreq.o(.revsh_text), (4 bytes).
    Removing usbd_ioreq.o(.rrx_text), (6 bytes).
    Removing usbd_ioreq.o(i.USBD_GetRxCount), (10 bytes).
    Removing usbd_core.o(.rev16_text), (4 bytes).
    Removing usbd_core.o(.revsh_text), (4 bytes).
    Removing usbd_core.o(.rrx_text), (6 bytes).
    Removing usbd_core.o(i.USBD_DeInit), (40 bytes).
    Removing usbd_core.o(i.USBD_RunTestMode), (4 bytes).
    Removing usbd_core.o(i.USBD_Stop), (28 bytes).
    Removing stm32746g_discovery_audio.o(.rev16_text), (4 bytes).
    Removing stm32746g_discovery_audio.o(.revsh_text), (4 bytes).
    Removing stm32746g_discovery_audio.o(.rrx_text), (6 bytes).
    Removing stm32746g_discovery_audio.o(i.BSP_AUDIO_IN_DeInit), (20 bytes).
    Removing stm32746g_discovery_audio.o(i.BSP_AUDIO_IN_HalfTransfer_CallBack), (2 bytes).
    Removing stm32746g_discovery_audio.o(i.BSP_AUDIO_IN_Init), (152 bytes).
    Removing stm32746g_discovery_audio.o(i.BSP_AUDIO_IN_MspDeInit), (72 bytes).
    Removing stm32746g_discovery_audio.o(i.BSP_AUDIO_IN_MspInit), (256 bytes).
    Removing stm32746g_discovery_audio.o(i.BSP_AUDIO_IN_OUT_Init), (164 bytes).
    Removing stm32746g_discovery_audio.o(i.BSP_AUDIO_IN_Pause), (16 bytes).
    Removing stm32746g_discovery_audio.o(i.BSP_AUDIO_IN_Record), (20 bytes).
    Removing stm32746g_discovery_audio.o(i.BSP_AUDIO_IN_Resume), (16 bytes).
    Removing stm32746g_discovery_audio.o(i.BSP_AUDIO_IN_SetVolume), (32 bytes).
    Removing stm32746g_discovery_audio.o(i.BSP_AUDIO_IN_Stop), (52 bytes).
    Removing stm32746g_discovery_audio.o(i.BSP_AUDIO_IN_TransferComplete_CallBack), (2 bytes).
    Removing stm32746g_discovery_audio.o(i.BSP_AUDIO_OUT_ClockConfig), (82 bytes).
    Removing stm32746g_discovery_audio.o(i.BSP_AUDIO_OUT_DeInit), (20 bytes).
    Removing stm32746g_discovery_audio.o(i.BSP_AUDIO_OUT_HalfTransfer_CallBack), (2 bytes).
    Removing stm32746g_discovery_audio.o(i.BSP_AUDIO_OUT_MspDeInit), (92 bytes).
    Removing stm32746g_discovery_audio.o(i.BSP_AUDIO_OUT_Pause), (36 bytes).
    Removing stm32746g_discovery_audio.o(i.BSP_AUDIO_OUT_Resume), (36 bytes).
    Removing stm32746g_discovery_audio.o(i.BSP_AUDIO_OUT_SetFrequency), (52 bytes).
    Removing stm32746g_discovery_audio.o(i.BSP_AUDIO_OUT_SetOutputMode), (28 bytes).
    Removing stm32746g_discovery_audio.o(i.BSP_AUDIO_OUT_TransferComplete_CallBack), (2 bytes).
    Removing stm32746g_discovery_audio.o(i.HAL_SAI_RxCpltCallback), (8 bytes).
    Removing stm32746g_discovery_audio.o(i.HAL_SAI_RxHalfCpltCallback), (8 bytes).
    Removing stm32746g_discovery_audio.o(i.SAIx_In_DeInit), (28 bytes).
    Removing stm32746g_discovery_audio.o(i.SAIx_In_Init), (232 bytes).
    Removing stm32746g_discovery_audio.o(.bss), (60 bytes).
    Removing stm32746g_discovery.o(.rev16_text), (4 bytes).
    Removing stm32746g_discovery.o(.revsh_text), (4 bytes).
    Removing stm32746g_discovery.o(.rrx_text), (6 bytes).
    Removing stm32746g_discovery.o(i.BSP_COM_DeInit), (44 bytes).
    Removing stm32746g_discovery.o(i.BSP_COM_Init), (172 bytes).
    Removing stm32746g_discovery.o(i.BSP_GetVersion), (6 bytes).
    Removing stm32746g_discovery.o(i.BSP_LED_DeInit), (44 bytes).
    Removing stm32746g_discovery.o(i.BSP_LED_Off), (28 bytes).
    Removing stm32746g_discovery.o(i.BSP_LED_On), (28 bytes).
    Removing stm32746g_discovery.o(i.BSP_PB_DeInit), (48 bytes).
    Removing stm32746g_discovery.o(i.BSP_PB_GetState), (24 bytes).
    Removing stm32746g_discovery.o(i.BSP_PB_Init), (148 bytes).
    Removing stm32746g_discovery.o(i.CAMERA_Delay), (4 bytes).
    Removing stm32746g_discovery.o(i.CAMERA_IO_Init), (12 bytes).
    Removing stm32746g_discovery.o(i.CAMERA_IO_Read), (40 bytes).
    Removing stm32746g_discovery.o(i.CAMERA_IO_Write), (32 bytes).
    Removing stm32746g_discovery.o(i.EEPROM_IO_Init), (12 bytes).
    Removing stm32746g_discovery.o(i.EEPROM_IO_IsDeviceReady), (20 bytes).
    Removing stm32746g_discovery.o(i.EEPROM_IO_ReadData), (28 bytes).
    Removing stm32746g_discovery.o(i.EEPROM_IO_WriteData), (28 bytes).
    Removing stm32746g_discovery.o(i.TS_IO_Delay), (4 bytes).
    Removing stm32746g_discovery.o(i.TS_IO_Init), (12 bytes).
    Removing stm32746g_discovery.o(i.TS_IO_Read), (40 bytes).
    Removing stm32746g_discovery.o(i.TS_IO_Write), (32 bytes).
    Removing stm32746g_discovery.o(.data), (24 bytes).
    Removing usbd_audio.o(.rev16_text), (4 bytes).
    Removing usbd_audio.o(.revsh_text), (4 bytes).
    Removing usbd_audio.o(.rrx_text), (6 bytes).

612 unused section(s) (total 38508 bytes) removed from the image.

==============================================================================

Image Symbol Table

    Local Symbols

    Symbol Name                              Value     Ov Type        Size  Object(Section)

    ../clib/../cmprslib/zerorunl2.c          0x00000000   Number         0  __dczerorl2.o ABSOLUTE
    ../clib/microlib/init/entry.s            0x00000000   Number         0  entry8b.o ABSOLUTE
    ../clib/microlib/init/entry.s            0x00000000   Number         0  entry8a.o ABSOLUTE
    ../clib/microlib/init/entry.s            0x00000000   Number         0  entry5.o ABSOLUTE
    ../clib/microlib/init/entry.s            0x00000000   Number         0  entry7b.o ABSOLUTE
    ../clib/microlib/init/entry.s            0x00000000   Number         0  entry11b.o ABSOLUTE
    ../clib/microlib/init/entry.s            0x00000000   Number         0  entry7a.o ABSOLUTE
    ../clib/microlib/init/entry.s            0x00000000   Number         0  entry.o ABSOLUTE
    ../clib/microlib/init/entry.s            0x00000000   Number         0  entry11a.o ABSOLUTE
    ../clib/microlib/init/entry.s            0x00000000   Number         0  entry10b.o ABSOLUTE
    ../clib/microlib/init/entry.s            0x00000000   Number         0  entry10a.o ABSOLUTE
    ../clib/microlib/init/entry.s            0x00000000   Number         0  entry9b.o ABSOLUTE
    ../clib/microlib/init/entry.s            0x00000000   Number         0  entry9a.o ABSOLUTE
    ../clib/microlib/init/entry.s            0x00000000   Number         0  entry2.o ABSOLUTE
    ../clib/microlib/malloc/malloc.c         0x00000000   Number         0  malloca.o ABSOLUTE
    ../clib/microlib/malloc/malloc.c         0x00000000   Number         0  mallocr.o ABSOLUTE
    ../clib/microlib/malloc/malloc.c         0x00000000   Number         0  malloc.o ABSOLUTE
    ../clib/microlib/malloc/malloc.c         0x00000000   Number         0  mallocra.o ABSOLUTE
    ../clib/microlib/malloc/mvars.c          0x00000000   Number         0  mvars.o ABSOLUTE
    ../clib/microlib/string/memcpy.c         0x00000000   Number         0  memcpya.o ABSOLUTE
    ../clib/microlib/string/memcpy.c         0x00000000   Number         0  memcpyb.o ABSOLUTE
    ../clib/microlib/string/memset.c         0x00000000   Number         0  memseta.o ABSOLUTE
    ..\..\..\..\..\..\Drivers\BSP\Components\wm8994\wm8994.c 0x00000000   Number         0  wm8994.o ABSOLUTE
    ..\..\..\..\..\..\Drivers\BSP\STM32746G-Discovery\stm32746g_discovery.c 0x00000000   Number         0  stm32746g_discovery.o ABSOLUTE
    ..\..\..\..\..\..\Drivers\BSP\STM32746G-Discovery\stm32746g_discovery_audio.c 0x00000000   Number         0  stm32746g_discovery_audio.o ABSOLUTE
    ..\..\..\..\..\..\Drivers\STM32F7xx_HAL_Driver\Src\stm32f7xx_hal.c 0x00000000   Number         0  stm32f7xx_hal.o ABSOLUTE
    ..\..\..\..\..\..\Drivers\STM32F7xx_HAL_Driver\Src\stm32f7xx_hal_cortex.c 0x00000000   Number         0  stm32f7xx_hal_cortex.o ABSOLUTE
    ..\..\..\..\..\..\Drivers\STM32F7xx_HAL_Driver\Src\stm32f7xx_hal_dma.c 0x00000000   Number         0  stm32f7xx_hal_dma.o ABSOLUTE
    ..\..\..\..\..\..\Drivers\STM32F7xx_HAL_Driver\Src\stm32f7xx_hal_flash.c 0x00000000   Number         0  stm32f7xx_hal_flash.o ABSOLUTE
    ..\..\..\..\..\..\Drivers\STM32F7xx_HAL_Driver\Src\stm32f7xx_hal_flash_ex.c 0x00000000   Number         0  stm32f7xx_hal_flash_ex.o ABSOLUTE
    ..\..\..\..\..\..\Drivers\STM32F7xx_HAL_Driver\Src\stm32f7xx_hal_gpio.c 0x00000000   Number         0  stm32f7xx_hal_gpio.o ABSOLUTE
    ..\..\..\..\..\..\Drivers\STM32F7xx_HAL_Driver\Src\stm32f7xx_hal_i2c.c 0x00000000   Number         0  stm32f7xx_hal_i2c.o ABSOLUTE
    ..\..\..\..\..\..\Drivers\STM32F7xx_HAL_Driver\Src\stm32f7xx_hal_i2s.c 0x00000000   Number         0  stm32f7xx_hal_i2s.o ABSOLUTE
    ..\..\..\..\..\..\Drivers\STM32F7xx_HAL_Driver\Src\stm32f7xx_hal_pcd.c 0x00000000   Number         0  stm32f7xx_hal_pcd.o ABSOLUTE
    ..\..\..\..\..\..\Drivers\STM32F7xx_HAL_Driver\Src\stm32f7xx_hal_pcd_ex.c 0x00000000   Number         0  stm32f7xx_hal_pcd_ex.o ABSOLUTE
    ..\..\..\..\..\..\Drivers\STM32F7xx_HAL_Driver\Src\stm32f7xx_hal_pwr.c 0x00000000   Number         0  stm32f7xx_hal_pwr.o ABSOLUTE
    ..\..\..\..\..\..\Drivers\STM32F7xx_HAL_Driver\Src\stm32f7xx_hal_pwr_ex.c 0x00000000   Number         0  stm32f7xx_hal_pwr_ex.o ABSOLUTE
    ..\..\..\..\..\..\Drivers\STM32F7xx_HAL_Driver\Src\stm32f7xx_hal_rcc.c 0x00000000   Number         0  stm32f7xx_hal_rcc.o ABSOLUTE
    ..\..\..\..\..\..\Drivers\STM32F7xx_HAL_Driver\Src\stm32f7xx_hal_rcc_ex.c 0x00000000   Number         0  stm32f7xx_hal_rcc_ex.o ABSOLUTE
    ..\..\..\..\..\..\Drivers\STM32F7xx_HAL_Driver\Src\stm32f7xx_hal_sai.c 0x00000000   Number         0  stm32f7xx_hal_sai.o ABSOLUTE
    ..\..\..\..\..\..\Drivers\STM32F7xx_HAL_Driver\Src\stm32f7xx_hal_sai_ex.c 0x00000000   Number         0  stm32f7xx_hal_sai_ex.o ABSOLUTE
    ..\..\..\..\..\..\Drivers\STM32F7xx_HAL_Driver\Src\stm32f7xx_hal_tim.c 0x00000000   Number         0  stm32f7xx_hal_tim.o ABSOLUTE
    ..\..\..\..\..\..\Drivers\STM32F7xx_HAL_Driver\Src\stm32f7xx_hal_tim_ex.c 0x00000000   Number         0  stm32f7xx_hal_tim_ex.o ABSOLUTE
    ..\..\..\..\..\..\Drivers\STM32F7xx_HAL_Driver\Src\stm32f7xx_hal_uart.c 0x00000000   Number         0  stm32f7xx_hal_uart.o ABSOLUTE
    ..\..\..\..\..\..\Drivers\STM32F7xx_HAL_Driver\Src\stm32f7xx_hal_usart.c 0x00000000   Number         0  stm32f7xx_hal_usart.o ABSOLUTE
    ..\..\..\..\..\..\Drivers\STM32F7xx_HAL_Driver\Src\stm32f7xx_ll_usb.c 0x00000000   Number         0  stm32f7xx_ll_usb.o ABSOLUTE
    ..\..\..\..\..\..\Middlewares\ST\STM32_USB_Device_Library\Class\AUDIO\Src\usbd_audio.c 0x00000000   Number         0  usbd_audio.o ABSOLUTE
    ..\..\..\..\..\..\Middlewares\ST\STM32_USB_Device_Library\Core\Src\usbd_core.c 0x00000000   Number         0  usbd_core.o ABSOLUTE
    ..\..\..\..\..\..\Middlewares\ST\STM32_USB_Device_Library\Core\Src\usbd_ctlreq.c 0x00000000   Number         0  usbd_ctlreq.o ABSOLUTE
    ..\..\..\..\..\..\Middlewares\ST\STM32_USB_Device_Library\Core\Src\usbd_ioreq.c 0x00000000   Number         0  usbd_ioreq.o ABSOLUTE
    ..\Src\main.c                            0x00000000   Number         0  main.o ABSOLUTE
    ..\Src\stm32f7xx_it.c                    0x00000000   Number         0  stm32f7xx_it.o ABSOLUTE
    ..\Src\system_stm32f7xx.c                0x00000000   Number         0  system_stm32f7xx.o ABSOLUTE
    ..\Src\usbd_audio_if.c                   0x00000000   Number         0  usbd_audio_if.o ABSOLUTE
    ..\Src\usbd_conf.c                       0x00000000   Number         0  usbd_conf.o ABSOLUTE
    ..\Src\usbd_desc.c                       0x00000000   Number         0  usbd_desc.o ABSOLUTE
    ..\\..\\..\\..\\..\\..\\Drivers\\BSP\\STM32746G-Discovery\\stm32746g_discovery.c 0x00000000   Number         0  stm32746g_discovery.o ABSOLUTE
    ..\\..\\..\\..\\..\\..\\Drivers\\BSP\\STM32746G-Discovery\\stm32746g_discovery_audio.c 0x00000000   Number         0  stm32746g_discovery_audio.o ABSOLUTE
    ..\\..\\..\\..\\..\\..\\Drivers\\STM32F7xx_HAL_Driver\\Src\\stm32f7xx_hal.c 0x00000000   Number         0  stm32f7xx_hal.o ABSOLUTE
    ..\\..\\..\\..\\..\\..\\Drivers\\STM32F7xx_HAL_Driver\\Src\\stm32f7xx_hal_cortex.c 0x00000000   Number         0  stm32f7xx_hal_cortex.o ABSOLUTE
    ..\\..\\..\\..\\..\\..\\Drivers\\STM32F7xx_HAL_Driver\\Src\\stm32f7xx_hal_dma.c 0x00000000   Number         0  stm32f7xx_hal_dma.o ABSOLUTE
    ..\\..\\..\\..\\..\\..\\Drivers\\STM32F7xx_HAL_Driver\\Src\\stm32f7xx_hal_flash.c 0x00000000   Number         0  stm32f7xx_hal_flash.o ABSOLUTE
    ..\\..\\..\\..\\..\\..\\Drivers\\STM32F7xx_HAL_Driver\\Src\\stm32f7xx_hal_flash_ex.c 0x00000000   Number         0  stm32f7xx_hal_flash_ex.o ABSOLUTE
    ..\\..\\..\\..\\..\\..\\Drivers\\STM32F7xx_HAL_Driver\\Src\\stm32f7xx_hal_gpio.c 0x00000000   Number         0  stm32f7xx_hal_gpio.o ABSOLUTE
    ..\\..\\..\\..\\..\\..\\Drivers\\STM32F7xx_HAL_Driver\\Src\\stm32f7xx_hal_i2c.c 0x00000000   Number         0  stm32f7xx_hal_i2c.o ABSOLUTE
    ..\\..\\..\\..\\..\\..\\Drivers\\STM32F7xx_HAL_Driver\\Src\\stm32f7xx_hal_i2s.c 0x00000000   Number         0  stm32f7xx_hal_i2s.o ABSOLUTE
    ..\\..\\..\\..\\..\\..\\Drivers\\STM32F7xx_HAL_Driver\\Src\\stm32f7xx_hal_pcd.c 0x00000000   Number         0  stm32f7xx_hal_pcd.o ABSOLUTE
    ..\\..\\..\\..\\..\\..\\Drivers\\STM32F7xx_HAL_Driver\\Src\\stm32f7xx_hal_pcd_ex.c 0x00000000   Number         0  stm32f7xx_hal_pcd_ex.o ABSOLUTE
    ..\\..\\..\\..\\..\\..\\Drivers\\STM32F7xx_HAL_Driver\\Src\\stm32f7xx_hal_pwr.c 0x00000000   Number         0  stm32f7xx_hal_pwr.o ABSOLUTE
    ..\\..\\..\\..\\..\\..\\Drivers\\STM32F7xx_HAL_Driver\\Src\\stm32f7xx_hal_pwr_ex.c 0x00000000   Number         0  stm32f7xx_hal_pwr_ex.o ABSOLUTE
    ..\\..\\..\\..\\..\\..\\Drivers\\STM32F7xx_HAL_Driver\\Src\\stm32f7xx_hal_rcc.c 0x00000000   Number         0  stm32f7xx_hal_rcc.o ABSOLUTE
    ..\\..\\..\\..\\..\\..\\Drivers\\STM32F7xx_HAL_Driver\\Src\\stm32f7xx_hal_rcc_ex.c 0x00000000   Number         0  stm32f7xx_hal_rcc_ex.o ABSOLUTE
    ..\\..\\..\\..\\..\\..\\Drivers\\STM32F7xx_HAL_Driver\\Src\\stm32f7xx_hal_sai.c 0x00000000   Number         0  stm32f7xx_hal_sai.o ABSOLUTE
    ..\\..\\..\\..\\..\\..\\Drivers\\STM32F7xx_HAL_Driver\\Src\\stm32f7xx_hal_sai_ex.c 0x00000000   Number         0  stm32f7xx_hal_sai_ex.o ABSOLUTE
    ..\\..\\..\\..\\..\\..\\Drivers\\STM32F7xx_HAL_Driver\\Src\\stm32f7xx_hal_tim.c 0x00000000   Number         0  stm32f7xx_hal_tim.o ABSOLUTE
    ..\\..\\..\\..\\..\\..\\Drivers\\STM32F7xx_HAL_Driver\\Src\\stm32f7xx_hal_tim_ex.c 0x00000000   Number         0  stm32f7xx_hal_tim_ex.o ABSOLUTE
    ..\\..\\..\\..\\..\\..\\Drivers\\STM32F7xx_HAL_Driver\\Src\\stm32f7xx_hal_uart.c 0x00000000   Number         0  stm32f7xx_hal_uart.o ABSOLUTE
    ..\\..\\..\\..\\..\\..\\Drivers\\STM32F7xx_HAL_Driver\\Src\\stm32f7xx_hal_usart.c 0x00000000   Number         0  stm32f7xx_hal_usart.o ABSOLUTE
    ..\\..\\..\\..\\..\\..\\Drivers\\STM32F7xx_HAL_Driver\\Src\\stm32f7xx_ll_usb.c 0x00000000   Number         0  stm32f7xx_ll_usb.o ABSOLUTE
    ..\\..\\..\\..\\..\\..\\Middlewares\\ST\\STM32_USB_Device_Library\\Class\\AUDIO\\Src\\usbd_audio.c 0x00000000   Number         0  usbd_audio.o ABSOLUTE
    ..\\..\\..\\..\\..\\..\\Middlewares\\ST\\STM32_USB_Device_Library\\Core\\Src\\usbd_core.c 0x00000000   Number         0  usbd_core.o ABSOLUTE
    ..\\..\\..\\..\\..\\..\\Middlewares\\ST\\STM32_USB_Device_Library\\Core\\Src\\usbd_ctlreq.c 0x00000000   Number         0  usbd_ctlreq.o ABSOLUTE
    ..\\..\\..\\..\\..\\..\\Middlewares\\ST\\STM32_USB_Device_Library\\Core\\Src\\usbd_ioreq.c 0x00000000   Number         0  usbd_ioreq.o ABSOLUTE
    ..\\Src\\main.c                          0x00000000   Number         0  main.o ABSOLUTE
    ..\\Src\\stm32f7xx_it.c                  0x00000000   Number         0  stm32f7xx_it.o ABSOLUTE
    ..\\Src\\system_stm32f7xx.c              0x00000000   Number         0  system_stm32f7xx.o ABSOLUTE
    ..\\Src\\usbd_audio_if.c                 0x00000000   Number         0  usbd_audio_if.o ABSOLUTE
    ..\\Src\\usbd_conf.c                     0x00000000   Number         0  usbd_conf.o ABSOLUTE
    ..\\Src\\usbd_desc.c                     0x00000000   Number         0  usbd_desc.o ABSOLUTE
    dc.s                                     0x00000000   Number         0  dc.o ABSOLUTE
    handlers.s                               0x00000000   Number         0  handlers.o ABSOLUTE
    init.s                                   0x00000000   Number         0  init.o ABSOLUTE
    startup_stm32f746xx.s                    0x00000000   Number         0  startup_stm32f746xx.o ABSOLUTE
    RESET                                    0x08000000   Section      456  startup_stm32f746xx.o(RESET)
    .ARM.Collect$$$$00000000                 0x080001c8   Section        0  entry.o(.ARM.Collect$$$$00000000)
    .ARM.Collect$$$$00000001                 0x080001c8   Section        4  entry2.o(.ARM.Collect$$$$00000001)
    .ARM.Collect$$$$00000004                 0x080001cc   Section        4  entry5.o(.ARM.Collect$$$$00000004)
    .ARM.Collect$$$$00000008                 0x080001d0   Section        0  entry7b.o(.ARM.Collect$$$$00000008)
    .ARM.Collect$$$$0000000A                 0x080001d0   Section        0  entry8b.o(.ARM.Collect$$$$0000000A)
    .ARM.Collect$$$$0000000B                 0x080001d0   Section        8  entry9a.o(.ARM.Collect$$$$0000000B)
    .ARM.Collect$$$$0000000D                 0x080001d8   Section        0  entry10a.o(.ARM.Collect$$$$0000000D)
    .ARM.Collect$$$$0000000F                 0x080001d8   Section        0  entry11a.o(.ARM.Collect$$$$0000000F)
    .ARM.Collect$$$$00002712                 0x080001d8   Section        4  entry2.o(.ARM.Collect$$$$00002712)
    __lit__00000000                          0x080001d8   Data           4  entry2.o(.ARM.Collect$$$$00002712)
    .text                                    0x080001dc   Section       36  startup_stm32f746xx.o(.text)
    $v0                                      0x080001dc   Number         0  startup_stm32f746xx.o(.text)
    .text                                    0x08000200   Section        0  memcpya.o(.text)
    .text                                    0x08000224   Section        0  memseta.o(.text)
    .text                                    0x08000248   Section       36  init.o(.text)
    .text                                    0x0800026c   Section        0  __dczerorl2.o(.text)
    i.AUDIO_IO_DeInit                        0x080002c2   Section        0  stm32746g_discovery.o(i.AUDIO_IO_DeInit)
    i.AUDIO_IO_Delay                         0x080002c4   Section        0  stm32746g_discovery.o(i.AUDIO_IO_Delay)
    i.AUDIO_IO_Init                          0x080002c8   Section        0  stm32746g_discovery.o(i.AUDIO_IO_Init)
    i.AUDIO_IO_Read                          0x080002d4   Section        0  stm32746g_discovery.o(i.AUDIO_IO_Read)
    i.AUDIO_IO_Write                         0x08000308   Section        0  stm32746g_discovery.o(i.AUDIO_IO_Write)
    i.Audio_DeInit                           0x0800033c   Section        0  usbd_audio_if.o(i.Audio_DeInit)
    Audio_DeInit                             0x0800033d   Thumb Code    12  usbd_audio_if.o(i.Audio_DeInit)
    i.Audio_GetState                         0x08000348   Section        0  usbd_audio_if.o(i.Audio_GetState)
    Audio_GetState                           0x08000349   Thumb Code     4  usbd_audio_if.o(i.Audio_GetState)
    i.Audio_Init                             0x0800034c   Section        0  usbd_audio_if.o(i.Audio_Init)
    Audio_Init                               0x0800034d   Thumb Code    22  usbd_audio_if.o(i.Audio_Init)
    i.Audio_MuteCtl                          0x08000362   Section        0  usbd_audio_if.o(i.Audio_MuteCtl)
    Audio_MuteCtl                            0x08000363   Thumb Code    10  usbd_audio_if.o(i.Audio_MuteCtl)
    i.Audio_PeriodicTC                       0x0800036c   Section        0  usbd_audio_if.o(i.Audio_PeriodicTC)
    Audio_PeriodicTC                         0x0800036d   Thumb Code     4  usbd_audio_if.o(i.Audio_PeriodicTC)
    i.Audio_PlaybackCmd                      0x08000370   Section        0  usbd_audio_if.o(i.Audio_PlaybackCmd)
    Audio_PlaybackCmd                        0x08000371   Thumb Code    42  usbd_audio_if.o(i.Audio_PlaybackCmd)
    i.Audio_VolumeCtl                        0x080003a0   Section        0  usbd_audio_if.o(i.Audio_VolumeCtl)
    Audio_VolumeCtl                          0x080003a1   Thumb Code    10  usbd_audio_if.o(i.Audio_VolumeCtl)
    i.BSP_AUDIO_IN_Error_CallBack            0x080003aa   Section        0  stm32746g_discovery_audio.o(i.BSP_AUDIO_IN_Error_CallBack)
    i.BSP_AUDIO_OUT_ChangeBuffer             0x080003ac   Section        0  stm32746g_discovery_audio.o(i.BSP_AUDIO_OUT_ChangeBuffer)
    i.BSP_AUDIO_OUT_ClockConfig              0x080003bc   Section        0  main.o(i.BSP_AUDIO_OUT_ClockConfig)
    i.BSP_AUDIO_OUT_Error_CallBack           0x08000414   Section        0  stm32746g_discovery_audio.o(i.BSP_AUDIO_OUT_Error_CallBack)
    i.BSP_AUDIO_OUT_HalfTransfer_CallBack    0x08000418   Section        0  usbd_audio_if.o(i.BSP_AUDIO_OUT_HalfTransfer_CallBack)
    i.BSP_AUDIO_OUT_Init                     0x08000424   Section        0  stm32746g_discovery_audio.o(i.BSP_AUDIO_OUT_Init)
    i.BSP_AUDIO_OUT_MspInit                  0x08000498   Section        0  stm32746g_discovery_audio.o(i.BSP_AUDIO_OUT_MspInit)
    i.BSP_AUDIO_OUT_Play                     0x080005cc   Section        0  stm32746g_discovery_audio.o(i.BSP_AUDIO_OUT_Play)
    i.BSP_AUDIO_OUT_SetAudioFrameSlot        0x0800060c   Section        0  stm32746g_discovery_audio.o(i.BSP_AUDIO_OUT_SetAudioFrameSlot)
    i.BSP_AUDIO_OUT_SetMute                  0x08000634   Section        0  stm32746g_discovery_audio.o(i.BSP_AUDIO_OUT_SetMute)
    i.BSP_AUDIO_OUT_SetVolume                0x08000650   Section        0  stm32746g_discovery_audio.o(i.BSP_AUDIO_OUT_SetVolume)
    i.BSP_AUDIO_OUT_Stop                     0x0800066c   Section        0  stm32746g_discovery_audio.o(i.BSP_AUDIO_OUT_Stop)
    i.BSP_AUDIO_OUT_TransferComplete_CallBack 0x080006a0   Section        0  usbd_audio_if.o(i.BSP_AUDIO_OUT_TransferComplete_CallBack)
    i.BSP_LED_Init                           0x080006ac   Section        0  stm32746g_discovery.o(i.BSP_LED_Init)
    i.BSP_LED_Toggle                         0x080006fc   Section        0  stm32746g_discovery.o(i.BSP_LED_Toggle)
    i.BusFault_Handler                       0x08000718   Section        0  stm32f7xx_it.o(i.BusFault_Handler)
    i.CODEC_IO_Write                         0x0800071a   Section        0  wm8994.o(i.CODEC_IO_Write)
    CODEC_IO_Write                           0x0800071b   Thumb Code    10  wm8994.o(i.CODEC_IO_Write)
    i.CPU_CACHE_Enable                       0x08000724   Section        0  main.o(i.CPU_CACHE_Enable)
    CPU_CACHE_Enable                         0x08000725   Thumb Code   108  main.o(i.CPU_CACHE_Enable)
    i.DMA2_Stream4_IRQHandler                0x08000798   Section        0  stm32f7xx_it.o(i.DMA2_Stream4_IRQHandler)
    i.DMA_CalcBaseAndBitshift                0x080007a4   Section        0  stm32f7xx_hal_dma.o(i.DMA_CalcBaseAndBitshift)
    DMA_CalcBaseAndBitshift                  0x080007a5   Thumb Code    34  stm32f7xx_hal_dma.o(i.DMA_CalcBaseAndBitshift)
    i.DMA_SetConfig                          0x080007cc   Section        0  stm32f7xx_hal_dma.o(i.DMA_SetConfig)
    DMA_SetConfig                            0x080007cd   Thumb Code    40  stm32f7xx_hal_dma.o(i.DMA_SetConfig)
    i.DebugMon_Handler                       0x080007f4   Section        0  stm32f7xx_it.o(i.DebugMon_Handler)
    i.HAL_DMA_Abort                          0x080007f8   Section        0  stm32f7xx_hal_dma.o(i.HAL_DMA_Abort)
    i.HAL_DMA_DeInit                         0x0800084e   Section        0  stm32f7xx_hal_dma.o(i.HAL_DMA_DeInit)
    i.HAL_DMA_IRQHandler                     0x080008a4   Section        0  stm32f7xx_hal_dma.o(i.HAL_DMA_IRQHandler)
    i.HAL_DMA_Init                           0x08000a3c   Section        0  stm32f7xx_hal_dma.o(i.HAL_DMA_Init)
    i.HAL_DMA_Start_IT                       0x08000ac8   Section        0  stm32f7xx_hal_dma.o(i.HAL_DMA_Start_IT)
    i.HAL_Delay                              0x08000b16   Section        0  stm32f7xx_hal.o(i.HAL_Delay)
    i.HAL_GPIO_DeInit                        0x08000b2c   Section        0  stm32f7xx_hal_gpio.o(i.HAL_GPIO_DeInit)
    i.HAL_GPIO_Init                          0x08000c80   Section        0  stm32f7xx_hal_gpio.o(i.HAL_GPIO_Init)
    i.HAL_GPIO_TogglePin                     0x08000e58   Section        0  stm32f7xx_hal_gpio.o(i.HAL_GPIO_TogglePin)
    i.HAL_GPIO_WritePin                      0x08000e60   Section        0  stm32f7xx_hal_gpio.o(i.HAL_GPIO_WritePin)
    i.HAL_GetTick                            0x08000e6c   Section        0  stm32f7xx_hal.o(i.HAL_GetTick)
    i.HAL_I2C_DeInit                         0x08000e78   Section        0  stm32f7xx_hal_i2c.o(i.HAL_I2C_DeInit)
    i.HAL_I2C_GetState                       0x08000ea6   Section        0  stm32f7xx_hal_i2c.o(i.HAL_I2C_GetState)
    i.HAL_I2C_Init                           0x08000eac   Section        0  stm32f7xx_hal_i2c.o(i.HAL_I2C_Init)
    i.HAL_I2C_Mem_Read                       0x08000f58   Section        0  stm32f7xx_hal_i2c.o(i.HAL_I2C_Mem_Read)
    i.HAL_I2C_Mem_Write                      0x08001068   Section        0  stm32f7xx_hal_i2c.o(i.HAL_I2C_Mem_Write)
    i.HAL_I2C_MspDeInit                      0x08001178   Section        0  stm32f7xx_hal_i2c.o(i.HAL_I2C_MspDeInit)
    i.HAL_I2C_MspInit                        0x0800117a   Section        0  stm32f7xx_hal_i2c.o(i.HAL_I2C_MspInit)
    i.HAL_IncTick                            0x0800117c   Section        0  stm32f7xx_hal.o(i.HAL_IncTick)
    i.HAL_Init                               0x0800118c   Section        0  stm32f7xx_hal.o(i.HAL_Init)
    i.HAL_InitTick                           0x080011b0   Section        0  stm32f7xx_hal.o(i.HAL_InitTick)
    i.HAL_MspInit                            0x080011d2   Section        0  stm32f7xx_hal.o(i.HAL_MspInit)
    i.HAL_NVIC_EnableIRQ                     0x080011da   Section        0  stm32f7xx_hal_cortex.o(i.HAL_NVIC_EnableIRQ)
    i.HAL_NVIC_SetPriority                   0x080011f0   Section        0  stm32f7xx_hal_cortex.o(i.HAL_NVIC_SetPriority)
    i.HAL_NVIC_SetPriorityGrouping           0x08001230   Section        0  stm32f7xx_hal_cortex.o(i.HAL_NVIC_SetPriorityGrouping)
    i.HAL_PCDEx_ActivateLPM                  0x08001254   Section        0  stm32f7xx_hal_pcd_ex.o(i.HAL_PCDEx_ActivateLPM)
    i.HAL_PCDEx_LPM_Callback                 0x0800127c   Section        0  stm32f7xx_hal_pcd_ex.o(i.HAL_PCDEx_LPM_Callback)
    i.HAL_PCDEx_SetRxFiFo                    0x0800127e   Section        0  stm32f7xx_hal_pcd_ex.o(i.HAL_PCDEx_SetRxFiFo)
    i.HAL_PCDEx_SetTxFiFo                    0x08001286   Section        0  stm32f7xx_hal_pcd_ex.o(i.HAL_PCDEx_SetTxFiFo)
    i.HAL_PCD_ConnectCallback                0x080012ce   Section        0  usbd_conf.o(i.HAL_PCD_ConnectCallback)
    i.HAL_PCD_DataInStageCallback            0x080012d6   Section        0  usbd_conf.o(i.HAL_PCD_DataInStageCallback)
    i.HAL_PCD_DataOutStageCallback           0x080012e8   Section        0  usbd_conf.o(i.HAL_PCD_DataOutStageCallback)
    i.HAL_PCD_DisconnectCallback             0x080012fc   Section        0  usbd_conf.o(i.HAL_PCD_DisconnectCallback)
    i.HAL_PCD_EP_Close                       0x08001304   Section        0  stm32f7xx_hal_pcd.o(i.HAL_PCD_EP_Close)
    i.HAL_PCD_EP_ClrStall                    0x08001348   Section        0  stm32f7xx_hal_pcd.o(i.HAL_PCD_EP_ClrStall)
    i.HAL_PCD_EP_Open                        0x08001398   Section        0  stm32f7xx_hal_pcd.o(i.HAL_PCD_EP_Open)
    i.HAL_PCD_EP_Receive                     0x080013f0   Section        0  stm32f7xx_hal_pcd.o(i.HAL_PCD_EP_Receive)
    i.HAL_PCD_EP_SetStall                    0x0800144e   Section        0  stm32f7xx_hal_pcd.o(i.HAL_PCD_EP_SetStall)
    i.HAL_PCD_EP_Transmit                    0x080014b0   Section        0  stm32f7xx_hal_pcd.o(i.HAL_PCD_EP_Transmit)
    i.HAL_PCD_IRQHandler                     0x0800150c   Section        0  stm32f7xx_hal_pcd.o(i.HAL_PCD_IRQHandler)
    i.HAL_PCD_ISOINIncompleteCallback        0x08001954   Section        0  usbd_conf.o(i.HAL_PCD_ISOINIncompleteCallback)
    i.HAL_PCD_ISOOUTIncompleteCallback       0x0800195c   Section        0  usbd_conf.o(i.HAL_PCD_ISOOUTIncompleteCallback)
    i.HAL_PCD_Init                           0x08001964   Section        0  stm32f7xx_hal_pcd.o(i.HAL_PCD_Init)
    i.HAL_PCD_MspInit                        0x08001a34   Section        0  usbd_conf.o(i.HAL_PCD_MspInit)
    i.HAL_PCD_ResetCallback                  0x08001bb8   Section        0  usbd_conf.o(i.HAL_PCD_ResetCallback)
    i.HAL_PCD_ResumeCallback                 0x08001bda   Section        0  usbd_conf.o(i.HAL_PCD_ResumeCallback)
    i.HAL_PCD_SOFCallback                    0x08001be2   Section        0  usbd_conf.o(i.HAL_PCD_SOFCallback)
    i.HAL_PCD_SetAddress                     0x08001bea   Section        0  stm32f7xx_hal_pcd.o(i.HAL_PCD_SetAddress)
    i.HAL_PCD_SetupStageCallback             0x08001c0e   Section        0  usbd_conf.o(i.HAL_PCD_SetupStageCallback)
    i.HAL_PCD_Start                          0x08001c1c   Section        0  stm32f7xx_hal_pcd.o(i.HAL_PCD_Start)
    i.HAL_PCD_SuspendCallback                0x08001c46   Section        0  usbd_conf.o(i.HAL_PCD_SuspendCallback)
    i.HAL_PWREx_EnableOverDrive              0x08001c50   Section        0  stm32f7xx_hal_pwr_ex.o(i.HAL_PWREx_EnableOverDrive)
    i.HAL_RCCEx_GetPeriphCLKConfig           0x08001cbc   Section        0  stm32f7xx_hal_rcc_ex.o(i.HAL_RCCEx_GetPeriphCLKConfig)
    i.HAL_RCCEx_GetPeriphCLKFreq             0x08001e70   Section        0  stm32f7xx_hal_rcc_ex.o(i.HAL_RCCEx_GetPeriphCLKFreq)
    i.HAL_RCCEx_PeriphCLKConfig              0x08001f90   Section        0  stm32f7xx_hal_rcc_ex.o(i.HAL_RCCEx_PeriphCLKConfig)
    i.HAL_RCC_ClockConfig                    0x08002640   Section        0  stm32f7xx_hal_rcc.o(i.HAL_RCC_ClockConfig)
    i.HAL_RCC_GetHCLKFreq                    0x0800280c   Section        0  stm32f7xx_hal_rcc.o(i.HAL_RCC_GetHCLKFreq)
    i.HAL_RCC_GetPCLK1Freq                   0x08002840   Section        0  stm32f7xx_hal_rcc.o(i.HAL_RCC_GetPCLK1Freq)
    i.HAL_RCC_GetPCLK2Freq                   0x0800286c   Section        0  stm32f7xx_hal_rcc.o(i.HAL_RCC_GetPCLK2Freq)
    i.HAL_RCC_GetSysClockFreq                0x08002898   Section        0  stm32f7xx_hal_rcc.o(i.HAL_RCC_GetSysClockFreq)
    i.HAL_RCC_OscConfig                      0x0800291c   Section        0  stm32f7xx_hal_rcc.o(i.HAL_RCC_OscConfig)
    i.HAL_SAI_DMAStop                        0x08002cc0   Section        0  stm32f7xx_hal_sai.o(i.HAL_SAI_DMAStop)
    i.HAL_SAI_DeInit                         0x08002d0c   Section        0  stm32f7xx_hal_sai.o(i.HAL_SAI_DeInit)
    i.HAL_SAI_ErrorCallback                  0x08002d50   Section        0  stm32746g_discovery_audio.o(i.HAL_SAI_ErrorCallback)
    i.HAL_SAI_GetState                       0x08002d94   Section        0  stm32f7xx_hal_sai.o(i.HAL_SAI_GetState)
    i.HAL_SAI_Init                           0x08002d9c   Section        0  stm32f7xx_hal_sai.o(i.HAL_SAI_Init)
    i.HAL_SAI_MspDeInit                      0x08002f28   Section        0  stm32f7xx_hal_sai.o(i.HAL_SAI_MspDeInit)
    i.HAL_SAI_MspInit                        0x08002f2a   Section        0  stm32f7xx_hal_sai.o(i.HAL_SAI_MspInit)
    i.HAL_SAI_Transmit_DMA                   0x08002f2c   Section        0  stm32f7xx_hal_sai.o(i.HAL_SAI_Transmit_DMA)
    i.HAL_SAI_TxCpltCallback                 0x08002fcc   Section        0  stm32746g_discovery_audio.o(i.HAL_SAI_TxCpltCallback)
    i.HAL_SAI_TxHalfCpltCallback             0x08002fd4   Section        0  stm32746g_discovery_audio.o(i.HAL_SAI_TxHalfCpltCallback)
    i.HAL_SYSTICK_Config                     0x08002fdc   Section        0  stm32f7xx_hal_cortex.o(i.HAL_SYSTICK_Config)
    i.HAL_UART_DeInit                        0x08003002   Section        0  stm32f7xx_hal_uart.o(i.HAL_UART_DeInit)
    i.HAL_UART_Init                          0x0800303e   Section        0  stm32f7xx_hal_uart.o(i.HAL_UART_Init)
    i.HAL_UART_MspDeInit                     0x080030a8   Section        0  main.o(i.HAL_UART_MspDeInit)
    i.HAL_UART_MspInit                       0x080030dc   Section        0  main.o(i.HAL_UART_MspInit)
    i.HAL_UART_Transmit                      0x08003148   Section        0  stm32f7xx_hal_uart.o(i.HAL_UART_Transmit)
    i.HardFault_Handler                      0x08003210   Section        0  stm32f7xx_it.o(i.HardFault_Handler)
    i.I2C_IsAcknowledgeFailed                0x08003214   Section        0  stm32f7xx_hal_i2c.o(i.I2C_IsAcknowledgeFailed)
    I2C_IsAcknowledgeFailed                  0x08003215   Thumb Code   124  stm32f7xx_hal_i2c.o(i.I2C_IsAcknowledgeFailed)
    i.I2C_RequestMemoryRead                  0x08003294   Section        0  stm32f7xx_hal_i2c.o(i.I2C_RequestMemoryRead)
    I2C_RequestMemoryRead                    0x08003295   Thumb Code   102  stm32f7xx_hal_i2c.o(i.I2C_RequestMemoryRead)
    i.I2C_RequestMemoryWrite                 0x080032fa   Section        0  stm32f7xx_hal_i2c.o(i.I2C_RequestMemoryWrite)
    I2C_RequestMemoryWrite                   0x080032fb   Thumb Code   102  stm32f7xx_hal_i2c.o(i.I2C_RequestMemoryWrite)
    i.I2C_TransferConfig                     0x08003360   Section        0  stm32f7xx_hal_i2c.o(i.I2C_TransferConfig)
    I2C_TransferConfig                       0x08003361   Thumb Code    30  stm32f7xx_hal_i2c.o(i.I2C_TransferConfig)
    i.I2C_WaitOnFlagUntilTimeout             0x08003384   Section        0  stm32f7xx_hal_i2c.o(i.I2C_WaitOnFlagUntilTimeout)
    I2C_WaitOnFlagUntilTimeout               0x08003385   Thumb Code   110  stm32f7xx_hal_i2c.o(i.I2C_WaitOnFlagUntilTimeout)
    i.I2C_WaitOnSTOPFlagUntilTimeout         0x080033f2   Section        0  stm32f7xx_hal_i2c.o(i.I2C_WaitOnSTOPFlagUntilTimeout)
    I2C_WaitOnSTOPFlagUntilTimeout           0x080033f3   Thumb Code    78  stm32f7xx_hal_i2c.o(i.I2C_WaitOnSTOPFlagUntilTimeout)
    i.I2C_WaitOnTXISFlagUntilTimeout         0x08003440   Section        0  stm32f7xx_hal_i2c.o(i.I2C_WaitOnTXISFlagUntilTimeout)
    I2C_WaitOnTXISFlagUntilTimeout           0x08003441   Thumb Code    82  stm32f7xx_hal_i2c.o(i.I2C_WaitOnTXISFlagUntilTimeout)
    i.I2Cx_Error                             0x08003492   Section        0  stm32746g_discovery.o(i.I2Cx_Error)
    I2Cx_Error                               0x08003493   Thumb Code    18  stm32746g_discovery.o(i.I2Cx_Error)
    i.I2Cx_Init                              0x080034a4   Section        0  stm32746g_discovery.o(i.I2Cx_Init)
    I2Cx_Init                                0x080034a5   Thumb Code    64  stm32746g_discovery.o(i.I2Cx_Init)
    i.I2Cx_MspInit                           0x080034f4   Section        0  stm32746g_discovery.o(i.I2Cx_MspInit)
    I2Cx_MspInit                             0x080034f5   Thumb Code   266  stm32746g_discovery.o(i.I2Cx_MspInit)
    i.I2Cx_ReadMultiple                      0x08003618   Section        0  stm32746g_discovery.o(i.I2Cx_ReadMultiple)
    I2Cx_ReadMultiple                        0x08003619   Thumb Code    42  stm32746g_discovery.o(i.I2Cx_ReadMultiple)
    i.I2Cx_WriteMultiple                     0x08003642   Section        0  stm32746g_discovery.o(i.I2Cx_WriteMultiple)
    I2Cx_WriteMultiple                       0x08003643   Thumb Code    42  stm32746g_discovery.o(i.I2Cx_WriteMultiple)
    i.IntToUnicode                           0x0800366c   Section        0  usbd_desc.o(i.IntToUnicode)
    IntToUnicode                             0x0800366d   Thumb Code    56  usbd_desc.o(i.IntToUnicode)
    i.MemManage_Handler                      0x080036a4   Section        0  stm32f7xx_it.o(i.MemManage_Handler)
    i.NMI_Handler                            0x080036a6   Section        0  stm32f7xx_it.o(i.NMI_Handler)
    i.NVIC_SetPriority                       0x080036a8   Section        0  stm32f7xx_hal_cortex.o(i.NVIC_SetPriority)
    NVIC_SetPriority                         0x080036a9   Thumb Code    34  stm32f7xx_hal_cortex.o(i.NVIC_SetPriority)
    i.OTG_FS_IRQHandler                      0x080036cc   Section        0  stm32f7xx_it.o(i.OTG_FS_IRQHandler)
    i.PCD_WriteEmptyTxFifo                   0x080036d8   Section        0  stm32f7xx_hal_pcd.o(i.PCD_WriteEmptyTxFifo)
    PCD_WriteEmptyTxFifo                     0x080036d9   Thumb Code   150  stm32f7xx_hal_pcd.o(i.PCD_WriteEmptyTxFifo)
    i.PendSV_Handler                         0x0800376e   Section        0  stm32f7xx_it.o(i.PendSV_Handler)
    i.SAI_BlockSynchroConfig                 0x08003770   Section        0  stm32f7xx_hal_sai_ex.o(i.SAI_BlockSynchroConfig)
    i.SAI_DMAError                           0x080037b4   Section        0  stm32f7xx_hal_sai.o(i.SAI_DMAError)
    SAI_DMAError                             0x080037b5   Thumb Code    30  stm32f7xx_hal_sai.o(i.SAI_DMAError)
    i.SAI_DMATxCplt                          0x080037d2   Section        0  stm32f7xx_hal_sai.o(i.SAI_DMATxCplt)
    SAI_DMATxCplt                            0x080037d3   Thumb Code    60  stm32f7xx_hal_sai.o(i.SAI_DMATxCplt)
    i.SAI_DMATxHalfCplt                      0x0800380e   Section        0  stm32f7xx_hal_sai.o(i.SAI_DMATxHalfCplt)
    SAI_DMATxHalfCplt                        0x0800380f   Thumb Code    10  stm32f7xx_hal_sai.o(i.SAI_DMATxHalfCplt)
    i.SAI_Disable                            0x08003818   Section        0  stm32f7xx_hal_sai.o(i.SAI_Disable)
    SAI_Disable                              0x08003819   Thumb Code    62  stm32f7xx_hal_sai.o(i.SAI_Disable)
    i.SAI_GetInputClock                      0x08003858   Section        0  stm32f7xx_hal_sai_ex.o(i.SAI_GetInputClock)
    i.SAI_InterruptFlag                      0x0800387c   Section        0  stm32f7xx_hal_sai.o(i.SAI_InterruptFlag)
    SAI_InterruptFlag                        0x0800387d   Thumb Code    50  stm32f7xx_hal_sai.o(i.SAI_InterruptFlag)
    i.SAIx_Out_DeInit                        0x080038b0   Section        0  stm32746g_discovery_audio.o(i.SAIx_Out_DeInit)
    SAIx_Out_DeInit                          0x080038b1   Thumb Code    20  stm32746g_discovery_audio.o(i.SAIx_Out_DeInit)
    i.SAIx_Out_Init                          0x080038cc   Section        0  stm32746g_discovery_audio.o(i.SAIx_Out_Init)
    SAIx_Out_Init                            0x080038cd   Thumb Code    98  stm32746g_discovery_audio.o(i.SAIx_Out_Init)
    i.SVC_Handler                            0x08003938   Section        0  stm32f7xx_it.o(i.SVC_Handler)
    i.SysTick_Handler                        0x0800393a   Section        0  stm32f7xx_it.o(i.SysTick_Handler)
    i.SystemInit                             0x08003940   Section        0  system_stm32f7xx.o(i.SystemInit)
    i.UART_AdvFeatureConfig                  0x08003994   Section        0  stm32f7xx_hal_uart.o(i.UART_AdvFeatureConfig)
    i.UART_CheckIdleState                    0x08003a5c   Section        0  stm32f7xx_hal_uart.o(i.UART_CheckIdleState)
    i.UART_SetConfig                         0x08003aac   Section        0  stm32f7xx_hal_uart.o(i.UART_SetConfig)
    i.UART_WaitOnFlagUntilTimeout            0x08003cf4   Section        0  stm32f7xx_hal_uart.o(i.UART_WaitOnFlagUntilTimeout)
    i.USBD_AUDIO_ConfigStrDescriptor         0x08003d88   Section        0  usbd_desc.o(i.USBD_AUDIO_ConfigStrDescriptor)
    i.USBD_AUDIO_DataIn                      0x08003dac   Section        0  usbd_audio.o(i.USBD_AUDIO_DataIn)
    USBD_AUDIO_DataIn                        0x08003dad   Thumb Code     4  usbd_audio.o(i.USBD_AUDIO_DataIn)
    i.USBD_AUDIO_DataOut                     0x08003db0   Section        0  usbd_audio.o(i.USBD_AUDIO_DataOut)
    USBD_AUDIO_DataOut                       0x08003db1   Thumb Code   116  usbd_audio.o(i.USBD_AUDIO_DataOut)
    i.USBD_AUDIO_DeInit                      0x08003e24   Section        0  usbd_audio.o(i.USBD_AUDIO_DeInit)
    USBD_AUDIO_DeInit                        0x08003e25   Thumb Code    44  usbd_audio.o(i.USBD_AUDIO_DeInit)
    i.USBD_AUDIO_DeviceDescriptor            0x08003e50   Section        0  usbd_desc.o(i.USBD_AUDIO_DeviceDescriptor)
    i.USBD_AUDIO_EP0_RxReady                 0x08003e5c   Section        0  usbd_audio.o(i.USBD_AUDIO_EP0_RxReady)
    USBD_AUDIO_EP0_RxReady                   0x08003e5d   Thumb Code    52  usbd_audio.o(i.USBD_AUDIO_EP0_RxReady)
    i.USBD_AUDIO_EP0_TxReady                 0x08003e90   Section        0  usbd_audio.o(i.USBD_AUDIO_EP0_TxReady)
    USBD_AUDIO_EP0_TxReady                   0x08003e91   Thumb Code     4  usbd_audio.o(i.USBD_AUDIO_EP0_TxReady)
    i.USBD_AUDIO_GetCfgDesc                  0x08003e94   Section        0  usbd_audio.o(i.USBD_AUDIO_GetCfgDesc)
    USBD_AUDIO_GetCfgDesc                    0x08003e95   Thumb Code     8  usbd_audio.o(i.USBD_AUDIO_GetCfgDesc)
    i.USBD_AUDIO_GetDeviceQualifierDesc      0x08003ea0   Section        0  usbd_audio.o(i.USBD_AUDIO_GetDeviceQualifierDesc)
    USBD_AUDIO_GetDeviceQualifierDesc        0x08003ea1   Thumb Code     8  usbd_audio.o(i.USBD_AUDIO_GetDeviceQualifierDesc)
    i.USBD_AUDIO_Init                        0x08003eac   Section        0  usbd_audio.o(i.USBD_AUDIO_Init)
    USBD_AUDIO_Init                          0x08003ead   Thumb Code    90  usbd_audio.o(i.USBD_AUDIO_Init)
    i.USBD_AUDIO_InterfaceStrDescriptor      0x08003f08   Section        0  usbd_desc.o(i.USBD_AUDIO_InterfaceStrDescriptor)
    i.USBD_AUDIO_IsoINIncomplete             0x08003f2c   Section        0  usbd_audio.o(i.USBD_AUDIO_IsoINIncomplete)
    USBD_AUDIO_IsoINIncomplete               0x08003f2d   Thumb Code     4  usbd_audio.o(i.USBD_AUDIO_IsoINIncomplete)
    i.USBD_AUDIO_IsoOutIncomplete            0x08003f30   Section        0  usbd_audio.o(i.USBD_AUDIO_IsoOutIncomplete)
    USBD_AUDIO_IsoOutIncomplete              0x08003f31   Thumb Code     4  usbd_audio.o(i.USBD_AUDIO_IsoOutIncomplete)
    i.USBD_AUDIO_LangIDStrDescriptor         0x08003f34   Section        0  usbd_desc.o(i.USBD_AUDIO_LangIDStrDescriptor)
    i.USBD_AUDIO_ManufacturerStrDescriptor   0x08003f40   Section        0  usbd_desc.o(i.USBD_AUDIO_ManufacturerStrDescriptor)
    i.USBD_AUDIO_ProductStrDescriptor        0x08003f68   Section        0  usbd_desc.o(i.USBD_AUDIO_ProductStrDescriptor)
    i.USBD_AUDIO_RegisterInterface           0x08003fcc   Section        0  usbd_audio.o(i.USBD_AUDIO_RegisterInterface)
    i.USBD_AUDIO_SOF                         0x08003fd6   Section        0  usbd_audio.o(i.USBD_AUDIO_SOF)
    USBD_AUDIO_SOF                           0x08003fd7   Thumb Code     4  usbd_audio.o(i.USBD_AUDIO_SOF)
    i.USBD_AUDIO_SerialStrDescriptor         0x08003fdc   Section        0  usbd_desc.o(i.USBD_AUDIO_SerialStrDescriptor)
    i.USBD_AUDIO_Setup                       0x08004018   Section        0  usbd_audio.o(i.USBD_AUDIO_Setup)
    USBD_AUDIO_Setup                         0x08004019   Thumb Code   186  usbd_audio.o(i.USBD_AUDIO_Setup)
    i.USBD_AUDIO_Sync                        0x080040d8   Section        0  usbd_audio.o(i.USBD_AUDIO_Sync)
    i.USBD_ClrClassConfig                    0x0800415e   Section        0  usbd_core.o(i.USBD_ClrClassConfig)
    i.USBD_CtlContinueRx                     0x0800416c   Section        0  usbd_ioreq.o(i.USBD_CtlContinueRx)
    i.USBD_CtlContinueSendData               0x0800417c   Section        0  usbd_ioreq.o(i.USBD_CtlContinueSendData)
    i.USBD_CtlError                          0x0800418c   Section        0  usbd_ctlreq.o(i.USBD_CtlError)
    i.USBD_CtlPrepareRx                      0x080041a2   Section        0  usbd_ioreq.o(i.USBD_CtlPrepareRx)
    i.USBD_CtlReceiveStatus                  0x080041c0   Section        0  usbd_ioreq.o(i.USBD_CtlReceiveStatus)
    i.USBD_CtlSendData                       0x080041d6   Section        0  usbd_ioreq.o(i.USBD_CtlSendData)
    i.USBD_CtlSendStatus                     0x080041f0   Section        0  usbd_ioreq.o(i.USBD_CtlSendStatus)
    i.USBD_GetDescriptor                     0x08004206   Section        0  usbd_ctlreq.o(i.USBD_GetDescriptor)
    USBD_GetDescriptor                       0x08004207   Thumb Code   224  usbd_ctlreq.o(i.USBD_GetDescriptor)
    i.USBD_GetString                         0x080042e6   Section        0  usbd_ctlreq.o(i.USBD_GetString)
    i.USBD_Init                              0x0800432e   Section        0  usbd_core.o(i.USBD_Init)
    i.USBD_LL_ClearStallEP                   0x08004358   Section        0  usbd_conf.o(i.USBD_LL_ClearStallEP)
    i.USBD_LL_CloseEP                        0x08004366   Section        0  usbd_conf.o(i.USBD_LL_CloseEP)
    i.USBD_LL_DataInStage                    0x08004374   Section        0  usbd_core.o(i.USBD_LL_DataInStage)
    i.USBD_LL_DataOutStage                   0x0800441e   Section        0  usbd_core.o(i.USBD_LL_DataOutStage)
    i.USBD_LL_DevConnected                   0x08004488   Section        0  usbd_core.o(i.USBD_LL_DevConnected)
    i.USBD_LL_DevDisconnected                0x0800448c   Section        0  usbd_core.o(i.USBD_LL_DevDisconnected)
    i.USBD_LL_Init                           0x080044a4   Section        0  usbd_conf.o(i.USBD_LL_Init)
    i.USBD_LL_IsStallEP                      0x080044f4   Section        0  usbd_conf.o(i.USBD_LL_IsStallEP)
    i.USBD_LL_IsoINIncomplete                0x08004514   Section        0  usbd_core.o(i.USBD_LL_IsoINIncomplete)
    i.USBD_LL_IsoOUTIncomplete               0x08004518   Section        0  usbd_core.o(i.USBD_LL_IsoOUTIncomplete)
    i.USBD_LL_OpenEP                         0x0800451c   Section        0  usbd_conf.o(i.USBD_LL_OpenEP)
    i.USBD_LL_PrepareReceive                 0x08004530   Section        0  usbd_conf.o(i.USBD_LL_PrepareReceive)
    i.USBD_LL_Reset                          0x0800453e   Section        0  usbd_core.o(i.USBD_LL_Reset)
    i.USBD_LL_Resume                         0x0800457e   Section        0  usbd_core.o(i.USBD_LL_Resume)
    i.USBD_LL_SOF                            0x0800458a   Section        0  usbd_core.o(i.USBD_LL_SOF)
    i.USBD_LL_SetSpeed                       0x080045a2   Section        0  usbd_core.o(i.USBD_LL_SetSpeed)
    i.USBD_LL_SetUSBAddress                  0x080045a8   Section        0  usbd_conf.o(i.USBD_LL_SetUSBAddress)
    i.USBD_LL_SetupStage                     0x080045b6   Section        0  usbd_core.o(i.USBD_LL_SetupStage)
    i.USBD_LL_StallEP                        0x0800460c   Section        0  usbd_conf.o(i.USBD_LL_StallEP)
    i.USBD_LL_Start                          0x0800461a   Section        0  usbd_conf.o(i.USBD_LL_Start)
    i.USBD_LL_Suspend                        0x08004628   Section        0  usbd_core.o(i.USBD_LL_Suspend)
    i.USBD_LL_Transmit                       0x0800463a   Section        0  usbd_conf.o(i.USBD_LL_Transmit)
    i.USBD_ParseSetupRequest                 0x08004648   Section        0  usbd_ctlreq.o(i.USBD_ParseSetupRequest)
    i.USBD_RegisterClass                     0x08004670   Section        0  usbd_core.o(i.USBD_RegisterClass)
    i.USBD_SetClassConfig                    0x08004682   Section        0  usbd_core.o(i.USBD_SetClassConfig)
    i.USBD_SetConfig                         0x08004698   Section        0  usbd_ctlreq.o(i.USBD_SetConfig)
    USBD_SetConfig                           0x08004699   Thumb Code   112  usbd_ctlreq.o(i.USBD_SetConfig)
    i.USBD_Start                             0x0800470c   Section        0  usbd_core.o(i.USBD_Start)
    i.USBD_StdDevReq                         0x08004716   Section        0  usbd_ctlreq.o(i.USBD_StdDevReq)
    i.USBD_StdEPReq                          0x08004808   Section        0  usbd_ctlreq.o(i.USBD_StdEPReq)
    i.USBD_StdItfReq                         0x080048e6   Section        0  usbd_ctlreq.o(i.USBD_StdItfReq)
    i.USB_ActivateEndpoint                   0x0800491c   Section        0  stm32f7xx_ll_usb.o(i.USB_ActivateEndpoint)
    i.USB_ActivateSetup                      0x0800499c   Section        0  stm32f7xx_ll_usb.o(i.USB_ActivateSetup)
    i.USB_CoreInit                           0x080049d0   Section        0  stm32f7xx_ll_usb.o(i.USB_CoreInit)
    i.USB_CoreReset                          0x08004a40   Section        0  stm32f7xx_ll_usb.o(i.USB_CoreReset)
    USB_CoreReset                            0x08004a41   Thumb Code    50  stm32f7xx_ll_usb.o(i.USB_CoreReset)
    i.USB_DeactivateEndpoint                 0x08004a78   Section        0  stm32f7xx_ll_usb.o(i.USB_DeactivateEndpoint)
    i.USB_DevConnect                         0x08004ae6   Section        0  stm32f7xx_ll_usb.o(i.USB_DevConnect)
    i.USB_DevDisconnect                      0x08004afe   Section        0  stm32f7xx_ll_usb.o(i.USB_DevDisconnect)
    i.USB_DevInit                            0x08004b18   Section        0  stm32f7xx_ll_usb.o(i.USB_DevInit)
    i.USB_DisableGlobalInt                   0x08004c74   Section        0  stm32f7xx_ll_usb.o(i.USB_DisableGlobalInt)
    i.USB_EP0StartXfer                       0x08004c80   Section        0  stm32f7xx_ll_usb.o(i.USB_EP0StartXfer)
    i.USB_EP0_OutStart                       0x08004dc0   Section        0  stm32f7xx_ll_usb.o(i.USB_EP0_OutStart)
    i.USB_EPClearStall                       0x08004dfe   Section        0  stm32f7xx_ll_usb.o(i.USB_EPClearStall)
    i.USB_EPSetStall                         0x08004e62   Section        0  stm32f7xx_ll_usb.o(i.USB_EPSetStall)
    i.USB_EPStartXfer                        0x08004ec0   Section        0  stm32f7xx_ll_usb.o(i.USB_EPStartXfer)
    i.USB_EnableGlobalInt                    0x080050dc   Section        0  stm32f7xx_ll_usb.o(i.USB_EnableGlobalInt)
    i.USB_FlushRxFifo                        0x080050e8   Section        0  stm32f7xx_ll_usb.o(i.USB_FlushRxFifo)
    i.USB_FlushTxFifo                        0x08005108   Section        0  stm32f7xx_ll_usb.o(i.USB_FlushTxFifo)
    i.USB_GetDevSpeed                        0x0800512c   Section        0  stm32f7xx_ll_usb.o(i.USB_GetDevSpeed)
    i.USB_GetMode                            0x0800516a   Section        0  stm32f7xx_ll_usb.o(i.USB_GetMode)
    i.USB_ReadDevAllInEpInterrupt            0x08005172   Section        0  stm32f7xx_ll_usb.o(i.USB_ReadDevAllInEpInterrupt)
    i.USB_ReadDevAllOutEpInterrupt           0x08005180   Section        0  stm32f7xx_ll_usb.o(i.USB_ReadDevAllOutEpInterrupt)
    i.USB_ReadDevInEPInterrupt               0x0800518e   Section        0  stm32f7xx_ll_usb.o(i.USB_ReadDevInEPInterrupt)
    i.USB_ReadDevOutEPInterrupt              0x080051ae   Section        0  stm32f7xx_ll_usb.o(i.USB_ReadDevOutEPInterrupt)
    i.USB_ReadInterrupts                     0x080051be   Section        0  stm32f7xx_ll_usb.o(i.USB_ReadInterrupts)
    i.USB_ReadPacket                         0x080051c6   Section        0  stm32f7xx_ll_usb.o(i.USB_ReadPacket)
    i.USB_SetCurrentMode                     0x080051e4   Section        0  stm32f7xx_ll_usb.o(i.USB_SetCurrentMode)
    i.USB_SetDevAddress                      0x08005210   Section        0  stm32f7xx_ll_usb.o(i.USB_SetDevAddress)
    i.USB_WritePacket                        0x08005234   Section        0  stm32f7xx_ll_usb.o(i.USB_WritePacket)
    i.UsageFault_Handler                     0x08005260   Section        0  stm32f7xx_it.o(i.UsageFault_Handler)
    i.__scatterload_copy                     0x08005262   Section       14  handlers.o(i.__scatterload_copy)
    i.__scatterload_null                     0x08005270   Section        2  handlers.o(i.__scatterload_null)
    i.__scatterload_zeroinit                 0x08005272   Section       14  handlers.o(i.__scatterload_zeroinit)
    i.free                                   0x08005280   Section        0  malloc.o(i.free)
    i.main                                   0x080052d0   Section        0  main.o(i.main)
    i.malloc                                 0x080053cc   Section        0  malloc.o(i.malloc)
    i.wm8994_DeInit                          0x08005438   Section        0  wm8994.o(i.wm8994_DeInit)
    i.wm8994_Init                            0x0800543c   Section        0  wm8994.o(i.wm8994_Init)
    i.wm8994_Pause                           0x080058c0   Section        0  wm8994.o(i.wm8994_Pause)
    i.wm8994_Play                            0x080058da   Section        0  wm8994.o(i.wm8994_Play)
    i.wm8994_ReadID                          0x080058e0   Section        0  wm8994.o(i.wm8994_ReadID)
    i.wm8994_Reset                           0x080058f4   Section        0  wm8994.o(i.wm8994_Reset)
    i.wm8994_Resume                          0x08005910   Section        0  wm8994.o(i.wm8994_Resume)
    i.wm8994_SetFrequency                    0x08005916   Section        0  wm8994.o(i.wm8994_SetFrequency)
    i.wm8994_SetMute                         0x0800598c   Section        0  wm8994.o(i.wm8994_SetMute)
    i.wm8994_SetOutputMode                   0x080059e4   Section        0  wm8994.o(i.wm8994_SetOutputMode)
    i.wm8994_SetVolume                       0x08005aa0   Section        0  wm8994.o(i.wm8994_SetVolume)
    i.wm8994_Stop                            0x08005bbc   Section        0  wm8994.o(i.wm8994_Stop)
    .constdata                               0x08005c38   Section       16  stm32f7xx_hal_rcc.o(.constdata)
    .constdata                               0x08005c48   Section        8  stm32f7xx_hal_dma.o(.constdata)
    flagBitshiftOffset                       0x08005c48   Data           8  stm32f7xx_hal_dma.o(.constdata)
    .constdata                               0x08005c50   Section       24  stm32746g_discovery.o(.constdata)
    .data                                    0x20000000   Section       20  system_stm32f7xx.o(.data)
    .data                                    0x20000014   Section        4  stm32f7xx_hal.o(.data)
    uwTick                                   0x20000014   Data           4  stm32f7xx_hal.o(.data)
    .data                                    0x20000018   Section       48  wm8994.o(.data)
    .data                                    0x20000048   Section        8  wm8994.o(.data)
    outputEnabled                            0x20000048   Data           4  wm8994.o(.data)
    inputEnabled                             0x2000004c   Data           4  wm8994.o(.data)
    .data                                    0x20000050   Section       28  usbd_audio_if.o(.data)
    .data                                    0x2000006c   Section        1  usbd_audio_if.o(.data)
    .data                                    0x20000070   Section       28  usbd_desc.o(.data)
    .data                                    0x2000008c   Section       48  usbd_desc.o(.data)
    .data                                    0x200000bc   Section        4  main.o(.data)
    ticks                                    0x200000bc   Data           4  main.o(.data)
    .data                                    0x200000c0   Section        1  usbd_ctlreq.o(.data)
    cfgidx                                   0x200000c0   Data           1  usbd_ctlreq.o(.data)
    .data                                    0x200000c4   Section        8  stm32746g_discovery_audio.o(.data)
    .data                                    0x200000cc   Section       56  usbd_audio.o(.data)
    .data                                    0x20000104   Section      122  usbd_audio.o(.data)
    USBD_AUDIO_CfgDesc                       0x20000104   Data         109  usbd_audio.o(.data)
    USBD_AUDIO_DeviceQualifierDesc           0x20000174   Data          10  usbd_audio.o(.data)
    .data                                    0x20000180   Section        4  mvars.o(.data)
    .data                                    0x20000184   Section        4  mvars.o(.data)
    .bss                                     0x20000188   Section      960  usbd_conf.o(.bss)
    .bss                                     0x20000548   Section      256  usbd_desc.o(.bss)
    .bss                                     0x20000648   Section      660  main.o(.bss)
    .bss                                     0x200008dc   Section      528  stm32746g_discovery_audio.o(.bss)
    hdma_sai_tx                              0x200009e4   Data          88  stm32746g_discovery_audio.o(.bss)
    hdma_sai_rx                              0x20000a3c   Data          88  stm32746g_discovery_audio.o(.bss)
    hdma_sai_rx                              0x20000a94   Data          88  stm32746g_discovery_audio.o(.bss)
    .bss                                     0x20000aec   Section      120  stm32746g_discovery.o(.bss)
    hI2cAudioHandler                         0x20000aec   Data          60  stm32746g_discovery.o(.bss)
    hI2cExtHandler                           0x20000b28   Data          60  stm32746g_discovery.o(.bss)
    HEAP                                     0x20000b68   Section    16384  startup_stm32f746xx.o(HEAP)
    STACK                                    0x20004b68   Section     8192  startup_stm32f746xx.o(STACK)

    Global Symbols

    Symbol Name                              Value     Ov Type        Size  Object(Section)

    BuildAttributes$$THM_ISAv4$E$P$D$K$B$S$7EM$VFPi5$EXTD16$VFPS$VFMA$PE$PLD8$A:L22UL41UL21$X:L11$S22US41US21$IEEE1$IW$USESV6$~STKCKD$USESV7$~SHL$OSPACE$EBA8$MICROLIB$REQ8$PRES8$EABIv2 0x00000000   Number         0  anon$$obj.o ABSOLUTE
    __ARM_use_no_argv                        0x00000000   Number         0  main.o ABSOLUTE
    __cpp_initialize__aeabi_                  - Undefined Weak Reference
    __cxa_finalize                            - Undefined Weak Reference
    _clock_init                               - Undefined Weak Reference
    _microlib_exit                            - Undefined Weak Reference
    __Vectors_Size                           0x000001c8   Number         0  startup_stm32f746xx.o ABSOLUTE
    __Vectors                                0x08000000   Data           4  startup_stm32f746xx.o(RESET)
    __Vectors_End                            0x080001c8   Data           0  startup_stm32f746xx.o(RESET)
    __main                                   0x080001c9   Thumb Code     0  entry.o(.ARM.Collect$$$$00000000)
    _main_stk                                0x080001c9   Thumb Code     0  entry2.o(.ARM.Collect$$$$00000001)
    _main_scatterload                        0x080001cd   Thumb Code     0  entry5.o(.ARM.Collect$$$$00000004)
    __main_after_scatterload                 0x080001d1   Thumb Code     0  entry5.o(.ARM.Collect$$$$00000004)
    _main_clock                              0x080001d1   Thumb Code     0  entry7b.o(.ARM.Collect$$$$00000008)
    _main_cpp_init                           0x080001d1   Thumb Code     0  entry8b.o(.ARM.Collect$$$$0000000A)
    _main_init                               0x080001d1   Thumb Code     0  entry9a.o(.ARM.Collect$$$$0000000B)
    __rt_final_cpp                           0x080001d9   Thumb Code     0  entry10a.o(.ARM.Collect$$$$0000000D)
    __rt_final_exit                          0x080001d9   Thumb Code     0  entry11a.o(.ARM.Collect$$$$0000000F)
    Reset_Handler                            0x080001dd   Thumb Code     8  startup_stm32f746xx.o(.text)
    ADC_IRQHandler                           0x080001f7   Thumb Code     0  startup_stm32f746xx.o(.text)
    CAN1_RX0_IRQHandler                      0x080001f7   Thumb Code     0  startup_stm32f746xx.o(.text)
    CAN1_RX1_IRQHandler                      0x080001f7   Thumb Code     0  startup_stm32f746xx.o(.text)
    CAN1_SCE_IRQHandler                      0x080001f7   Thumb Code     0  startup_stm32f746xx.o(.text)
    CAN1_TX_IRQHandler                       0x080001f7   Thumb Code     0  startup_stm32f746xx.o(.text)
    CAN2_RX0_IRQHandler                      0x080001f7   Thumb Code     0  startup_stm32f746xx.o(.text)
    CAN2_RX1_IRQHandler                      0x080001f7   Thumb Code     0  startup_stm32f746xx.o(.text)
    CAN2_SCE_IRQHandler                      0x080001f7   Thumb Code     0  startup_stm32f746xx.o(.text)
    CAN2_TX_IRQHandler                       0x080001f7   Thumb Code     0  startup_stm32f746xx.o(.text)
    CEC_IRQHandler                           0x080001f7   Thumb Code     0  startup_stm32f746xx.o(.text)
    DCMI_IRQHandler                          0x080001f7   Thumb Code     0  startup_stm32f746xx.o(.text)
    DMA1_Stream0_IRQHandler                  0x080001f7   Thumb Code     0  startup_stm32f746xx.o(.text)
    DMA1_Stream1_IRQHandler                  0x080001f7   Thumb Code     0  startup_stm32f746xx.o(.text)
    DMA1_Stream2_IRQHandler                  0x080001f7   Thumb Code     0  startup_stm32f746xx.o(.text)
    DMA1_Stream3_IRQHandler                  0x080001f7   Thumb Code     0  startup_stm32f746xx.o(.text)
    DMA1_Stream4_IRQHandler                  0x080001f7   Thumb Code     0  startup_stm32f746xx.o(.text)
    DMA1_Stream5_IRQHandler                  0x080001f7   Thumb Code     0  startup_stm32f746xx.o(.text)
    DMA1_Stream6_IRQHandler                  0x080001f7   Thumb Code     0  startup_stm32f746xx.o(.text)
    DMA1_Stream7_IRQHandler                  0x080001f7   Thumb Code     0  startup_stm32f746xx.o(.text)
    DMA2D_IRQHandler                         0x080001f7   Thumb Code     0  startup_stm32f746xx.o(.text)
    DMA2_Stream0_IRQHandler                  0x080001f7   Thumb Code     0  startup_stm32f746xx.o(.text)
    DMA2_Stream1_IRQHandler                  0x080001f7   Thumb Code     0  startup_stm32f746xx.o(.text)
    DMA2_Stream2_IRQHandler                  0x080001f7   Thumb Code     0  startup_stm32f746xx.o(.text)
    DMA2_Stream3_IRQHandler                  0x080001f7   Thumb Code     0  startup_stm32f746xx.o(.text)
    DMA2_Stream5_IRQHandler                  0x080001f7   Thumb Code     0  startup_stm32f746xx.o(.text)
    DMA2_Stream6_IRQHandler                  0x080001f7   Thumb Code     0  startup_stm32f746xx.o(.text)
    DMA2_Stream7_IRQHandler                  0x080001f7   Thumb Code     0  startup_stm32f746xx.o(.text)
    ETH_IRQHandler                           0x080001f7   Thumb Code     0  startup_stm32f746xx.o(.text)
    ETH_WKUP_IRQHandler                      0x080001f7   Thumb Code     0  startup_stm32f746xx.o(.text)
    EXTI0_IRQHandler                         0x080001f7   Thumb Code     0  startup_stm32f746xx.o(.text)
    EXTI15_10_IRQHandler                     0x080001f7   Thumb Code     0  startup_stm32f746xx.o(.text)
    EXTI1_IRQHandler                         0x080001f7   Thumb Code     0  startup_stm32f746xx.o(.text)
    EXTI2_IRQHandler                         0x080001f7   Thumb Code     0  startup_stm32f746xx.o(.text)
    EXTI3_IRQHandler                         0x080001f7   Thumb Code     0  startup_stm32f746xx.o(.text)
    EXTI4_IRQHandler                         0x080001f7   Thumb Code     0  startup_stm32f746xx.o(.text)
    EXTI9_5_IRQHandler                       0x080001f7   Thumb Code     0  startup_stm32f746xx.o(.text)
    FLASH_IRQHandler                         0x080001f7   Thumb Code     0  startup_stm32f746xx.o(.text)
    FMC_IRQHandler                           0x080001f7   Thumb Code     0  startup_stm32f746xx.o(.text)
    FPU_IRQHandler                           0x080001f7   Thumb Code     0  startup_stm32f746xx.o(.text)
    I2C1_ER_IRQHandler                       0x080001f7   Thumb Code     0  startup_stm32f746xx.o(.text)
    I2C1_EV_IRQHandler                       0x080001f7   Thumb Code     0  startup_stm32f746xx.o(.text)
    I2C2_ER_IRQHandler                       0x080001f7   Thumb Code     0  startup_stm32f746xx.o(.text)
    I2C2_EV_IRQHandler                       0x080001f7   Thumb Code     0  startup_stm32f746xx.o(.text)
    I2C3_ER_IRQHandler                       0x080001f7   Thumb Code     0  startup_stm32f746xx.o(.text)
    I2C3_EV_IRQHandler                       0x080001f7   Thumb Code     0  startup_stm32f746xx.o(.text)
    I2C4_ER_IRQHandler                       0x080001f7   Thumb Code     0  startup_stm32f746xx.o(.text)
    I2C4_EV_IRQHandler                       0x080001f7   Thumb Code     0  startup_stm32f746xx.o(.text)
    LPTIM1_IRQHandler                        0x080001f7   Thumb Code     0  startup_stm32f746xx.o(.text)
    LTDC_ER_IRQHandler                       0x080001f7   Thumb Code     0  startup_stm32f746xx.o(.text)
    LTDC_IRQHandler                          0x080001f7   Thumb Code     0  startup_stm32f746xx.o(.text)
    OTG_FS_WKUP_IRQHandler                   0x080001f7   Thumb Code     0  startup_stm32f746xx.o(.text)
    OTG_HS_EP1_IN_IRQHandler                 0x080001f7   Thumb Code     0  startup_stm32f746xx.o(.text)
    OTG_HS_EP1_OUT_IRQHandler                0x080001f7   Thumb Code     0  startup_stm32f746xx.o(.text)
    OTG_HS_IRQHandler                        0x080001f7   Thumb Code     0  startup_stm32f746xx.o(.text)
    OTG_HS_WKUP_IRQHandler                   0x080001f7   Thumb Code     0  startup_stm32f746xx.o(.text)
    PVD_IRQHandler                           0x080001f7   Thumb Code     0  startup_stm32f746xx.o(.text)
    QUADSPI_IRQHandler                       0x080001f7   Thumb Code     0  startup_stm32f746xx.o(.text)
    RCC_IRQHandler                           0x080001f7   Thumb Code     0  startup_stm32f746xx.o(.text)
    RNG_IRQHandler                           0x080001f7   Thumb Code     0  startup_stm32f746xx.o(.text)
    RTC_Alarm_IRQHandler                     0x080001f7   Thumb Code     0  startup_stm32f746xx.o(.text)
    RTC_WKUP_IRQHandler                      0x080001f7   Thumb Code     0  startup_stm32f746xx.o(.text)
    SAI1_IRQHandler                          0x080001f7   Thumb Code     0  startup_stm32f746xx.o(.text)
    SAI2_IRQHandler                          0x080001f7   Thumb Code     0  startup_stm32f746xx.o(.text)
    SDMMC1_IRQHandler                        0x080001f7   Thumb Code     0  startup_stm32f746xx.o(.text)
    SPDIF_RX_IRQHandler                      0x080001f7   Thumb Code     0  startup_stm32f746xx.o(.text)
    SPI1_IRQHandler                          0x080001f7   Thumb Code     0  startup_stm32f746xx.o(.text)
    SPI2_IRQHandler                          0x080001f7   Thumb Code     0  startup_stm32f746xx.o(.text)
    SPI3_IRQHandler                          0x080001f7   Thumb Code     0  startup_stm32f746xx.o(.text)
    SPI4_IRQHandler                          0x080001f7   Thumb Code     0  startup_stm32f746xx.o(.text)
    SPI5_IRQHandler                          0x080001f7   Thumb Code     0  startup_stm32f746xx.o(.text)
    SPI6_IRQHandler                          0x080001f7   Thumb Code     0  startup_stm32f746xx.o(.text)
    TAMP_STAMP_IRQHandler                    0x080001f7   Thumb Code     0  startup_stm32f746xx.o(.text)
    TIM1_BRK_TIM9_IRQHandler                 0x080001f7   Thumb Code     0  startup_stm32f746xx.o(.text)
    TIM1_CC_IRQHandler                       0x080001f7   Thumb Code     0  startup_stm32f746xx.o(.text)
    TIM1_TRG_COM_TIM11_IRQHandler            0x080001f7   Thumb Code     0  startup_stm32f746xx.o(.text)
    TIM1_UP_TIM10_IRQHandler                 0x080001f7   Thumb Code     0  startup_stm32f746xx.o(.text)
    TIM2_IRQHandler                          0x080001f7   Thumb Code     0  startup_stm32f746xx.o(.text)
    TIM3_IRQHandler                          0x080001f7   Thumb Code     0  startup_stm32f746xx.o(.text)
    TIM4_IRQHandler                          0x080001f7   Thumb Code     0  startup_stm32f746xx.o(.text)
    TIM5_IRQHandler                          0x080001f7   Thumb Code     0  startup_stm32f746xx.o(.text)
    TIM6_DAC_IRQHandler                      0x080001f7   Thumb Code     0  startup_stm32f746xx.o(.text)
    TIM7_IRQHandler                          0x080001f7   Thumb Code     0  startup_stm32f746xx.o(.text)
    TIM8_BRK_TIM12_IRQHandler                0x080001f7   Thumb Code     0  startup_stm32f746xx.o(.text)
    TIM8_CC_IRQHandler                       0x080001f7   Thumb Code     0  startup_stm32f746xx.o(.text)
    TIM8_TRG_COM_TIM14_IRQHandler            0x080001f7   Thumb Code     0  startup_stm32f746xx.o(.text)
    TIM8_UP_TIM13_IRQHandler                 0x080001f7   Thumb Code     0  startup_stm32f746xx.o(.text)
    UART4_IRQHandler                         0x080001f7   Thumb Code     0  startup_stm32f746xx.o(.text)
    UART5_IRQHandler                         0x080001f7   Thumb Code     0  startup_stm32f746xx.o(.text)
    UART7_IRQHandler                         0x080001f7   Thumb Code     0  startup_stm32f746xx.o(.text)
    UART8_IRQHandler                         0x080001f7   Thumb Code     0  startup_stm32f746xx.o(.text)
    USART1_IRQHandler                        0x080001f7   Thumb Code     0  startup_stm32f746xx.o(.text)
    USART2_IRQHandler                        0x080001f7   Thumb Code     0  startup_stm32f746xx.o(.text)
    USART3_IRQHandler                        0x080001f7   Thumb Code     0  startup_stm32f746xx.o(.text)
    USART6_IRQHandler                        0x080001f7   Thumb Code     0  startup_stm32f746xx.o(.text)
    WWDG_IRQHandler                          0x080001f7   Thumb Code     0  startup_stm32f746xx.o(.text)
    __aeabi_memcpy                           0x08000201   Thumb Code    36  memcpya.o(.text)
    __aeabi_memcpy4                          0x08000201   Thumb Code     0  memcpya.o(.text)
    __aeabi_memcpy8                          0x08000201   Thumb Code     0  memcpya.o(.text)
    __aeabi_memset                           0x08000225   Thumb Code    14  memseta.o(.text)
    __aeabi_memset4                          0x08000225   Thumb Code     0  memseta.o(.text)
    __aeabi_memset8                          0x08000225   Thumb Code     0  memseta.o(.text)
    __aeabi_memclr                           0x08000233   Thumb Code     4  memseta.o(.text)
    __aeabi_memclr4                          0x08000233   Thumb Code     0  memseta.o(.text)
    __aeabi_memclr8                          0x08000233   Thumb Code     0  memseta.o(.text)
    _memset$wrapper                          0x08000237   Thumb Code    18  memseta.o(.text)
    __scatterload                            0x08000249   Thumb Code    28  init.o(.text)
    __scatterload_rt2                        0x08000249   Thumb Code     0  init.o(.text)
    __decompress                             0x0800026d   Thumb Code     0  __dczerorl2.o(.text)
    __decompress1                            0x0800026d   Thumb Code    86  __dczerorl2.o(.text)
    AUDIO_IO_DeInit                          0x080002c3   Thumb Code     2  stm32746g_discovery.o(i.AUDIO_IO_DeInit)
    AUDIO_IO_Delay                           0x080002c5   Thumb Code     4  stm32746g_discovery.o(i.AUDIO_IO_Delay)
    AUDIO_IO_Init                            0x080002c9   Thumb Code     6  stm32746g_discovery.o(i.AUDIO_IO_Init)
    AUDIO_IO_Read                            0x080002d5   Thumb Code    46  stm32746g_discovery.o(i.AUDIO_IO_Read)
    AUDIO_IO_Write                           0x08000309   Thumb Code    46  stm32746g_discovery.o(i.AUDIO_IO_Write)
    BSP_AUDIO_IN_Error_CallBack              0x080003ab   Thumb Code     2  stm32746g_discovery_audio.o(i.BSP_AUDIO_IN_Error_CallBack)
    BSP_AUDIO_OUT_ChangeBuffer               0x080003ad   Thumb Code    10  stm32746g_discovery_audio.o(i.BSP_AUDIO_OUT_ChangeBuffer)
    BSP_AUDIO_OUT_ClockConfig                0x080003bd   Thumb Code    88  main.o(i.BSP_AUDIO_OUT_ClockConfig)
    BSP_AUDIO_OUT_Error_CallBack             0x08000415   Thumb Code     2  stm32746g_discovery_audio.o(i.BSP_AUDIO_OUT_Error_CallBack)
    BSP_AUDIO_OUT_HalfTransfer_CallBack      0x08000419   Thumb Code     8  usbd_audio_if.o(i.BSP_AUDIO_OUT_HalfTransfer_CallBack)
    BSP_AUDIO_OUT_Init                       0x08000425   Thumb Code   100  stm32746g_discovery_audio.o(i.BSP_AUDIO_OUT_Init)
    BSP_AUDIO_OUT_MspInit                    0x08000499   Thumb Code   288  stm32746g_discovery_audio.o(i.BSP_AUDIO_OUT_MspInit)
    BSP_AUDIO_OUT_Play                       0x080005cd   Thumb Code    54  stm32746g_discovery_audio.o(i.BSP_AUDIO_OUT_Play)
    BSP_AUDIO_OUT_SetAudioFrameSlot          0x0800060d   Thumb Code    34  stm32746g_discovery_audio.o(i.BSP_AUDIO_OUT_SetAudioFrameSlot)
    BSP_AUDIO_OUT_SetMute                    0x08000635   Thumb Code    22  stm32746g_discovery_audio.o(i.BSP_AUDIO_OUT_SetMute)
    BSP_AUDIO_OUT_SetVolume                  0x08000651   Thumb Code    22  stm32746g_discovery_audio.o(i.BSP_AUDIO_OUT_SetVolume)
    BSP_AUDIO_OUT_Stop                       0x0800066d   Thumb Code    42  stm32746g_discovery_audio.o(i.BSP_AUDIO_OUT_Stop)
    BSP_AUDIO_OUT_TransferComplete_CallBack  0x080006a1   Thumb Code     8  usbd_audio_if.o(i.BSP_AUDIO_OUT_TransferComplete_CallBack)
    BSP_LED_Init                             0x080006ad   Thumb Code    68  stm32746g_discovery.o(i.BSP_LED_Init)
    BSP_LED_Toggle                           0x080006fd   Thumb Code    18  stm32746g_discovery.o(i.BSP_LED_Toggle)
    BusFault_Handler                         0x08000719   Thumb Code     2  stm32f7xx_it.o(i.BusFault_Handler)
    DMA2_Stream4_IRQHandler                  0x08000799   Thumb Code     8  stm32f7xx_it.o(i.DMA2_Stream4_IRQHandler)
    DebugMon_Handler                         0x080007f5   Thumb Code     2  stm32f7xx_it.o(i.DebugMon_Handler)
    HAL_DMA_Abort                            0x080007f9   Thumb Code    86  stm32f7xx_hal_dma.o(i.HAL_DMA_Abort)
    HAL_DMA_DeInit                           0x0800084f   Thumb Code    86  stm32f7xx_hal_dma.o(i.HAL_DMA_DeInit)
    HAL_DMA_IRQHandler                       0x080008a5   Thumb Code   404  stm32f7xx_hal_dma.o(i.HAL_DMA_IRQHandler)
    HAL_DMA_Init                             0x08000a3d   Thumb Code   134  stm32f7xx_hal_dma.o(i.HAL_DMA_Init)
    HAL_DMA_Start_IT                         0x08000ac9   Thumb Code    78  stm32f7xx_hal_dma.o(i.HAL_DMA_Start_IT)
    HAL_Delay                                0x08000b17   Thumb Code    22  stm32f7xx_hal.o(i.HAL_Delay)
    HAL_GPIO_DeInit                          0x08000b2d   Thumb Code   292  stm32f7xx_hal_gpio.o(i.HAL_GPIO_DeInit)
    HAL_GPIO_Init                            0x08000c81   Thumb Code   418  stm32f7xx_hal_gpio.o(i.HAL_GPIO_Init)
    HAL_GPIO_TogglePin                       0x08000e59   Thumb Code     8  stm32f7xx_hal_gpio.o(i.HAL_GPIO_TogglePin)
    HAL_GPIO_WritePin                        0x08000e61   Thumb Code    10  stm32f7xx_hal_gpio.o(i.HAL_GPIO_WritePin)
    HAL_GetTick                              0x08000e6d   Thumb Code     6  stm32f7xx_hal.o(i.HAL_GetTick)
    HAL_I2C_DeInit                           0x08000e79   Thumb Code    46  stm32f7xx_hal_i2c.o(i.HAL_I2C_DeInit)
    HAL_I2C_GetState                         0x08000ea7   Thumb Code     6  stm32f7xx_hal_i2c.o(i.HAL_I2C_GetState)
    HAL_I2C_Init                             0x08000ead   Thumb Code   166  stm32f7xx_hal_i2c.o(i.HAL_I2C_Init)
    HAL_I2C_Mem_Read                         0x08000f59   Thumb Code   268  stm32f7xx_hal_i2c.o(i.HAL_I2C_Mem_Read)
    HAL_I2C_Mem_Write                        0x08001069   Thumb Code   268  stm32f7xx_hal_i2c.o(i.HAL_I2C_Mem_Write)
    HAL_I2C_MspDeInit                        0x08001179   Thumb Code     2  stm32f7xx_hal_i2c.o(i.HAL_I2C_MspDeInit)
    HAL_I2C_MspInit                          0x0800117b   Thumb Code     2  stm32f7xx_hal_i2c.o(i.HAL_I2C_MspInit)
    HAL_IncTick                              0x0800117d   Thumb Code    10  stm32f7xx_hal.o(i.HAL_IncTick)
    HAL_Init                                 0x0800118d   Thumb Code    32  stm32f7xx_hal.o(i.HAL_Init)
    HAL_InitTick                             0x080011b1   Thumb Code    34  stm32f7xx_hal.o(i.HAL_InitTick)
    HAL_MspInit                              0x080011d3   Thumb Code     8  stm32f7xx_hal.o(i.HAL_MspInit)
    HAL_NVIC_EnableIRQ                       0x080011db   Thumb Code    22  stm32f7xx_hal_cortex.o(i.HAL_NVIC_EnableIRQ)
    HAL_NVIC_SetPriority                     0x080011f1   Thumb Code    60  stm32f7xx_hal_cortex.o(i.HAL_NVIC_SetPriority)
    HAL_NVIC_SetPriorityGrouping             0x08001231   Thumb Code    28  stm32f7xx_hal_cortex.o(i.HAL_NVIC_SetPriorityGrouping)
    HAL_PCDEx_ActivateLPM                    0x08001255   Thumb Code    34  stm32f7xx_hal_pcd_ex.o(i.HAL_PCDEx_ActivateLPM)
    HAL_PCDEx_LPM_Callback                   0x0800127d   Thumb Code     2  stm32f7xx_hal_pcd_ex.o(i.HAL_PCDEx_LPM_Callback)
    HAL_PCDEx_SetRxFiFo                      0x0800127f   Thumb Code     8  stm32f7xx_hal_pcd_ex.o(i.HAL_PCDEx_SetRxFiFo)
    HAL_PCDEx_SetTxFiFo                      0x08001287   Thumb Code    72  stm32f7xx_hal_pcd_ex.o(i.HAL_PCDEx_SetTxFiFo)
    HAL_PCD_ConnectCallback                  0x080012cf   Thumb Code     8  usbd_conf.o(i.HAL_PCD_ConnectCallback)
    HAL_PCD_DataInStageCallback              0x080012d7   Thumb Code    18  usbd_conf.o(i.HAL_PCD_DataInStageCallback)
    HAL_PCD_DataOutStageCallback             0x080012e9   Thumb Code    20  usbd_conf.o(i.HAL_PCD_DataOutStageCallback)
    HAL_PCD_DisconnectCallback               0x080012fd   Thumb Code     8  usbd_conf.o(i.HAL_PCD_DisconnectCallback)
    HAL_PCD_EP_Close                         0x08001305   Thumb Code    68  stm32f7xx_hal_pcd.o(i.HAL_PCD_EP_Close)
    HAL_PCD_EP_ClrStall                      0x08001349   Thumb Code    80  stm32f7xx_hal_pcd.o(i.HAL_PCD_EP_ClrStall)
    HAL_PCD_EP_Open                          0x08001399   Thumb Code    86  stm32f7xx_hal_pcd.o(i.HAL_PCD_EP_Open)
    HAL_PCD_EP_Receive                       0x080013f1   Thumb Code    94  stm32f7xx_hal_pcd.o(i.HAL_PCD_EP_Receive)
    HAL_PCD_EP_SetStall                      0x0800144f   Thumb Code    96  stm32f7xx_hal_pcd.o(i.HAL_PCD_EP_SetStall)
    HAL_PCD_EP_Transmit                      0x080014b1   Thumb Code    92  stm32f7xx_hal_pcd.o(i.HAL_PCD_EP_Transmit)
    HAL_PCD_IRQHandler                       0x0800150d   Thumb Code  1096  stm32f7xx_hal_pcd.o(i.HAL_PCD_IRQHandler)
    HAL_PCD_ISOINIncompleteCallback          0x08001955   Thumb Code     8  usbd_conf.o(i.HAL_PCD_ISOINIncompleteCallback)
    HAL_PCD_ISOOUTIncompleteCallback         0x0800195d   Thumb Code     8  usbd_conf.o(i.HAL_PCD_ISOOUTIncompleteCallback)
    HAL_PCD_Init                             0x08001965   Thumb Code   208  stm32f7xx_hal_pcd.o(i.HAL_PCD_Init)
    HAL_PCD_MspInit                          0x08001a35   Thumb Code   362  usbd_conf.o(i.HAL_PCD_MspInit)
    HAL_PCD_ResetCallback                    0x08001bb9   Thumb Code    34  usbd_conf.o(i.HAL_PCD_ResetCallback)
    HAL_PCD_ResumeCallback                   0x08001bdb   Thumb Code     8  usbd_conf.o(i.HAL_PCD_ResumeCallback)
    HAL_PCD_SOFCallback                      0x08001be3   Thumb Code     8  usbd_conf.o(i.HAL_PCD_SOFCallback)
    HAL_PCD_SetAddress                       0x08001beb   Thumb Code    36  stm32f7xx_hal_pcd.o(i.HAL_PCD_SetAddress)
    HAL_PCD_SetupStageCallback               0x08001c0f   Thumb Code    14  usbd_conf.o(i.HAL_PCD_SetupStageCallback)
    HAL_PCD_Start                            0x08001c1d   Thumb Code    42  stm32f7xx_hal_pcd.o(i.HAL_PCD_Start)
    HAL_PCD_SuspendCallback                  0x08001c47   Thumb Code     8  usbd_conf.o(i.HAL_PCD_SuspendCallback)
    HAL_PWREx_EnableOverDrive                0x08001c51   Thumb Code   100  stm32f7xx_hal_pwr_ex.o(i.HAL_PWREx_EnableOverDrive)
    HAL_RCCEx_GetPeriphCLKConfig             0x08001cbd   Thumb Code   426  stm32f7xx_hal_rcc_ex.o(i.HAL_RCCEx_GetPeriphCLKConfig)
    HAL_RCCEx_GetPeriphCLKFreq               0x08001e71   Thumb Code   268  stm32f7xx_hal_rcc_ex.o(i.HAL_RCCEx_GetPeriphCLKFreq)
    HAL_RCCEx_PeriphCLKConfig                0x08001f91   Thumb Code  1708  stm32f7xx_hal_rcc_ex.o(i.HAL_RCCEx_PeriphCLKConfig)
    HAL_RCC_ClockConfig                      0x08002641   Thumb Code   450  stm32f7xx_hal_rcc.o(i.HAL_RCC_ClockConfig)
    HAL_RCC_GetHCLKFreq                      0x0800280d   Thumb Code    38  stm32f7xx_hal_rcc.o(i.HAL_RCC_GetHCLKFreq)
    HAL_RCC_GetPCLK1Freq                     0x08002841   Thumb Code    36  stm32f7xx_hal_rcc.o(i.HAL_RCC_GetPCLK1Freq)
    HAL_RCC_GetPCLK2Freq                     0x0800286d   Thumb Code    36  stm32f7xx_hal_rcc.o(i.HAL_RCC_GetPCLK2Freq)
    HAL_RCC_GetSysClockFreq                  0x08002899   Thumb Code   120  stm32f7xx_hal_rcc.o(i.HAL_RCC_GetSysClockFreq)
    HAL_RCC_OscConfig                        0x0800291d   Thumb Code   922  stm32f7xx_hal_rcc.o(i.HAL_RCC_OscConfig)
    HAL_SAI_DMAStop                          0x08002cc1   Thumb Code    76  stm32f7xx_hal_sai.o(i.HAL_SAI_DMAStop)
    HAL_SAI_DeInit                           0x08002d0d   Thumb Code    66  stm32f7xx_hal_sai.o(i.HAL_SAI_DeInit)
    HAL_SAI_ErrorCallback                    0x08002d51   Thumb Code    62  stm32746g_discovery_audio.o(i.HAL_SAI_ErrorCallback)
    HAL_SAI_GetState                         0x08002d95   Thumb Code     6  stm32f7xx_hal_sai.o(i.HAL_SAI_GetState)
    HAL_SAI_Init                             0x08002d9d   Thumb Code   388  stm32f7xx_hal_sai.o(i.HAL_SAI_Init)
    HAL_SAI_MspDeInit                        0x08002f29   Thumb Code     2  stm32f7xx_hal_sai.o(i.HAL_SAI_MspDeInit)
    HAL_SAI_MspInit                          0x08002f2b   Thumb Code     2  stm32f7xx_hal_sai.o(i.HAL_SAI_MspInit)
    HAL_SAI_Transmit_DMA                     0x08002f2d   Thumb Code   148  stm32f7xx_hal_sai.o(i.HAL_SAI_Transmit_DMA)
    HAL_SAI_TxCpltCallback                   0x08002fcd   Thumb Code     8  stm32746g_discovery_audio.o(i.HAL_SAI_TxCpltCallback)
    HAL_SAI_TxHalfCpltCallback               0x08002fd5   Thumb Code     8  stm32746g_discovery_audio.o(i.HAL_SAI_TxHalfCpltCallback)
    HAL_SYSTICK_Config                       0x08002fdd   Thumb Code    38  stm32f7xx_hal_cortex.o(i.HAL_SYSTICK_Config)
    HAL_UART_DeInit                          0x08003003   Thumb Code    60  stm32f7xx_hal_uart.o(i.HAL_UART_DeInit)
    HAL_UART_Init                            0x0800303f   Thumb Code   106  stm32f7xx_hal_uart.o(i.HAL_UART_Init)
    HAL_UART_MspDeInit                       0x080030a9   Thumb Code    42  main.o(i.HAL_UART_MspDeInit)
    HAL_UART_MspInit                         0x080030dd   Thumb Code   100  main.o(i.HAL_UART_MspInit)
    HAL_UART_Transmit                        0x08003149   Thumb Code   200  stm32f7xx_hal_uart.o(i.HAL_UART_Transmit)
    HardFault_Handler                        0x08003211   Thumb Code     2  stm32f7xx_it.o(i.HardFault_Handler)
    MemManage_Handler                        0x080036a5   Thumb Code     2  stm32f7xx_it.o(i.MemManage_Handler)
    NMI_Handler                              0x080036a7   Thumb Code     2  stm32f7xx_it.o(i.NMI_Handler)
    OTG_FS_IRQHandler                        0x080036cd   Thumb Code     6  stm32f7xx_it.o(i.OTG_FS_IRQHandler)
    PendSV_Handler                           0x0800376f   Thumb Code     2  stm32f7xx_it.o(i.PendSV_Handler)
    SAI_BlockSynchroConfig                   0x08003771   Thumb Code    60  stm32f7xx_hal_sai_ex.o(i.SAI_BlockSynchroConfig)
    SAI_GetInputClock                        0x08003859   Thumb Code    30  stm32f7xx_hal_sai_ex.o(i.SAI_GetInputClock)
    SVC_Handler                              0x08003939   Thumb Code     2  stm32f7xx_it.o(i.SVC_Handler)
    SysTick_Handler                          0x0800393b   Thumb Code     4  stm32f7xx_it.o(i.SysTick_Handler)
    SystemInit                               0x08003941   Thumb Code    68  system_stm32f7xx.o(i.SystemInit)
    UART_AdvFeatureConfig                    0x08003995   Thumb Code   200  stm32f7xx_hal_uart.o(i.UART_AdvFeatureConfig)
    UART_CheckIdleState                      0x08003a5d   Thumb Code    78  stm32f7xx_hal_uart.o(i.UART_CheckIdleState)
    UART_SetConfig                           0x08003aad   Thumb Code   534  stm32f7xx_hal_uart.o(i.UART_SetConfig)
    UART_WaitOnFlagUntilTimeout              0x08003cf5   Thumb Code   146  stm32f7xx_hal_uart.o(i.UART_WaitOnFlagUntilTimeout)
    USBD_AUDIO_ConfigStrDescriptor           0x08003d89   Thumb Code    16  usbd_desc.o(i.USBD_AUDIO_ConfigStrDescriptor)
    USBD_AUDIO_DeviceDescriptor              0x08003e51   Thumb Code     8  usbd_desc.o(i.USBD_AUDIO_DeviceDescriptor)
    USBD_AUDIO_InterfaceStrDescriptor        0x08003f09   Thumb Code    16  usbd_desc.o(i.USBD_AUDIO_InterfaceStrDescriptor)
    USBD_AUDIO_LangIDStrDescriptor           0x08003f35   Thumb Code     8  usbd_desc.o(i.USBD_AUDIO_LangIDStrDescriptor)
    USBD_AUDIO_ManufacturerStrDescriptor     0x08003f41   Thumb Code    16  usbd_desc.o(i.USBD_AUDIO_ManufacturerStrDescriptor)
    USBD_AUDIO_ProductStrDescriptor          0x08003f69   Thumb Code    24  usbd_desc.o(i.USBD_AUDIO_ProductStrDescriptor)
    USBD_AUDIO_RegisterInterface             0x08003fcd   Thumb Code    10  usbd_audio.o(i.USBD_AUDIO_RegisterInterface)
    USBD_AUDIO_SerialStrDescriptor           0x08003fdd   Thumb Code    50  usbd_desc.o(i.USBD_AUDIO_SerialStrDescriptor)
    USBD_AUDIO_Sync                          0x080040d9   Thumb Code   134  usbd_audio.o(i.USBD_AUDIO_Sync)
    USBD_ClrClassConfig                      0x0800415f   Thumb Code    14  usbd_core.o(i.USBD_ClrClassConfig)
    USBD_CtlContinueRx                       0x0800416d   Thumb Code    16  usbd_ioreq.o(i.USBD_CtlContinueRx)
    USBD_CtlContinueSendData                 0x0800417d   Thumb Code    16  usbd_ioreq.o(i.USBD_CtlContinueSendData)
    USBD_CtlError                            0x0800418d   Thumb Code    22  usbd_ctlreq.o(i.USBD_CtlError)
    USBD_CtlPrepareRx                        0x080041a3   Thumb Code    30  usbd_ioreq.o(i.USBD_CtlPrepareRx)
    USBD_CtlReceiveStatus                    0x080041c1   Thumb Code    22  usbd_ioreq.o(i.USBD_CtlReceiveStatus)
    USBD_CtlSendData                         0x080041d7   Thumb Code    26  usbd_ioreq.o(i.USBD_CtlSendData)
    USBD_CtlSendStatus                       0x080041f1   Thumb Code    22  usbd_ioreq.o(i.USBD_CtlSendStatus)
    USBD_GetString                           0x080042e7   Thumb Code    72  usbd_ctlreq.o(i.USBD_GetString)
    USBD_Init                                0x0800432f   Thumb Code    42  usbd_core.o(i.USBD_Init)
    USBD_LL_ClearStallEP                     0x08004359   Thumb Code    14  usbd_conf.o(i.USBD_LL_ClearStallEP)
    USBD_LL_CloseEP                          0x08004367   Thumb Code    14  usbd_conf.o(i.USBD_LL_CloseEP)
    USBD_LL_DataInStage                      0x08004375   Thumb Code   170  usbd_core.o(i.USBD_LL_DataInStage)
    USBD_LL_DataOutStage                     0x0800441f   Thumb Code   106  usbd_core.o(i.USBD_LL_DataOutStage)
    USBD_LL_DevConnected                     0x08004489   Thumb Code     4  usbd_core.o(i.USBD_LL_DevConnected)
    USBD_LL_DevDisconnected                  0x0800448d   Thumb Code    22  usbd_core.o(i.USBD_LL_DevDisconnected)
    USBD_LL_Init                             0x080044a5   Thumb Code    74  usbd_conf.o(i.USBD_LL_Init)
    USBD_LL_IsStallEP                        0x080044f5   Thumb Code    32  usbd_conf.o(i.USBD_LL_IsStallEP)
    USBD_LL_IsoINIncomplete                  0x08004515   Thumb Code     4  usbd_core.o(i.USBD_LL_IsoINIncomplete)
    USBD_LL_IsoOUTIncomplete                 0x08004519   Thumb Code     4  usbd_core.o(i.USBD_LL_IsoOUTIncomplete)
    USBD_LL_OpenEP                           0x0800451d   Thumb Code    20  usbd_conf.o(i.USBD_LL_OpenEP)
    USBD_LL_PrepareReceive                   0x08004531   Thumb Code    14  usbd_conf.o(i.USBD_LL_PrepareReceive)
    USBD_LL_Reset                            0x0800453f   Thumb Code    64  usbd_core.o(i.USBD_LL_Reset)
    USBD_LL_Resume                           0x0800457f   Thumb Code    12  usbd_core.o(i.USBD_LL_Resume)
    USBD_LL_SOF                              0x0800458b   Thumb Code    24  usbd_core.o(i.USBD_LL_SOF)
    USBD_LL_SetSpeed                         0x080045a3   Thumb Code     6  usbd_core.o(i.USBD_LL_SetSpeed)
    USBD_LL_SetUSBAddress                    0x080045a9   Thumb Code    14  usbd_conf.o(i.USBD_LL_SetUSBAddress)
    USBD_LL_SetupStage                       0x080045b7   Thumb Code    86  usbd_core.o(i.USBD_LL_SetupStage)
    USBD_LL_StallEP                          0x0800460d   Thumb Code    14  usbd_conf.o(i.USBD_LL_StallEP)
    USBD_LL_Start                            0x0800461b   Thumb Code    14  usbd_conf.o(i.USBD_LL_Start)
    USBD_LL_Suspend                          0x08004629   Thumb Code    18  usbd_core.o(i.USBD_LL_Suspend)
    USBD_LL_Transmit                         0x0800463b   Thumb Code    14  usbd_conf.o(i.USBD_LL_Transmit)
    USBD_ParseSetupRequest                   0x08004649   Thumb Code    40  usbd_ctlreq.o(i.USBD_ParseSetupRequest)
    USBD_RegisterClass                       0x08004671   Thumb Code    18  usbd_core.o(i.USBD_RegisterClass)
    USBD_SetClassConfig                      0x08004683   Thumb Code    22  usbd_core.o(i.USBD_SetClassConfig)
    USBD_Start                               0x0800470d   Thumb Code    10  usbd_core.o(i.USBD_Start)
    USBD_StdDevReq                           0x08004717   Thumb Code   242  usbd_ctlreq.o(i.USBD_StdDevReq)
    USBD_StdEPReq                            0x08004809   Thumb Code   222  usbd_ctlreq.o(i.USBD_StdEPReq)
    USBD_StdItfReq                           0x080048e7   Thumb Code    52  usbd_ctlreq.o(i.USBD_StdItfReq)
    USB_ActivateEndpoint                     0x0800491d   Thumb Code   124  stm32f7xx_ll_usb.o(i.USB_ActivateEndpoint)
    USB_ActivateSetup                        0x0800499d   Thumb Code    52  stm32f7xx_ll_usb.o(i.USB_ActivateSetup)
    USB_CoreInit                             0x080049d1   Thumb Code   106  stm32f7xx_ll_usb.o(i.USB_CoreInit)
    USB_DeactivateEndpoint                   0x08004a79   Thumb Code   110  stm32f7xx_ll_usb.o(i.USB_DeactivateEndpoint)
    USB_DevConnect                           0x08004ae7   Thumb Code    24  stm32f7xx_ll_usb.o(i.USB_DevConnect)
    USB_DevDisconnect                        0x08004aff   Thumb Code    24  stm32f7xx_ll_usb.o(i.USB_DevDisconnect)
    USB_DevInit                              0x08004b19   Thumb Code   330  stm32f7xx_ll_usb.o(i.USB_DevInit)
    USB_DisableGlobalInt                     0x08004c75   Thumb Code    12  stm32f7xx_ll_usb.o(i.USB_DisableGlobalInt)
    USB_EP0StartXfer                         0x08004c81   Thumb Code   316  stm32f7xx_ll_usb.o(i.USB_EP0StartXfer)
    USB_EP0_OutStart                         0x08004dc1   Thumb Code    62  stm32f7xx_ll_usb.o(i.USB_EP0_OutStart)
    USB_EPClearStall                         0x08004dff   Thumb Code   100  stm32f7xx_ll_usb.o(i.USB_EPClearStall)
    USB_EPSetStall                           0x08004e63   Thumb Code    94  stm32f7xx_ll_usb.o(i.USB_EPSetStall)
    USB_EPStartXfer                          0x08004ec1   Thumb Code   534  stm32f7xx_ll_usb.o(i.USB_EPStartXfer)
    USB_EnableGlobalInt                      0x080050dd   Thumb Code    12  stm32f7xx_ll_usb.o(i.USB_EnableGlobalInt)
    USB_FlushRxFifo                          0x080050e9   Thumb Code    28  stm32f7xx_ll_usb.o(i.USB_FlushRxFifo)
    USB_FlushTxFifo                          0x08005109   Thumb Code    32  stm32f7xx_ll_usb.o(i.USB_FlushTxFifo)
    USB_GetDevSpeed                          0x0800512d   Thumb Code    62  stm32f7xx_ll_usb.o(i.USB_GetDevSpeed)
    USB_GetMode                              0x0800516b   Thumb Code     8  stm32f7xx_ll_usb.o(i.USB_GetMode)
    USB_ReadDevAllInEpInterrupt              0x08005173   Thumb Code    14  stm32f7xx_ll_usb.o(i.USB_ReadDevAllInEpInterrupt)
    USB_ReadDevAllOutEpInterrupt             0x08005181   Thumb Code    14  stm32f7xx_ll_usb.o(i.USB_ReadDevAllOutEpInterrupt)
    USB_ReadDevInEPInterrupt                 0x0800518f   Thumb Code    32  stm32f7xx_ll_usb.o(i.USB_ReadDevInEPInterrupt)
    USB_ReadDevOutEPInterrupt                0x080051af   Thumb Code    16  stm32f7xx_ll_usb.o(i.USB_ReadDevOutEPInterrupt)
    USB_ReadInterrupts                       0x080051bf   Thumb Code     8  stm32f7xx_ll_usb.o(i.USB_ReadInterrupts)
    USB_ReadPacket                           0x080051c7   Thumb Code    30  stm32f7xx_ll_usb.o(i.USB_ReadPacket)
    USB_SetCurrentMode                       0x080051e5   Thumb Code    44  stm32f7xx_ll_usb.o(i.USB_SetCurrentMode)
    USB_SetDevAddress                        0x08005211   Thumb Code    34  stm32f7xx_ll_usb.o(i.USB_SetDevAddress)
    USB_WritePacket                          0x08005235   Thumb Code    44  stm32f7xx_ll_usb.o(i.USB_WritePacket)
    UsageFault_Handler                       0x08005261   Thumb Code     2  stm32f7xx_it.o(i.UsageFault_Handler)
    __scatterload_copy                       0x08005263   Thumb Code    14  handlers.o(i.__scatterload_copy)
    __scatterload_null                       0x08005271   Thumb Code     2  handlers.o(i.__scatterload_null)
    __scatterload_zeroinit                   0x08005273   Thumb Code    14  handlers.o(i.__scatterload_zeroinit)
    free                                     0x08005281   Thumb Code    76  malloc.o(i.free)
    main                                     0x080052d1   Thumb Code   218  main.o(i.main)
    malloc                                   0x080053cd   Thumb Code    92  malloc.o(i.malloc)
    wm8994_DeInit                            0x08005439   Thumb Code     4  wm8994.o(i.wm8994_DeInit)
    wm8994_Init                              0x0800543d   Thumb Code  1150  wm8994.o(i.wm8994_Init)
    wm8994_Pause                             0x080058c1   Thumb Code    26  wm8994.o(i.wm8994_Pause)
    wm8994_Play                              0x080058db   Thumb Code     6  wm8994.o(i.wm8994_Play)
    wm8994_ReadID                            0x080058e1   Thumb Code    20  wm8994.o(i.wm8994_ReadID)
    wm8994_Reset                             0x080058f5   Thumb Code    22  wm8994.o(i.wm8994_Reset)
    wm8994_Resume                            0x08005911   Thumb Code     6  wm8994.o(i.wm8994_Resume)
    wm8994_SetFrequency                      0x08005917   Thumb Code   118  wm8994.o(i.wm8994_SetFrequency)
    wm8994_SetMute                           0x0800598d   Thumb Code    82  wm8994.o(i.wm8994_SetMute)
    wm8994_SetOutputMode                     0x080059e5   Thumb Code   188  wm8994.o(i.wm8994_SetOutputMode)
    wm8994_SetVolume                         0x08005aa1   Thumb Code   280  wm8994.o(i.wm8994_SetVolume)
    wm8994_Stop                              0x08005bbd   Thumb Code   120  wm8994.o(i.wm8994_Stop)
    APBAHBPrescTable                         0x08005c38   Data          16  stm32f7xx_hal_rcc.o(.constdata)
    COM_TX_PIN                               0x08005c50   Data           2  stm32746g_discovery.o(.constdata)
    COM_RX_PIN                               0x08005c52   Data           2  stm32746g_discovery.o(.constdata)
    COM_TX_AF                                0x08005c54   Data           2  stm32746g_discovery.o(.constdata)
    COM_RX_AF                                0x08005c56   Data           2  stm32746g_discovery.o(.constdata)
    GPIO_PIN                                 0x08005c58   Data           4  stm32746g_discovery.o(.constdata)
    BUTTON_PIN                               0x08005c5c   Data           6  stm32746g_discovery.o(.constdata)
    BUTTON_IRQn                              0x08005c62   Data           6  stm32746g_discovery.o(.constdata)
    Region$$Table$$Base                      0x08005c68   Number         0  anon$$obj.o(Region$$Table)
    Region$$Table$$Limit                     0x08005c88   Number         0  anon$$obj.o(Region$$Table)
    SystemCoreClock                          0x20000000   Data           4  system_stm32f7xx.o(.data)
    AHBPrescTable                            0x20000004   Data          16  system_stm32f7xx.o(.data)
    wm8994_drv                               0x20000018   Data          48  wm8994.o(.data)
    USBD_AUDIO_fops                          0x20000050   Data          28  usbd_audio_if.o(.data)
    Buffer_USART_Senden                      0x2000006c   Data           1  usbd_audio_if.o(.data)
    AUDIO_Desc                               0x20000070   Data          28  usbd_desc.o(.data)
    USBD_LangIDDesc                          0x2000008c   Data           4  usbd_desc.o(.data)
    USBD_DeviceDesc                          0x20000090   Data          18  usbd_desc.o(.data)
    USBD_StringSerial                        0x200000a2   Data          26  usbd_desc.o(.data)
    AudioInVolume                            0x200000c4   Data           2  stm32746g_discovery_audio.o(.data)
    audio_drv                                0x200000c8   Data           4  stm32746g_discovery_audio.o(.data)
    USBD_AUDIO                               0x200000cc   Data          56  usbd_audio.o(.data)
    __microlib_freelist                      0x20000180   Data           4  mvars.o(.data)
    __microlib_freelist_initialised          0x20000184   Data           4  mvars.o(.data)
    hpcd                                     0x20000188   Data         960  usbd_conf.o(.bss)
    USBD_StrDesc                             0x20000548   Data         256  usbd_desc.o(.bss)
    USBD_Device                              0x20000648   Data         548  main.o(.bss)
    UartHandle                               0x2000086c   Data         112  main.o(.bss)
    haudio_out_sai                           0x200008dc   Data         132  stm32746g_discovery_audio.o(.bss)
    haudio_in_sai                            0x20000960   Data         132  stm32746g_discovery_audio.o(.bss)
    __heap_base                              0x20000b68   Data           0  startup_stm32f746xx.o(HEAP)
    __heap_limit                             0x20004b68   Data           0  startup_stm32f746xx.o(HEAP)
    __initial_sp                             0x20006b68   Data           0  startup_stm32f746xx.o(STACK)



==============================================================================

Memory Map of the image

  Image Entry point : 0x080001c9

  Load Region LR_IROM1 (Base: 0x08000000, Size: 0x00005e10, Max: 0x00100000, ABSOLUTE, COMPRESSED[0x00005d8c])

    Execution Region ER_IROM1 (Base: 0x08000000, Size: 0x00005c88, Max: 0x00100000, ABSOLUTE)

    Base Addr    Size         Type   Attr      Idx    E Section Name        Object

    0x08000000   0x000001c8   Data   RO         3928    RESET               startup_stm32f746xx.o
    0x080001c8   0x00000000   Code   RO         5302  * .ARM.Collect$$$$00000000  mc_w.l(entry.o)
    0x080001c8   0x00000004   Code   RO         5339    .ARM.Collect$$$$00000001  mc_w.l(entry2.o)
    0x080001cc   0x00000004   Code   RO         5342    .ARM.Collect$$$$00000004  mc_w.l(entry5.o)
    0x080001d0   0x00000000   Code   RO         5344    .ARM.Collect$$$$00000008  mc_w.l(entry7b.o)
    0x080001d0   0x00000000   Code   RO         5346    .ARM.Collect$$$$0000000A  mc_w.l(entry8b.o)
    0x080001d0   0x00000008   Code   RO         5347    .ARM.Collect$$$$0000000B  mc_w.l(entry9a.o)
    0x080001d8   0x00000000   Code   RO         5349    .ARM.Collect$$$$0000000D  mc_w.l(entry10a.o)
    0x080001d8   0x00000000   Code   RO         5351    .ARM.Collect$$$$0000000F  mc_w.l(entry11a.o)
    0x080001d8   0x00000004   Code   RO         5340    .ARM.Collect$$$$00002712  mc_w.l(entry2.o)
    0x080001dc   0x00000024   Code   RO         3929    .text               startup_stm32f746xx.o
    0x08000200   0x00000024   Code   RO         5305    .text               mc_w.l(memcpya.o)
    0x08000224   0x00000024   Code   RO         5307    .text               mc_w.l(memseta.o)
    0x08000248   0x00000024   Code   RO         5355    .text               mc_w.l(init.o)
    0x0800026c   0x00000056   Code   RO         5365    .text               mc_w.l(__dczerorl2.o)
    0x080002c2   0x00000002   Code   RO         4992    i.AUDIO_IO_DeInit   stm32746g_discovery.o
    0x080002c4   0x00000004   Code   RO         4993    i.AUDIO_IO_Delay    stm32746g_discovery.o
    0x080002c8   0x0000000c   Code   RO         4994    i.AUDIO_IO_Init     stm32746g_discovery.o
    0x080002d4   0x00000034   Code   RO         4995    i.AUDIO_IO_Read     stm32746g_discovery.o
    0x08000308   0x00000034   Code   RO         4996    i.AUDIO_IO_Write    stm32746g_discovery.o
    0x0800033c   0x0000000c   Code   RO         3936    i.Audio_DeInit      usbd_audio_if.o
    0x08000348   0x00000004   Code   RO         3937    i.Audio_GetState    usbd_audio_if.o
    0x0800034c   0x00000016   Code   RO         3938    i.Audio_Init        usbd_audio_if.o
    0x08000362   0x0000000a   Code   RO         3939    i.Audio_MuteCtl     usbd_audio_if.o
    0x0800036c   0x00000004   Code   RO         3940    i.Audio_PeriodicTC  usbd_audio_if.o
    0x08000370   0x00000030   Code   RO         3941    i.Audio_PlaybackCmd  usbd_audio_if.o
    0x080003a0   0x0000000a   Code   RO         3942    i.Audio_VolumeCtl   usbd_audio_if.o
    0x080003aa   0x00000002   Code   RO         4731    i.BSP_AUDIO_IN_Error_CallBack  stm32746g_discovery_audio.o
    0x080003ac   0x00000010   Code   RO         4743    i.BSP_AUDIO_OUT_ChangeBuffer  stm32746g_discovery_audio.o
    0x080003bc   0x00000058   Code   RO         4322    i.BSP_AUDIO_OUT_ClockConfig  main.o
    0x08000414   0x00000002   Code   RO         4746    i.BSP_AUDIO_OUT_Error_CallBack  stm32746g_discovery_audio.o
    0x08000416   0x00000002   PAD
    0x08000418   0x0000000c   Code   RO         3943    i.BSP_AUDIO_OUT_HalfTransfer_CallBack  usbd_audio_if.o
    0x08000424   0x00000074   Code   RO         4748    i.BSP_AUDIO_OUT_Init  stm32746g_discovery_audio.o
    0x08000498   0x00000134   Code   RO         4750    i.BSP_AUDIO_OUT_MspInit  stm32746g_discovery_audio.o
    0x080005cc   0x00000040   Code   RO         4752    i.BSP_AUDIO_OUT_Play  stm32746g_discovery_audio.o
    0x0800060c   0x00000028   Code   RO         4754    i.BSP_AUDIO_OUT_SetAudioFrameSlot  stm32746g_discovery_audio.o
    0x08000634   0x0000001c   Code   RO         4756    i.BSP_AUDIO_OUT_SetMute  stm32746g_discovery_audio.o
    0x08000650   0x0000001c   Code   RO         4758    i.BSP_AUDIO_OUT_SetVolume  stm32746g_discovery_audio.o
    0x0800066c   0x00000034   Code   RO         4759    i.BSP_AUDIO_OUT_Stop  stm32746g_discovery_audio.o
    0x080006a0   0x0000000c   Code   RO         3944    i.BSP_AUDIO_OUT_TransferComplete_CallBack  usbd_audio_if.o
    0x080006ac   0x00000050   Code   RO         5001    i.BSP_LED_Init      stm32746g_discovery.o
    0x080006fc   0x0000001c   Code   RO         5004    i.BSP_LED_Toggle    stm32746g_discovery.o
    0x08000718   0x00000002   Code   RO         4379    i.BusFault_Handler  stm32f7xx_it.o
    0x0800071a   0x0000000a   Code   RO         3833    i.CODEC_IO_Write    wm8994.o
    0x08000724   0x00000074   Code   RO         4323    i.CPU_CACHE_Enable  main.o
    0x08000798   0x0000000c   Code   RO         4380    i.DMA2_Stream4_IRQHandler  stm32f7xx_it.o
    0x080007a4   0x00000028   Code   RO         3045    i.DMA_CalcBaseAndBitshift  stm32f7xx_hal_dma.o
    0x080007cc   0x00000028   Code   RO         3046    i.DMA_SetConfig     stm32f7xx_hal_dma.o
    0x080007f4   0x00000002   Code   RO         4381    i.DebugMon_Handler  stm32f7xx_it.o
    0x080007f6   0x00000002   PAD
    0x080007f8   0x00000056   Code   RO         3047    i.HAL_DMA_Abort     stm32f7xx_hal_dma.o
    0x0800084e   0x00000056   Code   RO         3048    i.HAL_DMA_DeInit    stm32f7xx_hal_dma.o
    0x080008a4   0x00000198   Code   RO         3051    i.HAL_DMA_IRQHandler  stm32f7xx_hal_dma.o
    0x08000a3c   0x0000008c   Code   RO         3052    i.HAL_DMA_Init      stm32f7xx_hal_dma.o
    0x08000ac8   0x0000004e   Code   RO         3055    i.HAL_DMA_Start_IT  stm32f7xx_hal_dma.o
    0x08000b16   0x00000016   Code   RO          163    i.HAL_Delay         stm32f7xx_hal.o
    0x08000b2c   0x00000154   Code   RO         2261    i.HAL_GPIO_DeInit   stm32f7xx_hal_gpio.o
    0x08000c80   0x000001d8   Code   RO         2264    i.HAL_GPIO_Init     stm32f7xx_hal_gpio.o
    0x08000e58   0x00000008   Code   RO         2267    i.HAL_GPIO_TogglePin  stm32f7xx_hal_gpio.o
    0x08000e60   0x0000000a   Code   RO         2268    i.HAL_GPIO_WritePin  stm32f7xx_hal_gpio.o
    0x08000e6a   0x00000002   PAD
    0x08000e6c   0x0000000c   Code   RO          171    i.HAL_GetTick       stm32f7xx_hal.o
    0x08000e78   0x0000002e   Code   RO         1944    i.HAL_I2C_DeInit    stm32f7xx_hal_i2c.o
    0x08000ea6   0x00000006   Code   RO         1949    i.HAL_I2C_GetState  stm32f7xx_hal_i2c.o
    0x08000eac   0x000000ac   Code   RO         1950    i.HAL_I2C_Init      stm32f7xx_hal_i2c.o
    0x08000f58   0x00000110   Code   RO         1962    i.HAL_I2C_Mem_Read  stm32f7xx_hal_i2c.o
    0x08001068   0x00000110   Code   RO         1965    i.HAL_I2C_Mem_Write  stm32f7xx_hal_i2c.o
    0x08001178   0x00000002   Code   RO         1968    i.HAL_I2C_MspDeInit  stm32f7xx_hal_i2c.o
    0x0800117a   0x00000002   Code   RO         1969    i.HAL_I2C_MspInit   stm32f7xx_hal_i2c.o
    0x0800117c   0x00000010   Code   RO          172    i.HAL_IncTick       stm32f7xx_hal.o
    0x0800118c   0x00000024   Code   RO          173    i.HAL_Init          stm32f7xx_hal.o
    0x080011b0   0x00000022   Code   RO          174    i.HAL_InitTick      stm32f7xx_hal.o
    0x080011d2   0x00000008   Code   RO          176    i.HAL_MspInit       stm32f7xx_hal.o
    0x080011da   0x00000016   Code   RO          324    i.HAL_NVIC_EnableIRQ  stm32f7xx_hal_cortex.o
    0x080011f0   0x00000040   Code   RO          330    i.HAL_NVIC_SetPriority  stm32f7xx_hal_cortex.o
    0x08001230   0x00000024   Code   RO          331    i.HAL_NVIC_SetPriorityGrouping  stm32f7xx_hal_cortex.o
    0x08001254   0x00000028   Code   RO         2997    i.HAL_PCDEx_ActivateLPM  stm32f7xx_hal_pcd_ex.o
    0x0800127c   0x00000002   Code   RO         2999    i.HAL_PCDEx_LPM_Callback  stm32f7xx_hal_pcd_ex.o
    0x0800127e   0x00000008   Code   RO         3000    i.HAL_PCDEx_SetRxFiFo  stm32f7xx_hal_pcd_ex.o
    0x08001286   0x00000048   Code   RO         3001    i.HAL_PCDEx_SetTxFiFo  stm32f7xx_hal_pcd_ex.o
    0x080012ce   0x00000008   Code   RO         4048    i.HAL_PCD_ConnectCallback  usbd_conf.o
    0x080012d6   0x00000012   Code   RO         4049    i.HAL_PCD_DataInStageCallback  usbd_conf.o
    0x080012e8   0x00000014   Code   RO         4050    i.HAL_PCD_DataOutStageCallback  usbd_conf.o
    0x080012fc   0x00000008   Code   RO         4051    i.HAL_PCD_DisconnectCallback  usbd_conf.o
    0x08001304   0x00000044   Code   RO         1358    i.HAL_PCD_EP_Close  stm32f7xx_hal_pcd.o
    0x08001348   0x00000050   Code   RO         1359    i.HAL_PCD_EP_ClrStall  stm32f7xx_hal_pcd.o
    0x08001398   0x00000056   Code   RO         1362    i.HAL_PCD_EP_Open   stm32f7xx_hal_pcd.o
    0x080013ee   0x00000002   PAD
    0x080013f0   0x0000005e   Code   RO         1363    i.HAL_PCD_EP_Receive  stm32f7xx_hal_pcd.o
    0x0800144e   0x00000060   Code   RO         1364    i.HAL_PCD_EP_SetStall  stm32f7xx_hal_pcd.o
    0x080014ae   0x00000002   PAD
    0x080014b0   0x0000005c   Code   RO         1365    i.HAL_PCD_EP_Transmit  stm32f7xx_hal_pcd.o
    0x0800150c   0x00000448   Code   RO         1367    i.HAL_PCD_IRQHandler  stm32f7xx_hal_pcd.o
    0x08001954   0x00000008   Code   RO         4052    i.HAL_PCD_ISOINIncompleteCallback  usbd_conf.o
    0x0800195c   0x00000008   Code   RO         4053    i.HAL_PCD_ISOOUTIncompleteCallback  usbd_conf.o
    0x08001964   0x000000d0   Code   RO         1370    i.HAL_PCD_Init      stm32f7xx_hal_pcd.o
    0x08001a34   0x00000184   Code   RO         4055    i.HAL_PCD_MspInit   usbd_conf.o
    0x08001bb8   0x00000022   Code   RO         4056    i.HAL_PCD_ResetCallback  usbd_conf.o
    0x08001bda   0x00000008   Code   RO         4057    i.HAL_PCD_ResumeCallback  usbd_conf.o
    0x08001be2   0x00000008   Code   RO         4058    i.HAL_PCD_SOFCallback  usbd_conf.o
    0x08001bea   0x00000024   Code   RO         1376    i.HAL_PCD_SetAddress  stm32f7xx_hal_pcd.o
    0x08001c0e   0x0000000e   Code   RO         4059    i.HAL_PCD_SetupStageCallback  usbd_conf.o
    0x08001c1c   0x0000002a   Code   RO         1378    i.HAL_PCD_Start     stm32f7xx_hal_pcd.o
    0x08001c46   0x00000008   Code   RO         4060    i.HAL_PCD_SuspendCallback  usbd_conf.o
    0x08001c4e   0x00000002   PAD
    0x08001c50   0x0000006c   Code   RO          855    i.HAL_PWREx_EnableOverDrive  stm32f7xx_hal_pwr_ex.o
    0x08001cbc   0x000001b4   Code   RO         2327    i.HAL_RCCEx_GetPeriphCLKConfig  stm32f7xx_hal_rcc_ex.o
    0x08001e70   0x00000120   Code   RO         2328    i.HAL_RCCEx_GetPeriphCLKFreq  stm32f7xx_hal_rcc_ex.o
    0x08001f90   0x000006b0   Code   RO         2329    i.HAL_RCCEx_PeriphCLKConfig  stm32f7xx_hal_rcc_ex.o
    0x08002640   0x000001cc   Code   RO          942    i.HAL_RCC_ClockConfig  stm32f7xx_hal_rcc.o
    0x0800280c   0x00000034   Code   RO          947    i.HAL_RCC_GetHCLKFreq  stm32f7xx_hal_rcc.o
    0x08002840   0x0000002c   Code   RO          949    i.HAL_RCC_GetPCLK1Freq  stm32f7xx_hal_rcc.o
    0x0800286c   0x0000002c   Code   RO          950    i.HAL_RCC_GetPCLK2Freq  stm32f7xx_hal_rcc.o
    0x08002898   0x00000084   Code   RO          951    i.HAL_RCC_GetSysClockFreq  stm32f7xx_hal_rcc.o
    0x0800291c   0x000003a4   Code   RO          954    i.HAL_RCC_OscConfig  stm32f7xx_hal_rcc.o
    0x08002cc0   0x0000004c   Code   RO         1687    i.HAL_SAI_DMAStop   stm32f7xx_hal_sai.o
    0x08002d0c   0x00000042   Code   RO         1688    i.HAL_SAI_DeInit    stm32f7xx_hal_sai.o
    0x08002d4e   0x00000002   PAD
    0x08002d50   0x00000044   Code   RO         4761    i.HAL_SAI_ErrorCallback  stm32746g_discovery_audio.o
    0x08002d94   0x00000006   Code   RO         1695    i.HAL_SAI_GetState  stm32f7xx_hal_sai.o
    0x08002d9a   0x00000002   PAD
    0x08002d9c   0x0000018c   Code   RO         1697    i.HAL_SAI_Init      stm32f7xx_hal_sai.o
    0x08002f28   0x00000002   Code   RO         1699    i.HAL_SAI_MspDeInit  stm32f7xx_hal_sai.o
    0x08002f2a   0x00000002   Code   RO         1700    i.HAL_SAI_MspInit   stm32f7xx_hal_sai.o
    0x08002f2c   0x000000a0   Code   RO         1707    i.HAL_SAI_Transmit_DMA  stm32f7xx_hal_sai.o
    0x08002fcc   0x00000008   Code   RO         4764    i.HAL_SAI_TxCpltCallback  stm32746g_discovery_audio.o
    0x08002fd4   0x00000008   Code   RO         4765    i.HAL_SAI_TxHalfCpltCallback  stm32746g_discovery_audio.o
    0x08002fdc   0x00000026   Code   RO          335    i.HAL_SYSTICK_Config  stm32f7xx_hal_cortex.o
    0x08003002   0x0000003c   Code   RO         3417    i.HAL_UART_DeInit   stm32f7xx_hal_uart.o
    0x0800303e   0x0000006a   Code   RO         3422    i.HAL_UART_Init     stm32f7xx_hal_uart.o
    0x080030a8   0x00000034   Code   RO         4324    i.HAL_UART_MspDeInit  main.o
    0x080030dc   0x0000006c   Code   RO         4325    i.HAL_UART_MspInit  main.o
    0x08003148   0x000000c8   Code   RO         3430    i.HAL_UART_Transmit  stm32f7xx_hal_uart.o
    0x08003210   0x00000002   Code   RO         4382    i.HardFault_Handler  stm32f7xx_it.o
    0x08003212   0x00000002   PAD
    0x08003214   0x00000080   Code   RO         1985    i.I2C_IsAcknowledgeFailed  stm32f7xx_hal_i2c.o
    0x08003294   0x00000066   Code   RO         1988    i.I2C_RequestMemoryRead  stm32f7xx_hal_i2c.o
    0x080032fa   0x00000066   Code   RO         1989    i.I2C_RequestMemoryWrite  stm32f7xx_hal_i2c.o
    0x08003360   0x00000024   Code   RO         1992    i.I2C_TransferConfig  stm32f7xx_hal_i2c.o
    0x08003384   0x0000006e   Code   RO         1993    i.I2C_WaitOnFlagUntilTimeout  stm32f7xx_hal_i2c.o
    0x080033f2   0x0000004e   Code   RO         1995    i.I2C_WaitOnSTOPFlagUntilTimeout  stm32f7xx_hal_i2c.o
    0x08003440   0x00000052   Code   RO         1996    i.I2C_WaitOnTXISFlagUntilTimeout  stm32f7xx_hal_i2c.o
    0x08003492   0x00000012   Code   RO         5016    i.I2Cx_Error        stm32746g_discovery.o
    0x080034a4   0x00000050   Code   RO         5017    i.I2Cx_Init         stm32746g_discovery.o
    0x080034f4   0x00000124   Code   RO         5018    i.I2Cx_MspInit      stm32746g_discovery.o
    0x08003618   0x0000002a   Code   RO         5019    i.I2Cx_ReadMultiple  stm32746g_discovery.o
    0x08003642   0x0000002a   Code   RO         5020    i.I2Cx_WriteMultiple  stm32746g_discovery.o
    0x0800366c   0x00000038   Code   RO         4249    i.IntToUnicode      usbd_desc.o
    0x080036a4   0x00000002   Code   RO         4383    i.MemManage_Handler  stm32f7xx_it.o
    0x080036a6   0x00000002   Code   RO         4384    i.NMI_Handler       stm32f7xx_it.o
    0x080036a8   0x00000022   Code   RO          337    i.NVIC_SetPriority  stm32f7xx_hal_cortex.o
    0x080036ca   0x00000002   PAD
    0x080036cc   0x0000000c   Code   RO         4385    i.OTG_FS_IRQHandler  stm32f7xx_it.o
    0x080036d8   0x00000096   Code   RO         1381    i.PCD_WriteEmptyTxFifo  stm32f7xx_hal_pcd.o
    0x0800376e   0x00000002   Code   RO         4386    i.PendSV_Handler    stm32f7xx_it.o
    0x08003770   0x00000044   Code   RO         1319    i.SAI_BlockSynchroConfig  stm32f7xx_hal_sai_ex.o
    0x080037b4   0x0000001e   Code   RO         1711    i.SAI_DMAError      stm32f7xx_hal_sai.o
    0x080037d2   0x0000003c   Code   RO         1714    i.SAI_DMATxCplt     stm32f7xx_hal_sai.o
    0x0800380e   0x0000000a   Code   RO         1715    i.SAI_DMATxHalfCplt  stm32f7xx_hal_sai.o
    0x08003818   0x0000003e   Code   RO         1716    i.SAI_Disable       stm32f7xx_hal_sai.o
    0x08003856   0x00000002   PAD
    0x08003858   0x00000024   Code   RO         1320    i.SAI_GetInputClock  stm32f7xx_hal_sai_ex.o
    0x0800387c   0x00000032   Code   RO         1720    i.SAI_InterruptFlag  stm32f7xx_hal_sai.o
    0x080038ae   0x00000002   PAD
    0x080038b0   0x0000001c   Code   RO         4768    i.SAIx_Out_DeInit   stm32746g_discovery_audio.o
    0x080038cc   0x0000006c   Code   RO         4769    i.SAIx_Out_Init     stm32746g_discovery_audio.o
    0x08003938   0x00000002   Code   RO         4387    i.SVC_Handler       stm32f7xx_it.o
    0x0800393a   0x00000004   Code   RO         4388    i.SysTick_Handler   stm32f7xx_it.o
    0x0800393e   0x00000002   PAD
    0x08003940   0x00000054   Code   RO            5    i.SystemInit        system_stm32f7xx.o
    0x08003994   0x000000c8   Code   RO         3435    i.UART_AdvFeatureConfig  stm32f7xx_hal_uart.o
    0x08003a5c   0x0000004e   Code   RO         3436    i.UART_CheckIdleState  stm32f7xx_hal_uart.o
    0x08003aaa   0x00000002   PAD
    0x08003aac   0x00000248   Code   RO         3443    i.UART_SetConfig    stm32f7xx_hal_uart.o
    0x08003cf4   0x00000092   Code   RO         3445    i.UART_WaitOnFlagUntilTimeout  stm32f7xx_hal_uart.o
    0x08003d86   0x00000002   PAD
    0x08003d88   0x00000024   Code   RO         4250    i.USBD_AUDIO_ConfigStrDescriptor  usbd_desc.o
    0x08003dac   0x00000004   Code   RO         5208    i.USBD_AUDIO_DataIn  usbd_audio.o
    0x08003db0   0x00000074   Code   RO         5209    i.USBD_AUDIO_DataOut  usbd_audio.o
    0x08003e24   0x0000002c   Code   RO         5210    i.USBD_AUDIO_DeInit  usbd_audio.o
    0x08003e50   0x0000000c   Code   RO         4251    i.USBD_AUDIO_DeviceDescriptor  usbd_desc.o
    0x08003e5c   0x00000034   Code   RO         5211    i.USBD_AUDIO_EP0_RxReady  usbd_audio.o
    0x08003e90   0x00000004   Code   RO         5212    i.USBD_AUDIO_EP0_TxReady  usbd_audio.o
    0x08003e94   0x0000000c   Code   RO         5213    i.USBD_AUDIO_GetCfgDesc  usbd_audio.o
    0x08003ea0   0x0000000c   Code   RO         5214    i.USBD_AUDIO_GetDeviceQualifierDesc  usbd_audio.o
    0x08003eac   0x0000005a   Code   RO         5215    i.USBD_AUDIO_Init   usbd_audio.o
    0x08003f06   0x00000002   PAD
    0x08003f08   0x00000024   Code   RO         4252    i.USBD_AUDIO_InterfaceStrDescriptor  usbd_desc.o
    0x08003f2c   0x00000004   Code   RO         5216    i.USBD_AUDIO_IsoINIncomplete  usbd_audio.o
    0x08003f30   0x00000004   Code   RO         5217    i.USBD_AUDIO_IsoOutIncomplete  usbd_audio.o
    0x08003f34   0x0000000c   Code   RO         4253    i.USBD_AUDIO_LangIDStrDescriptor  usbd_desc.o
    0x08003f40   0x00000028   Code   RO         4254    i.USBD_AUDIO_ManufacturerStrDescriptor  usbd_desc.o
    0x08003f68   0x00000064   Code   RO         4255    i.USBD_AUDIO_ProductStrDescriptor  usbd_desc.o
    0x08003fcc   0x0000000a   Code   RO         5218    i.USBD_AUDIO_RegisterInterface  usbd_audio.o
    0x08003fd6   0x00000004   Code   RO         5219    i.USBD_AUDIO_SOF    usbd_audio.o
    0x08003fda   0x00000002   PAD
    0x08003fdc   0x0000003c   Code   RO         4256    i.USBD_AUDIO_SerialStrDescriptor  usbd_desc.o
    0x08004018   0x000000c0   Code   RO         5220    i.USBD_AUDIO_Setup  usbd_audio.o
    0x080040d8   0x00000086   Code   RO         5221    i.USBD_AUDIO_Sync   usbd_audio.o
    0x0800415e   0x0000000e   Code   RO         4592    i.USBD_ClrClassConfig  usbd_core.o
    0x0800416c   0x00000010   Code   RO         4532    i.USBD_CtlContinueRx  usbd_ioreq.o
    0x0800417c   0x00000010   Code   RO         4533    i.USBD_CtlContinueSendData  usbd_ioreq.o
    0x0800418c   0x00000016   Code   RO         4467    i.USBD_CtlError     usbd_ctlreq.o
    0x080041a2   0x0000001e   Code   RO         4534    i.USBD_CtlPrepareRx  usbd_ioreq.o
    0x080041c0   0x00000016   Code   RO         4535    i.USBD_CtlReceiveStatus  usbd_ioreq.o
    0x080041d6   0x0000001a   Code   RO         4536    i.USBD_CtlSendData  usbd_ioreq.o
    0x080041f0   0x00000016   Code   RO         4537    i.USBD_CtlSendStatus  usbd_ioreq.o
    0x08004206   0x000000e0   Code   RO         4468    i.USBD_GetDescriptor  usbd_ctlreq.o
    0x080042e6   0x00000048   Code   RO         4469    i.USBD_GetString    usbd_ctlreq.o
    0x0800432e   0x0000002a   Code   RO         4594    i.USBD_Init         usbd_core.o
    0x08004358   0x0000000e   Code   RO         4061    i.USBD_LL_ClearStallEP  usbd_conf.o
    0x08004366   0x0000000e   Code   RO         4062    i.USBD_LL_CloseEP   usbd_conf.o
    0x08004374   0x000000aa   Code   RO         4595    i.USBD_LL_DataInStage  usbd_core.o
    0x0800441e   0x0000006a   Code   RO         4596    i.USBD_LL_DataOutStage  usbd_core.o
    0x08004488   0x00000004   Code   RO         4597    i.USBD_LL_DevConnected  usbd_core.o
    0x0800448c   0x00000016   Code   RO         4598    i.USBD_LL_DevDisconnected  usbd_core.o
    0x080044a2   0x00000002   PAD
    0x080044a4   0x00000050   Code   RO         4067    i.USBD_LL_Init      usbd_conf.o
    0x080044f4   0x00000020   Code   RO         4068    i.USBD_LL_IsStallEP  usbd_conf.o
    0x08004514   0x00000004   Code   RO         4599    i.USBD_LL_IsoINIncomplete  usbd_core.o
    0x08004518   0x00000004   Code   RO         4600    i.USBD_LL_IsoOUTIncomplete  usbd_core.o
    0x0800451c   0x00000014   Code   RO         4069    i.USBD_LL_OpenEP    usbd_conf.o
    0x08004530   0x0000000e   Code   RO         4070    i.USBD_LL_PrepareReceive  usbd_conf.o
    0x0800453e   0x00000040   Code   RO         4601    i.USBD_LL_Reset     usbd_core.o
    0x0800457e   0x0000000c   Code   RO         4602    i.USBD_LL_Resume    usbd_core.o
    0x0800458a   0x00000018   Code   RO         4603    i.USBD_LL_SOF       usbd_core.o
    0x080045a2   0x00000006   Code   RO         4604    i.USBD_LL_SetSpeed  usbd_core.o
    0x080045a8   0x0000000e   Code   RO         4071    i.USBD_LL_SetUSBAddress  usbd_conf.o
    0x080045b6   0x00000056   Code   RO         4605    i.USBD_LL_SetupStage  usbd_core.o
    0x0800460c   0x0000000e   Code   RO         4072    i.USBD_LL_StallEP   usbd_conf.o
    0x0800461a   0x0000000e   Code   RO         4073    i.USBD_LL_Start     usbd_conf.o
    0x08004628   0x00000012   Code   RO         4606    i.USBD_LL_Suspend   usbd_core.o
    0x0800463a   0x0000000e   Code   RO         4075    i.USBD_LL_Transmit  usbd_conf.o
    0x08004648   0x00000028   Code   RO         4470    i.USBD_ParseSetupRequest  usbd_ctlreq.o
    0x08004670   0x00000012   Code   RO         4607    i.USBD_RegisterClass  usbd_core.o
    0x08004682   0x00000016   Code   RO         4609    i.USBD_SetClassConfig  usbd_core.o
    0x08004698   0x00000074   Code   RO         4471    i.USBD_SetConfig    usbd_ctlreq.o
    0x0800470c   0x0000000a   Code   RO         4610    i.USBD_Start        usbd_core.o
    0x08004716   0x000000f2   Code   RO         4472    i.USBD_StdDevReq    usbd_ctlreq.o
    0x08004808   0x000000de   Code   RO         4473    i.USBD_StdEPReq     usbd_ctlreq.o
    0x080048e6   0x00000034   Code   RO         4474    i.USBD_StdItfReq    usbd_ctlreq.o
    0x0800491a   0x00000002   PAD
    0x0800491c   0x00000080   Code   RO          445    i.USB_ActivateEndpoint  stm32f7xx_ll_usb.o
    0x0800499c   0x00000034   Code   RO          446    i.USB_ActivateSetup  stm32f7xx_ll_usb.o
    0x080049d0   0x00000070   Code   RO          448    i.USB_CoreInit      stm32f7xx_ll_usb.o
    0x08004a40   0x00000038   Code   RO          449    i.USB_CoreReset     stm32f7xx_ll_usb.o
    0x08004a78   0x0000006e   Code   RO          451    i.USB_DeactivateEndpoint  stm32f7xx_ll_usb.o
    0x08004ae6   0x00000018   Code   RO          452    i.USB_DevConnect    stm32f7xx_ll_usb.o
    0x08004afe   0x00000018   Code   RO          453    i.USB_DevDisconnect  stm32f7xx_ll_usb.o
    0x08004b16   0x00000002   PAD
    0x08004b18   0x0000015c   Code   RO          454    i.USB_DevInit       stm32f7xx_ll_usb.o
    0x08004c74   0x0000000c   Code   RO          455    i.USB_DisableGlobalInt  stm32f7xx_ll_usb.o
    0x08004c80   0x00000140   Code   RO          458    i.USB_EP0StartXfer  stm32f7xx_ll_usb.o
    0x08004dc0   0x0000003e   Code   RO          459    i.USB_EP0_OutStart  stm32f7xx_ll_usb.o
    0x08004dfe   0x00000064   Code   RO          460    i.USB_EPClearStall  stm32f7xx_ll_usb.o
    0x08004e62   0x0000005e   Code   RO          461    i.USB_EPSetStall    stm32f7xx_ll_usb.o
    0x08004ec0   0x0000021c   Code   RO          462    i.USB_EPStartXfer   stm32f7xx_ll_usb.o
    0x080050dc   0x0000000c   Code   RO          463    i.USB_EnableGlobalInt  stm32f7xx_ll_usb.o
    0x080050e8   0x00000020   Code   RO          464    i.USB_FlushRxFifo   stm32f7xx_ll_usb.o
    0x08005108   0x00000024   Code   RO          465    i.USB_FlushTxFifo   stm32f7xx_ll_usb.o
    0x0800512c   0x0000003e   Code   RO          467    i.USB_GetDevSpeed   stm32f7xx_ll_usb.o
    0x0800516a   0x00000008   Code   RO          469    i.USB_GetMode       stm32f7xx_ll_usb.o
    0x08005172   0x0000000e   Code   RO          476    i.USB_ReadDevAllInEpInterrupt  stm32f7xx_ll_usb.o
    0x08005180   0x0000000e   Code   RO          477    i.USB_ReadDevAllOutEpInterrupt  stm32f7xx_ll_usb.o
    0x0800518e   0x00000020   Code   RO          478    i.USB_ReadDevInEPInterrupt  stm32f7xx_ll_usb.o
    0x080051ae   0x00000010   Code   RO          479    i.USB_ReadDevOutEPInterrupt  stm32f7xx_ll_usb.o
    0x080051be   0x00000008   Code   RO          480    i.USB_ReadInterrupts  stm32f7xx_ll_usb.o
    0x080051c6   0x0000001e   Code   RO          481    i.USB_ReadPacket    stm32f7xx_ll_usb.o
    0x080051e4   0x0000002c   Code   RO          483    i.USB_SetCurrentMode  stm32f7xx_ll_usb.o
    0x08005210   0x00000022   Code   RO          484    i.USB_SetDevAddress  stm32f7xx_ll_usb.o
    0x08005232   0x00000002   PAD
    0x08005234   0x0000002c   Code   RO          488    i.USB_WritePacket   stm32f7xx_ll_usb.o
    0x08005260   0x00000002   Code   RO         4389    i.UsageFault_Handler  stm32f7xx_it.o
    0x08005262   0x0000000e   Code   RO         5359    i.__scatterload_copy  mc_w.l(handlers.o)
    0x08005270   0x00000002   Code   RO         5360    i.__scatterload_null  mc_w.l(handlers.o)
    0x08005272   0x0000000e   Code   RO         5361    i.__scatterload_zeroinit  mc_w.l(handlers.o)
    0x08005280   0x00000050   Code   RO         5311    i.free              mc_w.l(malloc.o)
    0x080052d0   0x000000fc   Code   RO         4326    i.main              main.o
    0x080053cc   0x0000006c   Code   RO         5312    i.malloc            mc_w.l(malloc.o)
    0x08005438   0x00000004   Code   RO         3834    i.wm8994_DeInit     wm8994.o
    0x0800543c   0x00000484   Code   RO         3835    i.wm8994_Init       wm8994.o
    0x080058c0   0x0000001a   Code   RO         3836    i.wm8994_Pause      wm8994.o
    0x080058da   0x00000006   Code   RO         3837    i.wm8994_Play       wm8994.o
    0x080058e0   0x00000014   Code   RO         3838    i.wm8994_ReadID     wm8994.o
    0x080058f4   0x0000001c   Code   RO         3839    i.wm8994_Reset      wm8994.o
    0x08005910   0x00000006   Code   RO         3840    i.wm8994_Resume     wm8994.o
    0x08005916   0x00000076   Code   RO         3841    i.wm8994_SetFrequency  wm8994.o
    0x0800598c   0x00000058   Code   RO         3842    i.wm8994_SetMute    wm8994.o
    0x080059e4   0x000000bc   Code   RO         3843    i.wm8994_SetOutputMode  wm8994.o
    0x08005aa0   0x0000011c   Code   RO         3844    i.wm8994_SetVolume  wm8994.o
    0x08005bbc   0x0000007c   Code   RO         3845    i.wm8994_Stop       wm8994.o
    0x08005c38   0x00000010   Data   RO          955    .constdata          stm32f7xx_hal_rcc.o
    0x08005c48   0x00000008   Data   RO         3056    .constdata          stm32f7xx_hal_dma.o
    0x08005c50   0x00000018   Data   RO         5026    .constdata          stm32746g_discovery.o
    0x08005c68   0x00000020   Data   RO         5357    Region$$Table       anon$$obj.o


    Execution Region RW_IRAM1 (Base: 0x20000000, Size: 0x00006b68, Max: 0x00050000, ABSOLUTE, COMPRESSED[0x00000104])

    Base Addr    Size         Type   Attr      Idx    E Section Name        Object

    0x20000000   0x00000014   Data   RW            6    .data               system_stm32f7xx.o
    0x20000014   0x00000004   Data   RW          179    .data               stm32f7xx_hal.o
    0x20000018   0x00000030   Data   RW         3846    .data               wm8994.o
    0x20000048   0x00000008   Data   RW         3847    .data               wm8994.o
    0x20000050   0x0000001c   Data   RW         3945    .data               usbd_audio_if.o
    0x2000006c   0x00000001   Data   RW         3946    .data               usbd_audio_if.o
    0x2000006d   0x00000003   PAD
    0x20000070   0x0000001c   Data   RW         4258    .data               usbd_desc.o
    0x2000008c   0x00000030   Data   RW         4259    .data               usbd_desc.o
    0x200000bc   0x00000004   Data   RW         4329    .data               main.o
    0x200000c0   0x00000001   Data   RW         4475    .data               usbd_ctlreq.o
    0x200000c1   0x00000003   PAD
    0x200000c4   0x00000008   Data   RW         4772    .data               stm32746g_discovery_audio.o
    0x200000cc   0x00000038   Data   RW         5222    .data               usbd_audio.o
    0x20000104   0x0000007a   Data   RW         5223    .data               usbd_audio.o
    0x2000017e   0x00000002   PAD
    0x20000180   0x00000004   Data   RW         5353    .data               mc_w.l(mvars.o)
    0x20000184   0x00000004   Data   RW         5354    .data               mc_w.l(mvars.o)
    0x20000188   0x000003c0   Zero   RW         4076    .bss                usbd_conf.o
    0x20000548   0x00000100   Zero   RW         4257    .bss                usbd_desc.o
    0x20000648   0x00000294   Zero   RW         4327    .bss                main.o
    0x200008dc   0x00000210   Zero   RW         4770    .bss                stm32746g_discovery_audio.o
    0x20000aec   0x00000078   Zero   RW         5025    .bss                stm32746g_discovery.o
    0x20000b64   0x00000004   PAD
    0x20000b68   0x00004000   Zero   RW         3927    HEAP                startup_stm32f746xx.o
    0x20004b68   0x00002000   Zero   RW         3926    STACK               startup_stm32f746xx.o


==============================================================================

Image component sizes


      Code (inc. data)   RO Data    RW Data    ZI Data      Debug   Object Name

       616         60          0          4        660      36723   main.o
        36          8        456          0      24576        912   startup_stm32f746xx.o
       704         82         24          0        120      11562   stm32746g_discovery.o
       876        104          0          8        528      15173   stm32746g_discovery_audio.o
       128         16          0          4          0       5404   stm32f7xx_hal.o
       194         12          0          0          0      36395   stm32f7xx_hal_cortex.o
       878         16          8          0          0       7176   stm32f7xx_hal_dma.o
       830        102          0          0          0       4879   stm32f7xx_hal_gpio.o
      1410         24          0          0          0      14776   stm32f7xx_hal_i2c.o
      2048          0          0          0          0      12453   stm32f7xx_hal_pcd.o
       122          6          0          0          0       3769   stm32f7xx_hal_pcd_ex.o
       108          8          0          0          0       1560   stm32f7xx_hal_pwr_ex.o
      1664         62         16          0          0       7127   stm32f7xx_hal_rcc.o
      2436         46          0          0          0       4892   stm32f7xx_hal_rcc_ex.o
       920         20          0          0          0      10726   stm32f7xx_hal_sai.o
       104         14          0          0          0       2125   stm32f7xx_hal_sai_ex.o
      1374         70          0          0          0       8055   stm32f7xx_hal_uart.o
        44         10          0          0          0       6200   stm32f7xx_it.o
      2368         52          0          0          0      24360   stm32f7xx_ll_usb.o
        84         16          0         20          0     484121   system_stm32f7xx.o
       682         14          0        178          0      15610   usbd_audio.o
       134         14          0         29          0      20101   usbd_audio_if.o
       760         32          0          0        960      16021   usbd_conf.o
       626          0          0          0          0      14502   usbd_core.o
       990         28          0          1          0       9324   usbd_ctlreq.o
       352        158          0         76        256       7282   usbd_desc.o
       132          0          0          0          0       5512   usbd_ioreq.o
      2058         26          0         56          0      13318   wm8994.o

    ----------------------------------------------------------------------
     22720       1000        536        384      27104     800058   Object Totals
         0          0         32          0          0          0   (incl. Generated)
        42          0          0          8          4          0   (incl. Padding)

    ----------------------------------------------------------------------

      Code (inc. data)   RO Data    RW Data    ZI Data      Debug   Library Member Name

        86          0          0          0          0          0   __dczerorl2.o
         0          0          0          0          0          0   entry.o
         0          0          0          0          0          0   entry10a.o
         0          0          0          0          0          0   entry11a.o
         8          4          0          0          0          0   entry2.o
         4          0          0          0          0          0   entry5.o
         0          0          0          0          0          0   entry7b.o
         0          0          0          0          0          0   entry8b.o
         8          4          0          0          0          0   entry9a.o
        30          0          0          0          0          0   handlers.o
        36          8          0          0          0         68   init.o
       188         20          0          0          0        160   malloc.o
        36          0          0          0          0         68   memcpya.o
        36          0          0          0          0        108   memseta.o
         0          0          0          8          0          0   mvars.o

    ----------------------------------------------------------------------
       432         36          0          8          0        404   Library Totals
         0          0          0          0          0          0   (incl. Padding)

    ----------------------------------------------------------------------

      Code (inc. data)   RO Data    RW Data    ZI Data      Debug   Library Name

       432         36          0          8          0        404   mc_w.l

    ----------------------------------------------------------------------
       432         36          0          8          0        404   Library Totals

    ----------------------------------------------------------------------

==============================================================================


      Code (inc. data)   RO Data    RW Data    ZI Data      Debug   

     23152       1036        536        392      27104     776190   Grand Totals
     23152       1036        536        260      27104     776190   ELF Image Totals (compressed)
     23152       1036        536        260          0          0   ROM Totals

==============================================================================

    Total RO  Size (Code + RO Data)                23688 (  23.13kB)
    Total RW  Size (RW Data + ZI Data)             27496 (  26.85kB)
    Total ROM Size (Code + RO Data + RW Data)      23948 (  23.39kB)

==============================================================================

